Microchip Technology Inc, vv1.24 (0)

Tool Name:
  c:\program files (x86)\microchip\xc16\v1.24\bin\bin\..\bin/elf-ld.exe

Command:
  -p33EP512MU810 \
  -o \
  dist/XC16_dsPIC33EP512MU810/debug/PLCD_P01V45.debug.elf \
  -Lc:/program files (x86)/microchip/xc16/v1.24/bin/bin/.. \
  -Lc:/program files (x86)/microchip/xc16/v1.24/bin/bin/../../lib \
  -Lc:/program files (x86)/microchip/xc16/v1.24/bin/bin/../../lib/PIC24E \
  -Lc:/program files (x86)/microchip/xc16/v1.24/bin/bin/../../support/PIC24E/gld \
  -Lc:/program files (x86)/microchip/xc16/v1.24/bin/bin/../../lib/PIC24F \
  -Lc:/program files (x86)/microchip/xc16/v1.24/bin/bin/../../support/PIC24F/gld \
  -Lc:/program files (x86)/microchip/xc16/v1.24/bin/bin/../../lib/PIC24H \
  -Lc:/program files (x86)/microchip/xc16/v1.24/bin/bin/../../support/PIC24H/gld \
  -Lc:/program files (x86)/microchip/xc16/v1.24/bin/bin/../../lib/dsPIC30F \
  -Lc:/program files (x86)/microchip/xc16/v1.24/bin/bin/../../support/dsPIC30F/gld \
  -Lc:/program files (x86)/microchip/xc16/v1.24/bin/bin/../../lib/dsPIC33E \
  -Lc:/program files (x86)/microchip/xc16/v1.24/bin/bin/../../support/dsPIC33E/gld \
  -Lc:/program files (x86)/microchip/xc16/v1.24/bin/bin/../../lib/dsPIC33F \
  -Lc:/program files (x86)/microchip/xc16/v1.24/bin/bin/../../support/dsPIC33F/gld \
  build/XC16_dsPIC33EP512MU810/debug/B40/par/abcc_handler_par.o \
  build/XC16_dsPIC33EP512MU810/debug/B40/par/abcc_par_drv.o \
  build/XC16_dsPIC33EP512MU810/debug/B40/spi/abcc_crc32.o \
  build/XC16_dsPIC33EP512MU810/debug/B40/spi/abcc_handler_spi.o \
  build/XC16_dsPIC33EP512MU810/debug/B40/spi/abcc_spi_drv.o \
  build/XC16_dsPIC33EP512MU810/debug/B40/abcc_cbf.o \
  build/XC16_dsPIC33EP512MU810/debug/B40/abcc_debug_err.o \
  build/XC16_dsPIC33EP512MU810/debug/B40/abcc_handler.o \
  build/XC16_dsPIC33EP512MU810/debug/B40/abcc_link.o \
  build/XC16_dsPIC33EP512MU810/debug/B40/abcc_mem.o \
  build/XC16_dsPIC33EP512MU810/debug/B40/abcc_remap.o \
  build/XC16_dsPIC33EP512MU810/debug/B40/abcc_setup.o \
  build/XC16_dsPIC33EP512MU810/debug/B40/abcc_sys_adapt.o \
  build/XC16_dsPIC33EP512MU810/debug/B40/abcc_timer.o \
  build/XC16_dsPIC33EP512MU810/debug/B40/ad_obj.o \
  build/XC16_dsPIC33EP512MU810/debug/B40/app_obj.o \
  build/XC16_dsPIC33EP512MU810/debug/B40/dpv1.o \
  build/XC16_dsPIC33EP512MU810/debug/B40/user_adi.o \
  build/XC16_dsPIC33EP512MU810/debug/B40/user_setup.o \
  build/XC16_dsPIC33EP512MU810/debug/ECAN/ECAN1Drv.o \
  build/XC16_dsPIC33EP512MU810/debug/BerkeleyTCPClient.o \
  build/XC16_dsPIC33EP512MU810/debug/BerkeleyTCPServer.o \
  build/XC16_dsPIC33EP512MU810/debug/BerkeleyUDPClient.o \
  build/XC16_dsPIC33EP512MU810/debug/MODBUSTCPServer.o \
  build/XC16_dsPIC33EP512MU810/debug/Regul.o \
  build/XC16_dsPIC33EP512MU810/debug/Pesage.o \
  build/XC16_dsPIC33EP512MU810/debug/Process.o \
  build/XC16_dsPIC33EP512MU810/debug/TCPIPStack/Announce.o \
  build/XC16_dsPIC33EP512MU810/debug/TCPIPStack/ARCFOUR.o \
  build/XC16_dsPIC33EP512MU810/debug/TCPIPStack/ARP.o \
  build/XC16_dsPIC33EP512MU810/debug/TCPIPStack/AutoIP.o \
  build/XC16_dsPIC33EP512MU810/debug/TCPIPStack/BerkeleyAPI.o \
  build/XC16_dsPIC33EP512MU810/debug/TCPIPStack/BigInt.o \
  build/XC16_dsPIC33EP512MU810/debug/TCPIPStack/Delay.o \
  build/XC16_dsPIC33EP512MU810/debug/TCPIPStack/DHCP.o \
  build/XC16_dsPIC33EP512MU810/debug/TCPIPStack/DHCPs.o \
  build/XC16_dsPIC33EP512MU810/debug/TCPIPStack/DNS.o \
  build/XC16_dsPIC33EP512MU810/debug/TCPIPStack/DNSs.o \
  build/XC16_dsPIC33EP512MU810/debug/TCPIPStack/DynDNS.o \
  build/XC16_dsPIC33EP512MU810/debug/TCPIPStack/ENC28J60.o \
  build/XC16_dsPIC33EP512MU810/debug/TCPIPStack/FileSystem.o \
  build/XC16_dsPIC33EP512MU810/debug/TCPIPStack/FTP.o \
  build/XC16_dsPIC33EP512MU810/debug/TCPIPStack/Hashes.o \
  build/XC16_dsPIC33EP512MU810/debug/TCPIPStack/Helpers.o \
  build/XC16_dsPIC33EP512MU810/debug/TCPIPStack/HTTP2.o \
  build/XC16_dsPIC33EP512MU810/debug/TCPIPStack/ICMP.o \
  build/XC16_dsPIC33EP512MU810/debug/TCPIPStack/IP.o \
  build/XC16_dsPIC33EP512MU810/debug/TCPIPStack/LCDBlocking.o \
  build/XC16_dsPIC33EP512MU810/debug/TCPIPStack/MPFS2.o \
  build/XC16_dsPIC33EP512MU810/debug/TCPIPStack/NBNS.o \
  build/XC16_dsPIC33EP512MU810/debug/TCPIPStack/Random.o \
  build/XC16_dsPIC33EP512MU810/debug/TCPIPStack/Reboot.o \
  build/XC16_dsPIC33EP512MU810/debug/TCPIPStack/RSA.o \
  build/XC16_dsPIC33EP512MU810/debug/TCPIPStack/SMTP.o \
  build/XC16_dsPIC33EP512MU810/debug/TCPIPStack/SNMP.o \
  build/XC16_dsPIC33EP512MU810/debug/TCPIPStack/SNMPv3.o \
  build/XC16_dsPIC33EP512MU810/debug/TCPIPStack/SNMPv3USM.o \
  build/XC16_dsPIC33EP512MU810/debug/TCPIPStack/SNTP.o \
  build/XC16_dsPIC33EP512MU810/debug/TCPIPStack/SPIEEPROM.o \
  build/XC16_dsPIC33EP512MU810/debug/TCPIPStack/SPIFlash.o \
  build/XC16_dsPIC33EP512MU810/debug/TCPIPStack/SPIRAM.o \
  build/XC16_dsPIC33EP512MU810/debug/TCPIPStack/SSL.o \
  build/XC16_dsPIC33EP512MU810/debug/TCPIPStack/StackTsk.o \
  build/XC16_dsPIC33EP512MU810/debug/TCPIPStack/TCP.o \
  build/XC16_dsPIC33EP512MU810/debug/TCPIPStack/TCPPerformanceTest.o \
  build/XC16_dsPIC33EP512MU810/debug/TCPIPStack/Telnet.o \
  build/XC16_dsPIC33EP512MU810/debug/TCPIPStack/TFTPc.o \
  build/XC16_dsPIC33EP512MU810/debug/TCPIPStack/Tick.o \
  build/XC16_dsPIC33EP512MU810/debug/TCPIPStack/UART.o \
  build/XC16_dsPIC33EP512MU810/debug/TCPIPStack/UART2TCPBridge.o \
  build/XC16_dsPIC33EP512MU810/debug/TCPIPStack/UDP.o \
  build/XC16_dsPIC33EP512MU810/debug/TCPIPStack/UDPPerformanceTest.o \
  build/XC16_dsPIC33EP512MU810/debug/TCPIPStack/ZeroconfHelper.o \
  build/XC16_dsPIC33EP512MU810/debug/TCPIPStack/ZeroconfLinkLocal.o \
  build/XC16_dsPIC33EP512MU810/debug/TCPIPStack/ZeroconfMulticastDNS.o \
  build/XC16_dsPIC33EP512MU810/debug/usb/src/usb_device.o \
  build/XC16_dsPIC33EP512MU810/debug/usb/src/usb_device_cdc.o \
  build/XC16_dsPIC33EP512MU810/debug/usb/src/usb_hal_dspic33e.o \
  build/XC16_dsPIC33EP512MU810/debug/configuration_bits.o \
  build/XC16_dsPIC33EP512MU810/debug/interrupts.o \
  build/XC16_dsPIC33EP512MU810/debug/main.o \
  build/XC16_dsPIC33EP512MU810/debug/system.o \
  build/XC16_dsPIC33EP512MU810/debug/traps.o \
  build/XC16_dsPIC33EP512MU810/debug/user.o \
  build/XC16_dsPIC33EP512MU810/debug/MPFSImg2.o \
  build/XC16_dsPIC33EP512MU810/debug/CustomHTTPApp.o \
  build/XC16_dsPIC33EP512MU810/debug/AD7190.o \
  build/XC16_dsPIC33EP512MU810/debug/ADComm.o \
  build/XC16_dsPIC33EP512MU810/debug/UARTsComm.o \
  build/XC16_dsPIC33EP512MU810/debug/MemFlash.o \
  build/XC16_dsPIC33EP512MU810/debug/ADC10bitsDrv.o \
  build/XC16_dsPIC33EP512MU810/debug/SPIFRAM.o \
  build/XC16_dsPIC33EP512MU810/debug/usb_descriptors.o \
  build/XC16_dsPIC33EP512MU810/debug/ModbusUartServer.o \
  -TC:\Users\David_2\AppData\Local\Temp\tmp000015dc.00 \
  -TC:\Users\David_2\AppData\Local\Temp\tmp000015dc.01 \
  -TC:\Users\David_2\AppData\Local\Temp\tmp000015dc.02 \
  -TC:\Users\David_2\AppData\Local\Temp\tmp000015dc.03 \
  -TC:\Users\David_2\AppData\Local\Temp\tmp000015dc.04 \
  -TC:\Users\David_2\AppData\Local\Temp\tmp000015dc.05 \
  -TC:\Users\David_2\AppData\Local\Temp\tmp000015dc.06 \
  --local-stack \
  --defsym=__MPLAB_BUILD=1 \
  --defsym=__MPLAB_DEBUG=1 \
  --defsym=__DEBUG=1 \
  --defsym=__MPLAB_DEBUGGER_PK3=1 \
  -Tp33EP512MU810.gld.07 \
  --stack=16 \
  --check-sections \
  --data-init \
  --pack-data \
  --handles \
  --isr \
  --no-gc-sections \
  --fill-upper=0 \
  --stackguard=16 \
  --no-force-link \
  --smart-io \
  -Map=dist/XC16_dsPIC33EP512MU810/debug/PLCD_P01V45.debug.map \
  --report-mem \
  -start-group \
  --library=pic30-elf \
  --library=m-elf \
  --library=c-elf \
  -end-group \

Archive member included because of file (symbol)

c:/program files (x86)/microchip/xc16/v1.24/bin/bin/../../lib/dsPIC33E\libp33EP512MU810-elf.a(CloseSPI1.o)
                              build/XC16_dsPIC33EP512MU810/debug/ADComm.o (_CloseSPI1)
c:/program files (x86)/microchip/xc16/v1.24/bin/bin/../../lib/dsPIC33E\libp33EP512MU810-elf.a(CloseSPI3.o)
                              build/XC16_dsPIC33EP512MU810/debug/B40/abcc_sys_adapt.o (_CloseSPI3)
c:/program files (x86)/microchip/xc16/v1.24/bin/bin/../../lib/dsPIC33E\libp33EP512MU810-elf.a(DataRdySPI1.o)
                              build/XC16_dsPIC33EP512MU810/debug/ADComm.o (_DataRdySPI1)
c:/program files (x86)/microchip/xc16/v1.24/bin/bin/../../lib/dsPIC33E\libp33EP512MU810-elf.a(DataRdySPI3.o)
                              build/XC16_dsPIC33EP512MU810/debug/B40/abcc_sys_adapt.o (_DataRdySPI3)
c:/program files (x86)/microchip/xc16/v1.24/bin/bin/../../lib/dsPIC33E\libp33EP512MU810-elf.a(OpenSPI1.o)
                              build/XC16_dsPIC33EP512MU810/debug/ADComm.o (_OpenSPI1)
c:/program files (x86)/microchip/xc16/v1.24/bin/bin/../../lib/dsPIC33E\libp33EP512MU810-elf.a(OpenSPI3.o)
                              build/XC16_dsPIC33EP512MU810/debug/B40/abcc_sys_adapt.o (_OpenSPI3)
c:/program files (x86)/microchip/xc16/v1.24/bin/bin/../../lib/dsPIC33E\libp33EP512MU810-elf.a(ReadSPI1.o)
                              build/XC16_dsPIC33EP512MU810/debug/ADComm.o (_ReadSPI1)
c:/program files (x86)/microchip/xc16/v1.24/bin/bin/../../lib/dsPIC33E\libp33EP512MU810-elf.a(ReadSPI3.o)
                              build/XC16_dsPIC33EP512MU810/debug/B40/abcc_sys_adapt.o (_ReadSPI3)
c:/program files (x86)/microchip/xc16/v1.24/bin/bin/../../lib/dsPIC33E\libp33EP512MU810-elf.a(WriteSPI1.o)
                              build/XC16_dsPIC33EP512MU810/debug/ADComm.o (_WriteSPI1)
c:/program files (x86)/microchip/xc16/v1.24/bin/bin/../../lib/dsPIC33E\libp33EP512MU810-elf.a(WriteSPI3.o)
                              build/XC16_dsPIC33EP512MU810/debug/B40/abcc_sys_adapt.o (_WriteSPI3)
c:/program files (x86)/microchip/xc16/v1.24/bin/bin/../../lib/dsPIC33E\libp33EP512MU810-elf.a(BusyUART2.o)
                              build/XC16_dsPIC33EP512MU810/debug/main.o (_BusyUART2)
c:/program files (x86)/microchip/xc16/v1.24/bin/bin/../../lib/dsPIC33E\libp33EP512MU810-elf.a(BusyUART3.o)
                              build/XC16_dsPIC33EP512MU810/debug/Process.o (_BusyUART3)
c:/program files (x86)/microchip/xc16/v1.24/bin/bin/../../lib/dsPIC33E\libp33EP512MU810-elf.a(BusyUART4.o)
                              build/XC16_dsPIC33EP512MU810/debug/Process.o (_BusyUART4)
c:/program files (x86)/microchip/xc16/v1.24/bin/bin/../../lib/dsPIC33E\libp33EP512MU810-elf.a(CloseUART1.o)
                              build/XC16_dsPIC33EP512MU810/debug/UARTsComm.o (_CloseUART1)
c:/program files (x86)/microchip/xc16/v1.24/bin/bin/../../lib/dsPIC33E\libp33EP512MU810-elf.a(CloseUART2.o)
                              build/XC16_dsPIC33EP512MU810/debug/UARTsComm.o (_CloseUART2)
c:/program files (x86)/microchip/xc16/v1.24/bin/bin/../../lib/dsPIC33E\libp33EP512MU810-elf.a(CloseUART3.o)
                              build/XC16_dsPIC33EP512MU810/debug/UARTsComm.o (_CloseUART3)
c:/program files (x86)/microchip/xc16/v1.24/bin/bin/../../lib/dsPIC33E\libp33EP512MU810-elf.a(CloseUART4.o)
                              build/XC16_dsPIC33EP512MU810/debug/UARTsComm.o (_CloseUART4)
c:/program files (x86)/microchip/xc16/v1.24/bin/bin/../../lib/dsPIC33E\libp33EP512MU810-elf.a(ConfigIntUART1.o)
                              build/XC16_dsPIC33EP512MU810/debug/UARTsComm.o (_ConfigIntUART1)
c:/program files (x86)/microchip/xc16/v1.24/bin/bin/../../lib/dsPIC33E\libp33EP512MU810-elf.a(ConfigIntUART2.o)
                              build/XC16_dsPIC33EP512MU810/debug/UARTsComm.o (_ConfigIntUART2)
c:/program files (x86)/microchip/xc16/v1.24/bin/bin/../../lib/dsPIC33E\libp33EP512MU810-elf.a(ConfigIntUART3.o)
                              build/XC16_dsPIC33EP512MU810/debug/UARTsComm.o (_ConfigIntUART3)
c:/program files (x86)/microchip/xc16/v1.24/bin/bin/../../lib/dsPIC33E\libp33EP512MU810-elf.a(ConfigIntUART4.o)
                              build/XC16_dsPIC33EP512MU810/debug/UARTsComm.o (_ConfigIntUART4)
c:/program files (x86)/microchip/xc16/v1.24/bin/bin/../../lib/dsPIC33E\libp33EP512MU810-elf.a(DataRdyUART1.o)
                              build/XC16_dsPIC33EP512MU810/debug/interrupts.o (_DataRdyUART1)
c:/program files (x86)/microchip/xc16/v1.24/bin/bin/../../lib/dsPIC33E\libp33EP512MU810-elf.a(DataRdyUART2.o)
                              build/XC16_dsPIC33EP512MU810/debug/interrupts.o (_DataRdyUART2)
c:/program files (x86)/microchip/xc16/v1.24/bin/bin/../../lib/dsPIC33E\libp33EP512MU810-elf.a(DataRdyUART3.o)
                              build/XC16_dsPIC33EP512MU810/debug/interrupts.o (_DataRdyUART3)
c:/program files (x86)/microchip/xc16/v1.24/bin/bin/../../lib/dsPIC33E\libp33EP512MU810-elf.a(DataRdyUART4.o)
                              build/XC16_dsPIC33EP512MU810/debug/interrupts.o (_DataRdyUART4)
c:/program files (x86)/microchip/xc16/v1.24/bin/bin/../../lib/dsPIC33E\libp33EP512MU810-elf.a(OpenUART1.o)
                              build/XC16_dsPIC33EP512MU810/debug/UARTsComm.o (_OpenUART1)
c:/program files (x86)/microchip/xc16/v1.24/bin/bin/../../lib/dsPIC33E\libp33EP512MU810-elf.a(OpenUART2.o)
                              build/XC16_dsPIC33EP512MU810/debug/UARTsComm.o (_OpenUART2)
c:/program files (x86)/microchip/xc16/v1.24/bin/bin/../../lib/dsPIC33E\libp33EP512MU810-elf.a(OpenUART3.o)
                              build/XC16_dsPIC33EP512MU810/debug/UARTsComm.o (_OpenUART3)
c:/program files (x86)/microchip/xc16/v1.24/bin/bin/../../lib/dsPIC33E\libp33EP512MU810-elf.a(OpenUART4.o)
                              build/XC16_dsPIC33EP512MU810/debug/UARTsComm.o (_OpenUART4)
c:/program files (x86)/microchip/xc16/v1.24/bin/bin/../../lib/dsPIC33E\libp33EP512MU810-elf.a(putsUART1.o)
                              build/XC16_dsPIC33EP512MU810/debug/Process.o (_putsUART1)
c:/program files (x86)/microchip/xc16/v1.24/bin/bin/../../lib/dsPIC33E\libp33EP512MU810-elf.a(putsUART2.o)
                              build/XC16_dsPIC33EP512MU810/debug/Process.o (_putsUART2)
c:/program files (x86)/microchip/xc16/v1.24/bin/bin/../../lib/dsPIC33E\libp33EP512MU810-elf.a(putsUART3.o)
                              build/XC16_dsPIC33EP512MU810/debug/main.o (_putsUART3)
c:/program files (x86)/microchip/xc16/v1.24/bin/bin/../../lib/dsPIC33E\libp33EP512MU810-elf.a(putsUART4.o)
                              build/XC16_dsPIC33EP512MU810/debug/main.o (_putsUART4)
c:/program files (x86)/microchip/xc16/v1.24/bin/bin/../../lib/dsPIC33E\libp33EP512MU810-elf.a(ReadUART1.o)
                              build/XC16_dsPIC33EP512MU810/debug/interrupts.o (_ReadUART1)
c:/program files (x86)/microchip/xc16/v1.24/bin/bin/../../lib/dsPIC33E\libp33EP512MU810-elf.a(ReadUART2.o)
                              build/XC16_dsPIC33EP512MU810/debug/interrupts.o (_ReadUART2)
c:/program files (x86)/microchip/xc16/v1.24/bin/bin/../../lib/dsPIC33E\libp33EP512MU810-elf.a(ReadUART3.o)
                              build/XC16_dsPIC33EP512MU810/debug/interrupts.o (_ReadUART3)
c:/program files (x86)/microchip/xc16/v1.24/bin/bin/../../lib/dsPIC33E\libp33EP512MU810-elf.a(ReadUART4.o)
                              build/XC16_dsPIC33EP512MU810/debug/interrupts.o (_ReadUART4)
c:/program files (x86)/microchip/xc16/v1.24/bin/bin/../../lib\libpic30-elf.a(crt0_extendedep.o)
                              (__resetPRI)
c:/program files (x86)/microchip/xc16/v1.24/bin/bin/../../lib\libpic30-elf.a(data_init_extendedep.o)
                              c:/program files (x86)/microchip/xc16/v1.24/bin/bin/../../lib\libpic30-elf.a(crt0_extendedep.o) (__data_init_extended)
c:/program files (x86)/microchip/xc16/v1.24/bin/bin/../../lib\libm-elf.a(addsf3.epeo)
                              build/XC16_dsPIC33EP512MU810/debug/Regul.o (___subsf3)
c:/program files (x86)/microchip/xc16/v1.24/bin/bin/../../lib\libm-elf.a(divsf3.epeo)
                              build/XC16_dsPIC33EP512MU810/debug/Regul.o (___divsf3)
c:/program files (x86)/microchip/xc16/v1.24/bin/bin/../../lib\libm-elf.a(divsi3.epeo)
                              build/XC16_dsPIC33EP512MU810/debug/Pesage.o (___divsi3)
c:/program files (x86)/microchip/xc16/v1.24/bin/bin/../../lib\libm-elf.a(feqltle.epeo)
                              build/XC16_dsPIC33EP512MU810/debug/Pesage.o (___eqsf2)
c:/program files (x86)/microchip/xc16/v1.24/bin/bin/../../lib\libm-elf.a(fgtge.epeo)
                              build/XC16_dsPIC33EP512MU810/debug/B40/ad_obj.o (___gtsf2)
c:/program files (x86)/microchip/xc16/v1.24/bin/bin/../../lib\libm-elf.a(fixsfsi.epeo)
                              build/XC16_dsPIC33EP512MU810/debug/Regul.o (_(float, int, long long, short, float, short, int))
c:/program files (x86)/microchip/xc16/v1.24/bin/bin/../../lib\libm-elf.a(fixunssfsi.epeo)
                              build/XC16_dsPIC33EP512MU810/debug/Regul.o (___fixunssfsi)
c:/program files (x86)/microchip/xc16/v1.24/bin/bin/../../lib\libm-elf.a(floatsisf.epeo)
                              build/XC16_dsPIC33EP512MU810/debug/Pesage.o (___floatsisf)
c:/program files (x86)/microchip/xc16/v1.24/bin/bin/../../lib\libm-elf.a(floatunsisf.epeo)
                              build/XC16_dsPIC33EP512MU810/debug/Regul.o (___floatunsisf)
c:/program files (x86)/microchip/xc16/v1.24/bin/bin/../../lib\libm-elf.a(fpack.epeo)
                              c:/program files (x86)/microchip/xc16/v1.24/bin/bin/../../lib\libm-elf.a(addsf3.epeo) (__fpack)
c:/program files (x86)/microchip/xc16/v1.24/bin/bin/../../lib\libm-elf.a(funpack.epeo)
                              c:/program files (x86)/microchip/xc16/v1.24/bin/bin/../../lib\libm-elf.a(fixsfsi.epeo) (__funpack)
c:/program files (x86)/microchip/xc16/v1.24/bin/bin/../../lib\libm-elf.a(funpack2.epeo)
                              c:/program files (x86)/microchip/xc16/v1.24/bin/bin/../../lib\libm-elf.a(addsf3.epeo) (__funpack2)
c:/program files (x86)/microchip/xc16/v1.24/bin/bin/../../lib\libm-elf.a(futil.epeo)
                              c:/program files (x86)/microchip/xc16/v1.24/bin/bin/../../lib\libm-elf.a(addsf3.epeo) (__fPropagateNaN)
c:/program files (x86)/microchip/xc16/v1.24/bin/bin/../../lib\libm-elf.a(mulsf3.epeo)
                              build/XC16_dsPIC33EP512MU810/debug/Regul.o (___mulsf3)
c:/program files (x86)/microchip/xc16/v1.24/bin/bin/../../lib\libm-elf.a(udivsi3.epeo)
                              build/XC16_dsPIC33EP512MU810/debug/TCPIPStack/MPFS2.o (___udivsi3)
c:/program files (x86)/microchip/xc16/v1.24/bin/bin/../../lib\libm-elf.a(umodsi3.epeo)
                              build/XC16_dsPIC33EP512MU810/debug/ModbusUartServer.o (___umodsi3)
c:/program files (x86)/microchip/xc16/v1.24/bin/bin/../../lib\libm-elf.a(fcompare.epeo)
                              c:/program files (x86)/microchip/xc16/v1.24/bin/bin/../../lib\libm-elf.a(feqltle.epeo) (__fcompare)
c:/program files (x86)/microchip/xc16/v1.24/bin/bin/../../lib\libm-elf.a(floatdisf.epeo)
                              c:/program files (x86)/microchip/xc16/v1.24/bin/bin/../../lib\libm-elf.a(floatsisf.epeo) (___floatdisf)
c:/program files (x86)/microchip/xc16/v1.24/bin/bin/../../lib\libm-elf.a(floatundisf.epeo)
                              c:/program files (x86)/microchip/xc16/v1.24/bin/bin/../../lib\libm-elf.a(floatunsisf.epeo) (___floatundisf)
c:/program files (x86)/microchip/xc16/v1.24/bin/bin/../../lib\libc-elf.a(atof.epeo)
                              build/XC16_dsPIC33EP512MU810/debug/ModbusUartServer.o (_atof)
c:/program files (x86)/microchip/xc16/v1.24/bin/bin/../../lib\libc-elf.a(atoi.epeo)
                              build/XC16_dsPIC33EP512MU810/debug/user.o (_atoi)
c:/program files (x86)/microchip/xc16/v1.24/bin/bin/../../lib\libc-elf.a(atol.epeo)
                              build/XC16_dsPIC33EP512MU810/debug/TCPIPStack/HTTP2.o (_atol)
c:/program files (x86)/microchip/xc16/v1.24/bin/bin/../../lib\libc-elf.a(errno.epeo)
                              c:/program files (x86)/microchip/xc16/v1.24/bin/bin/../../lib\libc-elf.a(atof.epeo) (_errno)
c:/program files (x86)/microchip/xc16/v1.24/bin/bin/../../lib\libc-elf.a(ltoa.epeo)
                              build/XC16_dsPIC33EP512MU810/debug/ModbusUartServer.o (_ltoa)
c:/program files (x86)/microchip/xc16/v1.24/bin/bin/../../lib\libc-elf.a(memcmp.epeo)
                              build/XC16_dsPIC33EP512MU810/debug/TCPIPStack/HTTP2.o (_memcmp)
c:/program files (x86)/microchip/xc16/v1.24/bin/bin/../../lib\libc-elf.a(memcpy.epeo)
                              build/XC16_dsPIC33EP512MU810/debug/B40/spi/abcc_spi_drv.o (_memcpy)
c:/program files (x86)/microchip/xc16/v1.24/bin/bin/../../lib\libc-elf.a(memset.epeo)
                              build/XC16_dsPIC33EP512MU810/debug/BerkeleyUDPClient.o (_memset)
c:/program files (x86)/microchip/xc16/v1.24/bin/bin/../../lib\libc-elf.a(rand.epeo)
                              build/XC16_dsPIC33EP512MU810/debug/ModbusUartServer.o (_srand)
c:/program files (x86)/microchip/xc16/v1.24/bin/bin/../../lib\libc-elf.a(sprintf.epeo)
                              build/XC16_dsPIC33EP512MU810/debug/Process.o (_sprintf)
c:/program files (x86)/microchip/xc16/v1.24/bin/bin/../../lib\libc-elf.a(strcmp.epeo)
                              build/XC16_dsPIC33EP512MU810/debug/TCPIPStack/HTTP2.o (_strcmp)
c:/program files (x86)/microchip/xc16/v1.24/bin/bin/../../lib\libc-elf.a(strcpy.epeo)
                              build/XC16_dsPIC33EP512MU810/debug/user.o (_strcpy)
c:/program files (x86)/microchip/xc16/v1.24/bin/bin/../../lib\libc-elf.a(strlen.epeo)
                              build/XC16_dsPIC33EP512MU810/debug/B40/ad_obj.o (_strlen)
c:/program files (x86)/microchip/xc16/v1.24/bin/bin/../../lib\libc-elf.a(strncpy.epeo)
                              build/XC16_dsPIC33EP512MU810/debug/TCPIPStack/Helpers.o (_strncpy)
c:/program files (x86)/microchip/xc16/v1.24/bin/bin/../../lib\libc-elf.a(strtok.epeo)
                              build/XC16_dsPIC33EP512MU810/debug/user.o (_strtok)
c:/program files (x86)/microchip/xc16/v1.24/bin/bin/../../lib\libc-elf.a(putchar.epeo)
                              build/XC16_dsPIC33EP512MU810/debug/B40/spi/abcc_handler_spi.o (_putchar)
c:/program files (x86)/microchip/xc16/v1.24/bin/bin/../../lib\libc-elf.a(_iob.epeo)
                              c:/program files (x86)/microchip/xc16/v1.24/bin/bin/../../lib\libc-elf.a(putchar.epeo) (__iob)
c:/program files (x86)/microchip/xc16/v1.24/bin/bin/../../lib\libc-elf.a(sprintf_cdnopuxX.EPeo)
                              build/XC16_dsPIC33EP512MU810/debug/AD7190.o (__sprintf_cdnopuxX)
c:/program files (x86)/microchip/xc16/v1.24/bin/bin/../../lib\libc-elf.a(doprnt_cdnopuxX.EPeo)
                              c:/program files (x86)/microchip/xc16/v1.24/bin/bin/../../lib\libc-elf.a(sprintf_cdnopuxX.EPeo) (__vfprintf_cdnopuxX)
c:/program files (x86)/microchip/xc16/v1.24/bin/bin/../../lib\libc-elf.a(printf_cdnopuxX.EPeo)
                              build/XC16_dsPIC33EP512MU810/debug/B40/spi/abcc_spi_drv.o (__printf_cdnopuxX)
c:/program files (x86)/microchip/xc16/v1.24/bin/bin/../../lib\libc-elf.a(sprintf_cdfFnopuxX.EPeo)
                              build/XC16_dsPIC33EP512MU810/debug/Process.o (__sprintf_cdfFnopuxX)
c:/program files (x86)/microchip/xc16/v1.24/bin/bin/../../lib\libc-elf.a(doprnt_cdfFnopuxX.EPeo)
                              c:/program files (x86)/microchip/xc16/v1.24/bin/bin/../../lib\libc-elf.a(sprintf_cdfFnopuxX.EPeo) (__vfprintf_cdfFnopuxX)
c:/program files (x86)/microchip/xc16/v1.24/bin/bin/../../lib\libc-elf.a(sprintf_cdfFnopsuxX.EPeo)
                              (__sprintf_cdfFnopsuxX)
c:/program files (x86)/microchip/xc16/v1.24/bin/bin/../../lib\libc-elf.a(doprnt_cdfFnopsuxX.EPeo)
                              c:/program files (x86)/microchip/xc16/v1.24/bin/bin/../../lib\libc-elf.a(sprintf_cdfFnopsuxX.EPeo) (__vfprintf_cdfFnopsuxX)
c:/program files (x86)/microchip/xc16/v1.24/bin/bin/../../lib\libc-elf.a(sprintf_cdnopsuxX.EPeo)
                              build/XC16_dsPIC33EP512MU810/debug/user.o (__sprintf_cdnopsuxX)
c:/program files (x86)/microchip/xc16/v1.24/bin/bin/../../lib\libc-elf.a(doprnt_cdnopsuxX.EPeo)
                              c:/program files (x86)/microchip/xc16/v1.24/bin/bin/../../lib\libc-elf.a(sprintf_cdnopsuxX.EPeo) (__vfprintf_cdnopsuxX)
c:/program files (x86)/microchip/xc16/v1.24/bin/bin/../../lib\libc-elf.a(printf_cdnopsuxX.EPeo)
                              build/XC16_dsPIC33EP512MU810/debug/B40/abcc_cbf.o (__printf_cdnopsuxX)
c:/program files (x86)/microchip/xc16/v1.24/bin/bin/../../lib\libc-elf.a(printf_s.EPeo)
                              build/XC16_dsPIC33EP512MU810/debug/B40/spi/abcc_handler_spi.o (__printf_0)
c:/program files (x86)/microchip/xc16/v1.24/bin/bin/../../lib\libc-elf.a(isspace.epeso)
                              c:/program files (x86)/microchip/xc16/v1.24/bin/bin/../../lib\libc-elf.a(atof.epeo) (_isspace)
c:/program files (x86)/microchip/xc16/v1.24/bin/bin/../../lib\libc-elf.a(doprnt.epeo)
                              c:/program files (x86)/microchip/xc16/v1.24/bin/bin/../../lib\libc-elf.a(sprintf.epeo) (_vfprintf)
c:/program files (x86)/microchip/xc16/v1.24/bin/bin/../../lib\libc-elf.a(fputc.epeo)
                              c:/program files (x86)/microchip/xc16/v1.24/bin/bin/../../lib\libc-elf.a(putchar.epeo) (_fputc)
c:/program files (x86)/microchip/xc16/v1.24/bin/bin/../../lib\libc-elf.a(powers.epeo)
                              c:/program files (x86)/microchip/xc16/v1.24/bin/bin/../../lib\libc-elf.a(doprnt_cdfFnopuxX.EPeo) (__powers_)
c:/program files (x86)/microchip/xc16/v1.24/bin/bin/../../lib\libc-elf.a(strcspn.epeo)
                              c:/program files (x86)/microchip/xc16/v1.24/bin/bin/../../lib\libc-elf.a(strtok.epeo) (_strcspn)
c:/program files (x86)/microchip/xc16/v1.24/bin/bin/../../lib\libc-elf.a(strspn.epeo)
                              c:/program files (x86)/microchip/xc16/v1.24/bin/bin/../../lib\libc-elf.a(strtok.epeo) (_strspn)
c:/program files (x86)/microchip/xc16/v1.24/bin/bin/../../lib\libc-elf.a(strchr.epelo)
                              c:/program files (x86)/microchip/xc16/v1.24/bin/bin/../../lib\libc-elf.a(strcspn.epeo) (_strchr)
c:/program files (x86)/microchip/xc16/v1.24/bin/bin/../../lib\libc-elf.a(doprnt_s.EPeo)
                              c:/program files (x86)/microchip/xc16/v1.24/bin/bin/../../lib\libc-elf.a(printf_s.EPeo) (__vfprintf_s)
c:/program files (x86)/microchip/xc16/v1.24/bin/bin/../../lib\libc-elf.a(flsbuf.epeo)
                              c:/program files (x86)/microchip/xc16/v1.24/bin/bin/../../lib\libc-elf.a(fputc.epeo) (__flsbuf)
c:/program files (x86)/microchip/xc16/v1.24/bin/bin/../../lib\libpic30-elf.a(writeep.eo)
                              c:/program files (x86)/microchip/xc16/v1.24/bin/bin/../../lib\libc-elf.a(fputc.epeo) (_write)
c:/program files (x86)/microchip/xc16/v1.24/bin/bin/../../lib\libm-elf.a(adddf3.epeo)
                              c:/program files (x86)/microchip/xc16/v1.24/bin/bin/../../lib\libc-elf.a(doprnt_cdfFnopuxX.EPeo) (___adddf3)
c:/program files (x86)/microchip/xc16/v1.24/bin/bin/../../lib\libm-elf.a(deqltle.epeo)
                              c:/program files (x86)/microchip/xc16/v1.24/bin/bin/../../lib\libc-elf.a(doprnt_cdfFnopuxX.EPeo) (___ltdf2)
c:/program files (x86)/microchip/xc16/v1.24/bin/bin/../../lib\libm-elf.a(dgtge.epeo)
                              c:/program files (x86)/microchip/xc16/v1.24/bin/bin/../../lib\libc-elf.a(doprnt_cdfFnopuxX.EPeo) (___gedf2)
c:/program files (x86)/microchip/xc16/v1.24/bin/bin/../../lib\libm-elf.a(divdf3.epeo)
                              c:/program files (x86)/microchip/xc16/v1.24/bin/bin/../../lib\libc-elf.a(doprnt_cdfFnopuxX.EPeo) (___divdf3)
c:/program files (x86)/microchip/xc16/v1.24/bin/bin/../../lib\libm-elf.a(dne.epeo)
                              c:/program files (x86)/microchip/xc16/v1.24/bin/bin/../../lib\libc-elf.a(doprnt_cdfFnopuxX.EPeo) (___nedf2)
c:/program files (x86)/microchip/xc16/v1.24/bin/bin/../../lib\libm-elf.a(dpack.epeo)
                              c:/program files (x86)/microchip/xc16/v1.24/bin/bin/../../lib\libm-elf.a(adddf3.epeo) (__dpack)
c:/program files (x86)/microchip/xc16/v1.24/bin/bin/../../lib\libm-elf.a(dunpack2.epeo)
                              c:/program files (x86)/microchip/xc16/v1.24/bin/bin/../../lib\libm-elf.a(adddf3.epeo) (__dunpack2)
c:/program files (x86)/microchip/xc16/v1.24/bin/bin/../../lib\libm-elf.a(extendsfdf.epeo)
                              c:/program files (x86)/microchip/xc16/v1.24/bin/bin/../../lib\libc-elf.a(doprnt_cdfFnopuxX.EPeo) (___extendsfdf2)
c:/program files (x86)/microchip/xc16/v1.24/bin/bin/../../lib\libm-elf.a(fixunsdfdi.epeo)
                              c:/program files (x86)/microchip/xc16/v1.24/bin/bin/../../lib\libc-elf.a(doprnt_cdfFnopuxX.EPeo) (___fixunsdfdi)
c:/program files (x86)/microchip/xc16/v1.24/bin/bin/../../lib\libm-elf.a(fixunsdfsi.epeo)
                              c:/program files (x86)/microchip/xc16/v1.24/bin/bin/../../lib\libc-elf.a(doprnt.epeo) (___fixunsdfsi)
c:/program files (x86)/microchip/xc16/v1.24/bin/bin/../../lib\libm-elf.a(floatundidf.epeo)
                              c:/program files (x86)/microchip/xc16/v1.24/bin/bin/../../lib\libc-elf.a(doprnt_cdfFnopuxX.EPeo) (___floatundidf)
c:/program files (x86)/microchip/xc16/v1.24/bin/bin/../../lib\libm-elf.a(floatunsidf.epeo)
                              c:/program files (x86)/microchip/xc16/v1.24/bin/bin/../../lib\libc-elf.a(doprnt.epeo) (___floatunsidf)
c:/program files (x86)/microchip/xc16/v1.24/bin/bin/../../lib\libm-elf.a(frexp.epeo)
                              c:/program files (x86)/microchip/xc16/v1.24/bin/bin/../../lib\libc-elf.a(doprnt_cdfFnopuxX.EPeo) (_frexpl)
c:/program files (x86)/microchip/xc16/v1.24/bin/bin/../../lib\libm-elf.a(muldf3.epeo)
                              c:/program files (x86)/microchip/xc16/v1.24/bin/bin/../../lib\libc-elf.a(doprnt_cdfFnopuxX.EPeo) (___muldf3)
c:/program files (x86)/microchip/xc16/v1.24/bin/bin/../../lib\libm-elf.a(subdf3.epeo)
                              c:/program files (x86)/microchip/xc16/v1.24/bin/bin/../../lib\libc-elf.a(doprnt_cdfFnopuxX.EPeo) (___subdf3)
c:/program files (x86)/microchip/xc16/v1.24/bin/bin/../../lib\libm-elf.a(mulsi3.epeo)
                              c:/program files (x86)/microchip/xc16/v1.24/bin/bin/../../lib\libc-elf.a(atof.epeo) (___mulsi3)
c:/program files (x86)/microchip/xc16/v1.24/bin/bin/../../lib\libm-elf.a(divmoddi3.epeo)
                              c:/program files (x86)/microchip/xc16/v1.24/bin/bin/../../lib\libc-elf.a(doprnt_cdnopuxX.EPeo) (___udivdi3)
c:/program files (x86)/microchip/xc16/v1.24/bin/bin/../../lib\libm-elf.a(muldi3.epeo)
                              c:/program files (x86)/microchip/xc16/v1.24/bin/bin/../../lib\libc-elf.a(doprnt_cdnopuxX.EPeo) (___muldi3)
c:/program files (x86)/microchip/xc16/v1.24/bin/bin/../../lib\libm-elf.a(dcompare.epeo)
                              c:/program files (x86)/microchip/xc16/v1.24/bin/bin/../../lib\libm-elf.a(deqltle.epeo) (__dcompare)
c:/program files (x86)/microchip/xc16/v1.24/bin/bin/../../lib\libm-elf.a(dpropagateNaN.epeo)
                              c:/program files (x86)/microchip/xc16/v1.24/bin/bin/../../lib\libm-elf.a(dunpack2.epeo) (__dPropagateNaN)
c:/program files (x86)/microchip/xc16/v1.24/bin/bin/../../lib\libm-elf.a(dtype.epeo)
                              c:/program files (x86)/microchip/xc16/v1.24/bin/bin/../../lib\libm-elf.a(dcompare.epeo) (__dtype)
c:/program files (x86)/microchip/xc16/v1.24/bin/bin/../../lib\libm-elf.a(dunpack.epeo)
                              c:/program files (x86)/microchip/xc16/v1.24/bin/bin/../../lib\libm-elf.a(dunpack2.epeo) (__dunpack)
c:/program files (x86)/microchip/xc16/v1.24/bin/bin/../../lib\libm-elf.a(umuldi3.epeo)
                              c:/program files (x86)/microchip/xc16/v1.24/bin/bin/../../lib\libm-elf.a(muldi3.epeo) (___umuldi3)


Program Memory  [Origin = 0x200, Length = 0x555fe]

section                    address   length (PC units)   length (bytes) (dec)
-------                    -------   -----------------   --------------------
.text                        0x200              0x3ee0          0x5e50  (24144)
.const                      0x40e0              0x16fe          0x227d  (8829)
.text                       0x57de              0x56ea          0x825f  (33375)
MPFSData                    0xaec8              0x51ea          0x7adf  (31455)
.text                      0x100b2             0x13658         0x1d184  (119172)
.dinit                     0x2370a               0x4fa           0x777  (1911)
.text                      0x23c04              0x4336          0x64d1  (25809)
MPFSHelpers                0x27f3a                 0xe            0x15  (21)

                     Total program memory used (bytes):        0x3bbec  (244716) 46%


Auxflash Memory  [Origin = 0x7fc000, Length = 0x3ff8]

section                    address   length (PC units)   length (bytes) (dec)
-------                    -------   -----------------   --------------------

                     Total auxflash memory used (bytes):              0  (0) <1%


Data Memory  [Origin = 0x1000, Length = 0xd000]

section                    address      alignment gaps    total length  (dec)
-------                    -------      --------------    -------------------
reserve_data_0x1000         0x1000                0x1c            0x1c  (28)
reserve_data_0x101c         0x101c                 0x2             0x2  (2)
reserve_data_0x101e         0x101e                 0x2             0x2  (2)
reserve_data_0x1020         0x1020                 0x2             0x2  (2)
reserve_data_0x1022         0x1022                 0x2             0x2  (2)
reserve_data_0x1024         0x1024                 0x4             0x4  (4)
reserve_data_0x1028         0x1028                0x28            0x28  (40)
.bss                        0x1050                   0          0x1ee4  (7908)
.data._powers_              0x2f34                   0            0xb0  (176)
.data._npowers_             0x2fe4                   0            0xb0  (176)
.bss                        0x3094                   0            0xac  (172)
.data.dpowers               0x3140                   0           0x140  (320)
.bss                        0x3280                   0            0xfc  (252)
.data                       0x337c                   0            0x70  (112)
.bss                        0x33ec                   0            0x14  (20)
_04C8D600560ab18f           0x3400                   0            0x60  (96)
.bss                        0x3460                   0           0x206  (518)
.bss                        0x3666                   0            0x6c  (108)
.data                       0x36d2                   0            0x66  (102)
.bss                        0x3738                   0            0x9a  (154)
.data                       0x37d2                   0            0x54  (84)
.bss                        0x3826                   0            0x24  (36)
.data._iob                  0x384a                   0            0x24  (36)
.bss                        0x386e                   0            0x5a  (90)
.bss                        0x38c8                   0            0x12  (18)
.data                       0x38da                   0            0x74  (116)
.bss                        0x394e                   0            0x90  (144)
.data                       0x39de                   0            0x10  (16)
.bss                        0x39ee                   0            0x28  (40)
.data                       0x3a16                   0             0x6  (6)
.bss                        0x3a1c                   0             0xc  (12)
_04DDDD20560ab18d           0x3a28                   0             0x6  (6)
.bss                        0x3a2e                   0             0xe  (14)
.data                       0x3a3c                   0             0x8  (8)
.bss                        0x3a44                   0             0xc  (12)
.data                       0x3a50                   0             0x4  (4)
.bss                        0x3a54                   0             0x8  (8)
.bss.randx                  0x3a5c                   0             0x4  (4)
.bss                        0x3a60                   0             0x2  (2)
.data                       0x3a62                   0             0x8  (8)
.pbss                       0x3a6a                   0             0x2  (2)
.data                       0x3a6c                   0             0x4  (4)
.pbss                       0x3a70                   0             0x2  (2)
.data                       0x3a72                   0             0x2  (2)
.pbss                       0x3a74                   0             0x2  (2)
.bss                        0x3a76                   0             0x4  (4)
.bss.errno                  0x3a7a                   0             0x2  (2)
.bss.randf                  0x3a7c                   0             0x2  (2)
.bss.sp.1310                0x3a7e                   0             0x2  (2)
.data._Files                0x3a80                   0             0x2  (2)
.bss._outdone               0x3a82                   0             0x2  (2)
.bss._sibuf                 0x3a84                   0             0x2  (2)
.bss._sobuf                 0x3a86                   0             0x2  (2)
_04697A20560ab195           0xd800                   0           0x210  (528)
_04793780560ab17d           0xdb00                   0             0xe  (14)
_04697840560ab195           0xdc00                   0           0x210  (528)
_047939C0560ab17d           0xdf00                   0            0x80  (128)

                        Total data memory used (bytes):         0x2f36  (12086) 22%


Dynamic Memory Usage

region                     address                      maximum length  (dec)
------                     -------                      ---------------------
heap                             0                                   0  (0)
stack                       0x3a88                              0x4578  (17784)

                        Maximum dynamic memory (bytes):         0x4578  (17784)


External Symbols in Data Memory (by address):

                    0x1050                  _U1Baudvalue
                    0x1052                  _U2Baudvalue
                    0x1054                  _U3Baudvalue
                    0x1056                  _U4Baudvalue
                    0x1058                  _U1MODEvalue
                    0x105a                  _U1STAvalue
                    0x105c                  _U2MODEvalue
                    0x105e                  _U2STAvalue
                    0x1060                  _U3MODEvalue
                    0x1062                  _U3STAvalue
                    0x1064                  _U4MODEvalue
                    0x1066                  _U4STAvalue
                    0x1068                  _TrameU1
                    0x126a                  _TrameU2
                    0x146c                  _TrameU3
                    0x166e                  _TrameU4
                    0x1870                  _PAR
                    0x1b38                  _EXP
                    0x1f4e                  _sorTOR
                    0x1f58                  _entTOR
                    0x1f62                  _Cav_USR1
                    0x1f64                  _Cav_CLR
                    0x1f66                  _T100
                    0x1fa2                  _T10
                    0x1fb6                  _AD7190_PoidsPret
                    0x1fb8                  _Compteur
                    0x1fba                  _NbTopTotal
                    0x1fbe                  _CompteurTot
                    0x1fc2                  _entreeTorVitesseMem
                    0x245c                  _link_bPool
                    0x28c8                  _MODBUS_COMMAND
                    0x28d4                  _WriteByteReverse
                    0x28d6                  _MODBUS_RX
                    0x2ad6                  _MODBUS_TX
                    0x2cd6                  _COIL
                    0x2cd8                  _COIL_REG
                    0x2e22                  _USB_In_Buffer
                    0x2e62                  _USB_Mess_head
                    0x2e64                  _USB_Mess
                    0x2f30                  _USB_list_count
                    0x2f34                  __powers_
                    0x2fe4                  __npowers_
                    0x3094                  _cdc_data_tx
                    0x30d4                  _cdc_data_rx
                    0x3114                  _line_coding
                    0x311c                  _cdc_notice
                    0x3126                  _cdc_rx_len
                    0x3127                  _cdc_trf_state
                    0x3128                  _pCDCSrc
                    0x312a                  _pCDCDst
                    0x312c                  _cdc_tx_len
                    0x312d                  _cdc_mem_type
                    0x312e                  _CDCDataOutHandle
                    0x3130                  _CDCDataInHandle
                    0x3132                  _control_signal_bitmap
                    0x3134                  _BaudRateGen
                    0x3138                  _dummy_encapsulated_cmd_response
                    0x3280                  _UDPSocketInfo
                    0x3370                  _activeUDPSocket
                    0x3372                  _UDPTxCount
                    0x3374                  _UDPRxCount
                    0x3400                  _BDT
                    0x3460                  _AD_asDefaultMap
                    0x3462                  _AD_asADIEntryList
                    0x35da                  _curHTTP
                    0x365c                  _httpStubs
                    0x3664                  _curHTTPID
                    0x36d2                  _ReadByteReverse
                    0x36d3                  _InputByteReverse
                    0x36d4                  _HOLDING_REG
                    0x3706                  _INPUT_REG
                    0x3738                  _fResetABCC
                    0x373a                  _ABCCPowerState
                    0x373c                  _address
                    0x3740                  _AppConfig
                    0x3788                  _USBDeviceState
                    0x378a                  _USBActiveConfiguration
                    0x378b                  _USBAlternateInterface
                    0x378e                  _pBDTEntryEP0OutCurrent
                    0x3790                  _pBDTEntryEP0OutNext
                    0x3792                  _pBDTEntryOut
                    0x3798                  _pBDTEntryIn
                    0x379e                  _shortPacketStatus
                    0x379f                  _controlTransferState
                    0x37a0                  _inPipes
                    0x37a6                  _outPipes
                    0x37ae                  _pDst
                    0x37b0                  _RemoteWakeup
                    0x37b1                  _USBBusIsSuspended
                    0x37b2                  _USTATcopy
                    0x37b3                  _endpoint_number
                    0x37b4                  _BothEP0OutUOWNsSet
                    0x37b5                  _ep_data_in
                    0x37b8                  _ep_data_out
                    0x37bb                  _USBStatusStageTimeoutCounter
                    0x37bc                  _USBDeferStatusStagePacket
                    0x37bd                  _USBStatusStageEnabledFlag1
                    0x37be                  _USBStatusStageEnabledFlag2
                    0x37bf                  _USBDeferINDataStagePackets
                    0x37c0                  _USBDeferOUTDataStagePackets
                    0x37c1                  _SetupPkt
                    0x37c9                  _CtrlTrfData
                    0x384a                  __iob
                    0x394e                  _ABCC_RunDriver
                    0x3950                  _ABCC_ISR
                    0x3952                  _pnABCC_DrvInit
                    0x3954                  _pnABCC_DrvISR
                    0x3956                  _pnABCC_DrvRunDriverTx
                    0x3958                  _pnABCC_DrvRunDriverRx
                    0x395a                  _pnABCC_DrvWriteMessage
                    0x395c                  _pnABCC_DrvWriteProcessData
                    0x395e                  _pnABCC_DrvISReadyForWrPd
                    0x3960                  _pnABCC_DrvISReadyForWriteMessage
                    0x3962                  _pnABCC_DrvISReadyForCmd
                    0x3964                  _pnABCC_DrvSetNbrOfCmds
                    0x3966                  _pnABCC_DrvSetAppStatus
                    0x3968                  _pnABCC_DrvSetPdSize
                    0x396a                  _pnABCC_DrvSetMsgReceiverBuffer
                    0x396c                  _pnABCC_DrvSetIntMask
                    0x396e                  _pnABCC_DrvGetWrPdBuffer
                    0x3970                  _pnABCC_DrvGetModCap
                    0x3972                  _pnABCC_DrvGetLedStatus
                    0x3974                  _pnABCC_DrvGetIntStatus
                    0x3976                  _pnABCC_DrvGetAnybusState
                    0x3978                  _pnABCC_DrvReadProcessData
                    0x397a                  _pnABCC_DrvReadMessage
                    0x397c                  _pnABCC_DrvIsSupervised
                    0x397e                  _pnABCC_DrvGetAnbStatus
                    0x398c                  _ADI_DebitInstan
                    0x3990                  _ADI_PoidsInstan
                    0x3994                  _ADI_PoidsMetre
                    0x3998                  _ADI_Vitesse
                    0x399c                  _ADI_TotalPartiel
                    0x39a0                  _ADI_TotalGlobal
                    0x39a4                  _ADI_Tare
                    0x39a8                  _ADI_EtatBascule
                    0x39ac                  _ADI_CmdsBascule
                    0x39b0                  _ADI_DigitalInput
                    0x39b1                  _ADI_DigitalOutput
                    0x39f0                  _remoteNode
                    0x39fc                  _receivedECANmsg
                    0x39fe                  _transmitNextECANmsg
                    0x3a00                  _sentPacketECANMSG
                    0x3a02                  _rxECANIndex
                    0x3a04                  _txECANBufferIndex
                    0x3a06                  _SPI3CON1Value
                    0x3a08                  _SPI3CON2Value
                    0x3a0a                  _SPI3STATValue
                    0x3a16                  _app_aacLanguages
                    0x3a18                  _app_sInstance
                    0x3a1c                  _us_bSwitch1
                    0x3a1d                  _us_bSwitch2
                    0x3a1e                  _us_fSwitch1Set
                    0x3a1f                  _us_fSwitch2Set
                    0x3a2e                  _SPICON1Value
                    0x3a30                  _SPICON2Value
                    0x3a32                  _SPISTATValue
                    0x3a50                  _ABCC_StateMachineEnabled
                    0x3a52                  ___C30_UART
                    0x3a58                  _Nb_Octets_Log
                    0x3a5a                  _Address_Log_L
                    0x3a5b                  _Address_Log_B
                    0x3a60                  _ErrorReporter
                    0x3a62                  _dpv_sInstance
                    0x3a64                  _rxECANBufferIndex
                    0x3a66                  _Demarrage1er
                    0x3a76                  _DmaBufferSwitch
                    0x3a7a                  _errno
                    0x3a80                  __Files
                    0x3a82                  __outdone
                    0x3a84                  __sibuf
                    0x3a86                  __sobuf
                    0xd800                  _BufferB
                    0xdb00                  _ecanTxMsgBuffer
                    0xdc00                  _BufferA
                    0xdf00                  _ecanRxMsgBuffer

External Symbols in Data Memory (by name):

                    0x373a                  _ABCCPowerState
                    0x3950                  _ABCC_ISR
                    0x394e                  _ABCC_RunDriver
                    0x3a50                  _ABCC_StateMachineEnabled
                    0x1fb6                  _AD7190_PoidsPret
                    0x39ac                  _ADI_CmdsBascule
                    0x398c                  _ADI_DebitInstan
                    0x39b0                  _ADI_DigitalInput
                    0x39b1                  _ADI_DigitalOutput
                    0x39a8                  _ADI_EtatBascule
                    0x3990                  _ADI_PoidsInstan
                    0x3994                  _ADI_PoidsMetre
                    0x39a4                  _ADI_Tare
                    0x39a0                  _ADI_TotalGlobal
                    0x399c                  _ADI_TotalPartiel
                    0x3998                  _ADI_Vitesse
                    0x3462                  _AD_asADIEntryList
                    0x3460                  _AD_asDefaultMap
                    0x3a5b                  _Address_Log_B
                    0x3a5a                  _Address_Log_L
                    0x3740                  _AppConfig
                    0x3400                  _BDT
                    0x3134                  _BaudRateGen
                    0x37b4                  _BothEP0OutUOWNsSet
                    0xdc00                  _BufferA
                    0xd800                  _BufferB
                    0x3130                  _CDCDataInHandle
                    0x312e                  _CDCDataOutHandle
                    0x2cd6                  _COIL
                    0x2cd8                  _COIL_REG
                    0x1f64                  _Cav_CLR
                    0x1f62                  _Cav_USR1
                    0x1fb8                  _Compteur
                    0x1fbe                  _CompteurTot
                    0x37c9                  _CtrlTrfData
                    0x3a66                  _Demarrage1er
                    0x3a76                  _DmaBufferSwitch
                    0x1b38                  _EXP
                    0x3a60                  _ErrorReporter
                    0x36d4                  _HOLDING_REG
                    0x3706                  _INPUT_REG
                    0x36d3                  _InputByteReverse
                    0x28c8                  _MODBUS_COMMAND
                    0x28d6                  _MODBUS_RX
                    0x2ad6                  _MODBUS_TX
                    0x1fba                  _NbTopTotal
                    0x3a58                  _Nb_Octets_Log
                    0x1870                  _PAR
                    0x36d2                  _ReadByteReverse
                    0x37b0                  _RemoteWakeup
                    0x3a06                  _SPI3CON1Value
                    0x3a08                  _SPI3CON2Value
                    0x3a0a                  _SPI3STATValue
                    0x3a2e                  _SPICON1Value
                    0x3a30                  _SPICON2Value
                    0x3a32                  _SPISTATValue
                    0x37c1                  _SetupPkt
                    0x1fa2                  _T10
                    0x1f66                  _T100
                    0x1068                  _TrameU1
                    0x126a                  _TrameU2
                    0x146c                  _TrameU3
                    0x166e                  _TrameU4
                    0x1050                  _U1Baudvalue
                    0x1058                  _U1MODEvalue
                    0x105a                  _U1STAvalue
                    0x1052                  _U2Baudvalue
                    0x105c                  _U2MODEvalue
                    0x105e                  _U2STAvalue
                    0x1054                  _U3Baudvalue
                    0x1060                  _U3MODEvalue
                    0x1062                  _U3STAvalue
                    0x1056                  _U4Baudvalue
                    0x1064                  _U4MODEvalue
                    0x1066                  _U4STAvalue
                    0x3374                  _UDPRxCount
                    0x3280                  _UDPSocketInfo
                    0x3372                  _UDPTxCount
                    0x378a                  _USBActiveConfiguration
                    0x378b                  _USBAlternateInterface
                    0x37b1                  _USBBusIsSuspended
                    0x37bf                  _USBDeferINDataStagePackets
                    0x37c0                  _USBDeferOUTDataStagePackets
                    0x37bc                  _USBDeferStatusStagePacket
                    0x3788                  _USBDeviceState
                    0x37bd                  _USBStatusStageEnabledFlag1
                    0x37be                  _USBStatusStageEnabledFlag2
                    0x37bb                  _USBStatusStageTimeoutCounter
                    0x2e22                  _USB_In_Buffer
                    0x2e64                  _USB_Mess
                    0x2e62                  _USB_Mess_head
                    0x2f30                  _USB_list_count
                    0x37b2                  _USTATcopy
                    0x28d4                  _WriteByteReverse
                    0x3a80                  __Files
                    0x3a52                  ___C30_UART
                    0x384a                  __iob
                    0x2fe4                  __npowers_
                    0x3a82                  __outdone
                    0x2f34                  __powers_
                    0x3a84                  __sibuf
                    0x3a86                  __sobuf
                    0x3370                  _activeUDPSocket
                    0x373c                  _address
                    0x3a16                  _app_aacLanguages
                    0x3a18                  _app_sInstance
                    0x30d4                  _cdc_data_rx
                    0x3094                  _cdc_data_tx
                    0x312d                  _cdc_mem_type
                    0x311c                  _cdc_notice
                    0x3126                  _cdc_rx_len
                    0x3127                  _cdc_trf_state
                    0x312c                  _cdc_tx_len
                    0x379f                  _controlTransferState
                    0x3132                  _control_signal_bitmap
                    0x35da                  _curHTTP
                    0x3664                  _curHTTPID
                    0x3a62                  _dpv_sInstance
                    0x3138                  _dummy_encapsulated_cmd_response
                    0xdf00                  _ecanRxMsgBuffer
                    0xdb00                  _ecanTxMsgBuffer
                    0x37b3                  _endpoint_number
                    0x1f58                  _entTOR
                    0x1fc2                  _entreeTorVitesseMem
                    0x37b5                  _ep_data_in
                    0x37b8                  _ep_data_out
                    0x3a7a                  _errno
                    0x3738                  _fResetABCC
                    0x365c                  _httpStubs
                    0x37a0                  _inPipes
                    0x3114                  _line_coding
                    0x245c                  _link_bPool
                    0x37a6                  _outPipes
                    0x378e                  _pBDTEntryEP0OutCurrent
                    0x3790                  _pBDTEntryEP0OutNext
                    0x3798                  _pBDTEntryIn
                    0x3792                  _pBDTEntryOut
                    0x312a                  _pCDCDst
                    0x3128                  _pCDCSrc
                    0x37ae                  _pDst
                    0x397e                  _pnABCC_DrvGetAnbStatus
                    0x3976                  _pnABCC_DrvGetAnybusState
                    0x3974                  _pnABCC_DrvGetIntStatus
                    0x3972                  _pnABCC_DrvGetLedStatus
                    0x3970                  _pnABCC_DrvGetModCap
                    0x396e                  _pnABCC_DrvGetWrPdBuffer
                    0x3954                  _pnABCC_DrvISR
                    0x3962                  _pnABCC_DrvISReadyForCmd
                    0x395e                  _pnABCC_DrvISReadyForWrPd
                    0x3960                  _pnABCC_DrvISReadyForWriteMessage
                    0x3952                  _pnABCC_DrvInit
                    0x397c                  _pnABCC_DrvIsSupervised
                    0x397a                  _pnABCC_DrvReadMessage
                    0x3978                  _pnABCC_DrvReadProcessData
                    0x3958                  _pnABCC_DrvRunDriverRx
                    0x3956                  _pnABCC_DrvRunDriverTx
                    0x3966                  _pnABCC_DrvSetAppStatus
                    0x396c                  _pnABCC_DrvSetIntMask
                    0x396a                  _pnABCC_DrvSetMsgReceiverBuffer
                    0x3964                  _pnABCC_DrvSetNbrOfCmds
                    0x3968                  _pnABCC_DrvSetPdSize
                    0x395a                  _pnABCC_DrvWriteMessage
                    0x395c                  _pnABCC_DrvWriteProcessData
                    0x39fc                  _receivedECANmsg
                    0x39f0                  _remoteNode
                    0x3a64                  _rxECANBufferIndex
                    0x3a02                  _rxECANIndex
                    0x3a00                  _sentPacketECANMSG
                    0x379e                  _shortPacketStatus
                    0x1f4e                  _sorTOR
                    0x39fe                  _transmitNextECANmsg
                    0x3a04                  _txECANBufferIndex
                    0x3a1c                  _us_bSwitch1
                    0x3a1d                  _us_bSwitch2
                    0x3a1e                  _us_fSwitch1Set
                    0x3a1f                  _us_fSwitch2Set

External Symbols in Program Memory (by address):

                  0x000200                  __resetPRI
                  0x00022c                  __psv_init
                  0x000238                  __data_init_extended
                  0x000238                  __data_init
                  0x000392                  __U1RXInterrupt
                  0x00041c                  __U2RXInterrupt
                  0x0004a6                  __U3RXInterrupt
                  0x000530                  __U4RXInterrupt
                  0x0005ba                  __DMA0Interrupt
                  0x00065e                  __INT1Interrupt
                  0x000698                  __INT2Interrupt
                  0x0006b4                  __INT3Interrupt
                  0x0006fa                  __INT4Interrupt
                  0x000728                  __USB1Interrupt
                  0x000750                  __C1Interrupt
                  0x000794                  __OscillatorFail
                  0x00079a                  __AddressError
                  0x0007a0                  __StackError
                  0x0007a6                  __MathError
                  0x0007ac                  __DMACError
                  0x0007b2                  __DefaultInterrupt
                  0x0007b6                  __HardTrapError
                  0x0007ba                  __SoftTrapError
                  0x0007be                  _isspace
                  0x00082e                  _CloseSPI1
                  0x00083a                  _CloseSPI3
                  0x000846                  _DataRdySPI1
                  0x000850                  _DataRdySPI3
                  0x00085a                  _OpenSPI1
                  0x000866                  _OpenSPI3
                  0x000872                  _ReadSPI1
                  0x000892                  _ReadSPI3
                  0x0008b2                  _WriteSPI1
                  0x0008c4                  _WriteSPI3
                  0x0008d6                  _BusyUART2
                  0x0008e4                  _BusyUART3
                  0x0008f2                  _BusyUART4
                  0x000900                  _CloseUART1
                  0x000910                  _CloseUART2
                  0x000920                  _CloseUART3
                  0x000930                  _CloseUART4
                  0x000940                  _ConfigIntUART1
                  0x00098c                  _ConfigIntUART2
                  0x0009d8                  _ConfigIntUART3
                  0x000a24                  _ConfigIntUART4
                  0x000a6c                  _DataRdyUART1
                  0x000a76                  _DataRdyUART2
                  0x000a80                  _DataRdyUART3
                  0x000a8a                  _DataRdyUART4
                  0x000a94                  _OpenUART1
                  0x000aa0                  _OpenUART2
                  0x000aac                  _OpenUART3
                  0x000ab8                  _OpenUART4
                  0x000ac4                  _putsUART1
                  0x000af0                  _putsUART2
                  0x000b1c                  _putsUART3
                  0x000b48                  _putsUART4
                  0x000b74                  _ReadUART1
                  0x000b8a                  _ReadUART2
                  0x000ba0                  _ReadUART3
                  0x000bb6                  _ReadUART4
                  0x000bcc                  ___subsf3
                  0x000bce                  ___addsf3
                  0x000c88                  ___divsf3
                  0x000d0c                  ___divsi3
                  0x000d2a                  ___lesf2
                  0x000d2a                  ___eqsf2
                  0x000d2a                  ___ltsf2
                  0x000d2e                  ___gtsf2
                  0x000d2e                  ___gesf2
                  0x000d32                  ___fixsfsi
                  0x000d74                  ___fixunssfsi
                  0x000daa                  ___floatsisf
                  0x000db0                  ___floatunsisf
                  0x000db4                  __fpack
                  0x000e00                  __funpack
                  0x000e2a                  __funpack2
                  0x000e3a                  __fPropagateNaN
                  0x000e4c                  __fbopExit
                  0x000e54                  __fbopReturnNaN
                  0x000e5a                  ___mulsf3
                  0x000ec2                  ___udivsi3
                  0x000ee2                  ___umodsi3
                  0x000ee8                  __fcompare
                  0x000f1e                  ___floatdisf
                  0x000f3e                  ___floatundisf
                  0x000f9c                  _strtof
                  0x001182                  _strtod
                  0x00118a                  _atof
                  0x001194                  _atoi
                  0x0011d6                  _atol
                  0x001230                  _ultoa
                  0x001280                  _ltoa
                  0x0012a4                  _memcmp
                  0x0012d2                  _memcpy
                  0x0012e4                  _memset
                  0x0012f6                  _srand
                  0x001308                  _rand
                  0x001334                  _sprintf
                  0x00135e                  _strcmp
                  0x001370                  _strcpy
                  0x001380                  _strlen
                  0x001392                  _strncpy
                  0x0013b8                  _strtok
                  0x0013fa                  _putchar
                  0x001404                  __sprintf_cdnopsuxX
                  0x001404                  __sprintf_cdfFnopsuxX
                  0x001404                  __sprintf_cdnopuxX
                  0x001404                  __sprintf_cdfFnopuxX
                  0x001590                  __vfprintf_cdnopuxX
                  0x001590                  __vfprintf_cdfFnopsuxX
                  0x001590                  __vfprintf_s
                  0x001590                  __vfprintf_0
                  0x001590                  __vfprintf_cdfFnopuxX
                  0x001590                  __vfprintf_cdnopsuxX
                  0x0021de                  __printf_cdnopuxX
                  0x0021de                  __printf_0
                  0x0021de                  __printf_s
                  0x0021de                  __printf_cdnopsuxX
                  0x00234e                  _vfprintf
                  0x003780                  _strcspn
                  0x0037aa                  _strspn
                  0x0037d4                  _strchr
                  0x003876                  ___adddf3
                  0x003970                  ___eqdf2
                  0x003970                  ___ltdf2
                  0x003970                  ___ledf2
                  0x00397a                  ___gedf2
                  0x00397a                  ___gtdf2
                  0x003984                  ___divdf3
                  0x003a38                  ___nedf2
                  0x003a42                  __dpack
                  0x003a9a                  __dunpack2
                  0x003abc                  __dreturnNaN
                  0x003ac2                  __dunpack2exit
                  0x003acc                  ___extendsfdf2
                  0x003b0a                  ___fixunsdfdi
                  0x003b6c                  ___fixunsdfsi
                  0x003bb8                  ___floatundidf
                  0x003c0e                  ___floatunsidf
                  0x003c12                  _frexp
                  0x003c12                  _frexpl
                  0x003c4c                  ___muldf3
                  0x003d36                  ___subdf3
                  0x003d3a                  ___mulp32peds3
                  0x003d3a                  ___mulp32eds3
                  0x003d3a                  ___mulsi3
                  0x003db4                  ___udivmoddi3
                  0x003e84                  ___udivdi3
                  0x003e96                  ___umoddi3
                  0x003ea2                  ___divdi3
                  0x003f06                  ___moddi3
                  0x003f66                  ___muldi3
                  0x003fbc                  __dcompare
                  0x00400e                  __dPropagateNaN
                  0x00402a                  __dtype
                  0x00404e                  __dunpack
                  0x00409c                  ___umuldi3
                  0x004b12                  _DELIMITER
                  0x004b16                  _DELIMITER_NULL
                  0x005285                  _HTML_UP_ARROW
                  0x005288                  _HTML_DOWN_ARROW
                  0x0055a6                  _device_dsc
                  0x0055b8                  _configDescriptor1
                  0x0055fc                  _sd000
                  0x005600                  _sd001
                  0x005618                  _sd002
                  0x005630                  _USB_CD_Ptr
                  0x005632                  _USB_SD_Ptr
                  0x005638                  _abBitReverseTable16
                  0x005648                  _crc_table32
                  0x00570e                  _TCPSocketInitializer
                  0x005746                  _app_sObject
                  0x005794                  _dpv1_sObject
                  0x0057da                  _MPFS_Start
                  0x0057de                  _ModbusUartServer
                  0x005886                  _ProcessMessageRecu
                  0x00592e                  _LectureMots
                  0x007f5a                  _LectureModbus
                  0x008018                  _envoieLongPF
                  0x008078                  _envoieLongPf
                  0x0080a4                  _envoieReelPF
                  0x008150                  _envoieReelPf
                  0x008202                  _EcritureMots
                  0x009dc6                  _AffectationIO
                  0x009e04                  _ModifParamMetro
                  0x00aa3e                  _LectureLong
                  0x00ab20                  _LectureReel
                  0x00ac4a                  _ValidationCodeMetrologie
                  0x00ad66                  _ModbusErreur
                  0x00ad94                  _Random
                  0x00adc4                  _ModifieVitesseComm
                  0x00aecc                  BEGIN_MPFS
                  0x0100b2                  _EcrFRAM_Param
                  0x0100fa                  _EcrFRAM
                  0x010142                  _LecFRAM_Param
                  0x0101a6                  _LecFRAM
                  0x0101ee                  _InitParams
                  0x010618                  _gestion_profibus
                  0x010844                  _process_plcd
                  0x010cc2                  _gestion_defauts
                  0x010f5a                  _gestion_cycle
                  0x0111a8                  _ValEntTOR
                  0x0111e0                  _gestion_vitesse
                  0x011472                  _EnvoieSerie
                  0x011554                  _gestion_totalisateurs
                  0x01186c                  _verif_totaux
                  0x011ac2                  _etatSortieTOR
                  0x011af6                  _sortiesTOR
                  0x011d42                  _gestion_poids_debit
                  0x011ff6                  _gestion_comm_serie
                  0x012054                  _envoyer_reel
                  0x012132                  _moyenne_glissante_debit
                  0x012156                  _moyenne_glissante_poids
                  0x0123b8                  _conversion_poids
                  0x012438                  _lecture_entrees_TOR
                  0x0124e4                  _EcritSortieAna
                  0x0129ba                  _TCPInit
                  0x012a8a                  _TCPOpen
                  0x012be4                  _TCPWasReset
                  0x012c12                  _TCPIsConnected
                  0x012c36                  _TCPDisconnect
                  0x012cd6                  _TCPClose
                  0x012cf6                  _TCPGetRemoteInfo
                  0x012d20                  _TCPFlush
                  0x012d46                  _TCPIsPutReady
                  0x012d94                  _TCPPut
                  0x012e3a                  _TCPPutArray
                  0x012f20                  _TCPPutString
                  0x012f44                  _TCPGetTxFIFOFull
                  0x012f70                  _TCPDiscard
                  0x012f90                  _TCPIsGetReady
                  0x012fc8                  _TCPGet
                  0x013042                  _TCPGetArray
                  0x01310e                  _TCPGetRxFIFOFree
                  0x013138                  _TCPPeekArray
                  0x0131e2                  _TCPPeek
                  0x0131fa                  _TCPFindArrayEx
                  0x01346a                  _TCPFindEx
                  0x01348e                  _TCPTick
                  0x01397e                  _TCPProcess
                  0x014b8c                  _TCPAdjustFIFOSize
                  0x014d8e                  _AD_Init
                  0x014f24                  _AD_GetAdiIndex
                  0x014f5a                  _AD_GetAdiInstEntry
                  0x014f80                  _AD_ProcObjectRequest
                  0x015f20                  _AD_GetAdiValue
                  0x0160c0                  _AD_SetAdiValue
                  0x01663a                  _AD_UpdatePdReadData
                  0x01668c                  _AD_UpdatePdWriteData
                  0x0166ee                  _AD_NewWrPd
                  0x0166f8                  _AD_AdiMappingReq
                  0x016b3e                  _AD_RemapDone
                  0x016b66                  _HTTPPrint
                  0x016db4                  _HTTPPrint_
                  0x016dd2                  _HTTPInit
                  0x016e60                  _HTTPServer
                  0x01818e                  _HTTPURLDecode
                  0x018262                  _HTTPGetArg
                  0x0182b8                  _HTTPReadPostName
                  0x0182e4                  _HTTPReadPostValue
                  0x018500                  _HTTPIncFile
                  0x0185e6                  _USBDeviceInit
                  0x0186fa                  _USBDeviceTasks
                  0x018896                  _USBEnableEndpoint
                  0x0188d0                  _USBTransferOnePacket
                  0x018a0a                  _USBStallEndpoint
                  0x018b98                  _USBCancelIO
                  0x018d2a                  _USBDeviceDetach
                  0x018d3c                  _USBDeviceAttach
                  0x018d7e                  _USBCtrlEPAllowStatusStage
                  0x018eb6                  _USBCtrlEPAllowDataStage
                  0x019eb4                  _GestionCyclePesage
                  0x01b0de                  _MACInit
                  0x01b20e                  _MACIsLinked
                  0x01b224                  _MACIsTxReady
                  0x01b23c                  _MACDiscardRx
                  0x01b278                  _MACGetFreeRxSize
                  0x01b302                  _MACGetHeader
                  0x01b3d4                  _MACPutHeader
                  0x01b42a                  _MACFlush
                  0x01b56c                  _MACSetReadPtrInRx
                  0x01b59e                  _MACSetWritePtr
                  0x01b5d4                  _MACSetReadPtr
                  0x01b60a                  _MACCalcRxChecksum
                  0x01b670                  _CalcIPBufferChecksum
                  0x01b726                  _MACMemCopyAsync
                  0x01b92c                  _MACIsMemCopyDone
                  0x01b944                  _MACGet
                  0x01b976                  _MACGetArray
                  0x01ba54                  _MACPut
                  0x01ba8c                  _MACPutArray
                  0x01bc46                  _ReadPHYReg
                  0x01bd8e                  _WritePHYReg
                  0x01bde6                  _MACPowerDown
                  0x01be1a                  _MACPowerUp
                  0x01be3c                  _SetCLKOUT
                  0x01be52                  _GetCLKOUT
                  0x01be70                  _InitApp
                  0x01be8c                  _putsUSB
                  0x01bef0                  _USB_enqMsg
                  0x01bf3c                  _DeviceCDCInitialize
                  0x01bf60                  _DeviceCDCTasks
                  0x01bffe                  _ProccessCmd
                  0x01c76e                  _CRC_Init
                  0x01c77e                  _CRC_ChecksumWord
                  0x01c7e4                  _ResetCounterMillis
                  0x01c7ee                  _GetCounterMillis
                  0x01c804                  _UpdateB40ADI
                  0x01ca24                  _BerkeleySocketInit
                  0x01ca50                  _socket
                  0x01caea                  _bind
                  0x01cb8a                  _listen
                  0x01cca6                  _accept
                  0x01cdec                  _connect
                  0x01cf6c                  _send
                  0x01cf8c                  _sendto
                  0x01d150                  _recv
                  0x01d1e8                  _recvfrom
                  0x01d348                  _gethostname
                  0x01d3aa                  _closesocket
                  0x01d582                  _HTTPNeedsAuth
                  0x01d5b6                  _HTTPCheckAuth
                  0x01d5e8                  _HTTPExecuteGet
                  0x01d66c                  _HTTPExecutePost
                  0x01d9de                  _HTTPPrint_builddate
                  0x01da2c                  _HTTPPrint_version
                  0x01da4c                  _HTTPPrint_btn
                  0x01daa2                  _HTTPPrint_led
                  0x01daf6                  _HTTPPrint_ledSelected
                  0x01db5a                  _HTTPPrint_pot
                  0x01db88                  _HTTPPrint_lcdtext
                  0x01dbc2                  _HTTPPrint_hellomsg
                  0x01dc0e                  _HTTPPrint_cookiename
                  0x01dc5c                  _HTTPPrint_uploadeImage
                  0x01dc62                  _HTTPPrint_uploadedmd5
                  0x01dcb4                  _HTTPPrintIP
                  0x01dd1a                  _HTTPPrint_config_hostname
                  0x01dd38                  _HTTPPrint_config_dhcpchecked
                  0x01dd62                  _HTTPPrint_config_ip
                  0x01dd90                  _HTTPPrint_config_gw
                  0x01ddbe                  _HTTPPrint_config_subnet
                  0x01ddec                  _HTTPPrint_config_dns1
                  0x01de1a                  _HTTPPrint_config_dns2
                  0x01de48                  _HTTPPrint_config_mac
                  0x01df00                  _HTTPPrint_read_comm
                  0x01df08                  _HTTPPrint_write_comm
                  0x01df10                  _HTTPPrint_reboot
                  0x01df18                  _HTTPPrint_rebootaddr
                  0x01df36                  _HTTPPrint_ddns_user
                  0x01df3c                  _HTTPPrint_ddns_pass
                  0x01df42                  _HTTPPrint_ddns_host
                  0x01df48                  _HTTPPrint_ddns_service
                  0x01df50                  _HTTPPrint_ddns_status
                  0x01df70                  _HTTPPrint_ddns_status_msg
                  0x01dfbe                  _HTTPPrint_smtps_en
                  0x01dfde                  _HTTPPrint_snmp_en
                  0x01dffe                  _HTTPPrint_status_ok
                  0x01e044                  _HTTPPrint_status_fail
                  0x01e08a                  _MPFSInit
                  0x01e0b6                  _MPFSOpen
                  0x01e20c                  _MPFSOpenID
                  0x01e296                  _MPFSClose
                  0x01e2bc                  _MPFSGet
                  0x01e44c                  _MPFSGetArray
                  0x01e676                  _MPFSGetLong
                  0x01e698                  _MPFSSeek
                  0x01e8aa                  _MPFSGetTimestamp
                  0x01e8f0                  _MPFSGetMicrotime
                  0x01e936                  _MPFSGetFlags
                  0x01e97a                  _MPFSGetSize
                  0x01e9c0                  _MPFSGetBytesRem
                  0x01e9fe                  _MPFSGetStartAddr
                  0x01ea46                  _MPFSGetEndAddr
                  0x01ea98                  _MPFSGetFilename
                  0x01eafc                  _MPFSGetPosition
                  0x01eb22                  _MPFSGetID
                  0x01eb7c                  _main
                  0x01ecac                  _ABCCMainStateMachine
                  0x01ed52                  _DisplayIPValue
                  0x01ed88                  _GestionReponseModbus
                  0x01eef4                  _ProcessIO
                  0x01f12a                  _InitTCPIPAppConfig
                  0x01f206                  _InitializeBoard
                  0x01f3d8                  _SaveAppConfig
                  0x01f410                  _ADInit
                  0x01f462                  _LEDUpdateUSBStatus
                  0x01f4d0                  _USER_USB_CALLBACK_EVENT_HANDLER
                  0x01f534                  _LFSRSeedRand
                  0x01f576                  _LFSRRand
                  0x01f5e6                  _GenerateRandomDWORD
                  0x01f6f0                  _StringToIPAddress
                  0x01f86a                  _Base64Decode
                  0x01f9d2                  _uitoa
                  0x01fa52                  _hexatob
                  0x01fabc                  _btohexa_high
                  0x01fade                  _btohexa_low
                  0x01fafc                  _stricmppgm2ram
                  0x01fb94                  _swaps
                  0x01fbb0                  _swapl
                  0x01fc10                  _CalcIPChecksum
                  0x01fc92                  _strupr
                  0x01fcd2                  _FormatNetBIOSName
                  0x01fd1c                  _strnchr
                  0x01fd6a                  _strncpy_m
                  0x01fde8                  _DNSBeginUsage
                  0x01fe08                  _DNSEndUsage
                  0x01fe40                  _DNSResolve
                  0x01fe80                  _DNSIsResolved
                  0x02067e                  _UDPInit
                  0x02069e                  _UDPOpenEx
                  0x0207b8                  _UDPTask
                  0x0209fa                  _UDPIsOpened
                  0x020a1c                  _UDPClose
                  0x020a5e                  _UDPSetTxBuffer
                  0x020a74                  _UDPSetRxBuffer
                  0x020a8a                  _UDPIsPutReady
                  0x020ac0                  _UDPPut
                  0x020af0                  _UDPPutArray
                  0x020b2c                  _UDPPutString
                  0x020b4a                  _UDPFlush
                  0x020c44                  _UDPIsGetReady
                  0x020c7a                  _UDPGet
                  0x020cae                  _UDPGetArray
                  0x020cfa                  _UDPDiscard
                  0x020d20                  _UDPProcess
                  0x020ef8                  _UARTs_Init
                  0x020fee                  _BaudrateIsValid
                  0x02105e                  _UART1_SetBaudrate
                  0x0210b4                  _UART2_SetBaudrate
                  0x02110a                  _UART3_SetBaudrate
                  0x021160                  _UART4_SetBaudrate
                  0x0211b6                  _UART1_SetStopBit
                  0x0211f4                  _UART2_SetStopBit
                  0x021232                  _UART1_SetParityNBits
                  0x02128a                  _UART2_SetParityNBits
                  0x0212e2                  _ReceiveUART1
                  0x021358                  _ReceiveUART2
                  0x021496                  _ReceiveUART3
                  0x0215c8                  _ReceiveUART4
                  0x0216fa                  _SendStrUART3
                  0x021726                  _SendStrUART4
                  0x02175e                  _ABCC_SetupInit
                  0x02178c                  _ABCC_SetupCommands
                  0x021abc                  _ABCC_SetupResponses
                  0x021e46                  _ABCC_UserInitComplete
                  0x021e7e                  _ABCC_NetworkType
                  0x021e88                  _ABCC_ModuleType
                  0x021e92                  _ABCC_NetFormatType
                  0x021e9c                  _ABCC_ParameterSupport
                  0x021ed4                  _ABCC_DrvSpiRunDriverTx
                  0x022010                  _ABCC_DrvSpiRunDriverRx
                  0x0221a2                  build/XC16_dsPIC33EP512MU810/debug/B40/spi/abcc_spi_drv.o:_spi_drv_DataReceived
                  0x0221e8                  build/XC16_dsPIC33EP512MU810/debug/B40/spi/abcc_spi_drv.o:_drv_WdTimeoutHandler
                  0x0221f6                  _ABCC_DrvSpiInit
                  0x02229e                  _ABCC_DrvSpiWriteMessage
                  0x02231a                  _ABCC_DrvSpiWriteProcessData
                  0x022350                  _ABCC_DrvSpiIsReadyForWriteMessage
                  0x022376                  _ABCC_DrvSpiIsReadyForCmd
                  0x022396                  _ABCC_DrvSpiSetNbrOfCmds
                  0x0223a2                  _ABCC_DrvSpiSetAppStatus
                  0x0223b2                  _ABCC_DrvSpiSetPdSize
                  0x02240e                  _ABCC_DrvSpiSetMsgReceiverBuffer
                  0x022456                  _ABCC_DrvSpiGetIntStatus
                  0x02247a                  _ABCC_DrvSpiGetAnybusState
                  0x022488                  _ABCC_DrvSpiReadProcessData
                  0x0224a0                  _ABCC_DrvSpiReadMessage
                  0x0224c2                  _ABCC_DrvSpiSetIntMask
                  0x0224d2                  _ABCC_DrvSpiGetWrPdBuffer
                  0x0224e2                  _ABCC_DrvSpiGetModCap
                  0x022506                  _ABCC_DrvSpiGetLedStatus
                  0x022510                  _ABCC_DrvSpiIsReadyForWrPd
                  0x022524                  _ABCC_DrvSpiIsSupervised
                  0x02253a                  _ABCC_DrvSpiGetAnbStatus
                  0x022548                  _AD7190_SetRegisterValue
                  0x02259a                  _AD7190_GetRegisterValue
                  0x02260c                  _AD7190_Init
                  0x022640                  _AD7190_Reset
                  0x02266c                  _AD7190_SetPower
                  0x0226fc                  _AD7190_WaitRdyGoLow
                  0x022730                  _AD7190_ChannelSelect
                  0x022790                  _AD7190_Calibrate
                  0x02281e                  _AD7190_RangeSetup
                  0x0228a4                  _AD7190_SingleConversion
                  0x0228e4                  _AD7190_ContinuousReadAvg
                  0x02294c                  _AD7190_TemperatureRead
                  0x0229ae                  _AD7190_StartContinuousRead
                  0x022a16                  _AD7190_StopContinuousRead
                  0x022a38                  _AD7190_PrintRegisters
                  0x022b72                  _ABCC_SetReadyForCommunication
                  0x022b7c                  _ABCC_SetMainStateError
                  0x022b86                  _ABCC_GetMainState
                  0x022b90                  _ABCC_CheckAnbStatus
                  0x022bb0                  _ABCC_CheckSendMessage
                  0x022bba                  _ABCC_StartDriver
                  0x022d52                  _ABCC_isReadyForCommunication
                  0x022dda                  _ABCC_NewWrPdEvent
                  0x022e08                  _ABCC_RdPdEvent
                  0x022e2c                  _ABCC_RdMsgEvent
                  0x022eb4                  _ABCC_SendCmdMsg
                  0x022f04                  _ABCC_GetCmdQueueSize
                  0x022f12                  _ABCC_SendRespMsg
                  0x022f24                  _ABCC_MsgAlloc
                  0x022f32                  _ABCC_MsgFree
                  0x022f44                  _ABCC_SetPdSize
                  0x022f6c                  _ABCC_HWReset
                  0x022f88                  _ABCC_ShutdownDriver
                  0x022faa                  _ABCC_ModuleDetect
                  0x022fb8                  _ABCC_ModCap
                  0x022fc6                  _ABCC_LedStatus
                  0x022fd4                  _ABCC_AnbState
                  0x022fe2                  _ABCC_IsSupervised
                  0x022ff0                  _ABCC_HWReleaseReset
                  0x022ffa                  _ABCC_SetAppStatus
                  0x023008                  _ABCC_ReadModuleId
                  0x023016                  _ABCC_RunTimerSystem
                  0x023024                  _ABCC_GetNewSourceId
                  0x023054                  _ABCC_GetOpmode
                  0x023062                  _ABCC_GetAttribute
                  0x0230ba                  _ABCC_SetByteAttribute
                  0x02311c                  _ABCC_VerifyMessage
                  0x023130                  _SetErrorReporter
                  0x02313c                  _ABCC_GetDataTypeSize
                  0x023278                  _ABCC_LinkInit
                  0x023302                  _ABCC_LinkReadMessage
                  0x023382                  _ABCC_LinkCheckSendMessage
                  0x02340c                  _ABCC_LinkRunDriverRx
                  0x02342a                  _ABCC_LinkGetNumCmdQueueEntries
                  0x02343e                  _ABCC_LinkWriteMessage
                  0x02355c                  _ABCC_LinkWrMsgWithNotification
                  0x0235a0                  _ABCC_LinkAlloc
                  0x0235b6                  _ABCC_LinkFree
                  0x023614                  _ABCC_LinkMapMsgHandler
                  0x023668                  _ABCC_LinkGetMsgHandler
                  0x0236c6                  _ABCC_LinkIsSrcIdUsed
                  0x023c04                  _Flash_N_Clock
                  0x023c22                  _Active_Flash
                  0x023c2a                  _Desactive_Flash
                  0x023c38                  _Flash_Ready
                  0x023c5a                  _Wait_Flash_Ready
                  0x023c6a                  _Write_Flash
                  0x023c9c                  _Charge_Pointeurs
                  0x023cb4                  _Lecture_Byte_In_Flash
                  0x023cd0                  _Direct_Byte_Write_In_Page
                  0x023ce8                  _Transfert_Page_To_Buffer
                  0x023d00                  _Read_Flash
                  0x023d3c                  _Incremente_Adresse_FlashDB32
                  0x023e0a                  _Incremente_Adresse_FlashDB64
                  0x023ed8                  _MakeAddrDB32
                  0x023f34                  _MakeAddrDB64
                  0x023f96                  _Ecriture_Memoire_Flash_Ligne_Str
                  0x024026                  _Lecture_Memoire_Flash_Ligne_Str
                  0x0240ae                  _USBCheckCDCRequest
                  0x0241f8                  _CDCInitEP
                  0x024248                  _USBCDCEventHandler
                  0x02428e                  _getsUSBUSART
                  0x024322                  _putUSBUSART
                  0x02434e                  _putsUSBUSART
                  0x0243a4                  _putrsUSBUSART
                  0x0243fa                  _CDCTxService
                  0x0244fc                  _APP_IsResetRequestAllowed
                  0x024512                  _APP_ProcResetRequest
                  0x02453e                  _APP_ProcessCmdMsg
                  0x024568                  _app_InstanceCommand
                  0x024772                  _app_ObjectCommand
                  0x02493c                  _NBNSTask
                  0x024cea                  _ARPSendPkt
                  0x024dbe                  _ARPInit
                  0x024df0                  _ARPProcess
                  0x024ec8                  _ARPResolve
                  0x024f92                  _ARPIsResolved
                  0x02505a                  _SwapARPPacket
                  0x025092                  _FRAMInit
                  0x0250aa                  _FRAMBeginRead
                  0x0250c2                  _FRAMRead
                  0x025106                  _FRAMReadArray
                  0x0251e2                  _FRAMBeginWrite
                  0x0251fa                  _FRAMWrite
                  0x02523c                  _FRAMWriteArray
                  0x02526a                  _FRAMEndWrite
                  0x025378                  _FRAMIsBusy
                  0x0253ea                  _XEEInit
                  0x025408                  _XEEBeginRead
                  0x025420                  _XEERead
                  0x025464                  _XEEEndRead
                  0x02546e                  _XEEReadArray
                  0x02552c                  _XEEBeginWrite
                  0x025544                  _XEEWrite
                  0x025586                  _XEEWriteArray
                  0x0255b4                  _XEEEndWrite
                  0x0256ae                  _XEEIsBusy
                  0x025720                  _ECANFilterSID
                  0x025750                  _ECANFilterEID
                  0x025762                  _ECAN1DMAConfig
                  0x0257aa                  _ECAN1ClockConfig
                  0x0257ba                  _ECAN1InterruptConfig
                  0x0257e4                  _ECAN1TxRxBuffersConfig
                  0x0257ee                  _ECAN1RxFiltersConfig
                  0x02585a                  _ECAN1SendPacket
                  0x025890                  _ECAN1SetOPMode
                  0x0258ac                  _ECANCreateSIDPacket
                  0x025900                  _ECANCreateEIDPacket
                  0x025a0c                  _DPV1_ProcessCmdMsg
                  0x025a36                  _dpv1_InstanceCommand
                  0x025b92                  _dpv1_ObjectCommand
                  0x025cf0                  _ICMPProcess
                  0x025ddc                  _ICMPSendPing
                  0x025e00                  _ICMPSendPingToHost
                  0x025e2a                  _ICMPGetReply
                  0x025f84                  _ICMPBeginUsage
                  0x025fa4                  _ICMPEndUsage
                  0x025fb2                  _BerkeleyUDPClient
                  0x0261da                  _BerkeleySNTPGetUTCSeconds
                  0x02622c                  _RegulationDoseur
                  0x02632c                  _RegulationPID
                  0x02649c                  _CRC_Crc32
                  0x0266ee                  _US_Init
                  0x0266f8                  _US_RunUserInitStateMachine
                  0x0267ee                  build/XC16_dsPIC33EP512MU810/debug/B40/user_setup.o:_US_ProcessRespMsg
                  0x026906                  _US_SetSwitch1
                  0x026918                  _US_SetSwitch2
                  0x02692a                  _TestModbus
                  0x02698e                  _BerkeleyTCPServer
                  0x026b66                  _ABCC_TimerInit
                  0x026b88                  _ABCC_TimerCreate
                  0x026bfa                  _ABCC_TimerStart
                  0x026c78                  _ABCC_TimerStop
                  0x026cba                  _ABCC_TimerTick
                  0x026d5a                  _IPGetHeader
                  0x026e24                  _IPPutHeader
                  0x026ed6                  _IPSetRxBuffer
                  0x026f24                  _AnnounceIP
                  0x026fce                  _DiscoveryTask
                  0x0270e6                  _StackInit
                  0x02711e                  _StackTask
                  0x027292                  _StackApplications
                  0x0272a8                  _ABCC_CbfUserInitReq
                  0x0272b6                  _ABCC_CbfAdiMappingReq
                  0x0272c8                  _ABCC_CbfRemapDone
                  0x0272d2                  _ABCC_CbfUpdateWriteProcessData
                  0x0272e4                  _ABCC_CbfNewReadPd
                  0x0272f2                  _ABCC_CbfDriverError
                  0x027314                  _ABCC_CbfReceiveMsg
                  0x027384                  _ABCC_CbfWdTimeout
                  0x02739a                  _ABCC_CbfWdTimeoutRecovered
                  0x0273b0                  _ABCC_CbfEvent
                  0x0273ea                  _ABCC_CbfAnbStatusChanged
                  0x027412                  _MODBUSTCPServer
                  0x0274b0                  _ProcessReceivedMessage
                  0x027544                  _ModbusError
                  0x027572                  _TickInit
                  0x027604                  _TickGet
                  0x027636                  _TickGetDiv256
                  0x027668                  _TickGetDiv64K
                  0x02769a                  _TickConvertToMilliseconds
                  0x0276b4                  __T1Interrupt
                  0x0276cc                  _BerkeleyTCPClient
                  0x0277fa                  _ABCC_SYS_Init
                  0x027824                  _ABCC_SYS_Close
                  0x02782e                  _ABCC_SYS_SetOpmode
                  0x027836                  _ABCC_SYS_GetOpmode
                  0x027840                  _ABCC_SYS_HWReset
                  0x027848                  _ABCC_SYS_HWReleaseReset
                  0x027850                  _ABCC_SYS_ReadModuleId
                  0x02785a                  _ABCC_SYS_ModuleDetect
                  0x027872                  _ABCC_SYS_AbccInterruptEnable
                  0x02787e                  _ABCC_SYS_AbccInterruptDisable
                  0x027886                  _ABCC_SYS_EnterCriticalImpl
                  0x02788c                  _ABCC_SYS_ExitCriticalImpl
                  0x027892                  _ABCC_SYS_UseCriticalImpl
                  0x027898                  _ABCC_SYS_SpiRegDataReceived
                  0x0278a4                  _ABCC_SYS_SpiSendReceive
                  0x027912                  _RebootTask
                  0x027a2a                  _InitAdc1
                  0x027a8a                  _InitTmr3
                  0x027a9e                  _InitDma0
                  0x027ad6                  _ProcessADCSamples
                  0x027b40                  _ADSPI_Init
                  0x027b66                  _SPI_Read
                  0x027bd8                  _SPI_Write
                  0x027c40                  _ABCC_MemCreatePool
                  0x027c8c                  _ABCC_MemAlloc
                  0x027cc8                  _ABCC_MemFree
                  0x027d08                  _ABCC_SpiRunDriver
                  0x027d64                  _ABCC_SpiISR
                  0x027d8e                  _ConfigureOscillator
                  0x027e0c                  _DelayMs
                  0x027e48                  _Delay10us
                  0x027e84                  _USBSleepOnSuspend
                  0x027eda                  build/XC16_dsPIC33EP512MU810/debug/B40/abcc_remap.o:_abcc_RemapRespMsgSent
                  0x027ef0                  _ABCC_SendRemapRespMsg
                  0x027f1c                  _AD_GetNumAdi
                  0x027f26                  _ADI_GetDefaultMap
                  0x027f30                  _ADI_GetADIEntryList
                  0x027f3a                  _ReadProgramMemory

External Symbols in Program Memory (by name):

                  0x00aecc                  BEGIN_MPFS
                  0x01ecac                  _ABCCMainStateMachine
                  0x022fd4                  _ABCC_AnbState
                  0x0272b6                  _ABCC_CbfAdiMappingReq
                  0x0273ea                  _ABCC_CbfAnbStatusChanged
                  0x0272f2                  _ABCC_CbfDriverError
                  0x0273b0                  _ABCC_CbfEvent
                  0x0272e4                  _ABCC_CbfNewReadPd
                  0x027314                  _ABCC_CbfReceiveMsg
                  0x0272c8                  _ABCC_CbfRemapDone
                  0x0272d2                  _ABCC_CbfUpdateWriteProcessData
                  0x0272a8                  _ABCC_CbfUserInitReq
                  0x027384                  _ABCC_CbfWdTimeout
                  0x02739a                  _ABCC_CbfWdTimeoutRecovered
                  0x022b90                  _ABCC_CheckAnbStatus
                  0x022bb0                  _ABCC_CheckSendMessage
                  0x02253a                  _ABCC_DrvSpiGetAnbStatus
                  0x02247a                  _ABCC_DrvSpiGetAnybusState
                  0x022456                  _ABCC_DrvSpiGetIntStatus
                  0x022506                  _ABCC_DrvSpiGetLedStatus
                  0x0224e2                  _ABCC_DrvSpiGetModCap
                  0x0224d2                  _ABCC_DrvSpiGetWrPdBuffer
                  0x0221f6                  _ABCC_DrvSpiInit
                  0x022376                  _ABCC_DrvSpiIsReadyForCmd
                  0x022510                  _ABCC_DrvSpiIsReadyForWrPd
                  0x022350                  _ABCC_DrvSpiIsReadyForWriteMessage
                  0x022524                  _ABCC_DrvSpiIsSupervised
                  0x0224a0                  _ABCC_DrvSpiReadMessage
                  0x022488                  _ABCC_DrvSpiReadProcessData
                  0x022010                  _ABCC_DrvSpiRunDriverRx
                  0x021ed4                  _ABCC_DrvSpiRunDriverTx
                  0x0223a2                  _ABCC_DrvSpiSetAppStatus
                  0x0224c2                  _ABCC_DrvSpiSetIntMask
                  0x02240e                  _ABCC_DrvSpiSetMsgReceiverBuffer
                  0x022396                  _ABCC_DrvSpiSetNbrOfCmds
                  0x0223b2                  _ABCC_DrvSpiSetPdSize
                  0x02229e                  _ABCC_DrvSpiWriteMessage
                  0x02231a                  _ABCC_DrvSpiWriteProcessData
                  0x023062                  _ABCC_GetAttribute
                  0x022f04                  _ABCC_GetCmdQueueSize
                  0x02313c                  _ABCC_GetDataTypeSize
                  0x022b86                  _ABCC_GetMainState
                  0x023024                  _ABCC_GetNewSourceId
                  0x023054                  _ABCC_GetOpmode
                  0x022ff0                  _ABCC_HWReleaseReset
                  0x022f6c                  _ABCC_HWReset
                  0x022fe2                  _ABCC_IsSupervised
                  0x022fc6                  _ABCC_LedStatus
                  0x0235a0                  _ABCC_LinkAlloc
                  0x023382                  _ABCC_LinkCheckSendMessage
                  0x0235b6                  _ABCC_LinkFree
                  0x023668                  _ABCC_LinkGetMsgHandler
                  0x02342a                  _ABCC_LinkGetNumCmdQueueEntries
                  0x023278                  _ABCC_LinkInit
                  0x0236c6                  _ABCC_LinkIsSrcIdUsed
                  0x023614                  _ABCC_LinkMapMsgHandler
                  0x023302                  _ABCC_LinkReadMessage
                  0x02340c                  _ABCC_LinkRunDriverRx
                  0x02355c                  _ABCC_LinkWrMsgWithNotification
                  0x02343e                  _ABCC_LinkWriteMessage
                  0x027c8c                  _ABCC_MemAlloc
                  0x027c40                  _ABCC_MemCreatePool
                  0x027cc8                  _ABCC_MemFree
                  0x022fb8                  _ABCC_ModCap
                  0x022faa                  _ABCC_ModuleDetect
                  0x021e88                  _ABCC_ModuleType
                  0x022f24                  _ABCC_MsgAlloc
                  0x022f32                  _ABCC_MsgFree
                  0x021e92                  _ABCC_NetFormatType
                  0x021e7e                  _ABCC_NetworkType
                  0x022dda                  _ABCC_NewWrPdEvent
                  0x021e9c                  _ABCC_ParameterSupport
                  0x022e2c                  _ABCC_RdMsgEvent
                  0x022e08                  _ABCC_RdPdEvent
                  0x023008                  _ABCC_ReadModuleId
                  0x023016                  _ABCC_RunTimerSystem
                  0x02787e                  _ABCC_SYS_AbccInterruptDisable
                  0x027872                  _ABCC_SYS_AbccInterruptEnable
                  0x027824                  _ABCC_SYS_Close
                  0x027886                  _ABCC_SYS_EnterCriticalImpl
                  0x02788c                  _ABCC_SYS_ExitCriticalImpl
                  0x027836                  _ABCC_SYS_GetOpmode
                  0x027848                  _ABCC_SYS_HWReleaseReset
                  0x027840                  _ABCC_SYS_HWReset
                  0x0277fa                  _ABCC_SYS_Init
                  0x02785a                  _ABCC_SYS_ModuleDetect
                  0x027850                  _ABCC_SYS_ReadModuleId
                  0x02782e                  _ABCC_SYS_SetOpmode
                  0x027898                  _ABCC_SYS_SpiRegDataReceived
                  0x0278a4                  _ABCC_SYS_SpiSendReceive
                  0x027892                  _ABCC_SYS_UseCriticalImpl
                  0x022eb4                  _ABCC_SendCmdMsg
                  0x027ef0                  _ABCC_SendRemapRespMsg
                  0x022f12                  _ABCC_SendRespMsg
                  0x022ffa                  _ABCC_SetAppStatus
                  0x0230ba                  _ABCC_SetByteAttribute
                  0x022b7c                  _ABCC_SetMainStateError
                  0x022f44                  _ABCC_SetPdSize
                  0x022b72                  _ABCC_SetReadyForCommunication
                  0x02178c                  _ABCC_SetupCommands
                  0x02175e                  _ABCC_SetupInit
                  0x021abc                  _ABCC_SetupResponses
                  0x022f88                  _ABCC_ShutdownDriver
                  0x027d64                  _ABCC_SpiISR
                  0x027d08                  _ABCC_SpiRunDriver
                  0x022bba                  _ABCC_StartDriver
                  0x026b88                  _ABCC_TimerCreate
                  0x026b66                  _ABCC_TimerInit
                  0x026bfa                  _ABCC_TimerStart
                  0x026c78                  _ABCC_TimerStop
                  0x026cba                  _ABCC_TimerTick
                  0x021e46                  _ABCC_UserInitComplete
                  0x02311c                  _ABCC_VerifyMessage
                  0x022d52                  _ABCC_isReadyForCommunication
                  0x022790                  _AD7190_Calibrate
                  0x022730                  _AD7190_ChannelSelect
                  0x0228e4                  _AD7190_ContinuousReadAvg
                  0x02259a                  _AD7190_GetRegisterValue
                  0x02260c                  _AD7190_Init
                  0x022a38                  _AD7190_PrintRegisters
                  0x02281e                  _AD7190_RangeSetup
                  0x022640                  _AD7190_Reset
                  0x02266c                  _AD7190_SetPower
                  0x022548                  _AD7190_SetRegisterValue
                  0x0228a4                  _AD7190_SingleConversion
                  0x0229ae                  _AD7190_StartContinuousRead
                  0x022a16                  _AD7190_StopContinuousRead
                  0x02294c                  _AD7190_TemperatureRead
                  0x0226fc                  _AD7190_WaitRdyGoLow
                  0x027f30                  _ADI_GetADIEntryList
                  0x027f26                  _ADI_GetDefaultMap
                  0x01f410                  _ADInit
                  0x027b40                  _ADSPI_Init
                  0x0166f8                  _AD_AdiMappingReq
                  0x014f24                  _AD_GetAdiIndex
                  0x014f5a                  _AD_GetAdiInstEntry
                  0x015f20                  _AD_GetAdiValue
                  0x027f1c                  _AD_GetNumAdi
                  0x014d8e                  _AD_Init
                  0x0166ee                  _AD_NewWrPd
                  0x014f80                  _AD_ProcObjectRequest
                  0x016b3e                  _AD_RemapDone
                  0x0160c0                  _AD_SetAdiValue
                  0x01663a                  _AD_UpdatePdReadData
                  0x01668c                  _AD_UpdatePdWriteData
                  0x0244fc                  _APP_IsResetRequestAllowed
                  0x024512                  _APP_ProcResetRequest
                  0x02453e                  _APP_ProcessCmdMsg
                  0x024dbe                  _ARPInit
                  0x024f92                  _ARPIsResolved
                  0x024df0                  _ARPProcess
                  0x024ec8                  _ARPResolve
                  0x024cea                  _ARPSendPkt
                  0x023c22                  _Active_Flash
                  0x009dc6                  _AffectationIO
                  0x026f24                  _AnnounceIP
                  0x01f86a                  _Base64Decode
                  0x020fee                  _BaudrateIsValid
                  0x0261da                  _BerkeleySNTPGetUTCSeconds
                  0x01ca24                  _BerkeleySocketInit
                  0x0276cc                  _BerkeleyTCPClient
                  0x02698e                  _BerkeleyTCPServer
                  0x025fb2                  _BerkeleyUDPClient
                  0x0008d6                  _BusyUART2
                  0x0008e4                  _BusyUART3
                  0x0008f2                  _BusyUART4
                  0x0241f8                  _CDCInitEP
                  0x0243fa                  _CDCTxService
                  0x01c77e                  _CRC_ChecksumWord
                  0x02649c                  _CRC_Crc32
                  0x01c76e                  _CRC_Init
                  0x01b670                  _CalcIPBufferChecksum
                  0x01fc10                  _CalcIPChecksum
                  0x023c9c                  _Charge_Pointeurs
                  0x00082e                  _CloseSPI1
                  0x00083a                  _CloseSPI3
                  0x000900                  _CloseUART1
                  0x000910                  _CloseUART2
                  0x000920                  _CloseUART3
                  0x000930                  _CloseUART4
                  0x000940                  _ConfigIntUART1
                  0x00098c                  _ConfigIntUART2
                  0x0009d8                  _ConfigIntUART3
                  0x000a24                  _ConfigIntUART4
                  0x027d8e                  _ConfigureOscillator
                  0x004b12                  _DELIMITER
                  0x004b16                  _DELIMITER_NULL
                  0x01fde8                  _DNSBeginUsage
                  0x01fe08                  _DNSEndUsage
                  0x01fe80                  _DNSIsResolved
                  0x01fe40                  _DNSResolve
                  0x025a0c                  _DPV1_ProcessCmdMsg
                  0x000846                  _DataRdySPI1
                  0x000850                  _DataRdySPI3
                  0x000a6c                  _DataRdyUART1
                  0x000a76                  _DataRdyUART2
                  0x000a80                  _DataRdyUART3
                  0x000a8a                  _DataRdyUART4
                  0x027e48                  _Delay10us
                  0x027e0c                  _DelayMs
                  0x023c2a                  _Desactive_Flash
                  0x01bf3c                  _DeviceCDCInitialize
                  0x01bf60                  _DeviceCDCTasks
                  0x023cd0                  _Direct_Byte_Write_In_Page
                  0x026fce                  _DiscoveryTask
                  0x01ed52                  _DisplayIPValue
                  0x0257aa                  _ECAN1ClockConfig
                  0x025762                  _ECAN1DMAConfig
                  0x0257ba                  _ECAN1InterruptConfig
                  0x0257ee                  _ECAN1RxFiltersConfig
                  0x02585a                  _ECAN1SendPacket
                  0x025890                  _ECAN1SetOPMode
                  0x0257e4                  _ECAN1TxRxBuffersConfig
                  0x025900                  _ECANCreateEIDPacket
                  0x0258ac                  _ECANCreateSIDPacket
                  0x025750                  _ECANFilterEID
                  0x025720                  _ECANFilterSID
                  0x0100fa                  _EcrFRAM
                  0x0100b2                  _EcrFRAM_Param
                  0x0124e4                  _EcritSortieAna
                  0x008202                  _EcritureMots
                  0x023f96                  _Ecriture_Memoire_Flash_Ligne_Str
                  0x011472                  _EnvoieSerie
                  0x0250aa                  _FRAMBeginRead
                  0x0251e2                  _FRAMBeginWrite
                  0x02526a                  _FRAMEndWrite
                  0x025092                  _FRAMInit
                  0x025378                  _FRAMIsBusy
                  0x0250c2                  _FRAMRead
                  0x025106                  _FRAMReadArray
                  0x0251fa                  _FRAMWrite
                  0x02523c                  _FRAMWriteArray
                  0x023c04                  _Flash_N_Clock
                  0x023c38                  _Flash_Ready
                  0x01fcd2                  _FormatNetBIOSName
                  0x01f5e6                  _GenerateRandomDWORD
                  0x019eb4                  _GestionCyclePesage
                  0x01ed88                  _GestionReponseModbus
                  0x01be52                  _GetCLKOUT
                  0x01c7ee                  _GetCounterMillis
                  0x005288                  _HTML_DOWN_ARROW
                  0x005285                  _HTML_UP_ARROW
                  0x01d5b6                  _HTTPCheckAuth
                  0x01d5e8                  _HTTPExecuteGet
                  0x01d66c                  _HTTPExecutePost
                  0x018262                  _HTTPGetArg
                  0x018500                  _HTTPIncFile
                  0x016dd2                  _HTTPInit
                  0x01d582                  _HTTPNeedsAuth
                  0x016b66                  _HTTPPrint
                  0x01dcb4                  _HTTPPrintIP
                  0x016db4                  _HTTPPrint_
                  0x01da4c                  _HTTPPrint_btn
                  0x01d9de                  _HTTPPrint_builddate
                  0x01dd38                  _HTTPPrint_config_dhcpchecked
                  0x01ddec                  _HTTPPrint_config_dns1
                  0x01de1a                  _HTTPPrint_config_dns2
                  0x01dd90                  _HTTPPrint_config_gw
                  0x01dd1a                  _HTTPPrint_config_hostname
                  0x01dd62                  _HTTPPrint_config_ip
                  0x01de48                  _HTTPPrint_config_mac
                  0x01ddbe                  _HTTPPrint_config_subnet
                  0x01dc0e                  _HTTPPrint_cookiename
                  0x01df42                  _HTTPPrint_ddns_host
                  0x01df3c                  _HTTPPrint_ddns_pass
                  0x01df48                  _HTTPPrint_ddns_service
                  0x01df50                  _HTTPPrint_ddns_status
                  0x01df70                  _HTTPPrint_ddns_status_msg
                  0x01df36                  _HTTPPrint_ddns_user
                  0x01dbc2                  _HTTPPrint_hellomsg
                  0x01db88                  _HTTPPrint_lcdtext
                  0x01daa2                  _HTTPPrint_led
                  0x01daf6                  _HTTPPrint_ledSelected
                  0x01db5a                  _HTTPPrint_pot
                  0x01df00                  _HTTPPrint_read_comm
                  0x01df10                  _HTTPPrint_reboot
                  0x01df18                  _HTTPPrint_rebootaddr
                  0x01dfbe                  _HTTPPrint_smtps_en
                  0x01dfde                  _HTTPPrint_snmp_en
                  0x01e044                  _HTTPPrint_status_fail
                  0x01dffe                  _HTTPPrint_status_ok
                  0x01dc5c                  _HTTPPrint_uploadeImage
                  0x01dc62                  _HTTPPrint_uploadedmd5
                  0x01da2c                  _HTTPPrint_version
                  0x01df08                  _HTTPPrint_write_comm
                  0x0182b8                  _HTTPReadPostName
                  0x0182e4                  _HTTPReadPostValue
                  0x016e60                  _HTTPServer
                  0x01818e                  _HTTPURLDecode
                  0x025f84                  _ICMPBeginUsage
                  0x025fa4                  _ICMPEndUsage
                  0x025e2a                  _ICMPGetReply
                  0x025cf0                  _ICMPProcess
                  0x025ddc                  _ICMPSendPing
                  0x025e00                  _ICMPSendPingToHost
                  0x026d5a                  _IPGetHeader
                  0x026e24                  _IPPutHeader
                  0x026ed6                  _IPSetRxBuffer
                  0x023d3c                  _Incremente_Adresse_FlashDB32
                  0x023e0a                  _Incremente_Adresse_FlashDB64
                  0x027a2a                  _InitAdc1
                  0x01be70                  _InitApp
                  0x027a9e                  _InitDma0
                  0x0101ee                  _InitParams
                  0x01f12a                  _InitTCPIPAppConfig
                  0x027a8a                  _InitTmr3
                  0x01f206                  _InitializeBoard
                  0x01f462                  _LEDUpdateUSBStatus
                  0x01f576                  _LFSRRand
                  0x01f534                  _LFSRSeedRand
                  0x0101a6                  _LecFRAM
                  0x010142                  _LecFRAM_Param
                  0x00aa3e                  _LectureLong
                  0x007f5a                  _LectureModbus
                  0x00592e                  _LectureMots
                  0x00ab20                  _LectureReel
                  0x023cb4                  _Lecture_Byte_In_Flash
                  0x024026                  _Lecture_Memoire_Flash_Ligne_Str
                  0x01b60a                  _MACCalcRxChecksum
                  0x01b23c                  _MACDiscardRx
                  0x01b42a                  _MACFlush
                  0x01b944                  _MACGet
                  0x01b976                  _MACGetArray
                  0x01b278                  _MACGetFreeRxSize
                  0x01b302                  _MACGetHeader
                  0x01b0de                  _MACInit
                  0x01b20e                  _MACIsLinked
                  0x01b92c                  _MACIsMemCopyDone
                  0x01b224                  _MACIsTxReady
                  0x01b726                  _MACMemCopyAsync
                  0x01bde6                  _MACPowerDown
                  0x01be1a                  _MACPowerUp
                  0x01ba54                  _MACPut
                  0x01ba8c                  _MACPutArray
                  0x01b3d4                  _MACPutHeader
                  0x01b5d4                  _MACSetReadPtr
                  0x01b56c                  _MACSetReadPtrInRx
                  0x01b59e                  _MACSetWritePtr
                  0x027412                  _MODBUSTCPServer
                  0x01e296                  _MPFSClose
                  0x01e2bc                  _MPFSGet
                  0x01e44c                  _MPFSGetArray
                  0x01e9c0                  _MPFSGetBytesRem
                  0x01ea46                  _MPFSGetEndAddr
                  0x01ea98                  _MPFSGetFilename
                  0x01e936                  _MPFSGetFlags
                  0x01eb22                  _MPFSGetID
                  0x01e676                  _MPFSGetLong
                  0x01e8f0                  _MPFSGetMicrotime
                  0x01eafc                  _MPFSGetPosition
                  0x01e97a                  _MPFSGetSize
                  0x01e9fe                  _MPFSGetStartAddr
                  0x01e8aa                  _MPFSGetTimestamp
                  0x01e08a                  _MPFSInit
                  0x01e0b6                  _MPFSOpen
                  0x01e20c                  _MPFSOpenID
                  0x01e698                  _MPFSSeek
                  0x0057da                  _MPFS_Start
                  0x023ed8                  _MakeAddrDB32
                  0x023f34                  _MakeAddrDB64
                  0x00ad66                  _ModbusErreur
                  0x027544                  _ModbusError
                  0x0057de                  _ModbusUartServer
                  0x009e04                  _ModifParamMetro
                  0x00adc4                  _ModifieVitesseComm
                  0x02493c                  _NBNSTask
                  0x00085a                  _OpenSPI1
                  0x000866                  _OpenSPI3
                  0x000a94                  _OpenUART1
                  0x000aa0                  _OpenUART2
                  0x000aac                  _OpenUART3
                  0x000ab8                  _OpenUART4
                  0x01bffe                  _ProccessCmd
                  0x027ad6                  _ProcessADCSamples
                  0x01eef4                  _ProcessIO
                  0x005886                  _ProcessMessageRecu
                  0x0274b0                  _ProcessReceivedMessage
                  0x00ad94                  _Random
                  0x01bc46                  _ReadPHYReg
                  0x027f3a                  _ReadProgramMemory
                  0x000872                  _ReadSPI1
                  0x000892                  _ReadSPI3
                  0x000b74                  _ReadUART1
                  0x000b8a                  _ReadUART2
                  0x000ba0                  _ReadUART3
                  0x000bb6                  _ReadUART4
                  0x023d00                  _Read_Flash
                  0x027912                  _RebootTask
                  0x0212e2                  _ReceiveUART1
                  0x021358                  _ReceiveUART2
                  0x021496                  _ReceiveUART3
                  0x0215c8                  _ReceiveUART4
                  0x02622c                  _RegulationDoseur
                  0x02632c                  _RegulationPID
                  0x01c7e4                  _ResetCounterMillis
                  0x027b66                  _SPI_Read
                  0x027bd8                  _SPI_Write
                  0x01f3d8                  _SaveAppConfig
                  0x0216fa                  _SendStrUART3
                  0x021726                  _SendStrUART4
                  0x01be3c                  _SetCLKOUT
                  0x023130                  _SetErrorReporter
                  0x027292                  _StackApplications
                  0x0270e6                  _StackInit
                  0x02711e                  _StackTask
                  0x01f6f0                  _StringToIPAddress
                  0x02505a                  _SwapARPPacket
                  0x014b8c                  _TCPAdjustFIFOSize
                  0x012cd6                  _TCPClose
                  0x012f70                  _TCPDiscard
                  0x012c36                  _TCPDisconnect
                  0x0131fa                  _TCPFindArrayEx
                  0x01346a                  _TCPFindEx
                  0x012d20                  _TCPFlush
                  0x012fc8                  _TCPGet
                  0x013042                  _TCPGetArray
                  0x012cf6                  _TCPGetRemoteInfo
                  0x01310e                  _TCPGetRxFIFOFree
                  0x012f44                  _TCPGetTxFIFOFull
                  0x0129ba                  _TCPInit
                  0x012c12                  _TCPIsConnected
                  0x012f90                  _TCPIsGetReady
                  0x012d46                  _TCPIsPutReady
                  0x012a8a                  _TCPOpen
                  0x0131e2                  _TCPPeek
                  0x013138                  _TCPPeekArray
                  0x01397e                  _TCPProcess
                  0x012d94                  _TCPPut
                  0x012e3a                  _TCPPutArray
                  0x012f20                  _TCPPutString
                  0x00570e                  _TCPSocketInitializer
                  0x01348e                  _TCPTick
                  0x012be4                  _TCPWasReset
                  0x02692a                  _TestModbus
                  0x02769a                  _TickConvertToMilliseconds
                  0x027604                  _TickGet
                  0x027636                  _TickGetDiv256
                  0x027668                  _TickGetDiv64K
                  0x027572                  _TickInit
                  0x023ce8                  _Transfert_Page_To_Buffer
                  0x02105e                  _UART1_SetBaudrate
                  0x021232                  _UART1_SetParityNBits
                  0x0211b6                  _UART1_SetStopBit
                  0x0210b4                  _UART2_SetBaudrate
                  0x02128a                  _UART2_SetParityNBits
                  0x0211f4                  _UART2_SetStopBit
                  0x02110a                  _UART3_SetBaudrate
                  0x021160                  _UART4_SetBaudrate
                  0x020ef8                  _UARTs_Init
                  0x020a1c                  _UDPClose
                  0x020cfa                  _UDPDiscard
                  0x020b4a                  _UDPFlush
                  0x020c7a                  _UDPGet
                  0x020cae                  _UDPGetArray
                  0x02067e                  _UDPInit
                  0x020c44                  _UDPIsGetReady
                  0x0209fa                  _UDPIsOpened
                  0x020a8a                  _UDPIsPutReady
                  0x02069e                  _UDPOpenEx
                  0x020d20                  _UDPProcess
                  0x020ac0                  _UDPPut
                  0x020af0                  _UDPPutArray
                  0x020b2c                  _UDPPutString
                  0x020a74                  _UDPSetRxBuffer
                  0x020a5e                  _UDPSetTxBuffer
                  0x0207b8                  _UDPTask
                  0x024248                  _USBCDCEventHandler
                  0x018b98                  _USBCancelIO
                  0x0240ae                  _USBCheckCDCRequest
                  0x018eb6                  _USBCtrlEPAllowDataStage
                  0x018d7e                  _USBCtrlEPAllowStatusStage
                  0x018d3c                  _USBDeviceAttach
                  0x018d2a                  _USBDeviceDetach
                  0x0185e6                  _USBDeviceInit
                  0x0186fa                  _USBDeviceTasks
                  0x018896                  _USBEnableEndpoint
                  0x027e84                  _USBSleepOnSuspend
                  0x018a0a                  _USBStallEndpoint
                  0x0188d0                  _USBTransferOnePacket
                  0x005630                  _USB_CD_Ptr
                  0x005632                  _USB_SD_Ptr
                  0x01bef0                  _USB_enqMsg
                  0x01f4d0                  _USER_USB_CALLBACK_EVENT_HANDLER
                  0x0266ee                  _US_Init
                  0x0266f8                  _US_RunUserInitStateMachine
                  0x026906                  _US_SetSwitch1
                  0x026918                  _US_SetSwitch2
                  0x01c804                  _UpdateB40ADI
                  0x0111a8                  _ValEntTOR
                  0x00ac4a                  _ValidationCodeMetrologie
                  0x023c5a                  _Wait_Flash_Ready
                  0x01bd8e                  _WritePHYReg
                  0x0008b2                  _WriteSPI1
                  0x0008c4                  _WriteSPI3
                  0x023c6a                  _Write_Flash
                  0x025408                  _XEEBeginRead
                  0x02552c                  _XEEBeginWrite
                  0x025464                  _XEEEndRead
                  0x0255b4                  _XEEEndWrite
                  0x0253ea                  _XEEInit
                  0x0256ae                  _XEEIsBusy
                  0x025420                  _XEERead
                  0x02546e                  _XEEReadArray
                  0x025544                  _XEEWrite
                  0x025586                  _XEEWriteArray
                  0x00079a                  __AddressError
                  0x000750                  __C1Interrupt
                  0x0005ba                  __DMA0Interrupt
                  0x0007ac                  __DMACError
                  0x0007b2                  __DefaultInterrupt
                  0x0007b6                  __HardTrapError
                  0x00065e                  __INT1Interrupt
                  0x000698                  __INT2Interrupt
                  0x0006b4                  __INT3Interrupt
                  0x0006fa                  __INT4Interrupt
                  0x0007a6                  __MathError
                  0x000794                  __OscillatorFail
                  0x0007ba                  __SoftTrapError
                  0x0007a0                  __StackError
                  0x0276b4                  __T1Interrupt
                  0x000392                  __U1RXInterrupt
                  0x00041c                  __U2RXInterrupt
                  0x0004a6                  __U3RXInterrupt
                  0x000530                  __U4RXInterrupt
                  0x000728                  __USB1Interrupt
                  0x003876                  ___adddf3
                  0x000bce                  ___addsf3
                  0x003984                  ___divdf3
                  0x003ea2                  ___divdi3
                  0x000c88                  ___divsf3
                  0x000d0c                  ___divsi3
                  0x003970                  ___eqdf2
                  0x000d2a                  ___eqsf2
                  0x003acc                  ___extendsfdf2
                  0x000d32                  ___fixsfsi
                  0x003b0a                  ___fixunsdfdi
                  0x003b6c                  ___fixunsdfsi
                  0x000d74                  ___fixunssfsi
                  0x000f1e                  ___floatdisf
                  0x000daa                  ___floatsisf
                  0x003bb8                  ___floatundidf
                  0x000f3e                  ___floatundisf
                  0x003c0e                  ___floatunsidf
                  0x000db0                  ___floatunsisf
                  0x00397a                  ___gedf2
                  0x000d2e                  ___gesf2
                  0x00397a                  ___gtdf2
                  0x000d2e                  ___gtsf2
                  0x003970                  ___ledf2
                  0x000d2a                  ___lesf2
                  0x003970                  ___ltdf2
                  0x000d2a                  ___ltsf2
                  0x003f06                  ___moddi3
                  0x003c4c                  ___muldf3
                  0x003f66                  ___muldi3
                  0x003d3a                  ___mulp32eds3
                  0x003d3a                  ___mulp32peds3
                  0x000e5a                  ___mulsf3
                  0x003d3a                  ___mulsi3
                  0x003a38                  ___nedf2
                  0x003d36                  ___subdf3
                  0x000bcc                  ___subsf3
                  0x003e84                  ___udivdi3
                  0x003db4                  ___udivmoddi3
                  0x000ec2                  ___udivsi3
                  0x003e96                  ___umoddi3
                  0x000ee2                  ___umodsi3
                  0x00409c                  ___umuldi3
                  0x00400e                  __dPropagateNaN
                  0x000238                  __data_init
                  0x000238                  __data_init_extended
                  0x003fbc                  __dcompare
                  0x003a42                  __dpack
                  0x003abc                  __dreturnNaN
                  0x00402a                  __dtype
                  0x00404e                  __dunpack
                  0x003a9a                  __dunpack2
                  0x003ac2                  __dunpack2exit
                  0x000e3a                  __fPropagateNaN
                  0x000e4c                  __fbopExit
                  0x000e54                  __fbopReturnNaN
                  0x000ee8                  __fcompare
                  0x000db4                  __fpack
                  0x000e00                  __funpack
                  0x000e2a                  __funpack2
                  0x0021de                  __printf_0
                  0x0021de                  __printf_cdnopsuxX
                  0x0021de                  __printf_cdnopuxX
                  0x0021de                  __printf_s
                  0x00022c                  __psv_init
                  0x000200                  __resetPRI
                  0x001404                  __sprintf_cdfFnopsuxX
                  0x001404                  __sprintf_cdfFnopuxX
                  0x001404                  __sprintf_cdnopsuxX
                  0x001404                  __sprintf_cdnopuxX
                  0x001590                  __vfprintf_0
                  0x001590                  __vfprintf_cdfFnopsuxX
                  0x001590                  __vfprintf_cdfFnopuxX
                  0x001590                  __vfprintf_cdnopsuxX
                  0x001590                  __vfprintf_cdnopuxX
                  0x001590                  __vfprintf_s
                  0x005638                  _abBitReverseTable16
                  0x01cca6                  _accept
                  0x024568                  _app_InstanceCommand
                  0x024772                  _app_ObjectCommand
                  0x005746                  _app_sObject
                  0x00118a                  _atof
                  0x001194                  _atoi
                  0x0011d6                  _atol
                  0x01caea                  _bind
                  0x01fabc                  _btohexa_high
                  0x01fade                  _btohexa_low
                  0x01d3aa                  _closesocket
                  0x0055b8                  _configDescriptor1
                  0x01cdec                  _connect
                  0x0123b8                  _conversion_poids
                  0x005648                  _crc_table32
                  0x0055a6                  _device_dsc
                  0x025a36                  _dpv1_InstanceCommand
                  0x025b92                  _dpv1_ObjectCommand
                  0x005794                  _dpv1_sObject
                  0x008018                  _envoieLongPF
                  0x008078                  _envoieLongPf
                  0x0080a4                  _envoieReelPF
                  0x008150                  _envoieReelPf
                  0x012054                  _envoyer_reel
                  0x011ac2                  _etatSortieTOR
                  0x003c12                  _frexp
                  0x003c12                  _frexpl
                  0x011ff6                  _gestion_comm_serie
                  0x010f5a                  _gestion_cycle
                  0x010cc2                  _gestion_defauts
                  0x011d42                  _gestion_poids_debit
                  0x010618                  _gestion_profibus
                  0x011554                  _gestion_totalisateurs
                  0x0111e0                  _gestion_vitesse
                  0x01d348                  _gethostname
                  0x02428e                  _getsUSBUSART
                  0x01fa52                  _hexatob
                  0x0007be                  _isspace
                  0x012438                  _lecture_entrees_TOR
                  0x01cb8a                  _listen
                  0x001280                  _ltoa
                  0x01eb7c                  _main
                  0x0012a4                  _memcmp
                  0x0012d2                  _memcpy
                  0x0012e4                  _memset
                  0x012132                  _moyenne_glissante_debit
                  0x012156                  _moyenne_glissante_poids
                  0x010844                  _process_plcd
                  0x024322                  _putUSBUSART
                  0x0013fa                  _putchar
                  0x0243a4                  _putrsUSBUSART
                  0x000ac4                  _putsUART1
                  0x000af0                  _putsUART2
                  0x000b1c                  _putsUART3
                  0x000b48                  _putsUART4
                  0x01be8c                  _putsUSB
                  0x02434e                  _putsUSBUSART
                  0x001308                  _rand
                  0x01d150                  _recv
                  0x01d1e8                  _recvfrom
                  0x0055fc                  _sd000
                  0x005600                  _sd001
                  0x005618                  _sd002
                  0x01cf6c                  _send
                  0x01cf8c                  _sendto
                  0x01ca50                  _socket
                  0x011af6                  _sortiesTOR
                  0x001334                  _sprintf
                  0x0012f6                  _srand
                  0x0037d4                  _strchr
                  0x00135e                  _strcmp
                  0x001370                  _strcpy
                  0x003780                  _strcspn
                  0x01fafc                  _stricmppgm2ram
                  0x001380                  _strlen
                  0x01fd1c                  _strnchr
                  0x001392                  _strncpy
                  0x01fd6a                  _strncpy_m
                  0x0037aa                  _strspn
                  0x001182                  _strtod
                  0x000f9c                  _strtof
                  0x0013b8                  _strtok
                  0x01fc92                  _strupr
                  0x01fbb0                  _swapl
                  0x01fb94                  _swaps
                  0x01f9d2                  _uitoa
                  0x001230                  _ultoa
                  0x01186c                  _verif_totaux
                  0x00234e                  _vfprintf
                  0x027eda                  build/XC16_dsPIC33EP512MU810/debug/B40/abcc_remap.o:_abcc_RemapRespMsgSent
                  0x0221e8                  build/XC16_dsPIC33EP512MU810/debug/B40/spi/abcc_spi_drv.o:_drv_WdTimeoutHandler
                  0x0221a2                  build/XC16_dsPIC33EP512MU810/debug/B40/spi/abcc_spi_drv.o:_spi_drv_DataReceived
                  0x0267ee                  build/XC16_dsPIC33EP512MU810/debug/B40/user_setup.o:_US_ProcessRespMsg

Memory Configuration

Name             Origin             Length             Attributes
data             0x001000           0x00d000           a !xr
reset            0x000000           0x000004  
ivt              0x000004           0x0001fc  
program          0x000200           0x0555fe           xr
auxflash         0x7fc000           0x003ff8           xr
FGS              0xf80004           0x000002  
FOSCSEL          0xf80006           0x000002  
FOSC             0xf80008           0x000002  
FWDT             0xf8000a           0x000002  
FPOR             0xf8000c           0x000002  
FICD             0xf8000e           0x000002  
FAS              0xf80010           0x000002  
FUID0            0xf80012           0x000002  
*default*        0x000000           0xffffffff  

Linker script and memory map

LOAD build/XC16_dsPIC33EP512MU810/debug/B40/par/abcc_handler_par.o
LOAD build/XC16_dsPIC33EP512MU810/debug/B40/par/abcc_par_drv.o
LOAD build/XC16_dsPIC33EP512MU810/debug/B40/spi/abcc_crc32.o
LOAD build/XC16_dsPIC33EP512MU810/debug/B40/spi/abcc_handler_spi.o
LOAD build/XC16_dsPIC33EP512MU810/debug/B40/spi/abcc_spi_drv.o
LOAD build/XC16_dsPIC33EP512MU810/debug/B40/abcc_cbf.o
LOAD build/XC16_dsPIC33EP512MU810/debug/B40/abcc_debug_err.o
LOAD build/XC16_dsPIC33EP512MU810/debug/B40/abcc_handler.o
LOAD build/XC16_dsPIC33EP512MU810/debug/B40/abcc_link.o
LOAD build/XC16_dsPIC33EP512MU810/debug/B40/abcc_mem.o
LOAD build/XC16_dsPIC33EP512MU810/debug/B40/abcc_remap.o
LOAD build/XC16_dsPIC33EP512MU810/debug/B40/abcc_setup.o
LOAD build/XC16_dsPIC33EP512MU810/debug/B40/abcc_sys_adapt.o
LOAD build/XC16_dsPIC33EP512MU810/debug/B40/abcc_timer.o
LOAD build/XC16_dsPIC33EP512MU810/debug/B40/ad_obj.o
LOAD build/XC16_dsPIC33EP512MU810/debug/B40/app_obj.o
LOAD build/XC16_dsPIC33EP512MU810/debug/B40/dpv1.o
LOAD build/XC16_dsPIC33EP512MU810/debug/B40/user_adi.o
LOAD build/XC16_dsPIC33EP512MU810/debug/B40/user_setup.o
LOAD build/XC16_dsPIC33EP512MU810/debug/ECAN/ECAN1Drv.o
LOAD build/XC16_dsPIC33EP512MU810/debug/BerkeleyTCPClient.o
LOAD build/XC16_dsPIC33EP512MU810/debug/BerkeleyTCPServer.o
LOAD build/XC16_dsPIC33EP512MU810/debug/BerkeleyUDPClient.o
LOAD build/XC16_dsPIC33EP512MU810/debug/MODBUSTCPServer.o
LOAD build/XC16_dsPIC33EP512MU810/debug/Regul.o
LOAD build/XC16_dsPIC33EP512MU810/debug/Pesage.o
LOAD build/XC16_dsPIC33EP512MU810/debug/Process.o
LOAD build/XC16_dsPIC33EP512MU810/debug/TCPIPStack/Announce.o
LOAD build/XC16_dsPIC33EP512MU810/debug/TCPIPStack/ARCFOUR.o
LOAD build/XC16_dsPIC33EP512MU810/debug/TCPIPStack/ARP.o
LOAD build/XC16_dsPIC33EP512MU810/debug/TCPIPStack/AutoIP.o
LOAD build/XC16_dsPIC33EP512MU810/debug/TCPIPStack/BerkeleyAPI.o
LOAD build/XC16_dsPIC33EP512MU810/debug/TCPIPStack/BigInt.o
LOAD build/XC16_dsPIC33EP512MU810/debug/TCPIPStack/Delay.o
LOAD build/XC16_dsPIC33EP512MU810/debug/TCPIPStack/DHCP.o
LOAD build/XC16_dsPIC33EP512MU810/debug/TCPIPStack/DHCPs.o
LOAD build/XC16_dsPIC33EP512MU810/debug/TCPIPStack/DNS.o
LOAD build/XC16_dsPIC33EP512MU810/debug/TCPIPStack/DNSs.o
LOAD build/XC16_dsPIC33EP512MU810/debug/TCPIPStack/DynDNS.o
LOAD build/XC16_dsPIC33EP512MU810/debug/TCPIPStack/ENC28J60.o
LOAD build/XC16_dsPIC33EP512MU810/debug/TCPIPStack/FileSystem.o
LOAD build/XC16_dsPIC33EP512MU810/debug/TCPIPStack/FTP.o
LOAD build/XC16_dsPIC33EP512MU810/debug/TCPIPStack/Hashes.o
LOAD build/XC16_dsPIC33EP512MU810/debug/TCPIPStack/Helpers.o
LOAD build/XC16_dsPIC33EP512MU810/debug/TCPIPStack/HTTP2.o
LOAD build/XC16_dsPIC33EP512MU810/debug/TCPIPStack/ICMP.o
LOAD build/XC16_dsPIC33EP512MU810/debug/TCPIPStack/IP.o
LOAD build/XC16_dsPIC33EP512MU810/debug/TCPIPStack/LCDBlocking.o
LOAD build/XC16_dsPIC33EP512MU810/debug/TCPIPStack/MPFS2.o
LOAD build/XC16_dsPIC33EP512MU810/debug/TCPIPStack/NBNS.o
LOAD build/XC16_dsPIC33EP512MU810/debug/TCPIPStack/Random.o
LOAD build/XC16_dsPIC33EP512MU810/debug/TCPIPStack/Reboot.o
LOAD build/XC16_dsPIC33EP512MU810/debug/TCPIPStack/RSA.o
LOAD build/XC16_dsPIC33EP512MU810/debug/TCPIPStack/SMTP.o
LOAD build/XC16_dsPIC33EP512MU810/debug/TCPIPStack/SNMP.o
LOAD build/XC16_dsPIC33EP512MU810/debug/TCPIPStack/SNMPv3.o
LOAD build/XC16_dsPIC33EP512MU810/debug/TCPIPStack/SNMPv3USM.o
LOAD build/XC16_dsPIC33EP512MU810/debug/TCPIPStack/SNTP.o
LOAD build/XC16_dsPIC33EP512MU810/debug/TCPIPStack/SPIEEPROM.o
LOAD build/XC16_dsPIC33EP512MU810/debug/TCPIPStack/SPIFlash.o
LOAD build/XC16_dsPIC33EP512MU810/debug/TCPIPStack/SPIRAM.o
LOAD build/XC16_dsPIC33EP512MU810/debug/TCPIPStack/SSL.o
LOAD build/XC16_dsPIC33EP512MU810/debug/TCPIPStack/StackTsk.o
LOAD build/XC16_dsPIC33EP512MU810/debug/TCPIPStack/TCP.o
LOAD build/XC16_dsPIC33EP512MU810/debug/TCPIPStack/TCPPerformanceTest.o
LOAD build/XC16_dsPIC33EP512MU810/debug/TCPIPStack/Telnet.o
LOAD build/XC16_dsPIC33EP512MU810/debug/TCPIPStack/TFTPc.o
LOAD build/XC16_dsPIC33EP512MU810/debug/TCPIPStack/Tick.o
LOAD build/XC16_dsPIC33EP512MU810/debug/TCPIPStack/UART.o
LOAD build/XC16_dsPIC33EP512MU810/debug/TCPIPStack/UART2TCPBridge.o
LOAD build/XC16_dsPIC33EP512MU810/debug/TCPIPStack/UDP.o
LOAD build/XC16_dsPIC33EP512MU810/debug/TCPIPStack/UDPPerformanceTest.o
LOAD build/XC16_dsPIC33EP512MU810/debug/TCPIPStack/ZeroconfHelper.o
LOAD build/XC16_dsPIC33EP512MU810/debug/TCPIPStack/ZeroconfLinkLocal.o
LOAD build/XC16_dsPIC33EP512MU810/debug/TCPIPStack/ZeroconfMulticastDNS.o
LOAD build/XC16_dsPIC33EP512MU810/debug/usb/src/usb_device.o
LOAD build/XC16_dsPIC33EP512MU810/debug/usb/src/usb_device_cdc.o
LOAD build/XC16_dsPIC33EP512MU810/debug/usb/src/usb_hal_dspic33e.o
LOAD build/XC16_dsPIC33EP512MU810/debug/configuration_bits.o
LOAD build/XC16_dsPIC33EP512MU810/debug/interrupts.o
LOAD build/XC16_dsPIC33EP512MU810/debug/main.o
LOAD build/XC16_dsPIC33EP512MU810/debug/system.o
LOAD build/XC16_dsPIC33EP512MU810/debug/traps.o
LOAD build/XC16_dsPIC33EP512MU810/debug/user.o
LOAD build/XC16_dsPIC33EP512MU810/debug/MPFSImg2.o
LOAD build/XC16_dsPIC33EP512MU810/debug/CustomHTTPApp.o
LOAD build/XC16_dsPIC33EP512MU810/debug/AD7190.o
LOAD build/XC16_dsPIC33EP512MU810/debug/ADComm.o
LOAD build/XC16_dsPIC33EP512MU810/debug/UARTsComm.o
LOAD build/XC16_dsPIC33EP512MU810/debug/MemFlash.o
LOAD build/XC16_dsPIC33EP512MU810/debug/ADC10bitsDrv.o
LOAD build/XC16_dsPIC33EP512MU810/debug/SPIFRAM.o
LOAD build/XC16_dsPIC33EP512MU810/debug/usb_descriptors.o
LOAD build/XC16_dsPIC33EP512MU810/debug/ModbusUartServer.o

reserve_data_0x1000
                    0x1000         0x1c
                    0x101c                  . = 0x1c
 *fill*             0x1000         0x1c00

reserve_data_0x101c
                    0x101c          0x2
                    0x101e                  . = 0x2
 *fill*             0x101c          0x200

reserve_data_0x101e
                    0x101e          0x2
                    0x1020                  . = 0x2
 *fill*             0x101e          0x200

reserve_data_0x1020
                    0x1020          0x2
                    0x1022                  . = 0x2
 *fill*             0x1020          0x200

reserve_data_0x1022
                    0x1022          0x2
                    0x1024                  . = 0x2
 *fill*             0x1022          0x200

reserve_data_0x1024
                    0x1024          0x4
                    0x1028                  . = 0x4
 *fill*             0x1024          0x400

reserve_data_0x1028
                    0x1028         0x28
                    0x1050                  . = 0x28
 *fill*             0x1028         0x2800
                    0x0001                  __MPLAB_BUILD = 0x1
                    0x0001                  __MPLAB_DEBUG = 0x1
                    0x0001                  __DEBUG = 0x1
                    0x0001                  __MPLAB_DEBUGGER_PK3 = 0x1
LOAD c:/program files (x86)/microchip/xc16/v1.24/bin/bin/../../lib/dsPIC33E\libp33EP512MU810-elf.a
                    0xf80004                  __FGS = 0xf80004
                    0xf80006                  __FOSCSEL = 0xf80006
                    0xf80008                  __FOSC = 0xf80008
                    0xf8000a                  __FWDT = 0xf8000a
                    0xf8000c                  __FPOR = 0xf8000c
                    0xf8000e                  __FICD = 0xf8000e
                    0xf80010                  __FAS = 0xf80010
                    0xf80012                  __FUID0 = 0xf80012
                    0x0004                  __IVT_BASE = 0x4
                    0x1000                  __DATA_BASE = 0x1000
                    0xd000                  __DATA_LENGTH = 0xd000
                    0x9000                  __YDATA_BASE = 0x9000
                    0xd000                  __DMA_BASE = 0xd000
                    0xdfff                  __DMA_END = 0xdfff
                    0x7fc000                  __CODE_BASE = 0x7fc000
                    0x3ffa                  __CODE_LENGTH = 0x3ffa

.reset            0x000000          0x4
                  0x000000          0x2 SHORT 0x200 ABSOLUTE (__reset)
                  0x000001          0x2 SHORT 0x4
                  0x000002          0x2 SHORT 0x0 ((ABSOLUTE (__reset) >> 0x10) & 0x7f)
                  0x000003          0x2 SHORT 0x0

.text             0x000200       0x3ee0
 *(.init)
 .init            0x000200         0x38 c:/program files (x86)/microchip/xc16/v1.24/bin/bin/../../lib\libpic30-elf.a(crt0_extendedep.o)
                  0x000200                  __resetPRI
                  0x000200                  __reset
                  0x00022c                  __psv_init
 .init            0x000238         0x9a c:/program files (x86)/microchip/xc16/v1.24/bin/bin/../../lib\libpic30-elf.a(data_init_extendedep.o)
                  0x000238                  __data_init
                  0x000238                  __data_init_extended
 *(.user_init)
 *(.handle)
 .handle          0x0002d2         0xc0 jump_table
 *(.isr*)
 .isr.text        0x000392        0x402 build/XC16_dsPIC33EP512MU810/debug/interrupts.o
                  0x000392                  __U1RXInterrupt
                  0x00041c                  __U2RXInterrupt
                  0x0004a6                  __U3RXInterrupt
                  0x000530                  __U4RXInterrupt
                  0x0005ba                  __DMA0Interrupt
                  0x00065e                  __INT1Interrupt
                  0x000698                  __INT2Interrupt
                  0x0006b4                  __INT3Interrupt
                  0x0006fa                  __INT4Interrupt
                  0x000728                  __USB1Interrupt
                  0x000750                  __C1Interrupt
 .isr.text        0x000794         0x2a build/XC16_dsPIC33EP512MU810/debug/traps.o
                  0x000794                  __OscillatorFail
                  0x00079a                  __AddressError
                  0x0007a0                  __StackError
                  0x0007a6                  __MathError
                  0x0007ac                  __DMACError
                  0x0007b2                  __DefaultInterrupt
                  0x0007b6                  __HardTrapError
                  0x0007ba                  __SoftTrapError
 *(.libc)
 .libc            0x0007be         0x10 c:/program files (x86)/microchip/xc16/v1.24/bin/bin/../../lib\libc-elf.a(isspace.epeso)
                  0x0007be                  _isspace
 .libc            0x0007ce         0x60 c:/program files (x86)/microchip/xc16/v1.24/bin/bin/../../lib\libpic30-elf.a(writeep.eo)
                  0x0007ce                  _write
 *(.libm)
 *(.libdsp)
 *(.lib*)
 .libperi         0x00082e          0xc c:/program files (x86)/microchip/xc16/v1.24/bin/bin/../../lib/dsPIC33E\libp33EP512MU810-elf.a(CloseSPI1.o)
                  0x00082e                  _CloseSPI1
 .libperi         0x00083a          0xc c:/program files (x86)/microchip/xc16/v1.24/bin/bin/../../lib/dsPIC33E\libp33EP512MU810-elf.a(CloseSPI3.o)
                  0x00083a                  _CloseSPI3
 .libperi         0x000846          0xa c:/program files (x86)/microchip/xc16/v1.24/bin/bin/../../lib/dsPIC33E\libp33EP512MU810-elf.a(DataRdySPI1.o)
                  0x000846                  _DataRdySPI1
 .libperi         0x000850          0xa c:/program files (x86)/microchip/xc16/v1.24/bin/bin/../../lib/dsPIC33E\libp33EP512MU810-elf.a(DataRdySPI3.o)
                  0x000850                  _DataRdySPI3
 .libperi         0x00085a          0xc c:/program files (x86)/microchip/xc16/v1.24/bin/bin/../../lib/dsPIC33E\libp33EP512MU810-elf.a(OpenSPI1.o)
                  0x00085a                  _OpenSPI1
 .libperi         0x000866          0xc c:/program files (x86)/microchip/xc16/v1.24/bin/bin/../../lib/dsPIC33E\libp33EP512MU810-elf.a(OpenSPI3.o)
                  0x000866                  _OpenSPI3
 .libperi         0x000872         0x20 c:/program files (x86)/microchip/xc16/v1.24/bin/bin/../../lib/dsPIC33E\libp33EP512MU810-elf.a(ReadSPI1.o)
                  0x000872                  _ReadSPI1
 .libperi         0x000892         0x20 c:/program files (x86)/microchip/xc16/v1.24/bin/bin/../../lib/dsPIC33E\libp33EP512MU810-elf.a(ReadSPI3.o)
                  0x000892                  _ReadSPI3
 .libperi         0x0008b2         0x12 c:/program files (x86)/microchip/xc16/v1.24/bin/bin/../../lib/dsPIC33E\libp33EP512MU810-elf.a(WriteSPI1.o)
                  0x0008b2                  _WriteSPI1
 .libperi         0x0008c4         0x12 c:/program files (x86)/microchip/xc16/v1.24/bin/bin/../../lib/dsPIC33E\libp33EP512MU810-elf.a(WriteSPI3.o)
                  0x0008c4                  _WriteSPI3
 .libperi         0x0008d6          0xe c:/program files (x86)/microchip/xc16/v1.24/bin/bin/../../lib/dsPIC33E\libp33EP512MU810-elf.a(BusyUART2.o)
                  0x0008d6                  _BusyUART2
 .libperi         0x0008e4          0xe c:/program files (x86)/microchip/xc16/v1.24/bin/bin/../../lib/dsPIC33E\libp33EP512MU810-elf.a(BusyUART3.o)
                  0x0008e4                  _BusyUART3
 .libperi         0x0008f2          0xe c:/program files (x86)/microchip/xc16/v1.24/bin/bin/../../lib/dsPIC33E\libp33EP512MU810-elf.a(BusyUART4.o)
                  0x0008f2                  _BusyUART4
 .libperi         0x000900         0x10 c:/program files (x86)/microchip/xc16/v1.24/bin/bin/../../lib/dsPIC33E\libp33EP512MU810-elf.a(CloseUART1.o)
                  0x000900                  _CloseUART1
 .libperi         0x000910         0x10 c:/program files (x86)/microchip/xc16/v1.24/bin/bin/../../lib/dsPIC33E\libp33EP512MU810-elf.a(CloseUART2.o)
                  0x000910                  _CloseUART2
 .libperi         0x000920         0x10 c:/program files (x86)/microchip/xc16/v1.24/bin/bin/../../lib/dsPIC33E\libp33EP512MU810-elf.a(CloseUART3.o)
                  0x000920                  _CloseUART3
 .libperi         0x000930         0x10 c:/program files (x86)/microchip/xc16/v1.24/bin/bin/../../lib/dsPIC33E\libp33EP512MU810-elf.a(CloseUART4.o)
                  0x000930                  _CloseUART4
 .libperi         0x000940         0x4c c:/program files (x86)/microchip/xc16/v1.24/bin/bin/../../lib/dsPIC33E\libp33EP512MU810-elf.a(ConfigIntUART1.o)
                  0x000940                  _ConfigIntUART1
 .libperi         0x00098c         0x4c c:/program files (x86)/microchip/xc16/v1.24/bin/bin/../../lib/dsPIC33E\libp33EP512MU810-elf.a(ConfigIntUART2.o)
                  0x00098c                  _ConfigIntUART2
 .libperi         0x0009d8         0x4c c:/program files (x86)/microchip/xc16/v1.24/bin/bin/../../lib/dsPIC33E\libp33EP512MU810-elf.a(ConfigIntUART3.o)
                  0x0009d8                  _ConfigIntUART3
 .libperi         0x000a24         0x48 c:/program files (x86)/microchip/xc16/v1.24/bin/bin/../../lib/dsPIC33E\libp33EP512MU810-elf.a(ConfigIntUART4.o)
                  0x000a24                  _ConfigIntUART4
 .libperi         0x000a6c          0xa c:/program files (x86)/microchip/xc16/v1.24/bin/bin/../../lib/dsPIC33E\libp33EP512MU810-elf.a(DataRdyUART1.o)
                  0x000a6c                  _DataRdyUART1
 .libperi         0x000a76          0xa c:/program files (x86)/microchip/xc16/v1.24/bin/bin/../../lib/dsPIC33E\libp33EP512MU810-elf.a(DataRdyUART2.o)
                  0x000a76                  _DataRdyUART2
 .libperi         0x000a80          0xa c:/program files (x86)/microchip/xc16/v1.24/bin/bin/../../lib/dsPIC33E\libp33EP512MU810-elf.a(DataRdyUART3.o)
                  0x000a80                  _DataRdyUART3
 .libperi         0x000a8a          0xa c:/program files (x86)/microchip/xc16/v1.24/bin/bin/../../lib/dsPIC33E\libp33EP512MU810-elf.a(DataRdyUART4.o)
                  0x000a8a                  _DataRdyUART4
 .libperi         0x000a94          0xc c:/program files (x86)/microchip/xc16/v1.24/bin/bin/../../lib/dsPIC33E\libp33EP512MU810-elf.a(OpenUART1.o)
                  0x000a94                  _OpenUART1
 .libperi         0x000aa0          0xc c:/program files (x86)/microchip/xc16/v1.24/bin/bin/../../lib/dsPIC33E\libp33EP512MU810-elf.a(OpenUART2.o)
                  0x000aa0                  _OpenUART2
 .libperi         0x000aac          0xc c:/program files (x86)/microchip/xc16/v1.24/bin/bin/../../lib/dsPIC33E\libp33EP512MU810-elf.a(OpenUART3.o)
                  0x000aac                  _OpenUART3
 .libperi         0x000ab8          0xc c:/program files (x86)/microchip/xc16/v1.24/bin/bin/../../lib/dsPIC33E\libp33EP512MU810-elf.a(OpenUART4.o)
                  0x000ab8                  _OpenUART4
 .libperi         0x000ac4         0x2c c:/program files (x86)/microchip/xc16/v1.24/bin/bin/../../lib/dsPIC33E\libp33EP512MU810-elf.a(putsUART1.o)
                  0x000ac4                  _putsUART1
 .libperi         0x000af0         0x2c c:/program files (x86)/microchip/xc16/v1.24/bin/bin/../../lib/dsPIC33E\libp33EP512MU810-elf.a(putsUART2.o)
                  0x000af0                  _putsUART2
 .libperi         0x000b1c         0x2c c:/program files (x86)/microchip/xc16/v1.24/bin/bin/../../lib/dsPIC33E\libp33EP512MU810-elf.a(putsUART3.o)
                  0x000b1c                  _putsUART3
 .libperi         0x000b48         0x2c c:/program files (x86)/microchip/xc16/v1.24/bin/bin/../../lib/dsPIC33E\libp33EP512MU810-elf.a(putsUART4.o)
                  0x000b48                  _putsUART4
 .libperi         0x000b74         0x16 c:/program files (x86)/microchip/xc16/v1.24/bin/bin/../../lib/dsPIC33E\libp33EP512MU810-elf.a(ReadUART1.o)
                  0x000b74                  _ReadUART1
 .libperi         0x000b8a         0x16 c:/program files (x86)/microchip/xc16/v1.24/bin/bin/../../lib/dsPIC33E\libp33EP512MU810-elf.a(ReadUART2.o)
                  0x000b8a                  _ReadUART2
 .libperi         0x000ba0         0x16 c:/program files (x86)/microchip/xc16/v1.24/bin/bin/../../lib/dsPIC33E\libp33EP512MU810-elf.a(ReadUART3.o)
                  0x000ba0                  _ReadUART3
 .libperi         0x000bb6         0x16 c:/program files (x86)/microchip/xc16/v1.24/bin/bin/../../lib/dsPIC33E\libp33EP512MU810-elf.a(ReadUART4.o)
                  0x000bb6                  _ReadUART4
 .libm.subsf3     0x000bcc         0xbc c:/program files (x86)/microchip/xc16/v1.24/bin/bin/../../lib\libm-elf.a(addsf3.epeo)
                  0x000bcc                  ___subsf3
                  0x000bce                  ___addsf3
 .libm.divfs3     0x000c88         0x84 c:/program files (x86)/microchip/xc16/v1.24/bin/bin/../../lib\libm-elf.a(divsf3.epeo)
                  0x000c88                  ___divsf3
 .libm.divsi3     0x000d0c         0x1e c:/program files (x86)/microchip/xc16/v1.24/bin/bin/../../lib\libm-elf.a(divsi3.epeo)
                  0x000d0c                  ___divsi3
 .libm.eqsf2      0x000d2a          0x4 c:/program files (x86)/microchip/xc16/v1.24/bin/bin/../../lib\libm-elf.a(feqltle.epeo)
                  0x000d2a                  ___eqsf2
                  0x000d2a                  ___ltsf2
                  0x000d2a                  ___lesf2
 .libm.gtsf2      0x000d2e          0x4 c:/program files (x86)/microchip/xc16/v1.24/bin/bin/../../lib\libm-elf.a(fgtge.epeo)
                  0x000d2e                  ___gesf2
                  0x000d2e                  ___gtsf2
 .libm.fixsfsi    0x000d32         0x42 c:/program files (x86)/microchip/xc16/v1.24/bin/bin/../../lib\libm-elf.a(fixsfsi.epeo)
                  0x000d32                  _(float, int, long long, short, float, short, int)
 .libm.fixunssfsi
                  0x000d74         0x36 c:/program files (x86)/microchip/xc16/v1.24/bin/bin/../../lib\libm-elf.a(fixunssfsi.epeo)
                  0x000d74                  ___fixunssfsi
 .libm.floatsisf
                  0x000daa          0x6 c:/program files (x86)/microchip/xc16/v1.24/bin/bin/../../lib\libm-elf.a(floatsisf.epeo)
                  0x000daa                  ___floatsisf
 .libm.floatunsisf
                  0x000db0          0x4 c:/program files (x86)/microchip/xc16/v1.24/bin/bin/../../lib\libm-elf.a(floatunsisf.epeo)
                  0x000db0                  ___floatunsisf
 .libm.fpack      0x000db4         0x4c c:/program files (x86)/microchip/xc16/v1.24/bin/bin/../../lib\libm-elf.a(fpack.epeo)
                  0x000db4                  __fpack
 .libm.funpack    0x000e00         0x2a c:/program files (x86)/microchip/xc16/v1.24/bin/bin/../../lib\libm-elf.a(funpack.epeo)
                  0x000e00                  __funpack
 .libm.funpack2
                  0x000e2a         0x10 c:/program files (x86)/microchip/xc16/v1.24/bin/bin/../../lib\libm-elf.a(funpack2.epeo)
                  0x000e2a                  __funpack2
 .libm.fPropagateNaN
                  0x000e3a         0x12 c:/program files (x86)/microchip/xc16/v1.24/bin/bin/../../lib\libm-elf.a(futil.epeo)
                  0x000e3a                  __fPropagateNaN
 .libm.fbobExit
                  0x000e4c          0x8 c:/program files (x86)/microchip/xc16/v1.24/bin/bin/../../lib\libm-elf.a(futil.epeo)
                  0x000e4c                  __fbopExit
 .libm.fbopReturnNaN
                  0x000e54          0x6 c:/program files (x86)/microchip/xc16/v1.24/bin/bin/../../lib\libm-elf.a(futil.epeo)
                  0x000e54                  __fbopReturnNaN
 .libm.mulsf3     0x000e5a         0x68 c:/program files (x86)/microchip/xc16/v1.24/bin/bin/../../lib\libm-elf.a(mulsf3.epeo)
                  0x000e5a                  ___mulsf3
 .libm.udivsi3    0x000ec2         0x20 c:/program files (x86)/microchip/xc16/v1.24/bin/bin/../../lib\libm-elf.a(udivsi3.epeo)
                  0x000ec2                  ___udivsi3
 .libm.umodsi3    0x000ee2          0x6 c:/program files (x86)/microchip/xc16/v1.24/bin/bin/../../lib\libm-elf.a(umodsi3.epeo)
                  0x000ee2                  ___umodsi3
 .libm.fcompare
                  0x000ee8         0x36 c:/program files (x86)/microchip/xc16/v1.24/bin/bin/../../lib\libm-elf.a(fcompare.epeo)
                  0x000ee8                  __fcompare
 .libm.floatdisf
                  0x000f1e         0x20 c:/program files (x86)/microchip/xc16/v1.24/bin/bin/../../lib\libm-elf.a(floatdisf.epeo)
                  0x000f1e                  ___floatdisf
 .libm.floatundisf
                  0x000f3e         0x5e c:/program files (x86)/microchip/xc16/v1.24/bin/bin/../../lib\libm-elf.a(floatundisf.epeo)
                  0x000f3e                  ___floatundisf
 .libc.strtof     0x000f9c        0x1e6 c:/program files (x86)/microchip/xc16/v1.24/bin/bin/../../lib\libc-elf.a(atof.epeo)
                  0x000f9c                  _strtof
 .libc.strtod     0x001182          0x8 c:/program files (x86)/microchip/xc16/v1.24/bin/bin/../../lib\libc-elf.a(atof.epeo)
                  0x001182                  _strtod
 .libc.atof       0x00118a          0xa c:/program files (x86)/microchip/xc16/v1.24/bin/bin/../../lib\libc-elf.a(atof.epeo)
                  0x00118a                  _atof
 .libc.atoi       0x001194         0x42 c:/program files (x86)/microchip/xc16/v1.24/bin/bin/../../lib\libc-elf.a(atoi.epeo)
                  0x001194                  _atoi
 .libc.atol       0x0011d6         0x5a c:/program files (x86)/microchip/xc16/v1.24/bin/bin/../../lib\libc-elf.a(atol.epeo)
                  0x0011d6                  _atol
 .libc.ultoa      0x001230         0x50 c:/program files (x86)/microchip/xc16/v1.24/bin/bin/../../lib\libc-elf.a(ltoa.epeo)
                  0x001230                  _ultoa
 .libc.ltoa       0x001280         0x24 c:/program files (x86)/microchip/xc16/v1.24/bin/bin/../../lib\libc-elf.a(ltoa.epeo)
                  0x001280                  _ltoa
 .libc.memcmp     0x0012a4         0x2e c:/program files (x86)/microchip/xc16/v1.24/bin/bin/../../lib\libc-elf.a(memcmp.epeo)
                  0x0012a4                  _memcmp
 .libc.memcpy     0x0012d2         0x12 c:/program files (x86)/microchip/xc16/v1.24/bin/bin/../../lib\libc-elf.a(memcpy.epeo)
                  0x0012d2                  _memcpy
 .libc.memset     0x0012e4         0x12 c:/program files (x86)/microchip/xc16/v1.24/bin/bin/../../lib\libc-elf.a(memset.epeo)
                  0x0012e4                  _memset
 .libc.srand      0x0012f6         0x12 c:/program files (x86)/microchip/xc16/v1.24/bin/bin/../../lib\libc-elf.a(rand.epeo)
                  0x0012f6                  _srand
 .libc.rand       0x001308         0x2c c:/program files (x86)/microchip/xc16/v1.24/bin/bin/../../lib\libc-elf.a(rand.epeo)
                  0x001308                  _rand
 .libc.sprintf    0x001334         0x2a c:/program files (x86)/microchip/xc16/v1.24/bin/bin/../../lib\libc-elf.a(sprintf.epeo)
                  0x001334                  _sprintf
 .libc.strcmp     0x00135e         0x12 c:/program files (x86)/microchip/xc16/v1.24/bin/bin/../../lib\libc-elf.a(strcmp.epeo)
                  0x00135e                  _strcmp
 .libc.strcpy     0x001370         0x10 c:/program files (x86)/microchip/xc16/v1.24/bin/bin/../../lib\libc-elf.a(strcpy.epeo)
                  0x001370                  _strcpy
 .libc.strlen     0x001380         0x12 c:/program files (x86)/microchip/xc16/v1.24/bin/bin/../../lib\libc-elf.a(strlen.epeo)
                  0x001380                  _strlen
 .libc.strncpy    0x001392         0x26 c:/program files (x86)/microchip/xc16/v1.24/bin/bin/../../lib\libc-elf.a(strncpy.epeo)
                  0x001392                  _strncpy
 .libc.strtok     0x0013b8         0x42 c:/program files (x86)/microchip/xc16/v1.24/bin/bin/../../lib\libc-elf.a(strtok.epeo)
                  0x0013b8                  _strtok
 .libc.putchar    0x0013fa          0xa c:/program files (x86)/microchip/xc16/v1.24/bin/bin/../../lib\libc-elf.a(putchar.epeo)
                  0x0013fa                  _putchar
 .libc._sprintf_cdfFnopsuxX
                  0x001404         0x2a c:/program files (x86)/microchip/xc16/v1.24/bin/bin/../../lib\libc-elf.a(sprintf_cdfFnopsuxX.EPeo)
                  0x001404                  __sprintf_cdfFnopuxX
                  0x001404                  __sprintf_cdfFnopsuxX
                  0x001404                  __sprintf_cdnopuxX
                  0x001404                  __sprintf_cdnopsuxX
 .libc.fround     0x00142e         0xaa c:/program files (x86)/microchip/xc16/v1.24/bin/bin/../../lib\libc-elf.a(doprnt_cdfFnopsuxX.EPeo)
 .libc.scale      0x0014d8         0xb8 c:/program files (x86)/microchip/xc16/v1.24/bin/bin/../../lib\libc-elf.a(doprnt_cdfFnopsuxX.EPeo)
 .libc._vfprintf_cdfFnopsuxX
                  0x001590        0xc4e c:/program files (x86)/microchip/xc16/v1.24/bin/bin/../../lib\libc-elf.a(doprnt_cdfFnopsuxX.EPeo)
                  0x001590                  __vfprintf_cdfFnopsuxX
                  0x001590                  __vfprintf_cdnopuxX
                  0x001590                  __vfprintf_cdnopsuxX
                  0x001590                  __vfprintf_cdfFnopuxX
                  0x001590                  __vfprintf_0
                  0x001590                  __vfprintf_s
 .libc._printf_cdnopsuxX
                  0x0021de          0xe c:/program files (x86)/microchip/xc16/v1.24/bin/bin/../../lib\libc-elf.a(printf_cdnopsuxX.EPeo)
                  0x0021de                  __printf_0
                  0x0021de                  __printf_s
                  0x0021de                  __printf_cdnopuxX
                  0x0021de                  __printf_cdnopsuxX
 .libc.fround     0x0021ec         0xaa c:/program files (x86)/microchip/xc16/v1.24/bin/bin/../../lib\libc-elf.a(doprnt.epeo)
 .libc.scale      0x002296         0xb8 c:/program files (x86)/microchip/xc16/v1.24/bin/bin/../../lib\libc-elf.a(doprnt.epeo)
 .libc.vfprintf
                  0x00234e       0x13a6 c:/program files (x86)/microchip/xc16/v1.24/bin/bin/../../lib\libc-elf.a(doprnt.epeo)
                  0x00234e                  _vfprintf
 .libc.fputc      0x0036f4         0x8c c:/program files (x86)/microchip/xc16/v1.24/bin/bin/../../lib\libc-elf.a(fputc.epeo)
                  0x0036f4                  _fputc
 .libc.strcspn    0x003780         0x2a c:/program files (x86)/microchip/xc16/v1.24/bin/bin/../../lib\libc-elf.a(strcspn.epeo)
                  0x003780                  _strcspn
 .libc.strspn     0x0037aa         0x2a c:/program files (x86)/microchip/xc16/v1.24/bin/bin/../../lib\libc-elf.a(strspn.epeo)
                  0x0037aa                  _strspn
 .libc.strchr     0x0037d4         0x1a c:/program files (x86)/microchip/xc16/v1.24/bin/bin/../../lib\libc-elf.a(strchr.epelo)
                  0x0037d4                  _strchr
 .libc._flsbuf    0x0037ee         0x80 c:/program files (x86)/microchip/xc16/v1.24/bin/bin/../../lib\libc-elf.a(flsbuf.epeo)
                  0x0037ee                  __flsbuf
 .libc.dowrite    0x00386e          0x8 c:/program files (x86)/microchip/xc16/v1.24/bin/bin/../../lib\libpic30-elf.a(writeep.eo)
 .libm.adddf3     0x003876         0xfa c:/program files (x86)/microchip/xc16/v1.24/bin/bin/../../lib\libm-elf.a(adddf3.epeo)
                  0x003876                  ___adddf3
 .libm.eqdf2      0x003970          0xa c:/program files (x86)/microchip/xc16/v1.24/bin/bin/../../lib\libm-elf.a(deqltle.epeo)
                  0x003970                  ___eqdf2
                  0x003970                  ___ltdf2
                  0x003970                  ___ledf2
 .libm.gtdf2      0x00397a          0xa c:/program files (x86)/microchip/xc16/v1.24/bin/bin/../../lib\libm-elf.a(dgtge.epeo)
                  0x00397a                  ___gtdf2
                  0x00397a                  ___gedf2
 .libm.divdf3     0x003984         0xb4 c:/program files (x86)/microchip/xc16/v1.24/bin/bin/../../lib\libm-elf.a(divdf3.epeo)
                  0x003984                  ___divdf3
 .libm.nedf2      0x003a38          0xa c:/program files (x86)/microchip/xc16/v1.24/bin/bin/../../lib\libm-elf.a(dne.epeo)
                  0x003a38                  ___nedf2
 .libm.dpack      0x003a42         0x58 c:/program files (x86)/microchip/xc16/v1.24/bin/bin/../../lib\libm-elf.a(dpack.epeo)
                  0x003a42                  __dpack
 .libm.dunpack2
                  0x003a9a         0x32 c:/program files (x86)/microchip/xc16/v1.24/bin/bin/../../lib\libm-elf.a(dunpack2.epeo)
                  0x003a9a                  __dunpack2
                  0x003abc                  __dreturnNaN
                  0x003ac2                  __dunpack2exit
 .libm.extendsfdf2
                  0x003acc         0x3e c:/program files (x86)/microchip/xc16/v1.24/bin/bin/../../lib\libm-elf.a(extendsfdf.epeo)
                  0x003acc                  ___extendsfdf2
 .libm.fixunsdfdi
                  0x003b0a         0x62 c:/program files (x86)/microchip/xc16/v1.24/bin/bin/../../lib\libm-elf.a(fixunsdfdi.epeo)
                  0x003b0a                  ___fixunsdfdi
 .libm.fixunsdfsi
                  0x003b6c         0x4c c:/program files (x86)/microchip/xc16/v1.24/bin/bin/../../lib\libm-elf.a(fixunsdfsi.epeo)
                  0x003b6c                  ___fixunsdfsi
 .libm.floatundidf
                  0x003bb8         0x56 c:/program files (x86)/microchip/xc16/v1.24/bin/bin/../../lib\libm-elf.a(floatundidf.epeo)
                  0x003bb8                  ___floatundidf
 .libm.floatunsidf
                  0x003c0e          0x4 c:/program files (x86)/microchip/xc16/v1.24/bin/bin/../../lib\libm-elf.a(floatunsidf.epeo)
                  0x003c0e                  ___floatunsidf
 .libm.frexp      0x003c12         0x3a c:/program files (x86)/microchip/xc16/v1.24/bin/bin/../../lib\libm-elf.a(frexp.epeo)
                  0x003c12                  _frexp
                  0x003c12                  _frexpl
 .libm.muldf3     0x003c4c         0xea c:/program files (x86)/microchip/xc16/v1.24/bin/bin/../../lib\libm-elf.a(muldf3.epeo)
                  0x003c4c                  ___muldf3
 .libm.subdf3     0x003d36          0x4 c:/program files (x86)/microchip/xc16/v1.24/bin/bin/../../lib\libm-elf.a(subdf3.epeo)
                  0x003d36                  ___subdf3
 .libm.mulsi3     0x003d3a          0xc c:/program files (x86)/microchip/xc16/v1.24/bin/bin/../../lib\libm-elf.a(mulsi3.epeo)
                  0x003d3a                  ___mulp32peds3
                  0x003d3a                  ___mulsi3
                  0x003d3a                  ___mulp32eds3
 .libm.__PplusBdi
                  0x003d46         0x2c c:/program files (x86)/microchip/xc16/v1.24/bin/bin/../../lib\libm-elf.a(divmoddi3.epeo)
 .libm.__PminusBdi
                  0x003d72         0x42 c:/program files (x86)/microchip/xc16/v1.24/bin/bin/../../lib\libm-elf.a(divmoddi3.epeo)
 .libm.__udivmoddi3
                  0x003db4         0xd0 c:/program files (x86)/microchip/xc16/v1.24/bin/bin/../../lib\libm-elf.a(divmoddi3.epeo)
                  0x003db4                  ___udivmoddi3
 .libm.__udivdi3
                  0x003e84         0x12 c:/program files (x86)/microchip/xc16/v1.24/bin/bin/../../lib\libm-elf.a(divmoddi3.epeo)
                  0x003e84                  ___udivdi3
 .libm.__umoddi3
                  0x003e96          0xc c:/program files (x86)/microchip/xc16/v1.24/bin/bin/../../lib\libm-elf.a(divmoddi3.epeo)
                  0x003e96                  ___umoddi3
 .libm.__divdi3
                  0x003ea2         0x64 c:/program files (x86)/microchip/xc16/v1.24/bin/bin/../../lib\libm-elf.a(divmoddi3.epeo)
                  0x003ea2                  ___divdi3
 .libm.__moddi3
                  0x003f06         0x60 c:/program files (x86)/microchip/xc16/v1.24/bin/bin/../../lib\libm-elf.a(divmoddi3.epeo)
                  0x003f06                  ___moddi3
 .libm.__muldi3
                  0x003f66         0x56 c:/program files (x86)/microchip/xc16/v1.24/bin/bin/../../lib\libm-elf.a(muldi3.epeo)
                  0x003f66                  ___muldi3
 .libm.dcompare
                  0x003fbc         0x52 c:/program files (x86)/microchip/xc16/v1.24/bin/bin/../../lib\libm-elf.a(dcompare.epeo)
                  0x003fbc                  __dcompare
 .libm.dPropagateNaN
                  0x00400e         0x1c c:/program files (x86)/microchip/xc16/v1.24/bin/bin/../../lib\libm-elf.a(dpropagateNaN.epeo)
                  0x00400e                  __dPropagateNaN
 .libm.dtype      0x00402a         0x24 c:/program files (x86)/microchip/xc16/v1.24/bin/bin/../../lib\libm-elf.a(dtype.epeo)
                  0x00402a                  __dtype
 .libm.dunpack    0x00404e         0x4e c:/program files (x86)/microchip/xc16/v1.24/bin/bin/../../lib\libm-elf.a(dunpack.epeo)
                  0x00404e                  __dunpack
 .libm.umuldi3    0x00409c         0x44 c:/program files (x86)/microchip/xc16/v1.24/bin/bin/../../lib\libm-elf.a(umuldi3.epeo)
                  0x00409c                  ___umuldi3

usercode
 *(usercode)

__FGS
 *(__FGS.sec*)

__FOSCSEL
 *(__FOSCSEL.sec*)

__FOSC
 *(__FOSC.sec*)

__FWDT
 *(__FWDT.sec*)

__FPOR
 *(__FPOR.sec*)

__FICD
 *(__FICD.sec*)

__FAS
 *(__FAS.sec*)

__FUID0
 *(__FUID0.sec*)

.comment
 *(.comment)

.debug_info       0x000000      0x44e85
 *(.debug_info)
 .debug_info      0x000000        0x14a build/XC16_dsPIC33EP512MU810/debug/B40/par/abcc_handler_par.o
 .debug_info      0x00014a        0x146 build/XC16_dsPIC33EP512MU810/debug/B40/par/abcc_par_drv.o
 .debug_info      0x000290        0x266 build/XC16_dsPIC33EP512MU810/debug/B40/spi/abcc_crc32.o
 .debug_info      0x0004f6        0x626 build/XC16_dsPIC33EP512MU810/debug/B40/spi/abcc_handler_spi.o
 .debug_info      0x000b1c       0x134c build/XC16_dsPIC33EP512MU810/debug/B40/spi/abcc_spi_drv.o
 .debug_info      0x001e68       0x1122 build/XC16_dsPIC33EP512MU810/debug/B40/abcc_cbf.o
 .debug_info      0x002f8a        0x4de build/XC16_dsPIC33EP512MU810/debug/B40/abcc_debug_err.o
 .debug_info      0x003468       0x1693 build/XC16_dsPIC33EP512MU810/debug/B40/abcc_handler.o
 .debug_info      0x004afb        0xfa5 build/XC16_dsPIC33EP512MU810/debug/B40/abcc_link.o
 .debug_info      0x005aa0        0x2ed build/XC16_dsPIC33EP512MU810/debug/B40/abcc_mem.o
 .debug_info      0x005d8d        0x3f1 build/XC16_dsPIC33EP512MU810/debug/B40/abcc_remap.o
 .debug_info      0x00617e       0x1195 build/XC16_dsPIC33EP512MU810/debug/B40/abcc_setup.o
 .debug_info      0x007313        0xe3f build/XC16_dsPIC33EP512MU810/debug/B40/abcc_sys_adapt.o
 .debug_info      0x008152        0x756 build/XC16_dsPIC33EP512MU810/debug/B40/abcc_timer.o
 .debug_info      0x0088a8       0x1638 build/XC16_dsPIC33EP512MU810/debug/B40/ad_obj.o
 .debug_info      0x009ee0        0x91a build/XC16_dsPIC33EP512MU810/debug/B40/app_obj.o
 .debug_info      0x00a7fa        0x920 build/XC16_dsPIC33EP512MU810/debug/B40/dpv1.o
 .debug_info      0x00b11a        0xb68 build/XC16_dsPIC33EP512MU810/debug/B40/user_adi.o
 .debug_info      0x00bc82        0x487 build/XC16_dsPIC33EP512MU810/debug/B40/user_setup.o
 .debug_info      0x00c109       0x2154 build/XC16_dsPIC33EP512MU810/debug/ECAN/ECAN1Drv.o
 .debug_info      0x00e25d        0xae8 build/XC16_dsPIC33EP512MU810/debug/BerkeleyTCPClient.o
 .debug_info      0x00ed45        0x797 build/XC16_dsPIC33EP512MU810/debug/BerkeleyTCPServer.o
 .debug_info      0x00f4dc        0xb7f build/XC16_dsPIC33EP512MU810/debug/BerkeleyUDPClient.o
 .debug_info      0x01005b        0x5e7 build/XC16_dsPIC33EP512MU810/debug/MODBUSTCPServer.o
 .debug_info      0x010642       0x18da build/XC16_dsPIC33EP512MU810/debug/Regul.o
 .debug_info      0x011f1c       0x1c2e build/XC16_dsPIC33EP512MU810/debug/Pesage.o
 .debug_info      0x013b4a       0x407a build/XC16_dsPIC33EP512MU810/debug/Process.o
 .debug_info      0x017bc4        0xb33 build/XC16_dsPIC33EP512MU810/debug/TCPIPStack/Announce.o
 .debug_info      0x0186f7        0x13b build/XC16_dsPIC33EP512MU810/debug/TCPIPStack/ARCFOUR.o
 .debug_info      0x018832        0xb63 build/XC16_dsPIC33EP512MU810/debug/TCPIPStack/ARP.o
 .debug_info      0x019395        0x13a build/XC16_dsPIC33EP512MU810/debug/TCPIPStack/AutoIP.o
 .debug_info      0x0194cf       0x1466 build/XC16_dsPIC33EP512MU810/debug/TCPIPStack/BerkeleyAPI.o
 .debug_info      0x01a935        0x13a build/XC16_dsPIC33EP512MU810/debug/TCPIPStack/BigInt.o
 .debug_info      0x01aa6f        0x1ce build/XC16_dsPIC33EP512MU810/debug/TCPIPStack/Delay.o
 .debug_info      0x01ac3d        0x138 build/XC16_dsPIC33EP512MU810/debug/TCPIPStack/DHCP.o
 .debug_info      0x01ad75        0x139 build/XC16_dsPIC33EP512MU810/debug/TCPIPStack/DHCPs.o
 .debug_info      0x01aeae        0xd85 build/XC16_dsPIC33EP512MU810/debug/TCPIPStack/DNS.o
 .debug_info      0x01bc33        0x138 build/XC16_dsPIC33EP512MU810/debug/TCPIPStack/DNSs.o
 .debug_info      0x01bd6b        0x13a build/XC16_dsPIC33EP512MU810/debug/TCPIPStack/DynDNS.o
 .debug_info      0x01bea5       0x2d29 build/XC16_dsPIC33EP512MU810/debug/TCPIPStack/ENC28J60.o
 .debug_info      0x01ebce        0x13e build/XC16_dsPIC33EP512MU810/debug/TCPIPStack/FileSystem.o
 .debug_info      0x01ed0c        0x137 build/XC16_dsPIC33EP512MU810/debug/TCPIPStack/FTP.o
 .debug_info      0x01ee43        0x13a build/XC16_dsPIC33EP512MU810/debug/TCPIPStack/Hashes.o
 .debug_info      0x01ef7d       0x1068 build/XC16_dsPIC33EP512MU810/debug/TCPIPStack/Helpers.o
 .debug_info      0x01ffe5       0x1305 build/XC16_dsPIC33EP512MU810/debug/TCPIPStack/HTTP2.o
 .debug_info      0x0212ea        0xac9 build/XC16_dsPIC33EP512MU810/debug/TCPIPStack/ICMP.o
 .debug_info      0x021db3        0xb16 build/XC16_dsPIC33EP512MU810/debug/TCPIPStack/IP.o
 .debug_info      0x0228c9        0x13f build/XC16_dsPIC33EP512MU810/debug/TCPIPStack/LCDBlocking.o
 .debug_info      0x022a08        0xe2f build/XC16_dsPIC33EP512MU810/debug/TCPIPStack/MPFS2.o
 .debug_info      0x023837        0xc6a build/XC16_dsPIC33EP512MU810/debug/TCPIPStack/NBNS.o
 .debug_info      0x0244a1        0x13a build/XC16_dsPIC33EP512MU810/debug/TCPIPStack/Random.o
 .debug_info      0x0245db        0xa51 build/XC16_dsPIC33EP512MU810/debug/TCPIPStack/Reboot.o
 .debug_info      0x02502c        0x137 build/XC16_dsPIC33EP512MU810/debug/TCPIPStack/RSA.o
 .debug_info      0x025163        0x138 build/XC16_dsPIC33EP512MU810/debug/TCPIPStack/SMTP.o
 .debug_info      0x02529b        0x138 build/XC16_dsPIC33EP512MU810/debug/TCPIPStack/SNMP.o
 .debug_info      0x0253d3        0x13a build/XC16_dsPIC33EP512MU810/debug/TCPIPStack/SNMPv3.o
 .debug_info      0x02550d        0x13d build/XC16_dsPIC33EP512MU810/debug/TCPIPStack/SNMPv3USM.o
 .debug_info      0x02564a        0x138 build/XC16_dsPIC33EP512MU810/debug/TCPIPStack/SNTP.o
 .debug_info      0x025782       0x1072 build/XC16_dsPIC33EP512MU810/debug/TCPIPStack/SPIEEPROM.o
 .debug_info      0x0267f4        0x13c build/XC16_dsPIC33EP512MU810/debug/TCPIPStack/SPIFlash.o
 .debug_info      0x026930        0x13a build/XC16_dsPIC33EP512MU810/debug/TCPIPStack/SPIRAM.o
 .debug_info      0x026a6a        0x137 build/XC16_dsPIC33EP512MU810/debug/TCPIPStack/SSL.o
 .debug_info      0x026ba1        0x9e1 build/XC16_dsPIC33EP512MU810/debug/TCPIPStack/StackTsk.o
 .debug_info      0x027582       0x21dc build/XC16_dsPIC33EP512MU810/debug/TCPIPStack/TCP.o
 .debug_info      0x02975e        0x146 build/XC16_dsPIC33EP512MU810/debug/TCPIPStack/TCPPerformanceTest.o
 .debug_info      0x0298a4        0x13a build/XC16_dsPIC33EP512MU810/debug/TCPIPStack/Telnet.o
 .debug_info      0x0299de        0x139 build/XC16_dsPIC33EP512MU810/debug/TCPIPStack/TFTPc.o
 .debug_info      0x029b17        0xb0e build/XC16_dsPIC33EP512MU810/debug/TCPIPStack/Tick.o
 .debug_info      0x02a625        0x138 build/XC16_dsPIC33EP512MU810/debug/TCPIPStack/UART.o
 .debug_info      0x02a75d        0x142 build/XC16_dsPIC33EP512MU810/debug/TCPIPStack/UART2TCPBridge.o
 .debug_info      0x02a89f       0x11e4 build/XC16_dsPIC33EP512MU810/debug/TCPIPStack/UDP.o
 .debug_info      0x02ba83        0x146 build/XC16_dsPIC33EP512MU810/debug/TCPIPStack/UDPPerformanceTest.o
 .debug_info      0x02bbc9        0x142 build/XC16_dsPIC33EP512MU810/debug/TCPIPStack/ZeroconfHelper.o
 .debug_info      0x02bd0b        0x145 build/XC16_dsPIC33EP512MU810/debug/TCPIPStack/ZeroconfLinkLocal.o
 .debug_info      0x02be50        0x148 build/XC16_dsPIC33EP512MU810/debug/TCPIPStack/ZeroconfMulticastDNS.o
 .debug_info      0x02bf98       0x2a14 build/XC16_dsPIC33EP512MU810/debug/usb/src/usb_device.o
 .debug_info      0x02e9ac       0x1620 build/XC16_dsPIC33EP512MU810/debug/usb/src/usb_device_cdc.o
 .debug_info      0x02ffcc        0x5d4 build/XC16_dsPIC33EP512MU810/debug/usb/src/usb_hal_dspic33e.o
 .debug_info      0x0305a0         0x9d build/XC16_dsPIC33EP512MU810/debug/configuration_bits.o
 .debug_info      0x03063d       0x1ea9 build/XC16_dsPIC33EP512MU810/debug/interrupts.o
 .debug_info      0x0324e6       0x6264 build/XC16_dsPIC33EP512MU810/debug/main.o
 .debug_info      0x03874a        0x895 build/XC16_dsPIC33EP512MU810/debug/system.o
 .debug_info      0x038fdf        0x37a build/XC16_dsPIC33EP512MU810/debug/traps.o
 .debug_info      0x039359       0x1a11 build/XC16_dsPIC33EP512MU810/debug/user.o
 .debug_info      0x03ad6a         0x6e build/XC16_dsPIC33EP512MU810/debug/MPFSImg2.o
 .debug_info      0x03add8       0x1be7 build/XC16_dsPIC33EP512MU810/debug/CustomHTTPApp.o
 .debug_info      0x03c9bf        0xb87 build/XC16_dsPIC33EP512MU810/debug/AD7190.o
 .debug_info      0x03d546        0x50c build/XC16_dsPIC33EP512MU810/debug/ADComm.o
 .debug_info      0x03da52       0x180d build/XC16_dsPIC33EP512MU810/debug/UARTsComm.o
 .debug_info      0x03f25f        0xb81 build/XC16_dsPIC33EP512MU810/debug/MemFlash.o
 .debug_info      0x03fde0       0x115b build/XC16_dsPIC33EP512MU810/debug/ADC10bitsDrv.o
 .debug_info      0x040f3b        0xf7a build/XC16_dsPIC33EP512MU810/debug/SPIFRAM.o
 .debug_info      0x041eb5        0x7b9 build/XC16_dsPIC33EP512MU810/debug/usb_descriptors.o
 .debug_info      0x04266e       0x2817 build/XC16_dsPIC33EP512MU810/debug/ModbusUartServer.o
 *(.gnu.linkonce.wi.*)

.debug_abbrev     0x000000       0x66c8
 *(.debug_abbrev)
 .debug_abbrev    0x000000         0x1f build/XC16_dsPIC33EP512MU810/debug/B40/par/abcc_handler_par.o
 .debug_abbrev    0x00001f         0x1f build/XC16_dsPIC33EP512MU810/debug/B40/par/abcc_par_drv.o
 .debug_abbrev    0x00003e         0xa7 build/XC16_dsPIC33EP512MU810/debug/B40/spi/abcc_crc32.o
 .debug_abbrev    0x0000e5         0xce build/XC16_dsPIC33EP512MU810/debug/B40/spi/abcc_handler_spi.o
 .debug_abbrev    0x0001b3        0x214 build/XC16_dsPIC33EP512MU810/debug/B40/spi/abcc_spi_drv.o
 .debug_abbrev    0x0003c7        0x1ac build/XC16_dsPIC33EP512MU810/debug/B40/abcc_cbf.o
 .debug_abbrev    0x000573         0x7b build/XC16_dsPIC33EP512MU810/debug/B40/abcc_debug_err.o
 .debug_abbrev    0x0005ee        0x260 build/XC16_dsPIC33EP512MU810/debug/B40/abcc_handler.o
 .debug_abbrev    0x00084e        0x250 build/XC16_dsPIC33EP512MU810/debug/B40/abcc_link.o
 .debug_abbrev    0x000a9e         0xc0 build/XC16_dsPIC33EP512MU810/debug/B40/abcc_mem.o
 .debug_abbrev    0x000b5e         0xe8 build/XC16_dsPIC33EP512MU810/debug/B40/abcc_remap.o
 .debug_abbrev    0x000c46        0x208 build/XC16_dsPIC33EP512MU810/debug/B40/abcc_setup.o
 .debug_abbrev    0x000e4e        0x151 build/XC16_dsPIC33EP512MU810/debug/B40/abcc_sys_adapt.o
 .debug_abbrev    0x000f9f        0x143 build/XC16_dsPIC33EP512MU810/debug/B40/abcc_timer.o
 .debug_abbrev    0x0010e2        0x290 build/XC16_dsPIC33EP512MU810/debug/B40/ad_obj.o
 .debug_abbrev    0x001372        0x153 build/XC16_dsPIC33EP512MU810/debug/B40/app_obj.o
 .debug_abbrev    0x0014c5        0x15e build/XC16_dsPIC33EP512MU810/debug/B40/dpv1.o
 .debug_abbrev    0x001623        0x14c build/XC16_dsPIC33EP512MU810/debug/B40/user_adi.o
 .debug_abbrev    0x00176f        0x13e build/XC16_dsPIC33EP512MU810/debug/B40/user_setup.o
 .debug_abbrev    0x0018ad        0x1b1 build/XC16_dsPIC33EP512MU810/debug/ECAN/ECAN1Drv.o
 .debug_abbrev    0x001a5e        0x145 build/XC16_dsPIC33EP512MU810/debug/BerkeleyTCPClient.o
 .debug_abbrev    0x001ba3        0x135 build/XC16_dsPIC33EP512MU810/debug/BerkeleyTCPServer.o
 .debug_abbrev    0x001cd8        0x154 build/XC16_dsPIC33EP512MU810/debug/BerkeleyUDPClient.o
 .debug_abbrev    0x001e2c        0x15e build/XC16_dsPIC33EP512MU810/debug/MODBUSTCPServer.o
 .debug_abbrev    0x001f8a         0xeb build/XC16_dsPIC33EP512MU810/debug/Regul.o
 .debug_abbrev    0x002075        0x102 build/XC16_dsPIC33EP512MU810/debug/Pesage.o
 .debug_abbrev    0x002177        0x38c build/XC16_dsPIC33EP512MU810/debug/Process.o
 .debug_abbrev    0x002503        0x159 build/XC16_dsPIC33EP512MU810/debug/TCPIPStack/Announce.o
 .debug_abbrev    0x00265c         0x1f build/XC16_dsPIC33EP512MU810/debug/TCPIPStack/ARCFOUR.o
 .debug_abbrev    0x00267b        0x1cb build/XC16_dsPIC33EP512MU810/debug/TCPIPStack/ARP.o
 .debug_abbrev    0x002846         0x1f build/XC16_dsPIC33EP512MU810/debug/TCPIPStack/AutoIP.o
 .debug_abbrev    0x002865        0x236 build/XC16_dsPIC33EP512MU810/debug/TCPIPStack/BerkeleyAPI.o
 .debug_abbrev    0x002a9b         0x1f build/XC16_dsPIC33EP512MU810/debug/TCPIPStack/BigInt.o
 .debug_abbrev    0x002aba         0x68 build/XC16_dsPIC33EP512MU810/debug/TCPIPStack/Delay.o
 .debug_abbrev    0x002b22         0x1f build/XC16_dsPIC33EP512MU810/debug/TCPIPStack/DHCP.o
 .debug_abbrev    0x002b41         0x1f build/XC16_dsPIC33EP512MU810/debug/TCPIPStack/DHCPs.o
 .debug_abbrev    0x002b60        0x1db build/XC16_dsPIC33EP512MU810/debug/TCPIPStack/DNS.o
 .debug_abbrev    0x002d3b         0x1f build/XC16_dsPIC33EP512MU810/debug/TCPIPStack/DNSs.o
 .debug_abbrev    0x002d5a         0x1f build/XC16_dsPIC33EP512MU810/debug/TCPIPStack/DynDNS.o
 .debug_abbrev    0x002d79        0x2b5 build/XC16_dsPIC33EP512MU810/debug/TCPIPStack/ENC28J60.o
 .debug_abbrev    0x00302e         0x1f build/XC16_dsPIC33EP512MU810/debug/TCPIPStack/FileSystem.o
 .debug_abbrev    0x00304d         0x1f build/XC16_dsPIC33EP512MU810/debug/TCPIPStack/FTP.o
 .debug_abbrev    0x00306c         0x1f build/XC16_dsPIC33EP512MU810/debug/TCPIPStack/Hashes.o
 .debug_abbrev    0x00308b        0x1aa build/XC16_dsPIC33EP512MU810/debug/TCPIPStack/Helpers.o
 .debug_abbrev    0x003235        0x225 build/XC16_dsPIC33EP512MU810/debug/TCPIPStack/HTTP2.o
 .debug_abbrev    0x00345a        0x19f build/XC16_dsPIC33EP512MU810/debug/TCPIPStack/ICMP.o
 .debug_abbrev    0x0035f9        0x198 build/XC16_dsPIC33EP512MU810/debug/TCPIPStack/IP.o
 .debug_abbrev    0x003791         0x1f build/XC16_dsPIC33EP512MU810/debug/TCPIPStack/LCDBlocking.o
 .debug_abbrev    0x0037b0        0x1eb build/XC16_dsPIC33EP512MU810/debug/TCPIPStack/MPFS2.o
 .debug_abbrev    0x00399b        0x1aa build/XC16_dsPIC33EP512MU810/debug/TCPIPStack/NBNS.o
 .debug_abbrev    0x003b45         0x1f build/XC16_dsPIC33EP512MU810/debug/TCPIPStack/Random.o
 .debug_abbrev    0x003b64        0x134 build/XC16_dsPIC33EP512MU810/debug/TCPIPStack/Reboot.o
 .debug_abbrev    0x003c98         0x1f build/XC16_dsPIC33EP512MU810/debug/TCPIPStack/RSA.o
 .debug_abbrev    0x003cb7         0x1f build/XC16_dsPIC33EP512MU810/debug/TCPIPStack/SMTP.o
 .debug_abbrev    0x003cd6         0x1f build/XC16_dsPIC33EP512MU810/debug/TCPIPStack/SNMP.o
 .debug_abbrev    0x003cf5         0x1f build/XC16_dsPIC33EP512MU810/debug/TCPIPStack/SNMPv3.o
 .debug_abbrev    0x003d14         0x1f build/XC16_dsPIC33EP512MU810/debug/TCPIPStack/SNMPv3USM.o
 .debug_abbrev    0x003d33         0x1f build/XC16_dsPIC33EP512MU810/debug/TCPIPStack/SNTP.o
 .debug_abbrev    0x003d52        0x214 build/XC16_dsPIC33EP512MU810/debug/TCPIPStack/SPIEEPROM.o
 .debug_abbrev    0x003f66         0x1f build/XC16_dsPIC33EP512MU810/debug/TCPIPStack/SPIFlash.o
 .debug_abbrev    0x003f85         0x1f build/XC16_dsPIC33EP512MU810/debug/TCPIPStack/SPIRAM.o
 .debug_abbrev    0x003fa4         0x1f build/XC16_dsPIC33EP512MU810/debug/TCPIPStack/SSL.o
 .debug_abbrev    0x003fc3        0x158 build/XC16_dsPIC33EP512MU810/debug/TCPIPStack/StackTsk.o
 .debug_abbrev    0x00411b        0x246 build/XC16_dsPIC33EP512MU810/debug/TCPIPStack/TCP.o
 .debug_abbrev    0x004361         0x1f build/XC16_dsPIC33EP512MU810/debug/TCPIPStack/TCPPerformanceTest.o
 .debug_abbrev    0x004380         0x1f build/XC16_dsPIC33EP512MU810/debug/TCPIPStack/Telnet.o
 .debug_abbrev    0x00439f         0x1f build/XC16_dsPIC33EP512MU810/debug/TCPIPStack/TFTPc.o
 .debug_abbrev    0x0043be        0x15f build/XC16_dsPIC33EP512MU810/debug/TCPIPStack/Tick.o
 .debug_abbrev    0x00451d         0x1f build/XC16_dsPIC33EP512MU810/debug/TCPIPStack/UART.o
 .debug_abbrev    0x00453c         0x1f build/XC16_dsPIC33EP512MU810/debug/TCPIPStack/UART2TCPBridge.o
 .debug_abbrev    0x00455b        0x258 build/XC16_dsPIC33EP512MU810/debug/TCPIPStack/UDP.o
 .debug_abbrev    0x0047b3         0x1f build/XC16_dsPIC33EP512MU810/debug/TCPIPStack/UDPPerformanceTest.o
 .debug_abbrev    0x0047d2         0x1f build/XC16_dsPIC33EP512MU810/debug/TCPIPStack/ZeroconfHelper.o
 .debug_abbrev    0x0047f1         0x1f build/XC16_dsPIC33EP512MU810/debug/TCPIPStack/ZeroconfLinkLocal.o
 .debug_abbrev    0x004810         0x1f build/XC16_dsPIC33EP512MU810/debug/TCPIPStack/ZeroconfMulticastDNS.o
 .debug_abbrev    0x00482f        0x2bc build/XC16_dsPIC33EP512MU810/debug/usb/src/usb_device.o
 .debug_abbrev    0x004aeb        0x25f build/XC16_dsPIC33EP512MU810/debug/usb/src/usb_device_cdc.o
 .debug_abbrev    0x004d4a         0xa1 build/XC16_dsPIC33EP512MU810/debug/usb/src/usb_hal_dspic33e.o
 .debug_abbrev    0x004deb         0x1f build/XC16_dsPIC33EP512MU810/debug/configuration_bits.o
 .debug_abbrev    0x004e0a        0x1a4 build/XC16_dsPIC33EP512MU810/debug/interrupts.o
 .debug_abbrev    0x004fae        0x2c7 build/XC16_dsPIC33EP512MU810/debug/main.o
 .debug_abbrev    0x005275         0xb8 build/XC16_dsPIC33EP512MU810/debug/system.o
 .debug_abbrev    0x00532d         0x7d build/XC16_dsPIC33EP512MU810/debug/traps.o
 .debug_abbrev    0x0053aa        0x2aa build/XC16_dsPIC33EP512MU810/debug/user.o
 .debug_abbrev    0x005654         0x10 build/XC16_dsPIC33EP512MU810/debug/MPFSImg2.o
 .debug_abbrev    0x005664        0x257 build/XC16_dsPIC33EP512MU810/debug/CustomHTTPApp.o
 .debug_abbrev    0x0058bb        0x196 build/XC16_dsPIC33EP512MU810/debug/AD7190.o
 .debug_abbrev    0x005a51        0x118 build/XC16_dsPIC33EP512MU810/debug/ADComm.o
 .debug_abbrev    0x005b69        0x211 build/XC16_dsPIC33EP512MU810/debug/UARTsComm.o
 .debug_abbrev    0x005d7a        0x1ec build/XC16_dsPIC33EP512MU810/debug/MemFlash.o
 .debug_abbrev    0x005f66        0x150 build/XC16_dsPIC33EP512MU810/debug/ADC10bitsDrv.o
 .debug_abbrev    0x0060b6        0x214 build/XC16_dsPIC33EP512MU810/debug/SPIFRAM.o
 .debug_abbrev    0x0062ca        0x102 build/XC16_dsPIC33EP512MU810/debug/usb_descriptors.o
 .debug_abbrev    0x0063cc        0x2fc build/XC16_dsPIC33EP512MU810/debug/ModbusUartServer.o

.debug_line       0x000000      0x1a637
 *(.debug_line)
 .debug_line      0x000000         0x24 build/XC16_dsPIC33EP512MU810/debug/B40/par/abcc_handler_par.o
 .debug_line      0x000024         0x24 build/XC16_dsPIC33EP512MU810/debug/B40/par/abcc_par_drv.o
 .debug_line      0x000048        0x13f build/XC16_dsPIC33EP512MU810/debug/B40/spi/abcc_crc32.o
 .debug_line      0x000187        0x190 build/XC16_dsPIC33EP512MU810/debug/B40/spi/abcc_handler_spi.o
 .debug_line      0x000317        0x980 build/XC16_dsPIC33EP512MU810/debug/B40/spi/abcc_spi_drv.o
 .debug_line      0x000c97        0x283 build/XC16_dsPIC33EP512MU810/debug/B40/abcc_cbf.o
 .debug_line      0x000f1a         0x79 build/XC16_dsPIC33EP512MU810/debug/B40/abcc_debug_err.o
 .debug_line      0x000f93        0x9d2 build/XC16_dsPIC33EP512MU810/debug/B40/abcc_handler.o
 .debug_line      0x001965        0x709 build/XC16_dsPIC33EP512MU810/debug/B40/abcc_link.o
 .debug_line      0x00206e        0x169 build/XC16_dsPIC33EP512MU810/debug/B40/abcc_mem.o
 .debug_line      0x0021d7         0xde build/XC16_dsPIC33EP512MU810/debug/B40/abcc_remap.o
 .debug_line      0x0022b5        0x695 build/XC16_dsPIC33EP512MU810/debug/B40/abcc_setup.o
 .debug_line      0x00294a        0x369 build/XC16_dsPIC33EP512MU810/debug/B40/abcc_sys_adapt.o
 .debug_line      0x002cb3        0x277 build/XC16_dsPIC33EP512MU810/debug/B40/abcc_timer.o
 .debug_line      0x002f2a        0xfde build/XC16_dsPIC33EP512MU810/debug/B40/ad_obj.o
 .debug_line      0x003f08        0x30c build/XC16_dsPIC33EP512MU810/debug/B40/app_obj.o
 .debug_line      0x004214        0x228 build/XC16_dsPIC33EP512MU810/debug/B40/dpv1.o
 .debug_line      0x00443c         0xe6 build/XC16_dsPIC33EP512MU810/debug/B40/user_adi.o
 .debug_line      0x004522        0x357 build/XC16_dsPIC33EP512MU810/debug/B40/user_setup.o
 .debug_line      0x004879        0x45e build/XC16_dsPIC33EP512MU810/debug/ECAN/ECAN1Drv.o
 .debug_line      0x004cd7        0x249 build/XC16_dsPIC33EP512MU810/debug/BerkeleyTCPClient.o
 .debug_line      0x004f20        0x277 build/XC16_dsPIC33EP512MU810/debug/BerkeleyTCPServer.o
 .debug_line      0x005197        0x2dc build/XC16_dsPIC33EP512MU810/debug/BerkeleyUDPClient.o
 .debug_line      0x005473        0x217 build/XC16_dsPIC33EP512MU810/debug/MODBUSTCPServer.o
 .debug_line      0x00568a        0x180 build/XC16_dsPIC33EP512MU810/debug/Regul.o
 .debug_line      0x00580a        0xc2f build/XC16_dsPIC33EP512MU810/debug/Pesage.o
 .debug_line      0x006439       0x1bd7 build/XC16_dsPIC33EP512MU810/debug/Process.o
 .debug_line      0x008010        0x25b build/XC16_dsPIC33EP512MU810/debug/TCPIPStack/Announce.o
 .debug_line      0x00826b         0x24 build/XC16_dsPIC33EP512MU810/debug/TCPIPStack/ARCFOUR.o
 .debug_line      0x00828f        0x3e5 build/XC16_dsPIC33EP512MU810/debug/TCPIPStack/ARP.o
 .debug_line      0x008674         0x24 build/XC16_dsPIC33EP512MU810/debug/TCPIPStack/AutoIP.o
 .debug_line      0x008698        0xb3a build/XC16_dsPIC33EP512MU810/debug/TCPIPStack/BerkeleyAPI.o
 .debug_line      0x0091d2         0x24 build/XC16_dsPIC33EP512MU810/debug/TCPIPStack/BigInt.o
 .debug_line      0x0091f6        0x106 build/XC16_dsPIC33EP512MU810/debug/TCPIPStack/Delay.o
 .debug_line      0x0092fc         0x24 build/XC16_dsPIC33EP512MU810/debug/TCPIPStack/DHCP.o
 .debug_line      0x009320         0x24 build/XC16_dsPIC33EP512MU810/debug/TCPIPStack/DHCPs.o
 .debug_line      0x009344        0x7f7 build/XC16_dsPIC33EP512MU810/debug/TCPIPStack/DNS.o
 .debug_line      0x009b3b         0x24 build/XC16_dsPIC33EP512MU810/debug/TCPIPStack/DNSs.o
 .debug_line      0x009b5f         0x24 build/XC16_dsPIC33EP512MU810/debug/TCPIPStack/DynDNS.o
 .debug_line      0x009b83       0x1285 build/XC16_dsPIC33EP512MU810/debug/TCPIPStack/ENC28J60.o
 .debug_line      0x00ae08         0x24 build/XC16_dsPIC33EP512MU810/debug/TCPIPStack/FileSystem.o
 .debug_line      0x00ae2c         0x24 build/XC16_dsPIC33EP512MU810/debug/TCPIPStack/FTP.o
 .debug_line      0x00ae50         0x24 build/XC16_dsPIC33EP512MU810/debug/TCPIPStack/Hashes.o
 .debug_line      0x00ae74        0xade build/XC16_dsPIC33EP512MU810/debug/TCPIPStack/Helpers.o
 .debug_line      0x00b952       0x14bf build/XC16_dsPIC33EP512MU810/debug/TCPIPStack/HTTP2.o
 .debug_line      0x00ce11        0x427 build/XC16_dsPIC33EP512MU810/debug/TCPIPStack/ICMP.o
 .debug_line      0x00d238        0x249 build/XC16_dsPIC33EP512MU810/debug/TCPIPStack/IP.o
 .debug_line      0x00d481         0x24 build/XC16_dsPIC33EP512MU810/debug/TCPIPStack/LCDBlocking.o
 .debug_line      0x00d4a5        0x94b build/XC16_dsPIC33EP512MU810/debug/TCPIPStack/MPFS2.o
 .debug_line      0x00ddf0        0x3cd build/XC16_dsPIC33EP512MU810/debug/TCPIPStack/NBNS.o
 .debug_line      0x00e1bd         0x24 build/XC16_dsPIC33EP512MU810/debug/TCPIPStack/Random.o
 .debug_line      0x00e1e1        0x185 build/XC16_dsPIC33EP512MU810/debug/TCPIPStack/Reboot.o
 .debug_line      0x00e366         0x24 build/XC16_dsPIC33EP512MU810/debug/TCPIPStack/RSA.o
 .debug_line      0x00e38a         0x24 build/XC16_dsPIC33EP512MU810/debug/TCPIPStack/SMTP.o
 .debug_line      0x00e3ae         0x24 build/XC16_dsPIC33EP512MU810/debug/TCPIPStack/SNMP.o
 .debug_line      0x00e3d2         0x24 build/XC16_dsPIC33EP512MU810/debug/TCPIPStack/SNMPv3.o
 .debug_line      0x00e3f6         0x24 build/XC16_dsPIC33EP512MU810/debug/TCPIPStack/SNMPv3USM.o
 .debug_line      0x00e41a         0x24 build/XC16_dsPIC33EP512MU810/debug/TCPIPStack/SNTP.o
 .debug_line      0x00e43e        0x5ab build/XC16_dsPIC33EP512MU810/debug/TCPIPStack/SPIEEPROM.o
 .debug_line      0x00e9e9         0x24 build/XC16_dsPIC33EP512MU810/debug/TCPIPStack/SPIFlash.o
 .debug_line      0x00ea0d         0x24 build/XC16_dsPIC33EP512MU810/debug/TCPIPStack/SPIRAM.o
 .debug_line      0x00ea31         0x24 build/XC16_dsPIC33EP512MU810/debug/TCPIPStack/SSL.o
 .debug_line      0x00ea55        0x24d build/XC16_dsPIC33EP512MU810/debug/TCPIPStack/StackTsk.o
 .debug_line      0x00eca2       0x2726 build/XC16_dsPIC33EP512MU810/debug/TCPIPStack/TCP.o
 .debug_line      0x0113c8         0x24 build/XC16_dsPIC33EP512MU810/debug/TCPIPStack/TCPPerformanceTest.o
 .debug_line      0x0113ec         0x24 build/XC16_dsPIC33EP512MU810/debug/TCPIPStack/Telnet.o
 .debug_line      0x011410         0x24 build/XC16_dsPIC33EP512MU810/debug/TCPIPStack/TFTPc.o
 .debug_line      0x011434        0x326 build/XC16_dsPIC33EP512MU810/debug/TCPIPStack/Tick.o
 .debug_line      0x01175a         0x24 build/XC16_dsPIC33EP512MU810/debug/TCPIPStack/UART.o
 .debug_line      0x01177e         0x24 build/XC16_dsPIC33EP512MU810/debug/TCPIPStack/UART2TCPBridge.o
 .debug_line      0x0117a2        0x936 build/XC16_dsPIC33EP512MU810/debug/TCPIPStack/UDP.o
 .debug_line      0x0120d8         0x24 build/XC16_dsPIC33EP512MU810/debug/TCPIPStack/UDPPerformanceTest.o
 .debug_line      0x0120fc         0x24 build/XC16_dsPIC33EP512MU810/debug/TCPIPStack/ZeroconfHelper.o
 .debug_line      0x012120         0x24 build/XC16_dsPIC33EP512MU810/debug/TCPIPStack/ZeroconfLinkLocal.o
 .debug_line      0x012144         0x24 build/XC16_dsPIC33EP512MU810/debug/TCPIPStack/ZeroconfMulticastDNS.o
 .debug_line      0x012168       0x131a build/XC16_dsPIC33EP512MU810/debug/usb/src/usb_device.o
 .debug_line      0x013482        0x5f8 build/XC16_dsPIC33EP512MU810/debug/usb/src/usb_device_cdc.o
 .debug_line      0x013a7a        0x144 build/XC16_dsPIC33EP512MU810/debug/usb/src/usb_hal_dspic33e.o
 .debug_line      0x013bbe         0x24 build/XC16_dsPIC33EP512MU810/debug/configuration_bits.o
 .debug_line      0x013be2        0x4f3 build/XC16_dsPIC33EP512MU810/debug/interrupts.o
 .debug_line      0x0140d5        0xde0 build/XC16_dsPIC33EP512MU810/debug/main.o
 .debug_line      0x014eb5        0x11a build/XC16_dsPIC33EP512MU810/debug/system.o
 .debug_line      0x014fcf        0x187 build/XC16_dsPIC33EP512MU810/debug/traps.o
 .debug_line      0x015156        0x917 build/XC16_dsPIC33EP512MU810/debug/user.o
 .debug_line      0x015a6d         0x50 build/XC16_dsPIC33EP512MU810/debug/MPFSImg2.o
 .debug_line      0x015abd        0xb08 build/XC16_dsPIC33EP512MU810/debug/CustomHTTPApp.o
 .debug_line      0x0165c5        0x6a3 build/XC16_dsPIC33EP512MU810/debug/AD7190.o
 .debug_line      0x016c68        0x1ce build/XC16_dsPIC33EP512MU810/debug/ADComm.o
 .debug_line      0x016e36        0x957 build/XC16_dsPIC33EP512MU810/debug/UARTsComm.o
 .debug_line      0x01778d        0x708 build/XC16_dsPIC33EP512MU810/debug/MemFlash.o
 .debug_line      0x017e95        0x29b build/XC16_dsPIC33EP512MU810/debug/ADC10bitsDrv.o
 .debug_line      0x018130        0x531 build/XC16_dsPIC33EP512MU810/debug/SPIFRAM.o
 .debug_line      0x018661         0xbc build/XC16_dsPIC33EP512MU810/debug/usb_descriptors.o
 .debug_line      0x01871d       0x1f1a build/XC16_dsPIC33EP512MU810/debug/ModbusUartServer.o

.debug_frame      0x000000       0x3924
 *(.debug_frame)
 .debug_frame     0x000000         0x24 build/XC16_dsPIC33EP512MU810/debug/B40/spi/abcc_crc32.o
 .debug_frame     0x000024         0x50 build/XC16_dsPIC33EP512MU810/debug/B40/spi/abcc_handler_spi.o
 .debug_frame     0x000074        0x2e4 build/XC16_dsPIC33EP512MU810/debug/B40/spi/abcc_spi_drv.o
 .debug_frame     0x000358        0x138 build/XC16_dsPIC33EP512MU810/debug/B40/abcc_cbf.o
 .debug_frame     0x000490        0x380 build/XC16_dsPIC33EP512MU810/debug/B40/abcc_handler.o
 .debug_frame     0x000810        0x1c8 build/XC16_dsPIC33EP512MU810/debug/B40/abcc_link.o
 .debug_frame     0x0009d8         0x44 build/XC16_dsPIC33EP512MU810/debug/B40/abcc_mem.o
 .debug_frame     0x000a1c         0x34 build/XC16_dsPIC33EP512MU810/debug/B40/abcc_remap.o
 .debug_frame     0x000a50        0x30c build/XC16_dsPIC33EP512MU810/debug/B40/abcc_setup.o
 .debug_frame     0x000d5c        0x104 build/XC16_dsPIC33EP512MU810/debug/B40/abcc_sys_adapt.o
 .debug_frame     0x000e60         0x80 build/XC16_dsPIC33EP512MU810/debug/B40/abcc_timer.o
 .debug_frame     0x000ee0         0xd4 build/XC16_dsPIC33EP512MU810/debug/B40/ad_obj.o
 .debug_frame     0x000fb4         0x64 build/XC16_dsPIC33EP512MU810/debug/B40/app_obj.o
 .debug_frame     0x001018         0x44 build/XC16_dsPIC33EP512MU810/debug/B40/dpv1.o
 .debug_frame     0x00105c         0x44 build/XC16_dsPIC33EP512MU810/debug/B40/user_adi.o
 .debug_frame     0x0010a0        0x15c build/XC16_dsPIC33EP512MU810/debug/B40/user_setup.o
 .debug_frame     0x0011fc         0xc4 build/XC16_dsPIC33EP512MU810/debug/ECAN/ECAN1Drv.o
 .debug_frame     0x0012c0         0x24 build/XC16_dsPIC33EP512MU810/debug/BerkeleyTCPClient.o
 .debug_frame     0x0012e4         0x34 build/XC16_dsPIC33EP512MU810/debug/BerkeleyTCPServer.o
 .debug_frame     0x001318         0x34 build/XC16_dsPIC33EP512MU810/debug/BerkeleyUDPClient.o
 .debug_frame     0x00134c         0x44 build/XC16_dsPIC33EP512MU810/debug/MODBUSTCPServer.o
 .debug_frame     0x001390         0x34 build/XC16_dsPIC33EP512MU810/debug/Regul.o
 .debug_frame     0x0013c4         0x24 build/XC16_dsPIC33EP512MU810/debug/Pesage.o
 .debug_frame     0x0013e8        0x3b0 build/XC16_dsPIC33EP512MU810/debug/Process.o
 .debug_frame     0x001798         0x34 build/XC16_dsPIC33EP512MU810/debug/TCPIPStack/Announce.o
 .debug_frame     0x0017cc         0x84 build/XC16_dsPIC33EP512MU810/debug/TCPIPStack/ARP.o
 .debug_frame     0x001850         0xe4 build/XC16_dsPIC33EP512MU810/debug/TCPIPStack/BerkeleyAPI.o
 .debug_frame     0x001934         0x34 build/XC16_dsPIC33EP512MU810/debug/TCPIPStack/Delay.o
 .debug_frame     0x001968         0x74 build/XC16_dsPIC33EP512MU810/debug/TCPIPStack/DNS.o
 .debug_frame     0x0019dc        0x214 build/XC16_dsPIC33EP512MU810/debug/TCPIPStack/ENC28J60.o
 .debug_frame     0x001bf0        0x124 build/XC16_dsPIC33EP512MU810/debug/TCPIPStack/Helpers.o
 .debug_frame     0x001d14        0x124 build/XC16_dsPIC33EP512MU810/debug/TCPIPStack/HTTP2.o
 .debug_frame     0x001e38         0x74 build/XC16_dsPIC33EP512MU810/debug/TCPIPStack/ICMP.o
 .debug_frame     0x001eac         0x54 build/XC16_dsPIC33EP512MU810/debug/TCPIPStack/IP.o
 .debug_frame     0x001f00        0x154 build/XC16_dsPIC33EP512MU810/debug/TCPIPStack/MPFS2.o
 .debug_frame     0x002054         0x44 build/XC16_dsPIC33EP512MU810/debug/TCPIPStack/NBNS.o
 .debug_frame     0x002098         0x24 build/XC16_dsPIC33EP512MU810/debug/TCPIPStack/Reboot.o
 .debug_frame     0x0020bc         0xc4 build/XC16_dsPIC33EP512MU810/debug/TCPIPStack/SPIEEPROM.o
 .debug_frame     0x002180         0x44 build/XC16_dsPIC33EP512MU810/debug/TCPIPStack/StackTsk.o
 .debug_frame     0x0021c4        0x234 build/XC16_dsPIC33EP512MU810/debug/TCPIPStack/TCP.o
 .debug_frame     0x0023f8         0x84 build/XC16_dsPIC33EP512MU810/debug/TCPIPStack/Tick.o
 .debug_frame     0x00247c        0x134 build/XC16_dsPIC33EP512MU810/debug/TCPIPStack/UDP.o
 .debug_frame     0x0025b0        0x1b4 build/XC16_dsPIC33EP512MU810/debug/usb/src/usb_device.o
 .debug_frame     0x002764         0x94 build/XC16_dsPIC33EP512MU810/debug/usb/src/usb_device_cdc.o
 .debug_frame     0x0027f8         0x24 build/XC16_dsPIC33EP512MU810/debug/usb/src/usb_hal_dspic33e.o
 .debug_frame     0x00281c         0xc4 build/XC16_dsPIC33EP512MU810/debug/interrupts.o
 .debug_frame     0x0028e0         0xc4 build/XC16_dsPIC33EP512MU810/debug/main.o
 .debug_frame     0x0029a4         0x24 build/XC16_dsPIC33EP512MU810/debug/system.o
 .debug_frame     0x0029c8         0x94 build/XC16_dsPIC33EP512MU810/debug/traps.o
 .debug_frame     0x002a5c        0x268 build/XC16_dsPIC33EP512MU810/debug/user.o
 .debug_frame     0x002cc4        0x284 build/XC16_dsPIC33EP512MU810/debug/CustomHTTPApp.o
 .debug_frame     0x002f48        0x21c build/XC16_dsPIC33EP512MU810/debug/AD7190.o
 .debug_frame     0x003164         0x44 build/XC16_dsPIC33EP512MU810/debug/ADComm.o
 .debug_frame     0x0031a8        0x114 build/XC16_dsPIC33EP512MU810/debug/UARTsComm.o
 .debug_frame     0x0032bc        0x124 build/XC16_dsPIC33EP512MU810/debug/MemFlash.o
 .debug_frame     0x0033e0         0x54 build/XC16_dsPIC33EP512MU810/debug/ADC10bitsDrv.o
 .debug_frame     0x003434         0xb4 build/XC16_dsPIC33EP512MU810/debug/SPIFRAM.o
 .debug_frame     0x0034e8        0x43c build/XC16_dsPIC33EP512MU810/debug/ModbusUartServer.o

.debug_str        0x000000       0x25b5
 *(.debug_str)
 .debug_str       0x000000         0x20 build/XC16_dsPIC33EP512MU810/debug/B40/spi/abcc_crc32.o
 .debug_str       0x000020         0x67 build/XC16_dsPIC33EP512MU810/debug/B40/spi/abcc_handler_spi.o
 .debug_str       0x000087         0xb8 build/XC16_dsPIC33EP512MU810/debug/B40/spi/abcc_spi_drv.o
 .debug_str       0x00013f        0x16d build/XC16_dsPIC33EP512MU810/debug/B40/abcc_cbf.o
 .debug_str       0x0002ac         0x25 build/XC16_dsPIC33EP512MU810/debug/B40/abcc_debug_err.o
 .debug_str       0x0002d1        0x2ce build/XC16_dsPIC33EP512MU810/debug/B40/abcc_handler.o
 .debug_str       0x00059f        0x154 build/XC16_dsPIC33EP512MU810/debug/B40/abcc_link.o
 .debug_str       0x0006f3          0xd build/XC16_dsPIC33EP512MU810/debug/B40/abcc_mem.o
 .debug_str       0x000700         0x1e build/XC16_dsPIC33EP512MU810/debug/B40/abcc_remap.o
 .debug_str       0x00071e        0x1ce build/XC16_dsPIC33EP512MU810/debug/B40/abcc_setup.o
 .debug_str       0x0008ec         0x71 build/XC16_dsPIC33EP512MU810/debug/B40/abcc_sys_adapt.o
 .debug_str       0x00095d         0x61 build/XC16_dsPIC33EP512MU810/debug/B40/abcc_timer.o
 .debug_str       0x0009be        0x225 build/XC16_dsPIC33EP512MU810/debug/B40/ad_obj.o
 .debug_str       0x000be3         0x97 build/XC16_dsPIC33EP512MU810/debug/B40/app_obj.o
 .debug_str       0x000c7a         0x68 build/XC16_dsPIC33EP512MU810/debug/B40/dpv1.o
 .debug_str       0x000ce2        0x1c8 build/XC16_dsPIC33EP512MU810/debug/B40/user_adi.o
 .debug_str       0x000eaa         0x54 build/XC16_dsPIC33EP512MU810/debug/B40/user_setup.o
 .debug_str       0x000efe        0x16d build/XC16_dsPIC33EP512MU810/debug/ECAN/ECAN1Drv.o
 .debug_str       0x00106b          0xa build/XC16_dsPIC33EP512MU810/debug/BerkeleyTCPClient.o
 .debug_str       0x001075         0x14 build/XC16_dsPIC33EP512MU810/debug/BerkeleyTCPServer.o
 .debug_str       0x001089         0x23 build/XC16_dsPIC33EP512MU810/debug/MODBUSTCPServer.o
 .debug_str       0x0010ac         0x50 build/XC16_dsPIC33EP512MU810/debug/Regul.o
 .debug_str       0x0010fc         0x50 build/XC16_dsPIC33EP512MU810/debug/Pesage.o
 .debug_str       0x00114c        0x2d8 build/XC16_dsPIC33EP512MU810/debug/Process.o
 .debug_str       0x001424         0x2c build/XC16_dsPIC33EP512MU810/debug/TCPIPStack/Announce.o
 .debug_str       0x001450         0x18 build/XC16_dsPIC33EP512MU810/debug/TCPIPStack/ARP.o
 .debug_str       0x001468         0x5a build/XC16_dsPIC33EP512MU810/debug/TCPIPStack/BerkeleyAPI.o
 .debug_str       0x0014c2          0xa build/XC16_dsPIC33EP512MU810/debug/TCPIPStack/DNS.o
 .debug_str       0x0014cc         0xbf build/XC16_dsPIC33EP512MU810/debug/TCPIPStack/ENC28J60.o
 .debug_str       0x00158b          0x9 build/XC16_dsPIC33EP512MU810/debug/TCPIPStack/Helpers.o
 .debug_str       0x001594         0x2c build/XC16_dsPIC33EP512MU810/debug/TCPIPStack/HTTP2.o
 .debug_str       0x0015c0         0x13 build/XC16_dsPIC33EP512MU810/debug/TCPIPStack/IP.o
 .debug_str       0x0015d3         0x11 build/XC16_dsPIC33EP512MU810/debug/TCPIPStack/MPFS2.o
 .debug_str       0x0015e4         0x23 build/XC16_dsPIC33EP512MU810/debug/TCPIPStack/NBNS.o
 .debug_str       0x001607         0x1e build/XC16_dsPIC33EP512MU810/debug/TCPIPStack/Reboot.o
 .debug_str       0x001625         0x64 build/XC16_dsPIC33EP512MU810/debug/TCPIPStack/SPIEEPROM.o
 .debug_str       0x001689         0x15 build/XC16_dsPIC33EP512MU810/debug/TCPIPStack/StackTsk.o
 .debug_str       0x00169e         0xcb build/XC16_dsPIC33EP512MU810/debug/TCPIPStack/TCP.o
 .debug_str       0x001769         0x25 build/XC16_dsPIC33EP512MU810/debug/TCPIPStack/Tick.o
 .debug_str       0x00178e         0x7f build/XC16_dsPIC33EP512MU810/debug/TCPIPStack/UDP.o
 .debug_str       0x00180d        0x290 build/XC16_dsPIC33EP512MU810/debug/usb/src/usb_device.o
 .debug_str       0x001a9d         0xde build/XC16_dsPIC33EP512MU810/debug/usb/src/usb_device_cdc.o
 .debug_str       0x001b7b         0x1e build/XC16_dsPIC33EP512MU810/debug/usb/src/usb_hal_dspic33e.o
 .debug_str       0x001b99        0x10b build/XC16_dsPIC33EP512MU810/debug/interrupts.o
 .debug_str       0x001ca4        0x2e1 build/XC16_dsPIC33EP512MU810/debug/main.o
 .debug_str       0x001f85         0x3e build/XC16_dsPIC33EP512MU810/debug/system.o
 .debug_str       0x001fc3          0xc build/XC16_dsPIC33EP512MU810/debug/traps.o
 .debug_str       0x001fcf         0xf6 build/XC16_dsPIC33EP512MU810/debug/user.o
 .debug_str       0x0020c5         0x61 build/XC16_dsPIC33EP512MU810/debug/CustomHTTPApp.o
 .debug_str       0x002126         0x7b build/XC16_dsPIC33EP512MU810/debug/AD7190.o
 .debug_str       0x0021a1         0x58 build/XC16_dsPIC33EP512MU810/debug/ADComm.o
 .debug_str       0x0021f9         0xdf build/XC16_dsPIC33EP512MU810/debug/UARTsComm.o
 .debug_str       0x0022d8         0x65 build/XC16_dsPIC33EP512MU810/debug/MemFlash.o
 .debug_str       0x00233d         0x9b build/XC16_dsPIC33EP512MU810/debug/ADC10bitsDrv.o
 .debug_str       0x0023d8         0x5a build/XC16_dsPIC33EP512MU810/debug/SPIFRAM.o
 .debug_str       0x002432         0x2a build/XC16_dsPIC33EP512MU810/debug/usb_descriptors.o
 .debug_str       0x00245c        0x159 build/XC16_dsPIC33EP512MU810/debug/ModbusUartServer.o

.debug_loc
 *(.debug_loc)

.debug_macinfo
 *(.debug_macinfo)

.debug_pubnames
                  0x000000       0x3b5a
 *(.debug_pubnames)
 .debug_pubnames
                  0x000000         0x48 build/XC16_dsPIC33EP512MU810/debug/B40/spi/abcc_crc32.o
 .debug_pubnames
                  0x000048         0x38 build/XC16_dsPIC33EP512MU810/debug/B40/spi/abcc_handler_spi.o
 .debug_pubnames
                  0x000080        0x286 build/XC16_dsPIC33EP512MU810/debug/B40/spi/abcc_spi_drv.o
 .debug_pubnames
                  0x000306        0x126 build/XC16_dsPIC33EP512MU810/debug/B40/abcc_cbf.o
 .debug_pubnames
                  0x00042c         0x24 build/XC16_dsPIC33EP512MU810/debug/B40/abcc_debug_err.o
 .debug_pubnames
                  0x000450        0x598 build/XC16_dsPIC33EP512MU810/debug/B40/abcc_handler.o
 .debug_pubnames
                  0x0009e8        0x157 build/XC16_dsPIC33EP512MU810/debug/B40/abcc_link.o
 .debug_pubnames
                  0x000b3f         0x4c build/XC16_dsPIC33EP512MU810/debug/B40/abcc_mem.o
 .debug_pubnames
                  0x000b8b         0x2c build/XC16_dsPIC33EP512MU810/debug/B40/abcc_remap.o
 .debug_pubnames
                  0x000bb7         0xc8 build/XC16_dsPIC33EP512MU810/debug/B40/abcc_setup.o
 .debug_pubnames
                  0x000c7f        0x1d9 build/XC16_dsPIC33EP512MU810/debug/B40/abcc_sys_adapt.o
 .debug_pubnames
                  0x000e58         0x74 build/XC16_dsPIC33EP512MU810/debug/B40/abcc_timer.o
 .debug_pubnames
                  0x000ecc        0x117 build/XC16_dsPIC33EP512MU810/debug/B40/ad_obj.o
 .debug_pubnames
                  0x000fe3         0xc4 build/XC16_dsPIC33EP512MU810/debug/B40/app_obj.o
 .debug_pubnames
                  0x0010a7         0x7c build/XC16_dsPIC33EP512MU810/debug/B40/dpv1.o
 .debug_pubnames
                  0x001123        0x125 build/XC16_dsPIC33EP512MU810/debug/B40/user_adi.o
 .debug_pubnames
                  0x001248         0xa7 build/XC16_dsPIC33EP512MU810/debug/B40/user_setup.o
 .debug_pubnames
                  0x0012ef        0x1a8 build/XC16_dsPIC33EP512MU810/debug/ECAN/ECAN1Drv.o
 .debug_pubnames
                  0x001497         0x28 build/XC16_dsPIC33EP512MU810/debug/BerkeleyTCPClient.o
 .debug_pubnames
                  0x0014bf         0x37 build/XC16_dsPIC33EP512MU810/debug/BerkeleyTCPServer.o
 .debug_pubnames
                  0x0014f6         0x46 build/XC16_dsPIC33EP512MU810/debug/BerkeleyUDPClient.o
 .debug_pubnames
                  0x00153c         0xf2 build/XC16_dsPIC33EP512MU810/debug/MODBUSTCPServer.o
 .debug_pubnames
                  0x00162e         0x39 build/XC16_dsPIC33EP512MU810/debug/Regul.o
 .debug_pubnames
                  0x001667         0x29 build/XC16_dsPIC33EP512MU810/debug/Pesage.o
 .debug_pubnames
                  0x001690        0x299 build/XC16_dsPIC33EP512MU810/debug/Process.o
 .debug_pubnames
                  0x001929         0x33 build/XC16_dsPIC33EP512MU810/debug/TCPIPStack/Announce.o
 .debug_pubnames
                  0x00195c         0x6f build/XC16_dsPIC33EP512MU810/debug/TCPIPStack/ARP.o
 .debug_pubnames
                  0x0019cb         0xa9 build/XC16_dsPIC33EP512MU810/debug/TCPIPStack/BerkeleyAPI.o
 .debug_pubnames
                  0x001a74         0x2c build/XC16_dsPIC33EP512MU810/debug/TCPIPStack/Delay.o
 .debug_pubnames
                  0x001aa0         0x55 build/XC16_dsPIC33EP512MU810/debug/TCPIPStack/DNS.o
 .debug_pubnames
                  0x001af5        0x1b8 build/XC16_dsPIC33EP512MU810/debug/TCPIPStack/ENC28J60.o
 .debug_pubnames
                  0x001cad        0x11b build/XC16_dsPIC33EP512MU810/debug/TCPIPStack/Helpers.o
 .debug_pubnames
                  0x001dc8         0xcf build/XC16_dsPIC33EP512MU810/debug/TCPIPStack/HTTP2.o
 .debug_pubnames
                  0x001e97         0x7f build/XC16_dsPIC33EP512MU810/debug/TCPIPStack/ICMP.o
 .debug_pubnames
                  0x001f16         0x44 build/XC16_dsPIC33EP512MU810/debug/TCPIPStack/IP.o
 .debug_pubnames
                  0x001f5a        0x140 build/XC16_dsPIC33EP512MU810/debug/TCPIPStack/MPFS2.o
 .debug_pubnames
                  0x00209a         0x1f build/XC16_dsPIC33EP512MU810/debug/TCPIPStack/NBNS.o
 .debug_pubnames
                  0x0020b9         0x21 build/XC16_dsPIC33EP512MU810/debug/TCPIPStack/Reboot.o
 .debug_pubnames
                  0x0020da         0xaa build/XC16_dsPIC33EP512MU810/debug/TCPIPStack/SPIEEPROM.o
 .debug_pubnames
                  0x002184         0x53 build/XC16_dsPIC33EP512MU810/debug/TCPIPStack/StackTsk.o
 .debug_pubnames
                  0x0021d7        0x1ba build/XC16_dsPIC33EP512MU810/debug/TCPIPStack/TCP.o
 .debug_pubnames
                  0x002391         0x7e build/XC16_dsPIC33EP512MU810/debug/TCPIPStack/Tick.o
 .debug_pubnames
                  0x00240f        0x155 build/XC16_dsPIC33EP512MU810/debug/TCPIPStack/UDP.o
 .debug_pubnames
                  0x002564        0x33a build/XC16_dsPIC33EP512MU810/debug/usb/src/usb_device.o
 .debug_pubnames
                  0x00289e        0x1b2 build/XC16_dsPIC33EP512MU810/debug/usb/src/usb_device_cdc.o
 .debug_pubnames
                  0x002a50         0x28 build/XC16_dsPIC33EP512MU810/debug/usb/src/usb_hal_dspic33e.o
 .debug_pubnames
                  0x002a78         0xe1 build/XC16_dsPIC33EP512MU810/debug/interrupts.o
 .debug_pubnames
                  0x002b59        0x159 build/XC16_dsPIC33EP512MU810/debug/main.o
 .debug_pubnames
                  0x002cb2         0x2a build/XC16_dsPIC33EP512MU810/debug/system.o
 .debug_pubnames
                  0x002cdc         0xa2 build/XC16_dsPIC33EP512MU810/debug/traps.o
 .debug_pubnames
                  0x002d7e        0x138 build/XC16_dsPIC33EP512MU810/debug/user.o
 .debug_pubnames
                  0x002eb6        0x3bd build/XC16_dsPIC33EP512MU810/debug/CustomHTTPApp.o
 .debug_pubnames
                  0x003273        0x186 build/XC16_dsPIC33EP512MU810/debug/AD7190.o
 .debug_pubnames
                  0x0033f9         0x6f build/XC16_dsPIC33EP512MU810/debug/ADComm.o
 .debug_pubnames
                  0x003468        0x23b build/XC16_dsPIC33EP512MU810/debug/UARTsComm.o
 .debug_pubnames
                  0x0036a3        0x1da build/XC16_dsPIC33EP512MU810/debug/MemFlash.o
 .debug_pubnames
                  0x00387d         0x7b build/XC16_dsPIC33EP512MU810/debug/ADC10bitsDrv.o
 .debug_pubnames
                  0x0038f8         0xa4 build/XC16_dsPIC33EP512MU810/debug/SPIFRAM.o
 .debug_pubnames
                  0x00399c         0x73 build/XC16_dsPIC33EP512MU810/debug/usb_descriptors.o
 .debug_pubnames
                  0x003a0f        0x14b build/XC16_dsPIC33EP512MU810/debug/ModbusUartServer.o

.debug_ranges
 *(.debug_ranges)

.debug_aranges    0x000000        0x590
 *(.debug_aranges)
 .debug_aranges
                  0x000000         0x18 build/XC16_dsPIC33EP512MU810/debug/B40/spi/abcc_crc32.o
 .debug_aranges
                  0x000018         0x18 build/XC16_dsPIC33EP512MU810/debug/B40/spi/abcc_handler_spi.o
 .debug_aranges
                  0x000030         0x18 build/XC16_dsPIC33EP512MU810/debug/B40/spi/abcc_spi_drv.o
 .debug_aranges
                  0x000048         0x18 build/XC16_dsPIC33EP512MU810/debug/B40/abcc_cbf.o
 .debug_aranges
                  0x000060         0x18 build/XC16_dsPIC33EP512MU810/debug/B40/abcc_handler.o
 .debug_aranges
                  0x000078         0x18 build/XC16_dsPIC33EP512MU810/debug/B40/abcc_link.o
 .debug_aranges
                  0x000090         0x18 build/XC16_dsPIC33EP512MU810/debug/B40/abcc_mem.o
 .debug_aranges
                  0x0000a8         0x18 build/XC16_dsPIC33EP512MU810/debug/B40/abcc_remap.o
 .debug_aranges
                  0x0000c0         0x18 build/XC16_dsPIC33EP512MU810/debug/B40/abcc_setup.o
 .debug_aranges
                  0x0000d8         0x18 build/XC16_dsPIC33EP512MU810/debug/B40/abcc_sys_adapt.o
 .debug_aranges
                  0x0000f0         0x18 build/XC16_dsPIC33EP512MU810/debug/B40/abcc_timer.o
 .debug_aranges
                  0x000108         0x18 build/XC16_dsPIC33EP512MU810/debug/B40/ad_obj.o
 .debug_aranges
                  0x000120         0x18 build/XC16_dsPIC33EP512MU810/debug/B40/app_obj.o
 .debug_aranges
                  0x000138         0x18 build/XC16_dsPIC33EP512MU810/debug/B40/dpv1.o
 .debug_aranges
                  0x000150         0x18 build/XC16_dsPIC33EP512MU810/debug/B40/user_adi.o
 .debug_aranges
                  0x000168         0x18 build/XC16_dsPIC33EP512MU810/debug/B40/user_setup.o
 .debug_aranges
                  0x000180         0x18 build/XC16_dsPIC33EP512MU810/debug/ECAN/ECAN1Drv.o
 .debug_aranges
                  0x000198         0x18 build/XC16_dsPIC33EP512MU810/debug/BerkeleyTCPClient.o
 .debug_aranges
                  0x0001b0         0x18 build/XC16_dsPIC33EP512MU810/debug/BerkeleyTCPServer.o
 .debug_aranges
                  0x0001c8         0x18 build/XC16_dsPIC33EP512MU810/debug/BerkeleyUDPClient.o
 .debug_aranges
                  0x0001e0         0x18 build/XC16_dsPIC33EP512MU810/debug/MODBUSTCPServer.o
 .debug_aranges
                  0x0001f8         0x18 build/XC16_dsPIC33EP512MU810/debug/Regul.o
 .debug_aranges
                  0x000210         0x18 build/XC16_dsPIC33EP512MU810/debug/Pesage.o
 .debug_aranges
                  0x000228         0x18 build/XC16_dsPIC33EP512MU810/debug/Process.o
 .debug_aranges
                  0x000240         0x18 build/XC16_dsPIC33EP512MU810/debug/TCPIPStack/Announce.o
 .debug_aranges
                  0x000258         0x18 build/XC16_dsPIC33EP512MU810/debug/TCPIPStack/ARP.o
 .debug_aranges
                  0x000270         0x18 build/XC16_dsPIC33EP512MU810/debug/TCPIPStack/BerkeleyAPI.o
 .debug_aranges
                  0x000288         0x18 build/XC16_dsPIC33EP512MU810/debug/TCPIPStack/Delay.o
 .debug_aranges
                  0x0002a0         0x18 build/XC16_dsPIC33EP512MU810/debug/TCPIPStack/DNS.o
 .debug_aranges
                  0x0002b8         0x18 build/XC16_dsPIC33EP512MU810/debug/TCPIPStack/ENC28J60.o
 .debug_aranges
                  0x0002d0         0x18 build/XC16_dsPIC33EP512MU810/debug/TCPIPStack/Helpers.o
 .debug_aranges
                  0x0002e8         0x18 build/XC16_dsPIC33EP512MU810/debug/TCPIPStack/HTTP2.o
 .debug_aranges
                  0x000300         0x18 build/XC16_dsPIC33EP512MU810/debug/TCPIPStack/ICMP.o
 .debug_aranges
                  0x000318         0x18 build/XC16_dsPIC33EP512MU810/debug/TCPIPStack/IP.o
 .debug_aranges
                  0x000330         0x18 build/XC16_dsPIC33EP512MU810/debug/TCPIPStack/MPFS2.o
 .debug_aranges
                  0x000348         0x18 build/XC16_dsPIC33EP512MU810/debug/TCPIPStack/NBNS.o
 .debug_aranges
                  0x000360         0x18 build/XC16_dsPIC33EP512MU810/debug/TCPIPStack/Reboot.o
 .debug_aranges
                  0x000378         0x18 build/XC16_dsPIC33EP512MU810/debug/TCPIPStack/SPIEEPROM.o
 .debug_aranges
                  0x000390         0x18 build/XC16_dsPIC33EP512MU810/debug/TCPIPStack/StackTsk.o
 .debug_aranges
                  0x0003a8         0x18 build/XC16_dsPIC33EP512MU810/debug/TCPIPStack/TCP.o
 .debug_aranges
                  0x0003c0         0x18 build/XC16_dsPIC33EP512MU810/debug/TCPIPStack/Tick.o
 .debug_aranges
                  0x0003d8         0x18 build/XC16_dsPIC33EP512MU810/debug/TCPIPStack/UDP.o
 .debug_aranges
                  0x0003f0         0x18 build/XC16_dsPIC33EP512MU810/debug/usb/src/usb_device.o
 .debug_aranges
                  0x000408         0x18 build/XC16_dsPIC33EP512MU810/debug/usb/src/usb_device_cdc.o
 .debug_aranges
                  0x000420         0x18 build/XC16_dsPIC33EP512MU810/debug/usb/src/usb_hal_dspic33e.o
 .debug_aranges
                  0x000438         0x18 build/XC16_dsPIC33EP512MU810/debug/interrupts.o
 .debug_aranges
                  0x000450         0x18 build/XC16_dsPIC33EP512MU810/debug/main.o
 .debug_aranges
                  0x000468         0x18 build/XC16_dsPIC33EP512MU810/debug/system.o
 .debug_aranges
                  0x000480         0x18 build/XC16_dsPIC33EP512MU810/debug/traps.o
 .debug_aranges
                  0x000498         0x18 build/XC16_dsPIC33EP512MU810/debug/user.o
 .debug_aranges
                  0x0004b0         0x20 build/XC16_dsPIC33EP512MU810/debug/MPFSImg2.o
 .debug_aranges
                  0x0004d0         0x18 build/XC16_dsPIC33EP512MU810/debug/CustomHTTPApp.o
 .debug_aranges
                  0x0004e8         0x18 build/XC16_dsPIC33EP512MU810/debug/AD7190.o
 .debug_aranges
                  0x000500         0x18 build/XC16_dsPIC33EP512MU810/debug/ADComm.o
 .debug_aranges
                  0x000518         0x18 build/XC16_dsPIC33EP512MU810/debug/UARTsComm.o
 .debug_aranges
                  0x000530         0x18 build/XC16_dsPIC33EP512MU810/debug/MemFlash.o
 .debug_aranges
                  0x000548         0x18 build/XC16_dsPIC33EP512MU810/debug/ADC10bitsDrv.o
 .debug_aranges
                  0x000560         0x18 build/XC16_dsPIC33EP512MU810/debug/SPIFRAM.o
 .debug_aranges
                  0x000578         0x18 build/XC16_dsPIC33EP512MU810/debug/ModbusUartServer.o

.ivt              0x000004        0x130
                  0x000004          0x4 LONG 0x794 DEFINED (__OscillatorFail)?ABSOLUTE (__OscillatorFail):ABSOLUTE (__DefaultInterrupt)
                  0x000006          0x4 LONG 0x79a DEFINED (__AddressError)?ABSOLUTE (__AddressError):ABSOLUTE (__DefaultInterrupt)
                  0x000008          0x4 LONG 0x7b6 DEFINED (__HardTrapError)?ABSOLUTE (__HardTrapError):ABSOLUTE (__DefaultInterrupt)
                  0x00000a          0x4 LONG 0x7a0 DEFINED (__StackError)?ABSOLUTE (__StackError):ABSOLUTE (__DefaultInterrupt)
                  0x00000c          0x4 LONG 0x7a6 DEFINED (__MathError)?ABSOLUTE (__MathError):ABSOLUTE (__DefaultInterrupt)
                  0x00000e          0x4 LONG 0x7ac DEFINED (__DMACError)?ABSOLUTE (__DMACError):ABSOLUTE (__DefaultInterrupt)
                  0x000010          0x4 LONG 0x7ba DEFINED (__SoftTrapError)?ABSOLUTE (__SoftTrapError):ABSOLUTE (__DefaultInterrupt)
                  0x000012          0x4 LONG 0x7b2 DEFINED (__ReservedTrap7)?ABSOLUTE (__ReservedTrap7):ABSOLUTE (__DefaultInterrupt)
                  0x000014          0x4 LONG 0x7b2 DEFINED (__INT0Interrupt)?ABSOLUTE (__INT0Interrupt):ABSOLUTE (__DefaultInterrupt)
                  0x000016          0x4 LONG 0x7b2 DEFINED (__IC1Interrupt)?ABSOLUTE (__IC1Interrupt):ABSOLUTE (__DefaultInterrupt)
                  0x000018          0x4 LONG 0x7b2 DEFINED (__OC1Interrupt)?ABSOLUTE (__OC1Interrupt):ABSOLUTE (__DefaultInterrupt)
                  0x00001a          0x4 LONG 0x276b4 DEFINED (__T1Interrupt)?ABSOLUTE (__T1Interrupt):ABSOLUTE (__DefaultInterrupt)
                  0x00001c          0x4 LONG 0x5ba DEFINED (__DMA0Interrupt)?ABSOLUTE (__DMA0Interrupt):ABSOLUTE (__DefaultInterrupt)
                  0x00001e          0x4 LONG 0x7b2 DEFINED (__IC2Interrupt)?ABSOLUTE (__IC2Interrupt):ABSOLUTE (__DefaultInterrupt)
                  0x000020          0x4 LONG 0x7b2 DEFINED (__OC2Interrupt)?ABSOLUTE (__OC2Interrupt):ABSOLUTE (__DefaultInterrupt)
                  0x000022          0x4 LONG 0x7b2 DEFINED (__T2Interrupt)?ABSOLUTE (__T2Interrupt):ABSOLUTE (__DefaultInterrupt)
                  0x000024          0x4 LONG 0x7b2 DEFINED (__T3Interrupt)?ABSOLUTE (__T3Interrupt):ABSOLUTE (__DefaultInterrupt)
                  0x000026          0x4 LONG 0x7b2 DEFINED (__SPI1ErrInterrupt)?ABSOLUTE (__SPI1ErrInterrupt):ABSOLUTE (__DefaultInterrupt)
                  0x000028          0x4 LONG 0x7b2 DEFINED (__SPI1Interrupt)?ABSOLUTE (__SPI1Interrupt):ABSOLUTE (__DefaultInterrupt)
                  0x00002a          0x4 LONG 0x392 DEFINED (__U1RXInterrupt)?ABSOLUTE (__U1RXInterrupt):ABSOLUTE (__DefaultInterrupt)
                  0x00002c          0x4 LONG 0x7b2 DEFINED (__U1TXInterrupt)?ABSOLUTE (__U1TXInterrupt):ABSOLUTE (__DefaultInterrupt)
                  0x00002e          0x4 LONG 0x7b2 DEFINED (__AD1Interrupt)?ABSOLUTE (__AD1Interrupt):ABSOLUTE (__DefaultInterrupt)
                  0x000030          0x4 LONG 0x7b2 DEFINED (__DMA1Interrupt)?ABSOLUTE (__DMA1Interrupt):ABSOLUTE (__DefaultInterrupt)
                  0x000032          0x4 LONG 0x7b2 DEFINED (__NVMInterrupt)?ABSOLUTE (__NVMInterrupt):ABSOLUTE (__DefaultInterrupt)
                  0x000034          0x4 LONG 0x7b2 DEFINED (__SI2C1Interrupt)?ABSOLUTE (__SI2C1Interrupt):ABSOLUTE (__DefaultInterrupt)
                  0x000036          0x4 LONG 0x7b2 DEFINED (__MI2C1Interrupt)?ABSOLUTE (__MI2C1Interrupt):ABSOLUTE (__DefaultInterrupt)
                  0x000038          0x4 LONG 0x7b2 DEFINED (__CM1Interrupt)?ABSOLUTE (__CM1Interrupt):ABSOLUTE (__DefaultInterrupt)
                  0x00003a          0x4 LONG 0x7b2 DEFINED (__CNInterrupt)?ABSOLUTE (__CNInterrupt):ABSOLUTE (__DefaultInterrupt)
                  0x00003c          0x4 LONG 0x65e DEFINED (__INT1Interrupt)?ABSOLUTE (__INT1Interrupt):ABSOLUTE (__DefaultInterrupt)
                  0x00003e          0x4 LONG 0x7b2 DEFINED (__AD2Interrupt)?ABSOLUTE (__AD2Interrupt):ABSOLUTE (__DefaultInterrupt)
                  0x000040          0x4 LONG 0x7b2 DEFINED (__IC7Interrupt)?ABSOLUTE (__IC7Interrupt):ABSOLUTE (__DefaultInterrupt)
                  0x000042          0x4 LONG 0x7b2 DEFINED (__IC8Interrupt)?ABSOLUTE (__IC8Interrupt):ABSOLUTE (__DefaultInterrupt)
                  0x000044          0x4 LONG 0x7b2 DEFINED (__DMA2Interrupt)?ABSOLUTE (__DMA2Interrupt):ABSOLUTE (__DefaultInterrupt)
                  0x000046          0x4 LONG 0x7b2 DEFINED (__OC3Interrupt)?ABSOLUTE (__OC3Interrupt):ABSOLUTE (__DefaultInterrupt)
                  0x000048          0x4 LONG 0x7b2 DEFINED (__OC4Interrupt)?ABSOLUTE (__OC4Interrupt):ABSOLUTE (__DefaultInterrupt)
                  0x00004a          0x4 LONG 0x7b2 DEFINED (__T4Interrupt)?ABSOLUTE (__T4Interrupt):ABSOLUTE (__DefaultInterrupt)
                  0x00004c          0x4 LONG 0x7b2 DEFINED (__T5Interrupt)?ABSOLUTE (__T5Interrupt):ABSOLUTE (__DefaultInterrupt)
                  0x00004e          0x4 LONG 0x698 DEFINED (__INT2Interrupt)?ABSOLUTE (__INT2Interrupt):ABSOLUTE (__DefaultInterrupt)
                  0x000050          0x4 LONG 0x41c DEFINED (__U2RXInterrupt)?ABSOLUTE (__U2RXInterrupt):ABSOLUTE (__DefaultInterrupt)
                  0x000052          0x4 LONG 0x7b2 DEFINED (__U2TXInterrupt)?ABSOLUTE (__U2TXInterrupt):ABSOLUTE (__DefaultInterrupt)
                  0x000054          0x4 LONG 0x7b2 DEFINED (__SPI2ErrInterrupt)?ABSOLUTE (__SPI2ErrInterrupt):ABSOLUTE (__DefaultInterrupt)
                  0x000056          0x4 LONG 0x7b2 DEFINED (__SPI2Interrupt)?ABSOLUTE (__SPI2Interrupt):ABSOLUTE (__DefaultInterrupt)
                  0x000058          0x4 LONG 0x7b2 DEFINED (__C1RxRdyInterrupt)?ABSOLUTE (__C1RxRdyInterrupt):ABSOLUTE (__DefaultInterrupt)
                  0x00005a          0x4 LONG 0x750 DEFINED (__C1Interrupt)?ABSOLUTE (__C1Interrupt):ABSOLUTE (__DefaultInterrupt)
                  0x00005c          0x4 LONG 0x7b2 DEFINED (__DMA3Interrupt)?ABSOLUTE (__DMA3Interrupt):ABSOLUTE (__DefaultInterrupt)
                  0x00005e          0x4 LONG 0x7b2 DEFINED (__IC3Interrupt)?ABSOLUTE (__IC3Interrupt):ABSOLUTE (__DefaultInterrupt)
                  0x000060          0x4 LONG 0x7b2 DEFINED (__IC4Interrupt)?ABSOLUTE (__IC4Interrupt):ABSOLUTE (__DefaultInterrupt)
                  0x000062          0x4 LONG 0x7b2 DEFINED (__IC5Interrupt)?ABSOLUTE (__IC5Interrupt):ABSOLUTE (__DefaultInterrupt)
                  0x000064          0x4 LONG 0x7b2 DEFINED (__IC6Interrupt)?ABSOLUTE (__IC6Interrupt):ABSOLUTE (__DefaultInterrupt)
                  0x000066          0x4 LONG 0x7b2 DEFINED (__OC5Interrupt)?ABSOLUTE (__OC5Interrupt):ABSOLUTE (__DefaultInterrupt)
                  0x000068          0x4 LONG 0x7b2 DEFINED (__OC6Interrupt)?ABSOLUTE (__OC6Interrupt):ABSOLUTE (__DefaultInterrupt)
                  0x00006a          0x4 LONG 0x7b2 DEFINED (__OC7Interrupt)?ABSOLUTE (__OC7Interrupt):ABSOLUTE (__DefaultInterrupt)
                  0x00006c          0x4 LONG 0x7b2 DEFINED (__OC8Interrupt)?ABSOLUTE (__OC8Interrupt):ABSOLUTE (__DefaultInterrupt)
                  0x00006e          0x4 LONG 0x7b2 DEFINED (__PMPInterrupt)?ABSOLUTE (__PMPInterrupt):ABSOLUTE (__DefaultInterrupt)
                  0x000070          0x4 LONG 0x7b2 DEFINED (__DMA4Interrupt)?ABSOLUTE (__DMA4Interrupt):ABSOLUTE (__DefaultInterrupt)
                  0x000072          0x4 LONG 0x7b2 DEFINED (__T6Interrupt)?ABSOLUTE (__T6Interrupt):ABSOLUTE (__DefaultInterrupt)
                  0x000074          0x4 LONG 0x7b2 DEFINED (__T7Interrupt)?ABSOLUTE (__T7Interrupt):ABSOLUTE (__DefaultInterrupt)
                  0x000076          0x4 LONG 0x7b2 DEFINED (__SI2C2Interrupt)?ABSOLUTE (__SI2C2Interrupt):ABSOLUTE (__DefaultInterrupt)
                  0x000078          0x4 LONG 0x7b2 DEFINED (__MI2C2Interrupt)?ABSOLUTE (__MI2C2Interrupt):ABSOLUTE (__DefaultInterrupt)
                  0x00007a          0x4 LONG 0x7b2 DEFINED (__T8Interrupt)?ABSOLUTE (__T8Interrupt):ABSOLUTE (__DefaultInterrupt)
                  0x00007c          0x4 LONG 0x7b2 DEFINED (__T9Interrupt)?ABSOLUTE (__T9Interrupt):ABSOLUTE (__DefaultInterrupt)
                  0x00007e          0x4 LONG 0x6b4 DEFINED (__INT3Interrupt)?ABSOLUTE (__INT3Interrupt):ABSOLUTE (__DefaultInterrupt)
                  0x000080          0x4 LONG 0x6fa DEFINED (__INT4Interrupt)?ABSOLUTE (__INT4Interrupt):ABSOLUTE (__DefaultInterrupt)
                  0x000082          0x4 LONG 0x7b2 DEFINED (__C2RxRdyInterrupt)?ABSOLUTE (__C2RxRdyInterrupt):ABSOLUTE (__DefaultInterrupt)
                  0x000084          0x4 LONG 0x7b2 DEFINED (__C2Interrupt)?ABSOLUTE (__C2Interrupt):ABSOLUTE (__DefaultInterrupt)
                  0x000086          0x4 LONG 0x7b2 DEFINED (__PWMSpEventMatchInterrupt)?ABSOLUTE (__PWMSpEventMatchInterrupt):ABSOLUTE (__DefaultInterrupt)
                  0x000088          0x4 LONG 0x7b2 DEFINED (__QEI1Interrupt)?ABSOLUTE (__QEI1Interrupt):ABSOLUTE (__DefaultInterrupt)
                  0x00008a          0x4 LONG 0x7b2 DEFINED (__DCIEInterrupt)?ABSOLUTE (__DCIEInterrupt):ABSOLUTE (__DefaultInterrupt)
                  0x00008c          0x4 LONG 0x7b2 DEFINED (__DCIInterrupt)?ABSOLUTE (__DCIInterrupt):ABSOLUTE (__DefaultInterrupt)
                  0x00008e          0x4 LONG 0x7b2 DEFINED (__DMA5Interrupt)?ABSOLUTE (__DMA5Interrupt):ABSOLUTE (__DefaultInterrupt)
                  0x000090          0x4 LONG 0x7b2 DEFINED (__RTCCInterrupt)?ABSOLUTE (__RTCCInterrupt):ABSOLUTE (__DefaultInterrupt)
                  0x000092          0x4 LONG 0x7b2 DEFINED (__Interrupt63)?ABSOLUTE (__Interrupt63):ABSOLUTE (__DefaultInterrupt)
                  0x000094          0x4 LONG 0x7b2 DEFINED (__Interrupt64)?ABSOLUTE (__Interrupt64):ABSOLUTE (__DefaultInterrupt)
                  0x000096          0x4 LONG 0x7b2 DEFINED (__U1ErrInterrupt)?ABSOLUTE (__U1ErrInterrupt):ABSOLUTE (__DefaultInterrupt)
                  0x000098          0x4 LONG 0x7b2 DEFINED (__U2ErrInterrupt)?ABSOLUTE (__U2ErrInterrupt):ABSOLUTE (__DefaultInterrupt)
                  0x00009a          0x4 LONG 0x7b2 DEFINED (__CRCInterrupt)?ABSOLUTE (__CRCInterrupt):ABSOLUTE (__DefaultInterrupt)
                  0x00009c          0x4 LONG 0x7b2 DEFINED (__DMA6Interrupt)?ABSOLUTE (__DMA6Interrupt):ABSOLUTE (__DefaultInterrupt)
                  0x00009e          0x4 LONG 0x7b2 DEFINED (__DMA7Interrupt)?ABSOLUTE (__DMA7Interrupt):ABSOLUTE (__DefaultInterrupt)
                  0x0000a0          0x4 LONG 0x7b2 DEFINED (__C1TxReqInterrupt)?ABSOLUTE (__C1TxReqInterrupt):ABSOLUTE (__DefaultInterrupt)
                  0x0000a2          0x4 LONG 0x7b2 DEFINED (__C2TxReqInterrupt)?ABSOLUTE (__C2TxReqInterrupt):ABSOLUTE (__DefaultInterrupt)
                  0x0000a4          0x4 LONG 0x7b2 DEFINED (__Interrupt72)?ABSOLUTE (__Interrupt72):ABSOLUTE (__DefaultInterrupt)
                  0x0000a6          0x4 LONG 0x7b2 DEFINED (__PWMSecSpEventMatchInterrupt)?ABSOLUTE (__PWMSecSpEventMatchInterrupt):ABSOLUTE (__DefaultInterrupt)
                  0x0000a8          0x4 LONG 0x7b2 DEFINED (__Interrupt74)?ABSOLUTE (__Interrupt74):ABSOLUTE (__DefaultInterrupt)
                  0x0000aa          0x4 LONG 0x7b2 DEFINED (__QEI2Interrupt)?ABSOLUTE (__QEI2Interrupt):ABSOLUTE (__DefaultInterrupt)
                  0x0000ac          0x4 LONG 0x7b2 DEFINED (__Interrupt76)?ABSOLUTE (__Interrupt76):ABSOLUTE (__DefaultInterrupt)
                  0x0000ae          0x4 LONG 0x7b2 DEFINED (__Interrupt77)?ABSOLUTE (__Interrupt77):ABSOLUTE (__DefaultInterrupt)
                  0x0000b0          0x4 LONG 0x7b2 DEFINED (__Interrupt78)?ABSOLUTE (__Interrupt78):ABSOLUTE (__DefaultInterrupt)
                  0x0000b2          0x4 LONG 0x7b2 DEFINED (__Interrupt79)?ABSOLUTE (__Interrupt79):ABSOLUTE (__DefaultInterrupt)
                  0x0000b4          0x4 LONG 0x7b2 DEFINED (__Interrupt80)?ABSOLUTE (__Interrupt80):ABSOLUTE (__DefaultInterrupt)
                  0x0000b6          0x4 LONG 0x7b2 DEFINED (__U3ErrInterrupt)?ABSOLUTE (__U3ErrInterrupt):ABSOLUTE (__DefaultInterrupt)
                  0x0000b8          0x4 LONG 0x4a6 DEFINED (__U3RXInterrupt)?ABSOLUTE (__U3RXInterrupt):ABSOLUTE (__DefaultInterrupt)
                  0x0000ba          0x4 LONG 0x7b2 DEFINED (__U3TXInterrupt)?ABSOLUTE (__U3TXInterrupt):ABSOLUTE (__DefaultInterrupt)
                  0x0000bc          0x4 LONG 0x7b2 DEFINED (__Interrupt84)?ABSOLUTE (__Interrupt84):ABSOLUTE (__DefaultInterrupt)
                  0x0000be          0x4 LONG 0x7b2 DEFINED (__Interrupt85)?ABSOLUTE (__Interrupt85):ABSOLUTE (__DefaultInterrupt)
                  0x0000c0          0x4 LONG 0x728 DEFINED (__USB1Interrupt)?ABSOLUTE (__USB1Interrupt):ABSOLUTE (__DefaultInterrupt)
                  0x0000c2          0x4 LONG 0x7b2 DEFINED (__U4ErrInterrupt)?ABSOLUTE (__U4ErrInterrupt):ABSOLUTE (__DefaultInterrupt)
                  0x0000c4          0x4 LONG 0x530 DEFINED (__U4RXInterrupt)?ABSOLUTE (__U4RXInterrupt):ABSOLUTE (__DefaultInterrupt)
                  0x0000c6          0x4 LONG 0x7b2 DEFINED (__U4TXInterrupt)?ABSOLUTE (__U4TXInterrupt):ABSOLUTE (__DefaultInterrupt)
                  0x0000c8          0x4 LONG 0x7b2 DEFINED (__SPI3ErrInterrupt)?ABSOLUTE (__SPI3ErrInterrupt):ABSOLUTE (__DefaultInterrupt)
                  0x0000ca          0x4 LONG 0x7b2 DEFINED (__SPI3Interrupt)?ABSOLUTE (__SPI3Interrupt):ABSOLUTE (__DefaultInterrupt)
                  0x0000cc          0x4 LONG 0x7b2 DEFINED (__OC9Interrupt)?ABSOLUTE (__OC9Interrupt):ABSOLUTE (__DefaultInterrupt)
                  0x0000ce          0x4 LONG 0x7b2 DEFINED (__IC9Interrupt)?ABSOLUTE (__IC9Interrupt):ABSOLUTE (__DefaultInterrupt)
                  0x0000d0          0x4 LONG 0x7b2 DEFINED (__PWM1Interrupt)?ABSOLUTE (__PWM1Interrupt):ABSOLUTE (__DefaultInterrupt)
                  0x0000d2          0x4 LONG 0x7b2 DEFINED (__PWM2Interrupt)?ABSOLUTE (__PWM2Interrupt):ABSOLUTE (__DefaultInterrupt)
                  0x0000d4          0x4 LONG 0x7b2 DEFINED (__PWM3Interrupt)?ABSOLUTE (__PWM3Interrupt):ABSOLUTE (__DefaultInterrupt)
                  0x0000d6          0x4 LONG 0x7b2 DEFINED (__PWM4Interrupt)?ABSOLUTE (__PWM4Interrupt):ABSOLUTE (__DefaultInterrupt)
                  0x0000d8          0x4 LONG 0x7b2 DEFINED (__PWM5Interrupt)?ABSOLUTE (__PWM5Interrupt):ABSOLUTE (__DefaultInterrupt)
                  0x0000da          0x4 LONG 0x7b2 DEFINED (__PWM6Interrupt)?ABSOLUTE (__PWM6Interrupt):ABSOLUTE (__DefaultInterrupt)
                  0x0000dc          0x4 LONG 0x7b2 DEFINED (__Interrupt100)?ABSOLUTE (__Interrupt100):ABSOLUTE (__DefaultInterrupt)
                  0x0000de          0x4 LONG 0x7b2 DEFINED (__Interrupt101)?ABSOLUTE (__Interrupt101):ABSOLUTE (__DefaultInterrupt)
                  0x0000e0          0x4 LONG 0x7b2 DEFINED (__Interrupt102)?ABSOLUTE (__Interrupt102):ABSOLUTE (__DefaultInterrupt)
                  0x0000e2          0x4 LONG 0x7b2 DEFINED (__Interrupt103)?ABSOLUTE (__Interrupt103):ABSOLUTE (__DefaultInterrupt)
                  0x0000e4          0x4 LONG 0x7b2 DEFINED (__Interrupt104)?ABSOLUTE (__Interrupt104):ABSOLUTE (__DefaultInterrupt)
                  0x0000e6          0x4 LONG 0x7b2 DEFINED (__Interrupt105)?ABSOLUTE (__Interrupt105):ABSOLUTE (__DefaultInterrupt)
                  0x0000e8          0x4 LONG 0x7b2 DEFINED (__Interrupt106)?ABSOLUTE (__Interrupt106):ABSOLUTE (__DefaultInterrupt)
                  0x0000ea          0x4 LONG 0x7b2 DEFINED (__Interrupt107)?ABSOLUTE (__Interrupt107):ABSOLUTE (__DefaultInterrupt)
                  0x0000ec          0x4 LONG 0x7b2 DEFINED (__Interrupt108)?ABSOLUTE (__Interrupt108):ABSOLUTE (__DefaultInterrupt)
                  0x0000ee          0x4 LONG 0x7b2 DEFINED (__Interrupt109)?ABSOLUTE (__Interrupt109):ABSOLUTE (__DefaultInterrupt)
                  0x0000f0          0x4 LONG 0x7b2 DEFINED (__Interrupt110)?ABSOLUTE (__Interrupt110):ABSOLUTE (__DefaultInterrupt)
                  0x0000f2          0x4 LONG 0x7b2 DEFINED (__Interrupt111)?ABSOLUTE (__Interrupt111):ABSOLUTE (__DefaultInterrupt)
                  0x0000f4          0x4 LONG 0x7b2 DEFINED (__Interrupt112)?ABSOLUTE (__Interrupt112):ABSOLUTE (__DefaultInterrupt)
                  0x0000f6          0x4 LONG 0x7b2 DEFINED (__Interrupt113)?ABSOLUTE (__Interrupt113):ABSOLUTE (__DefaultInterrupt)
                  0x0000f8          0x4 LONG 0x7b2 DEFINED (__Interrupt114)?ABSOLUTE (__Interrupt114):ABSOLUTE (__DefaultInterrupt)
                  0x0000fa          0x4 LONG 0x7b2 DEFINED (__Interrupt115)?ABSOLUTE (__Interrupt115):ABSOLUTE (__DefaultInterrupt)
                  0x0000fc          0x4 LONG 0x7b2 DEFINED (__Interrupt116)?ABSOLUTE (__Interrupt116):ABSOLUTE (__DefaultInterrupt)
                  0x0000fe          0x4 LONG 0x7b2 DEFINED (__Interrupt117)?ABSOLUTE (__Interrupt117):ABSOLUTE (__DefaultInterrupt)
                  0x000100          0x4 LONG 0x7b2 DEFINED (__DMA8Interrupt)?ABSOLUTE (__DMA8Interrupt):ABSOLUTE (__DefaultInterrupt)
                  0x000102          0x4 LONG 0x7b2 DEFINED (__DMA9Interrupt)?ABSOLUTE (__DMA9Interrupt):ABSOLUTE (__DefaultInterrupt)
                  0x000104          0x4 LONG 0x7b2 DEFINED (__DMA10Interrupt)?ABSOLUTE (__DMA10Interrupt):ABSOLUTE (__DefaultInterrupt)
                  0x000106          0x4 LONG 0x7b2 DEFINED (__DMA11Interrupt)?ABSOLUTE (__DMA11Interrupt):ABSOLUTE (__DefaultInterrupt)
                  0x000108          0x4 LONG 0x7b2 DEFINED (__SPI4ErrInterrupt)?ABSOLUTE (__SPI4ErrInterrupt):ABSOLUTE (__DefaultInterrupt)
                  0x00010a          0x4 LONG 0x7b2 DEFINED (__SPI4Interrupt)?ABSOLUTE (__SPI4Interrupt):ABSOLUTE (__DefaultInterrupt)
                  0x00010c          0x4 LONG 0x7b2 DEFINED (__OC10Interrupt)?ABSOLUTE (__OC10Interrupt):ABSOLUTE (__DefaultInterrupt)
                  0x00010e          0x4 LONG 0x7b2 DEFINED (__IC10Interrupt)?ABSOLUTE (__IC10Interrupt):ABSOLUTE (__DefaultInterrupt)
                  0x000110          0x4 LONG 0x7b2 DEFINED (__OC11Interrupt)?ABSOLUTE (__OC11Interrupt):ABSOLUTE (__DefaultInterrupt)
                  0x000112          0x4 LONG 0x7b2 DEFINED (__IC11Interrupt)?ABSOLUTE (__IC11Interrupt):ABSOLUTE (__DefaultInterrupt)
                  0x000114          0x4 LONG 0x7b2 DEFINED (__OC12Interrupt)?ABSOLUTE (__OC12Interrupt):ABSOLUTE (__DefaultInterrupt)
                  0x000116          0x4 LONG 0x7b2 DEFINED (__IC12Interrupt)?ABSOLUTE (__IC12Interrupt):ABSOLUTE (__DefaultInterrupt)
                  0x000118          0x4 LONG 0x7b2 DEFINED (__DMA12Interrupt)?ABSOLUTE (__DMA12Interrupt):ABSOLUTE (__DefaultInterrupt)
                  0x00011a          0x4 LONG 0x7b2 DEFINED (__DMA13Interrupt)?ABSOLUTE (__DMA13Interrupt):ABSOLUTE (__DefaultInterrupt)
                  0x00011c          0x4 LONG 0x7b2 DEFINED (__DMA14Interrupt)?ABSOLUTE (__DMA14Interrupt):ABSOLUTE (__DefaultInterrupt)
                  0x00011e          0x4 LONG 0x7b2 DEFINED (__Interrupt133)?ABSOLUTE (__Interrupt133):ABSOLUTE (__DefaultInterrupt)
                  0x000120          0x4 LONG 0x7b2 DEFINED (__OC13Interrupt)?ABSOLUTE (__OC13Interrupt):ABSOLUTE (__DefaultInterrupt)
                  0x000122          0x4 LONG 0x7b2 DEFINED (__IC13Interrupt)?ABSOLUTE (__IC13Interrupt):ABSOLUTE (__DefaultInterrupt)
                  0x000124          0x4 LONG 0x7b2 DEFINED (__OC14Interrupt)?ABSOLUTE (__OC14Interrupt):ABSOLUTE (__DefaultInterrupt)
                  0x000126          0x4 LONG 0x7b2 DEFINED (__IC14Interrupt)?ABSOLUTE (__IC14Interrupt):ABSOLUTE (__DefaultInterrupt)
                  0x000128          0x4 LONG 0x7b2 DEFINED (__OC15Interrupt)?ABSOLUTE (__OC15Interrupt):ABSOLUTE (__DefaultInterrupt)
                  0x00012a          0x4 LONG 0x7b2 DEFINED (__IC15Interrupt)?ABSOLUTE (__IC15Interrupt):ABSOLUTE (__DefaultInterrupt)
                  0x00012c          0x4 LONG 0x7b2 DEFINED (__OC16Interrupt)?ABSOLUTE (__OC16Interrupt):ABSOLUTE (__DefaultInterrupt)
                  0x00012e          0x4 LONG 0x7b2 DEFINED (__IC16Interrupt)?ABSOLUTE (__IC16Interrupt):ABSOLUTE (__DefaultInterrupt)
                  0x000130          0x4 LONG 0x7b2 DEFINED (__ICDInterrupt)?ABSOLUTE (__ICDInterrupt):ABSOLUTE (__DefaultInterrupt)
                  0x000132          0x4 LONG 0x7b2 DEFINED (__JTAGInterrupt)?ABSOLUTE (__JTAGInterrupt):ABSOLUTE (__DefaultInterrupt)
                    0x0000                  WREG0 = 0x0
                    0x0000                  _WREG0 = 0x0
                    0x0002                  WREG1 = 0x2
                    0x0002                  _WREG1 = 0x2
                    0x0004                  WREG2 = 0x4
                    0x0004                  _WREG2 = 0x4
                    0x0006                  WREG3 = 0x6
                    0x0006                  _WREG3 = 0x6
                    0x0008                  WREG4 = 0x8
                    0x0008                  _WREG4 = 0x8
                    0x000a                  WREG5 = 0xa
                    0x000a                  _WREG5 = 0xa
                    0x000c                  WREG6 = 0xc
                    0x000c                  _WREG6 = 0xc
                    0x000e                  WREG7 = 0xe
                    0x000e                  _WREG7 = 0xe
                    0x0010                  WREG8 = 0x10
                    0x0010                  _WREG8 = 0x10
                    0x0012                  WREG9 = 0x12
                    0x0012                  _WREG9 = 0x12
                    0x0014                  WREG10 = 0x14
                    0x0014                  _WREG10 = 0x14
                    0x0016                  WREG11 = 0x16
                    0x0016                  _WREG11 = 0x16
                    0x0018                  WREG12 = 0x18
                    0x0018                  _WREG12 = 0x18
                    0x001a                  WREG13 = 0x1a
                    0x001a                  _WREG13 = 0x1a
                    0x001c                  WREG14 = 0x1c
                    0x001c                  _WREG14 = 0x1c
                    0x001e                  WREG15 = 0x1e
                    0x001e                  _WREG15 = 0x1e
                    0x0020                  SPLIM = 0x20
                    0x0020                  _SPLIM = 0x20
                    0x0022                  ACCAL = 0x22
                    0x0022                  _ACCAL = 0x22
                    0x0024                  ACCAH = 0x24
                    0x0024                  _ACCAH = 0x24
                    0x0026                  ACCAU = 0x26
                    0x0026                  _ACCAU = 0x26
                    0x0028                  ACCBL = 0x28
                    0x0028                  _ACCBL = 0x28
                    0x002a                  ACCBH = 0x2a
                    0x002a                  _ACCBH = 0x2a
                    0x002c                  ACCBU = 0x2c
                    0x002c                  _ACCBU = 0x2c
                    0x002e                  PCL = 0x2e
                    0x002e                  _PCL = 0x2e
                    0x0030                  PCH = 0x30
                    0x0030                  _PCH = 0x30
                    0x0032                  DSRPAG = 0x32
                    0x0032                  _DSRPAG = 0x32
                    0x0032                  _DSRPAGbits = 0x32
                    0x0034                  DSWPAG = 0x34
                    0x0034                  _DSWPAG = 0x34
                    0x0034                  _DSWPAGbits = 0x34
                    0x0036                  RCOUNT = 0x36
                    0x0036                  _RCOUNT = 0x36
                    0x0038                  DCOUNT = 0x38
                    0x0038                  _DCOUNT = 0x38
                    0x003a                  DOSTARTL = 0x3a
                    0x003a                  _DOSTARTL = 0x3a
                    0x003c                  DOSTARTH = 0x3c
                    0x003c                  _DOSTARTH = 0x3c
                    0x003e                  DOENDL = 0x3e
                    0x003e                  _DOENDL = 0x3e
                    0x0040                  DOENDH = 0x40
                    0x0040                  _DOENDH = 0x40
                    0x0042                  SR = 0x42
                    0x0042                  _SR = 0x42
                    0x0042                  _SRbits = 0x42
                    0x0044                  CORCON = 0x44
                    0x0044                  _CORCON = 0x44
                    0x0044                  _CORCONbits = 0x44
                    0x0046                  MODCON = 0x46
                    0x0046                  _MODCON = 0x46
                    0x0046                  _MODCONbits = 0x46
                    0x0048                  XMODSRT = 0x48
                    0x0048                  _XMODSRT = 0x48
                    0x004a                  XMODEND = 0x4a
                    0x004a                  _XMODEND = 0x4a
                    0x004c                  YMODSRT = 0x4c
                    0x004c                  _YMODSRT = 0x4c
                    0x004e                  YMODEND = 0x4e
                    0x004e                  _YMODEND = 0x4e
                    0x0050                  XBREV = 0x50
                    0x0050                  _XBREV = 0x50
                    0x0050                  _XBREVbits = 0x50
                    0x0052                  DISICNT = 0x52
                    0x0052                  _DISICNT = 0x52
                    0x0054                  TBLPAG = 0x54
                    0x0054                  _TBLPAG = 0x54
                    0x0054                  _TBLPAGbits = 0x54
                    0x0058                  MSTRPR = 0x58
                    0x0058                  _MSTRPR = 0x58
                    0x0100                  TMR1 = 0x100
                    0x0100                  _TMR1 = 0x100
                    0x0102                  PR1 = 0x102
                    0x0102                  _PR1 = 0x102
                    0x0104                  T1CON = 0x104
                    0x0104                  _T1CON = 0x104
                    0x0104                  _T1CONbits = 0x104
                    0x0106                  TMR2 = 0x106
                    0x0106                  _TMR2 = 0x106
                    0x0108                  TMR3HLD = 0x108
                    0x0108                  _TMR3HLD = 0x108
                    0x010a                  TMR3 = 0x10a
                    0x010a                  _TMR3 = 0x10a
                    0x010c                  PR2 = 0x10c
                    0x010c                  _PR2 = 0x10c
                    0x010e                  PR3 = 0x10e
                    0x010e                  _PR3 = 0x10e
                    0x0110                  T2CON = 0x110
                    0x0110                  _T2CON = 0x110
                    0x0110                  _T2CONbits = 0x110
                    0x0112                  T3CON = 0x112
                    0x0112                  _T3CON = 0x112
                    0x0112                  _T3CONbits = 0x112
                    0x0114                  TMR4 = 0x114
                    0x0114                  _TMR4 = 0x114
                    0x0116                  TMR5HLD = 0x116
                    0x0116                  _TMR5HLD = 0x116
                    0x0118                  TMR5 = 0x118
                    0x0118                  _TMR5 = 0x118
                    0x011a                  PR4 = 0x11a
                    0x011a                  _PR4 = 0x11a
                    0x011c                  PR5 = 0x11c
                    0x011c                  _PR5 = 0x11c
                    0x011e                  T4CON = 0x11e
                    0x011e                  _T4CON = 0x11e
                    0x011e                  _T4CONbits = 0x11e
                    0x0120                  T5CON = 0x120
                    0x0120                  _T5CON = 0x120
                    0x0120                  _T5CONbits = 0x120
                    0x0122                  TMR6 = 0x122
                    0x0122                  _TMR6 = 0x122
                    0x0124                  TMR7HLD = 0x124
                    0x0124                  _TMR7HLD = 0x124
                    0x0126                  TMR7 = 0x126
                    0x0126                  _TMR7 = 0x126
                    0x0128                  PR6 = 0x128
                    0x0128                  _PR6 = 0x128
                    0x012a                  PR7 = 0x12a
                    0x012a                  _PR7 = 0x12a
                    0x012c                  T6CON = 0x12c
                    0x012c                  _T6CON = 0x12c
                    0x012c                  _T6CONbits = 0x12c
                    0x012e                  T7CON = 0x12e
                    0x012e                  _T7CON = 0x12e
                    0x012e                  _T7CONbits = 0x12e
                    0x0130                  TMR8 = 0x130
                    0x0130                  _TMR8 = 0x130
                    0x0132                  TMR9HLD = 0x132
                    0x0132                  _TMR9HLD = 0x132
                    0x0134                  TMR9 = 0x134
                    0x0134                  _TMR9 = 0x134
                    0x0136                  PR8 = 0x136
                    0x0136                  _PR8 = 0x136
                    0x0138                  PR9 = 0x138
                    0x0138                  _PR9 = 0x138
                    0x013a                  T8CON = 0x13a
                    0x013a                  _T8CON = 0x13a
                    0x013a                  _T8CONbits = 0x13a
                    0x013c                  T9CON = 0x13c
                    0x013c                  _T9CON = 0x13c
                    0x013c                  _T9CONbits = 0x13c
                    0x0140                  IC1CON1 = 0x140
                    0x0140                  _IC1CON1 = 0x140
                    0x0140                  _IC1CON1bits = 0x140
                    0x0142                  IC1CON2 = 0x142
                    0x0142                  _IC1CON2 = 0x142
                    0x0142                  _IC1CON2bits = 0x142
                    0x0144                  IC1BUF = 0x144
                    0x0144                  _IC1BUF = 0x144
                    0x0146                  IC1TMR = 0x146
                    0x0146                  _IC1TMR = 0x146
                    0x0148                  IC2CON1 = 0x148
                    0x0148                  _IC2CON1 = 0x148
                    0x0148                  _IC2CON1bits = 0x148
                    0x014a                  IC2CON2 = 0x14a
                    0x014a                  _IC2CON2 = 0x14a
                    0x014a                  _IC2CON2bits = 0x14a
                    0x014c                  IC2BUF = 0x14c
                    0x014c                  _IC2BUF = 0x14c
                    0x014e                  IC2TMR = 0x14e
                    0x014e                  _IC2TMR = 0x14e
                    0x0150                  IC3CON1 = 0x150
                    0x0150                  _IC3CON1 = 0x150
                    0x0150                  _IC3CON1bits = 0x150
                    0x0152                  IC3CON2 = 0x152
                    0x0152                  _IC3CON2 = 0x152
                    0x0152                  _IC3CON2bits = 0x152
                    0x0154                  IC3BUF = 0x154
                    0x0154                  _IC3BUF = 0x154
                    0x0156                  IC3TMR = 0x156
                    0x0156                  _IC3TMR = 0x156
                    0x0158                  IC4CON1 = 0x158
                    0x0158                  _IC4CON1 = 0x158
                    0x0158                  _IC4CON1bits = 0x158
                    0x015a                  IC4CON2 = 0x15a
                    0x015a                  _IC4CON2 = 0x15a
                    0x015a                  _IC4CON2bits = 0x15a
                    0x015c                  IC4BUF = 0x15c
                    0x015c                  _IC4BUF = 0x15c
                    0x015e                  IC4TMR = 0x15e
                    0x015e                  _IC4TMR = 0x15e
                    0x0160                  IC5CON1 = 0x160
                    0x0160                  _IC5CON1 = 0x160
                    0x0160                  _IC5CON1bits = 0x160
                    0x0162                  IC5CON2 = 0x162
                    0x0162                  _IC5CON2 = 0x162
                    0x0162                  _IC5CON2bits = 0x162
                    0x0164                  IC5BUF = 0x164
                    0x0164                  _IC5BUF = 0x164
                    0x0166                  IC5TMR = 0x166
                    0x0166                  _IC5TMR = 0x166
                    0x0168                  IC6CON1 = 0x168
                    0x0168                  _IC6CON1 = 0x168
                    0x0168                  _IC6CON1bits = 0x168
                    0x016a                  IC6CON2 = 0x16a
                    0x016a                  _IC6CON2 = 0x16a
                    0x016a                  _IC6CON2bits = 0x16a
                    0x016c                  IC6BUF = 0x16c
                    0x016c                  _IC6BUF = 0x16c
                    0x016e                  IC6TMR = 0x16e
                    0x016e                  _IC6TMR = 0x16e
                    0x0170                  IC7CON1 = 0x170
                    0x0170                  _IC7CON1 = 0x170
                    0x0170                  _IC7CON1bits = 0x170
                    0x0172                  IC7CON2 = 0x172
                    0x0172                  _IC7CON2 = 0x172
                    0x0172                  _IC7CON2bits = 0x172
                    0x0174                  IC7BUF = 0x174
                    0x0174                  _IC7BUF = 0x174
                    0x0176                  IC7TMR = 0x176
                    0x0176                  _IC7TMR = 0x176
                    0x0178                  IC8CON1 = 0x178
                    0x0178                  _IC8CON1 = 0x178
                    0x0178                  _IC8CON1bits = 0x178
                    0x017a                  IC8CON2 = 0x17a
                    0x017a                  _IC8CON2 = 0x17a
                    0x017a                  _IC8CON2bits = 0x17a
                    0x017c                  IC8BUF = 0x17c
                    0x017c                  _IC8BUF = 0x17c
                    0x017e                  IC8TMR = 0x17e
                    0x017e                  _IC8TMR = 0x17e
                    0x0180                  IC9CON1 = 0x180
                    0x0180                  _IC9CON1 = 0x180
                    0x0180                  _IC9CON1bits = 0x180
                    0x0182                  IC9CON2 = 0x182
                    0x0182                  _IC9CON2 = 0x182
                    0x0182                  _IC9CON2bits = 0x182
                    0x0184                  IC9BUF = 0x184
                    0x0184                  _IC9BUF = 0x184
                    0x0186                  IC9TMR = 0x186
                    0x0186                  _IC9TMR = 0x186
                    0x0188                  IC10CON1 = 0x188
                    0x0188                  _IC10CON1 = 0x188
                    0x0188                  _IC10CON1bits = 0x188
                    0x018a                  IC10CON2 = 0x18a
                    0x018a                  _IC10CON2 = 0x18a
                    0x018a                  _IC10CON2bits = 0x18a
                    0x018c                  IC10BUF = 0x18c
                    0x018c                  _IC10BUF = 0x18c
                    0x018e                  IC10TMR = 0x18e
                    0x018e                  _IC10TMR = 0x18e
                    0x0190                  IC11CON1 = 0x190
                    0x0190                  _IC11CON1 = 0x190
                    0x0190                  _IC11CON1bits = 0x190
                    0x0192                  IC11CON2 = 0x192
                    0x0192                  _IC11CON2 = 0x192
                    0x0192                  _IC11CON2bits = 0x192
                    0x0194                  IC11BUF = 0x194
                    0x0194                  _IC11BUF = 0x194
                    0x0196                  IC11TMR = 0x196
                    0x0196                  _IC11TMR = 0x196
                    0x0198                  IC12CON1 = 0x198
                    0x0198                  _IC12CON1 = 0x198
                    0x0198                  _IC12CON1bits = 0x198
                    0x019a                  IC12CON2 = 0x19a
                    0x019a                  _IC12CON2 = 0x19a
                    0x019a                  _IC12CON2bits = 0x19a
                    0x019c                  IC12BUF = 0x19c
                    0x019c                  _IC12BUF = 0x19c
                    0x019e                  IC12TMR = 0x19e
                    0x019e                  _IC12TMR = 0x19e
                    0x01a0                  IC13CON1 = 0x1a0
                    0x01a0                  _IC13CON1 = 0x1a0
                    0x01a0                  _IC13CON1bits = 0x1a0
                    0x01a2                  IC13CON2 = 0x1a2
                    0x01a2                  _IC13CON2 = 0x1a2
                    0x01a2                  _IC13CON2bits = 0x1a2
                    0x01a4                  IC13BUF = 0x1a4
                    0x01a4                  _IC13BUF = 0x1a4
                    0x01a6                  IC13TMR = 0x1a6
                    0x01a6                  _IC13TMR = 0x1a6
                    0x01a8                  IC14CON1 = 0x1a8
                    0x01a8                  _IC14CON1 = 0x1a8
                    0x01a8                  _IC14CON1bits = 0x1a8
                    0x01aa                  IC14CON2 = 0x1aa
                    0x01aa                  _IC14CON2 = 0x1aa
                    0x01aa                  _IC14CON2bits = 0x1aa
                    0x01ac                  IC14BUF = 0x1ac
                    0x01ac                  _IC14BUF = 0x1ac
                    0x01ae                  IC14TMR = 0x1ae
                    0x01ae                  _IC14TMR = 0x1ae
                    0x01b0                  IC15CON1 = 0x1b0
                    0x01b0                  _IC15CON1 = 0x1b0
                    0x01b0                  _IC15CON1bits = 0x1b0
                    0x01b2                  IC15CON2 = 0x1b2
                    0x01b2                  _IC15CON2 = 0x1b2
                    0x01b2                  _IC15CON2bits = 0x1b2
                    0x01b4                  IC15BUF = 0x1b4
                    0x01b4                  _IC15BUF = 0x1b4
                    0x01b6                  IC15TMR = 0x1b6
                    0x01b6                  _IC15TMR = 0x1b6
                    0x01b8                  IC16CON1 = 0x1b8
                    0x01b8                  _IC16CON1 = 0x1b8
                    0x01b8                  _IC16CON1bits = 0x1b8
                    0x01ba                  IC16CON2 = 0x1ba
                    0x01ba                  _IC16CON2 = 0x1ba
                    0x01ba                  _IC16CON2bits = 0x1ba
                    0x01bc                  IC16BUF = 0x1bc
                    0x01bc                  _IC16BUF = 0x1bc
                    0x01be                  IC16TMR = 0x1be
                    0x01be                  _IC16TMR = 0x1be
                    0x01c0                  QEI1CON = 0x1c0
                    0x01c0                  _QEI1CON = 0x1c0
                    0x01c0                  _QEI1CONbits = 0x1c0
                    0x01c2                  QEI1IOC = 0x1c2
                    0x01c2                  _QEI1IOC = 0x1c2
                    0x01c2                  _QEI1IOCbits = 0x1c2
                    0x01c4                  QEI1STAT = 0x1c4
                    0x01c4                  _QEI1STAT = 0x1c4
                    0x01c4                  _QEI1STATbits = 0x1c4
                    0x01c6                  POS1CNTL = 0x1c6
                    0x01c6                  _POS1CNTL = 0x1c6
                    0x01c8                  POS1CNTH = 0x1c8
                    0x01c8                  _POS1CNTH = 0x1c8
                    0x01ca                  POS1HLD = 0x1ca
                    0x01ca                  _POS1HLD = 0x1ca
                    0x01cc                  VEL1CNT = 0x1cc
                    0x01cc                  _VEL1CNT = 0x1cc
                    0x01ce                  INT1TMRL = 0x1ce
                    0x01ce                  _INT1TMRL = 0x1ce
                    0x01d0                  INT1TMRH = 0x1d0
                    0x01d0                  _INT1TMRH = 0x1d0
                    0x01d2                  INT1HLDL = 0x1d2
                    0x01d2                  _INT1HLDL = 0x1d2
                    0x01d4                  INT1HLDH = 0x1d4
                    0x01d4                  _INT1HLDH = 0x1d4
                    0x01d6                  INDX1CNTL = 0x1d6
                    0x01d6                  _INDX1CNTL = 0x1d6
                    0x01d8                  INDX1CNTH = 0x1d8
                    0x01d8                  _INDX1CNTH = 0x1d8
                    0x01da                  INDX1HLD = 0x1da
                    0x01da                  _INDX1HLD = 0x1da
                    0x01dc                  QEI1GECL = 0x1dc
                    0x01dc                  _QEI1GECL = 0x1dc
                    0x01dc                  QEI1ICL = 0x1dc
                    0x01dc                  _QEI1ICL = 0x1dc
                    0x01de                  QEI1GECH = 0x1de
                    0x01de                  _QEI1GECH = 0x1de
                    0x01de                  QEI1ICH = 0x1de
                    0x01de                  _QEI1ICH = 0x1de
                    0x01e0                  QEI1LECL = 0x1e0
                    0x01e0                  _QEI1LECL = 0x1e0
                    0x01e2                  QEI1LECH = 0x1e2
                    0x01e2                  _QEI1LECH = 0x1e2
                    0x0200                  I2C1RCV = 0x200
                    0x0200                  _I2C1RCV = 0x200
                    0x0202                  I2C1TRN = 0x202
                    0x0202                  _I2C1TRN = 0x202
                    0x0204                  I2C1BRG = 0x204
                    0x0204                  _I2C1BRG = 0x204
                    0x0206                  I2C1CON = 0x206
                    0x0206                  _I2C1CON = 0x206
                    0x0206                  _I2C1CONbits = 0x206
                    0x0208                  I2C1STAT = 0x208
                    0x0208                  _I2C1STAT = 0x208
                    0x0208                  _I2C1STATbits = 0x208
                    0x020a                  I2C1ADD = 0x20a
                    0x020a                  _I2C1ADD = 0x20a
                    0x020c                  I2C1MSK = 0x20c
                    0x020c                  _I2C1MSK = 0x20c
                    0x0210                  I2C2RCV = 0x210
                    0x0210                  _I2C2RCV = 0x210
                    0x0212                  I2C2TRN = 0x212
                    0x0212                  _I2C2TRN = 0x212
                    0x0214                  I2C2BRG = 0x214
                    0x0214                  _I2C2BRG = 0x214
                    0x0216                  I2C2CON = 0x216
                    0x0216                  _I2C2CON = 0x216
                    0x0216                  _I2C2CONbits = 0x216
                    0x0218                  I2C2STAT = 0x218
                    0x0218                  _I2C2STAT = 0x218
                    0x0218                  _I2C2STATbits = 0x218
                    0x021a                  I2C2ADD = 0x21a
                    0x021a                  _I2C2ADD = 0x21a
                    0x021c                  I2C2MSK = 0x21c
                    0x021c                  _I2C2MSK = 0x21c
                    0x0220                  U1MODE = 0x220
                    0x0220                  _U1MODE = 0x220
                    0x0220                  _U1MODEbits = 0x220
                    0x0222                  U1STA = 0x222
                    0x0222                  _U1STA = 0x222
                    0x0222                  _U1STAbits = 0x222
                    0x0224                  U1TXREG = 0x224
                    0x0224                  _U1TXREG = 0x224
                    0x0226                  U1RXREG = 0x226
                    0x0226                  _U1RXREG = 0x226
                    0x0228                  U1BRG = 0x228
                    0x0228                  _U1BRG = 0x228
                    0x0230                  U2MODE = 0x230
                    0x0230                  _U2MODE = 0x230
                    0x0230                  _U2MODEbits = 0x230
                    0x0232                  U2STA = 0x232
                    0x0232                  _U2STA = 0x232
                    0x0232                  _U2STAbits = 0x232
                    0x0234                  U2TXREG = 0x234
                    0x0234                  _U2TXREG = 0x234
                    0x0236                  U2RXREG = 0x236
                    0x0236                  _U2RXREG = 0x236
                    0x0238                  U2BRG = 0x238
                    0x0238                  _U2BRG = 0x238
                    0x0240                  SPI1STAT = 0x240
                    0x0240                  _SPI1STAT = 0x240
                    0x0240                  _SPI1STATbits = 0x240
                    0x0242                  SPI1CON1 = 0x242
                    0x0242                  _SPI1CON1 = 0x242
                    0x0242                  _SPI1CON1bits = 0x242
                    0x0244                  SPI1CON2 = 0x244
                    0x0244                  _SPI1CON2 = 0x244
                    0x0244                  _SPI1CON2bits = 0x244
                    0x0248                  SPI1BUF = 0x248
                    0x0248                  _SPI1BUF = 0x248
                    0x0250                  U3MODE = 0x250
                    0x0250                  _U3MODE = 0x250
                    0x0250                  _U3MODEbits = 0x250
                    0x0252                  U3STA = 0x252
                    0x0252                  _U3STA = 0x252
                    0x0252                  _U3STAbits = 0x252
                    0x0254                  U3TXREG = 0x254
                    0x0254                  _U3TXREG = 0x254
                    0x0256                  U3RXREG = 0x256
                    0x0256                  _U3RXREG = 0x256
                    0x0258                  U3BRG = 0x258
                    0x0258                  _U3BRG = 0x258
                    0x0260                  SPI2STAT = 0x260
                    0x0260                  _SPI2STAT = 0x260
                    0x0260                  _SPI2STATbits = 0x260
                    0x0262                  SPI2CON1 = 0x262
                    0x0262                  _SPI2CON1 = 0x262
                    0x0262                  _SPI2CON1bits = 0x262
                    0x0264                  SPI2CON2 = 0x264
                    0x0264                  _SPI2CON2 = 0x264
                    0x0264                  _SPI2CON2bits = 0x264
                    0x0268                  SPI2BUF = 0x268
                    0x0268                  _SPI2BUF = 0x268
                    0x0280                  DCICON1 = 0x280
                    0x0280                  _DCICON1 = 0x280
                    0x0280                  _DCICON1bits = 0x280
                    0x0282                  DCICON2 = 0x282
                    0x0282                  _DCICON2 = 0x282
                    0x0282                  _DCICON2bits = 0x282
                    0x0284                  DCICON3 = 0x284
                    0x0284                  _DCICON3 = 0x284
                    0x0284                  _DCICON3bits = 0x284
                    0x0286                  DCISTAT = 0x286
                    0x0286                  _DCISTAT = 0x286
                    0x0286                  _DCISTATbits = 0x286
                    0x0288                  TSCON = 0x288
                    0x0288                  _TSCON = 0x288
                    0x0288                  _TSCONbits = 0x288
                    0x028c                  RSCON = 0x28c
                    0x028c                  _RSCON = 0x28c
                    0x028c                  _RSCONbits = 0x28c
                    0x0290                  RXBUF0 = 0x290
                    0x0290                  _RXBUF0 = 0x290
                    0x0292                  RXBUF1 = 0x292
                    0x0292                  _RXBUF1 = 0x292
                    0x0294                  RXBUF2 = 0x294
                    0x0294                  _RXBUF2 = 0x294
                    0x0296                  RXBUF3 = 0x296
                    0x0296                  _RXBUF3 = 0x296
                    0x0298                  TXBUF0 = 0x298
                    0x0298                  _TXBUF0 = 0x298
                    0x029a                  TXBUF1 = 0x29a
                    0x029a                  _TXBUF1 = 0x29a
                    0x029c                  TXBUF2 = 0x29c
                    0x029c                  _TXBUF2 = 0x29c
                    0x029e                  TXBUF3 = 0x29e
                    0x029e                  _TXBUF3 = 0x29e
                    0x02a0                  SPI3STAT = 0x2a0
                    0x02a0                  _SPI3STAT = 0x2a0
                    0x02a0                  _SPI3STATbits = 0x2a0
                    0x02a2                  SPI3CON1 = 0x2a2
                    0x02a2                  _SPI3CON1 = 0x2a2
                    0x02a2                  _SPI3CON1bits = 0x2a2
                    0x02a4                  SPI3CON2 = 0x2a4
                    0x02a4                  _SPI3CON2 = 0x2a4
                    0x02a4                  _SPI3CON2bits = 0x2a4
                    0x02a8                  SPI3BUF = 0x2a8
                    0x02a8                  _SPI3BUF = 0x2a8
                    0x02b0                  U4MODE = 0x2b0
                    0x02b0                  _U4MODE = 0x2b0
                    0x02b0                  _U4MODEbits = 0x2b0
                    0x02b2                  U4STA = 0x2b2
                    0x02b2                  _U4STA = 0x2b2
                    0x02b2                  _U4STAbits = 0x2b2
                    0x02b4                  U4TXREG = 0x2b4
                    0x02b4                  _U4TXREG = 0x2b4
                    0x02b6                  U4RXREG = 0x2b6
                    0x02b6                  _U4RXREG = 0x2b6
                    0x02b8                  U4BRG = 0x2b8
                    0x02b8                  _U4BRG = 0x2b8
                    0x02c0                  SPI4STAT = 0x2c0
                    0x02c0                  _SPI4STAT = 0x2c0
                    0x02c0                  _SPI4STATbits = 0x2c0
                    0x02c2                  SPI4CON1 = 0x2c2
                    0x02c2                  _SPI4CON1 = 0x2c2
                    0x02c2                  _SPI4CON1bits = 0x2c2
                    0x02c4                  SPI4CON2 = 0x2c4
                    0x02c4                  _SPI4CON2 = 0x2c4
                    0x02c4                  _SPI4CON2bits = 0x2c4
                    0x02c8                  SPI4BUF = 0x2c8
                    0x02c8                  _SPI4BUF = 0x2c8
                    0x0300                  ADC1BUF0 = 0x300
                    0x0300                  _ADC1BUF0 = 0x300
                    0x0302                  ADC1BUF1 = 0x302
                    0x0302                  _ADC1BUF1 = 0x302
                    0x0304                  ADC1BUF2 = 0x304
                    0x0304                  _ADC1BUF2 = 0x304
                    0x0306                  ADC1BUF3 = 0x306
                    0x0306                  _ADC1BUF3 = 0x306
                    0x0308                  ADC1BUF4 = 0x308
                    0x0308                  _ADC1BUF4 = 0x308
                    0x030a                  ADC1BUF5 = 0x30a
                    0x030a                  _ADC1BUF5 = 0x30a
                    0x030c                  ADC1BUF6 = 0x30c
                    0x030c                  _ADC1BUF6 = 0x30c
                    0x030e                  ADC1BUF7 = 0x30e
                    0x030e                  _ADC1BUF7 = 0x30e
                    0x0310                  ADC1BUF8 = 0x310
                    0x0310                  _ADC1BUF8 = 0x310
                    0x0312                  ADC1BUF9 = 0x312
                    0x0312                  _ADC1BUF9 = 0x312
                    0x0314                  ADC1BUFA = 0x314
                    0x0314                  _ADC1BUFA = 0x314
                    0x0316                  ADC1BUFB = 0x316
                    0x0316                  _ADC1BUFB = 0x316
                    0x0318                  ADC1BUFC = 0x318
                    0x0318                  _ADC1BUFC = 0x318
                    0x031a                  ADC1BUFD = 0x31a
                    0x031a                  _ADC1BUFD = 0x31a
                    0x031c                  ADC1BUFE = 0x31c
                    0x031c                  _ADC1BUFE = 0x31c
                    0x031e                  ADC1BUFF = 0x31e
                    0x031e                  _ADC1BUFF = 0x31e
                    0x0320                  AD1CON1 = 0x320
                    0x0320                  _AD1CON1 = 0x320
                    0x0320                  _AD1CON1bits = 0x320
                    0x0322                  AD1CON2 = 0x322
                    0x0322                  _AD1CON2 = 0x322
                    0x0322                  _AD1CON2bits = 0x322
                    0x0324                  AD1CON3 = 0x324
                    0x0324                  _AD1CON3 = 0x324
                    0x0324                  _AD1CON3bits = 0x324
                    0x0326                  AD1CHS123 = 0x326
                    0x0326                  _AD1CHS123 = 0x326
                    0x0326                  _AD1CHS123bits = 0x326
                    0x0328                  AD1CHS0 = 0x328
                    0x0328                  _AD1CHS0 = 0x328
                    0x0328                  _AD1CHS0bits = 0x328
                    0x032e                  AD1CSSH = 0x32e
                    0x032e                  _AD1CSSH = 0x32e
                    0x032e                  _AD1CSSHbits = 0x32e
                    0x0330                  AD1CSSL = 0x330
                    0x0330                  _AD1CSSL = 0x330
                    0x0330                  _AD1CSSLbits = 0x330
                    0x0332                  AD1CON4 = 0x332
                    0x0332                  _AD1CON4 = 0x332
                    0x0332                  _AD1CON4bits = 0x332
                    0x0340                  ADC2BUF0 = 0x340
                    0x0340                  _ADC2BUF0 = 0x340
                    0x0342                  ADC2BUF1 = 0x342
                    0x0342                  _ADC2BUF1 = 0x342
                    0x0344                  ADC2BUF2 = 0x344
                    0x0344                  _ADC2BUF2 = 0x344
                    0x0346                  ADC2BUF3 = 0x346
                    0x0346                  _ADC2BUF3 = 0x346
                    0x0348                  ADC2BUF4 = 0x348
                    0x0348                  _ADC2BUF4 = 0x348
                    0x034a                  ADC2BUF5 = 0x34a
                    0x034a                  _ADC2BUF5 = 0x34a
                    0x034c                  ADC2BUF6 = 0x34c
                    0x034c                  _ADC2BUF6 = 0x34c
                    0x034e                  ADC2BUF7 = 0x34e
                    0x034e                  _ADC2BUF7 = 0x34e
                    0x0350                  ADC2BUF8 = 0x350
                    0x0350                  _ADC2BUF8 = 0x350
                    0x0352                  ADC2BUF9 = 0x352
                    0x0352                  _ADC2BUF9 = 0x352
                    0x0354                  ADC2BUFA = 0x354
                    0x0354                  _ADC2BUFA = 0x354
                    0x0356                  ADC2BUFB = 0x356
                    0x0356                  _ADC2BUFB = 0x356
                    0x0358                  ADC2BUFC = 0x358
                    0x0358                  _ADC2BUFC = 0x358
                    0x035a                  ADC2BUFD = 0x35a
                    0x035a                  _ADC2BUFD = 0x35a
                    0x035c                  ADC2BUFE = 0x35c
                    0x035c                  _ADC2BUFE = 0x35c
                    0x035e                  ADC2BUFF = 0x35e
                    0x035e                  _ADC2BUFF = 0x35e
                    0x0360                  AD2CON1 = 0x360
                    0x0360                  _AD2CON1 = 0x360
                    0x0360                  _AD2CON1bits = 0x360
                    0x0362                  AD2CON2 = 0x362
                    0x0362                  _AD2CON2 = 0x362
                    0x0362                  _AD2CON2bits = 0x362
                    0x0364                  AD2CON3 = 0x364
                    0x0364                  _AD2CON3 = 0x364
                    0x0364                  _AD2CON3bits = 0x364
                    0x0366                  AD2CHS123 = 0x366
                    0x0366                  _AD2CHS123 = 0x366
                    0x0366                  _AD2CHS123bits = 0x366
                    0x0368                  AD2CHS0 = 0x368
                    0x0368                  _AD2CHS0 = 0x368
                    0x0368                  _AD2CHS0bits = 0x368
                    0x0370                  AD2CSSL = 0x370
                    0x0370                  _AD2CSSL = 0x370
                    0x0370                  _AD2CSSLbits = 0x370
                    0x0372                  AD2CON4 = 0x372
                    0x0372                  _AD2CON4 = 0x372
                    0x0372                  _AD2CON4bits = 0x372
                    0x0400                  C1CTRL1 = 0x400
                    0x0400                  _C1CTRL1 = 0x400
                    0x0400                  _C1CTRL1bits = 0x400
                    0x0402                  C1CTRL2 = 0x402
                    0x0402                  _C1CTRL2 = 0x402
                    0x0402                  _C1CTRL2bits = 0x402
                    0x0404                  C1VEC = 0x404
                    0x0404                  _C1VEC = 0x404
                    0x0404                  _C1VECbits = 0x404
                    0x0406                  C1FCTRL = 0x406
                    0x0406                  _C1FCTRL = 0x406
                    0x0406                  _C1FCTRLbits = 0x406
                    0x0408                  C1FIFO = 0x408
                    0x0408                  _C1FIFO = 0x408
                    0x0408                  _C1FIFObits = 0x408
                    0x040a                  C1INTF = 0x40a
                    0x040a                  _C1INTF = 0x40a
                    0x040a                  _C1INTFbits = 0x40a
                    0x040c                  C1INTE = 0x40c
                    0x040c                  _C1INTE = 0x40c
                    0x040c                  _C1INTEbits = 0x40c
                    0x040e                  C1EC = 0x40e
                    0x040e                  _C1EC = 0x40e
                    0x040e                  _C1ECbits = 0x40e
                    0x040e                  C1RERRCNT = 0x40e
                    0x040e                  _C1RERRCNT = 0x40e
                    0x040f                  C1TERRCNT = 0x40f
                    0x040f                  _C1TERRCNT = 0x40f
                    0x0410                  C1CFG1 = 0x410
                    0x0410                  _C1CFG1 = 0x410
                    0x0410                  _C1CFG1bits = 0x410
                    0x0412                  C1CFG2 = 0x412
                    0x0412                  _C1CFG2 = 0x412
                    0x0412                  _C1CFG2bits = 0x412
                    0x0414                  C1FEN1 = 0x414
                    0x0414                  _C1FEN1 = 0x414
                    0x0414                  _C1FEN1bits = 0x414
                    0x0418                  C1FMSKSEL1 = 0x418
                    0x0418                  _C1FMSKSEL1 = 0x418
                    0x0418                  _C1FMSKSEL1bits = 0x418
                    0x041a                  C1FMSKSEL2 = 0x41a
                    0x041a                  _C1FMSKSEL2 = 0x41a
                    0x041a                  _C1FMSKSEL2bits = 0x41a
                    0x0420                  C1BUFPNT1 = 0x420
                    0x0420                  _C1BUFPNT1 = 0x420
                    0x0420                  _C1BUFPNT1bits = 0x420
                    0x0420                  C1RXFUL1 = 0x420
                    0x0420                  _C1RXFUL1 = 0x420
                    0x0420                  _C1RXFUL1bits = 0x420
                    0x0422                  C1BUFPNT2 = 0x422
                    0x0422                  _C1BUFPNT2 = 0x422
                    0x0422                  _C1BUFPNT2bits = 0x422
                    0x0422                  C1RXFUL2 = 0x422
                    0x0422                  _C1RXFUL2 = 0x422
                    0x0422                  _C1RXFUL2bits = 0x422
                    0x0424                  C1BUFPNT3 = 0x424
                    0x0424                  _C1BUFPNT3 = 0x424
                    0x0424                  _C1BUFPNT3bits = 0x424
                    0x0426                  C1BUFPNT4 = 0x426
                    0x0426                  _C1BUFPNT4 = 0x426
                    0x0426                  _C1BUFPNT4bits = 0x426
                    0x0428                  C1RXOVF1 = 0x428
                    0x0428                  _C1RXOVF1 = 0x428
                    0x0428                  _C1RXOVF1bits = 0x428
                    0x042a                  C1RXOVF2 = 0x42a
                    0x042a                  _C1RXOVF2 = 0x42a
                    0x042a                  _C1RXOVF2bits = 0x42a
                    0x0430                  C1RXM0SID = 0x430
                    0x0430                  _C1RXM0SID = 0x430
                    0x0430                  _C1RXM0SIDbits = 0x430
                    0x0430                  C1TR01CON = 0x430
                    0x0430                  _C1TR01CON = 0x430
                    0x0430                  _C1TR01CONbits = 0x430
                    0x0432                  C1RXM0EID = 0x432
                    0x0432                  _C1RXM0EID = 0x432
                    0x0432                  _C1RXM0EIDbits = 0x432
                    0x0432                  C1TR23CON = 0x432
                    0x0432                  _C1TR23CON = 0x432
                    0x0432                  _C1TR23CONbits = 0x432
                    0x0434                  C1RXM1SID = 0x434
                    0x0434                  _C1RXM1SID = 0x434
                    0x0434                  _C1RXM1SIDbits = 0x434
                    0x0434                  C1TR45CON = 0x434
                    0x0434                  _C1TR45CON = 0x434
                    0x0434                  _C1TR45CONbits = 0x434
                    0x0436                  C1RXM1EID = 0x436
                    0x0436                  _C1RXM1EID = 0x436
                    0x0436                  _C1RXM1EIDbits = 0x436
                    0x0436                  C1TR67CON = 0x436
                    0x0436                  _C1TR67CON = 0x436
                    0x0436                  _C1TR67CONbits = 0x436
                    0x0438                  C1RXM2SID = 0x438
                    0x0438                  _C1RXM2SID = 0x438
                    0x0438                  _C1RXM2SIDbits = 0x438
                    0x043a                  C1RXM2EID = 0x43a
                    0x043a                  _C1RXM2EID = 0x43a
                    0x043a                  _C1RXM2EIDbits = 0x43a
                    0x0440                  C1RXD = 0x440
                    0x0440                  _C1RXD = 0x440
                    0x0440                  C1RXF0SID = 0x440
                    0x0440                  _C1RXF0SID = 0x440
                    0x0440                  _C1RXF0SIDbits = 0x440
                    0x0442                  C1RXF0EID = 0x442
                    0x0442                  _C1RXF0EID = 0x442
                    0x0442                  _C1RXF0EIDbits = 0x442
                    0x0442                  C1TXD = 0x442
                    0x0442                  _C1TXD = 0x442
                    0x0442                  _C1TXDbits = 0x442
                    0x0444                  C1RXF1SID = 0x444
                    0x0444                  _C1RXF1SID = 0x444
                    0x0444                  _C1RXF1SIDbits = 0x444
                    0x0446                  C1RXF1EID = 0x446
                    0x0446                  _C1RXF1EID = 0x446
                    0x0446                  _C1RXF1EIDbits = 0x446
                    0x0448                  C1RXF2SID = 0x448
                    0x0448                  _C1RXF2SID = 0x448
                    0x0448                  _C1RXF2SIDbits = 0x448
                    0x044a                  C1RXF2EID = 0x44a
                    0x044a                  _C1RXF2EID = 0x44a
                    0x044a                  _C1RXF2EIDbits = 0x44a
                    0x044c                  C1RXF3SID = 0x44c
                    0x044c                  _C1RXF3SID = 0x44c
                    0x044c                  _C1RXF3SIDbits = 0x44c
                    0x044e                  C1RXF3EID = 0x44e
                    0x044e                  _C1RXF3EID = 0x44e
                    0x044e                  _C1RXF3EIDbits = 0x44e
                    0x0450                  C1RXF4SID = 0x450
                    0x0450                  _C1RXF4SID = 0x450
                    0x0450                  _C1RXF4SIDbits = 0x450
                    0x0452                  C1RXF4EID = 0x452
                    0x0452                  _C1RXF4EID = 0x452
                    0x0452                  _C1RXF4EIDbits = 0x452
                    0x0454                  C1RXF5SID = 0x454
                    0x0454                  _C1RXF5SID = 0x454
                    0x0454                  _C1RXF5SIDbits = 0x454
                    0x0456                  C1RXF5EID = 0x456
                    0x0456                  _C1RXF5EID = 0x456
                    0x0456                  _C1RXF5EIDbits = 0x456
                    0x0458                  C1RXF6SID = 0x458
                    0x0458                  _C1RXF6SID = 0x458
                    0x0458                  _C1RXF6SIDbits = 0x458
                    0x045a                  C1RXF6EID = 0x45a
                    0x045a                  _C1RXF6EID = 0x45a
                    0x045a                  _C1RXF6EIDbits = 0x45a
                    0x045c                  C1RXF7SID = 0x45c
                    0x045c                  _C1RXF7SID = 0x45c
                    0x045c                  _C1RXF7SIDbits = 0x45c
                    0x045e                  C1RXF7EID = 0x45e
                    0x045e                  _C1RXF7EID = 0x45e
                    0x045e                  _C1RXF7EIDbits = 0x45e
                    0x0460                  C1RXF8SID = 0x460
                    0x0460                  _C1RXF8SID = 0x460
                    0x0460                  _C1RXF8SIDbits = 0x460
                    0x0462                  C1RXF8EID = 0x462
                    0x0462                  _C1RXF8EID = 0x462
                    0x0462                  _C1RXF8EIDbits = 0x462
                    0x0464                  C1RXF9SID = 0x464
                    0x0464                  _C1RXF9SID = 0x464
                    0x0464                  _C1RXF9SIDbits = 0x464
                    0x0466                  C1RXF9EID = 0x466
                    0x0466                  _C1RXF9EID = 0x466
                    0x0466                  _C1RXF9EIDbits = 0x466
                    0x0468                  C1RXF10SID = 0x468
                    0x0468                  _C1RXF10SID = 0x468
                    0x0468                  _C1RXF10SIDbits = 0x468
                    0x046a                  C1RXF10EID = 0x46a
                    0x046a                  _C1RXF10EID = 0x46a
                    0x046a                  _C1RXF10EIDbits = 0x46a
                    0x046c                  C1RXF11SID = 0x46c
                    0x046c                  _C1RXF11SID = 0x46c
                    0x046c                  _C1RXF11SIDbits = 0x46c
                    0x046e                  C1RXF11EID = 0x46e
                    0x046e                  _C1RXF11EID = 0x46e
                    0x046e                  _C1RXF11EIDbits = 0x46e
                    0x0470                  C1RXF12SID = 0x470
                    0x0470                  _C1RXF12SID = 0x470
                    0x0470                  _C1RXF12SIDbits = 0x470
                    0x0472                  C1RXF12EID = 0x472
                    0x0472                  _C1RXF12EID = 0x472
                    0x0472                  _C1RXF12EIDbits = 0x472
                    0x0474                  C1RXF13SID = 0x474
                    0x0474                  _C1RXF13SID = 0x474
                    0x0474                  _C1RXF13SIDbits = 0x474
                    0x0476                  C1RXF13EID = 0x476
                    0x0476                  _C1RXF13EID = 0x476
                    0x0476                  _C1RXF13EIDbits = 0x476
                    0x0478                  C1RXF14SID = 0x478
                    0x0478                  _C1RXF14SID = 0x478
                    0x0478                  _C1RXF14SIDbits = 0x478
                    0x047a                  C1RXF14EID = 0x47a
                    0x047a                  _C1RXF14EID = 0x47a
                    0x047a                  _C1RXF14EIDbits = 0x47a
                    0x047c                  C1RXF15SID = 0x47c
                    0x047c                  _C1RXF15SID = 0x47c
                    0x047c                  _C1RXF15SIDbits = 0x47c
                    0x047e                  C1RXF15EID = 0x47e
                    0x047e                  _C1RXF15EID = 0x47e
                    0x047e                  _C1RXF15EIDbits = 0x47e
                    0x0488                  U1OTGIR = 0x488
                    0x0488                  _U1OTGIR = 0x488
                    0x0488                  _U1OTGIRbits = 0x488
                    0x048a                  U1OTGIE = 0x48a
                    0x048a                  _U1OTGIE = 0x48a
                    0x048a                  _U1OTGIEbits = 0x48a
                    0x048c                  U1OTGSTAT = 0x48c
                    0x048c                  _U1OTGSTAT = 0x48c
                    0x048c                  _U1OTGSTATbits = 0x48c
                    0x048e                  U1OTGCON = 0x48e
                    0x048e                  _U1OTGCON = 0x48e
                    0x048e                  _U1OTGCONbits = 0x48e
                    0x0490                  U1PWRC = 0x490
                    0x0490                  _U1PWRC = 0x490
                    0x0490                  _U1PWRCbits = 0x490
                    0x04c0                  U1IR = 0x4c0
                    0x04c0                  _U1IR = 0x4c0
                    0x04c0                  _U1IRbits = 0x4c0
                    0x04c2                  U1IE = 0x4c2
                    0x04c2                  _U1IE = 0x4c2
                    0x04c2                  _U1IEbits = 0x4c2
                    0x04c4                  U1EIR = 0x4c4
                    0x04c4                  _U1EIR = 0x4c4
                    0x04c4                  _U1EIRbits = 0x4c4
                    0x04c6                  U1EIE = 0x4c6
                    0x04c6                  _U1EIE = 0x4c6
                    0x04c6                  _U1EIEbits = 0x4c6
                    0x04c8                  U1STAT = 0x4c8
                    0x04c8                  _U1STAT = 0x4c8
                    0x04c8                  _U1STATbits = 0x4c8
                    0x04ca                  U1CON = 0x4ca
                    0x04ca                  _U1CON = 0x4ca
                    0x04ca                  _U1CONbits = 0x4ca
                    0x04cc                  U1ADDR = 0x4cc
                    0x04cc                  _U1ADDR = 0x4cc
                    0x04cc                  _U1ADDRbits = 0x4cc
                    0x04ce                  U1BDTP1 = 0x4ce
                    0x04ce                  _U1BDTP1 = 0x4ce
                    0x04ce                  _U1BDTP1bits = 0x4ce
                    0x04d0                  U1FRML = 0x4d0
                    0x04d0                  _U1FRML = 0x4d0
                    0x04d0                  _U1FRMLbits = 0x4d0
                    0x04d2                  U1FRMH = 0x4d2
                    0x04d2                  _U1FRMH = 0x4d2
                    0x04d2                  _U1FRMHbits = 0x4d2
                    0x04d4                  U1TOK = 0x4d4
                    0x04d4                  _U1TOK = 0x4d4
                    0x04d4                  _U1TOKbits = 0x4d4
                    0x04d6                  U1SOF = 0x4d6
                    0x04d6                  _U1SOF = 0x4d6
                    0x04d6                  _U1SOFbits = 0x4d6
                    0x04d8                  U1BDTP2 = 0x4d8
                    0x04d8                  _U1BDTP2 = 0x4d8
                    0x04d8                  _U1BDTP2bits = 0x4d8
                    0x04da                  U1BDTP3 = 0x4da
                    0x04da                  _U1BDTP3 = 0x4da
                    0x04da                  _U1BDTP3bits = 0x4da
                    0x04dc                  U1CNFG1 = 0x4dc
                    0x04dc                  _U1CNFG1 = 0x4dc
                    0x04dc                  _U1CNFG1bits = 0x4dc
                    0x04de                  U1CNFG2 = 0x4de
                    0x04de                  _U1CNFG2 = 0x4de
                    0x04de                  _U1CNFG2bits = 0x4de
                    0x04e0                  U1EP0 = 0x4e0
                    0x04e0                  _U1EP0 = 0x4e0
                    0x04e0                  _U1EP0bits = 0x4e0
                    0x04e2                  U1EP1 = 0x4e2
                    0x04e2                  _U1EP1 = 0x4e2
                    0x04e2                  _U1EP1bits = 0x4e2
                    0x04e4                  U1EP2 = 0x4e4
                    0x04e4                  _U1EP2 = 0x4e4
                    0x04e4                  _U1EP2bits = 0x4e4
                    0x04e6                  U1EP3 = 0x4e6
                    0x04e6                  _U1EP3 = 0x4e6
                    0x04e6                  _U1EP3bits = 0x4e6
                    0x04e8                  U1EP4 = 0x4e8
                    0x04e8                  _U1EP4 = 0x4e8
                    0x04e8                  _U1EP4bits = 0x4e8
                    0x04ea                  U1EP5 = 0x4ea
                    0x04ea                  _U1EP5 = 0x4ea
                    0x04ea                  _U1EP5bits = 0x4ea
                    0x04ec                  U1EP6 = 0x4ec
                    0x04ec                  _U1EP6 = 0x4ec
                    0x04ec                  _U1EP6bits = 0x4ec
                    0x04ee                  U1EP7 = 0x4ee
                    0x04ee                  _U1EP7 = 0x4ee
                    0x04ee                  _U1EP7bits = 0x4ee
                    0x04f0                  U1EP8 = 0x4f0
                    0x04f0                  _U1EP8 = 0x4f0
                    0x04f0                  _U1EP8bits = 0x4f0
                    0x04f2                  U1EP9 = 0x4f2
                    0x04f2                  _U1EP9 = 0x4f2
                    0x04f2                  _U1EP9bits = 0x4f2
                    0x04f4                  U1EP10 = 0x4f4
                    0x04f4                  _U1EP10 = 0x4f4
                    0x04f4                  _U1EP10bits = 0x4f4
                    0x04f6                  U1EP11 = 0x4f6
                    0x04f6                  _U1EP11 = 0x4f6
                    0x04f6                  _U1EP11bits = 0x4f6
                    0x04f8                  U1EP12 = 0x4f8
                    0x04f8                  _U1EP12 = 0x4f8
                    0x04f8                  _U1EP12bits = 0x4f8
                    0x04fa                  U1EP13 = 0x4fa
                    0x04fa                  _U1EP13 = 0x4fa
                    0x04fa                  _U1EP13bits = 0x4fa
                    0x04fc                  U1EP14 = 0x4fc
                    0x04fc                  _U1EP14 = 0x4fc
                    0x04fc                  _U1EP14bits = 0x4fc
                    0x04fe                  U1EP15 = 0x4fe
                    0x04fe                  _U1EP15 = 0x4fe
                    0x04fe                  _U1EP15bits = 0x4fe
                    0x0500                  C2CTRL1 = 0x500
                    0x0500                  _C2CTRL1 = 0x500
                    0x0500                  _C2CTRL1bits = 0x500
                    0x0502                  C2CTRL2 = 0x502
                    0x0502                  _C2CTRL2 = 0x502
                    0x0502                  _C2CTRL2bits = 0x502
                    0x0504                  C2VEC = 0x504
                    0x0504                  _C2VEC = 0x504
                    0x0504                  _C2VECbits = 0x504
                    0x0506                  C2FCTRL = 0x506
                    0x0506                  _C2FCTRL = 0x506
                    0x0506                  _C2FCTRLbits = 0x506
                    0x0508                  C2FIFO = 0x508
                    0x0508                  _C2FIFO = 0x508
                    0x0508                  _C2FIFObits = 0x508
                    0x050a                  C2INTF = 0x50a
                    0x050a                  _C2INTF = 0x50a
                    0x050a                  _C2INTFbits = 0x50a
                    0x050c                  C2INTE = 0x50c
                    0x050c                  _C2INTE = 0x50c
                    0x050c                  _C2INTEbits = 0x50c
                    0x050e                  C2EC = 0x50e
                    0x050e                  _C2EC = 0x50e
                    0x050e                  _C2ECbits = 0x50e
                    0x050e                  C2RERRCNT = 0x50e
                    0x050e                  _C2RERRCNT = 0x50e
                    0x050f                  C2TERRCNT = 0x50f
                    0x050f                  _C2TERRCNT = 0x50f
                    0x0510                  C2CFG1 = 0x510
                    0x0510                  _C2CFG1 = 0x510
                    0x0510                  _C2CFG1bits = 0x510
                    0x0512                  C2CFG2 = 0x512
                    0x0512                  _C2CFG2 = 0x512
                    0x0512                  _C2CFG2bits = 0x512
                    0x0514                  C2FEN1 = 0x514
                    0x0514                  _C2FEN1 = 0x514
                    0x0514                  _C2FEN1bits = 0x514
                    0x0518                  C2FMSKSEL1 = 0x518
                    0x0518                  _C2FMSKSEL1 = 0x518
                    0x0518                  _C2FMSKSEL1bits = 0x518
                    0x051a                  C2FMSKSEL2 = 0x51a
                    0x051a                  _C2FMSKSEL2 = 0x51a
                    0x051a                  _C2FMSKSEL2bits = 0x51a
                    0x0520                  C2BUFPNT1 = 0x520
                    0x0520                  _C2BUFPNT1 = 0x520
                    0x0520                  _C2BUFPNT1bits = 0x520
                    0x0520                  C2RXFUL1 = 0x520
                    0x0520                  _C2RXFUL1 = 0x520
                    0x0520                  _C2RXFUL1bits = 0x520
                    0x0522                  C2BUFPNT2 = 0x522
                    0x0522                  _C2BUFPNT2 = 0x522
                    0x0522                  _C2BUFPNT2bits = 0x522
                    0x0522                  C2RXFUL2 = 0x522
                    0x0522                  _C2RXFUL2 = 0x522
                    0x0522                  _C2RXFUL2bits = 0x522
                    0x0524                  C2BUFPNT3 = 0x524
                    0x0524                  _C2BUFPNT3 = 0x524
                    0x0524                  _C2BUFPNT3bits = 0x524
                    0x0526                  C2BUFPNT4 = 0x526
                    0x0526                  _C2BUFPNT4 = 0x526
                    0x0526                  _C2BUFPNT4bits = 0x526
                    0x0528                  C2RXOVF1 = 0x528
                    0x0528                  _C2RXOVF1 = 0x528
                    0x0528                  _C2RXOVF1bits = 0x528
                    0x052a                  C2RXOVF2 = 0x52a
                    0x052a                  _C2RXOVF2 = 0x52a
                    0x052a                  _C2RXOVF2bits = 0x52a
                    0x0530                  C2RXM0SID = 0x530
                    0x0530                  _C2RXM0SID = 0x530
                    0x0530                  _C2RXM0SIDbits = 0x530
                    0x0530                  C2TR01CON = 0x530
                    0x0530                  _C2TR01CON = 0x530
                    0x0530                  _C2TR01CONbits = 0x530
                    0x0532                  C2RXM0EID = 0x532
                    0x0532                  _C2RXM0EID = 0x532
                    0x0532                  _C2RXM0EIDbits = 0x532
                    0x0532                  C2TR23CON = 0x532
                    0x0532                  _C2TR23CON = 0x532
                    0x0532                  _C2TR23CONbits = 0x532
                    0x0534                  C2RXM1SID = 0x534
                    0x0534                  _C2RXM1SID = 0x534
                    0x0534                  _C2RXM1SIDbits = 0x534
                    0x0534                  C2TR45CON = 0x534
                    0x0534                  _C2TR45CON = 0x534
                    0x0534                  _C2TR45CONbits = 0x534
                    0x0536                  C2RXM1EID = 0x536
                    0x0536                  _C2RXM1EID = 0x536
                    0x0536                  _C2RXM1EIDbits = 0x536
                    0x0536                  C2TR67CON = 0x536
                    0x0536                  _C2TR67CON = 0x536
                    0x0536                  _C2TR67CONbits = 0x536
                    0x0538                  C2RXM2SID = 0x538
                    0x0538                  _C2RXM2SID = 0x538
                    0x0538                  _C2RXM2SIDbits = 0x538
                    0x053a                  C2RXM2EID = 0x53a
                    0x053a                  _C2RXM2EID = 0x53a
                    0x053a                  _C2RXM2EIDbits = 0x53a
                    0x0540                  C2RXD = 0x540
                    0x0540                  _C2RXD = 0x540
                    0x0540                  C2RXF0SID = 0x540
                    0x0540                  _C2RXF0SID = 0x540
                    0x0540                  _C2RXF0SIDbits = 0x540
                    0x0542                  C2RXF0EID = 0x542
                    0x0542                  _C2RXF0EID = 0x542
                    0x0542                  _C2RXF0EIDbits = 0x542
                    0x0542                  C2TXD = 0x542
                    0x0542                  _C2TXD = 0x542
                    0x0542                  _C2TXDbits = 0x542
                    0x0544                  C2RXF1SID = 0x544
                    0x0544                  _C2RXF1SID = 0x544
                    0x0544                  _C2RXF1SIDbits = 0x544
                    0x0546                  C2RXF1EID = 0x546
                    0x0546                  _C2RXF1EID = 0x546
                    0x0546                  _C2RXF1EIDbits = 0x546
                    0x0548                  C2RXF2SID = 0x548
                    0x0548                  _C2RXF2SID = 0x548
                    0x0548                  _C2RXF2SIDbits = 0x548
                    0x054a                  C2RXF2EID = 0x54a
                    0x054a                  _C2RXF2EID = 0x54a
                    0x054a                  _C2RXF2EIDbits = 0x54a
                    0x054c                  C2RXF3SID = 0x54c
                    0x054c                  _C2RXF3SID = 0x54c
                    0x054c                  _C2RXF3SIDbits = 0x54c
                    0x054e                  C2RXF3EID = 0x54e
                    0x054e                  _C2RXF3EID = 0x54e
                    0x054e                  _C2RXF3EIDbits = 0x54e
                    0x0550                  C2RXF4SID = 0x550
                    0x0550                  _C2RXF4SID = 0x550
                    0x0550                  _C2RXF4SIDbits = 0x550
                    0x0552                  C2RXF4EID = 0x552
                    0x0552                  _C2RXF4EID = 0x552
                    0x0552                  _C2RXF4EIDbits = 0x552
                    0x0554                  C2RXF5SID = 0x554
                    0x0554                  _C2RXF5SID = 0x554
                    0x0554                  _C2RXF5SIDbits = 0x554
                    0x0556                  C2RXF5EID = 0x556
                    0x0556                  _C2RXF5EID = 0x556
                    0x0556                  _C2RXF5EIDbits = 0x556
                    0x0558                  C2RXF6SID = 0x558
                    0x0558                  _C2RXF6SID = 0x558
                    0x0558                  _C2RXF6SIDbits = 0x558
                    0x055a                  C2RXF6EID = 0x55a
                    0x055a                  _C2RXF6EID = 0x55a
                    0x055a                  _C2RXF6EIDbits = 0x55a
                    0x055c                  C2RXF7SID = 0x55c
                    0x055c                  _C2RXF7SID = 0x55c
                    0x055c                  _C2RXF7SIDbits = 0x55c
                    0x055e                  C2RXF7EID = 0x55e
                    0x055e                  _C2RXF7EID = 0x55e
                    0x055e                  _C2RXF7EIDbits = 0x55e
                    0x0560                  C2RXF8SID = 0x560
                    0x0560                  _C2RXF8SID = 0x560
                    0x0560                  _C2RXF8SIDbits = 0x560
                    0x0562                  C2RXF8EID = 0x562
                    0x0562                  _C2RXF8EID = 0x562
                    0x0562                  _C2RXF8EIDbits = 0x562
                    0x0564                  C2RXF9SID = 0x564
                    0x0564                  _C2RXF9SID = 0x564
                    0x0564                  _C2RXF9SIDbits = 0x564
                    0x0566                  C2RXF9EID = 0x566
                    0x0566                  _C2RXF9EID = 0x566
                    0x0566                  _C2RXF9EIDbits = 0x566
                    0x0568                  C2RXF10SID = 0x568
                    0x0568                  _C2RXF10SID = 0x568
                    0x0568                  _C2RXF10SIDbits = 0x568
                    0x056a                  C2RXF10EID = 0x56a
                    0x056a                  _C2RXF10EID = 0x56a
                    0x056a                  _C2RXF10EIDbits = 0x56a
                    0x056c                  C2RXF11SID = 0x56c
                    0x056c                  _C2RXF11SID = 0x56c
                    0x056c                  _C2RXF11SIDbits = 0x56c
                    0x056e                  C2RXF11EID = 0x56e
                    0x056e                  _C2RXF11EID = 0x56e
                    0x056e                  _C2RXF11EIDbits = 0x56e
                    0x0570                  C2RXF12SID = 0x570
                    0x0570                  _C2RXF12SID = 0x570
                    0x0570                  _C2RXF12SIDbits = 0x570
                    0x0572                  C2RXF12EID = 0x572
                    0x0572                  _C2RXF12EID = 0x572
                    0x0572                  _C2RXF12EIDbits = 0x572
                    0x0574                  C2RXF13SID = 0x574
                    0x0574                  _C2RXF13SID = 0x574
                    0x0574                  _C2RXF13SIDbits = 0x574
                    0x0576                  C2RXF13EID = 0x576
                    0x0576                  _C2RXF13EID = 0x576
                    0x0576                  _C2RXF13EIDbits = 0x576
                    0x0578                  C2RXF14SID = 0x578
                    0x0578                  _C2RXF14SID = 0x578
                    0x0578                  _C2RXF14SIDbits = 0x578
                    0x057a                  C2RXF14EID = 0x57a
                    0x057a                  _C2RXF14EID = 0x57a
                    0x057a                  _C2RXF14EIDbits = 0x57a
                    0x057c                  C2RXF15SID = 0x57c
                    0x057c                  _C2RXF15SID = 0x57c
                    0x057c                  _C2RXF15SIDbits = 0x57c
                    0x057e                  C2RXF15EID = 0x57e
                    0x057e                  _C2RXF15EID = 0x57e
                    0x057e                  _C2RXF15EIDbits = 0x57e
                    0x0580                  U1PWMRRS = 0x580
                    0x0580                  _U1PWMRRS = 0x580
                    0x0580                  _U1PWMRRSbits = 0x580
                    0x0582                  U1PWMCON = 0x582
                    0x0582                  _U1PWMCON = 0x582
                    0x0582                  _U1PWMCONbits = 0x582
                    0x05c0                  QEI2CON = 0x5c0
                    0x05c0                  _QEI2CON = 0x5c0
                    0x05c0                  _QEI2CONbits = 0x5c0
                    0x05c2                  QEI2IOC = 0x5c2
                    0x05c2                  _QEI2IOC = 0x5c2
                    0x05c2                  _QEI2IOCbits = 0x5c2
                    0x05c4                  QEI2STAT = 0x5c4
                    0x05c4                  _QEI2STAT = 0x5c4
                    0x05c4                  _QEI2STATbits = 0x5c4
                    0x05c6                  POS2CNTL = 0x5c6
                    0x05c6                  _POS2CNTL = 0x5c6
                    0x05c8                  POS2CNTH = 0x5c8
                    0x05c8                  _POS2CNTH = 0x5c8
                    0x05ca                  POS2HLD = 0x5ca
                    0x05ca                  _POS2HLD = 0x5ca
                    0x05cc                  VEL2CNT = 0x5cc
                    0x05cc                  _VEL2CNT = 0x5cc
                    0x05ce                  INT2TMRL = 0x5ce
                    0x05ce                  _INT2TMRL = 0x5ce
                    0x05d0                  INT2TMRH = 0x5d0
                    0x05d0                  _INT2TMRH = 0x5d0
                    0x05d2                  INT2HLDL = 0x5d2
                    0x05d2                  _INT2HLDL = 0x5d2
                    0x05d4                  INT2HLDH = 0x5d4
                    0x05d4                  _INT2HLDH = 0x5d4
                    0x05d6                  INDX2CNTL = 0x5d6
                    0x05d6                  _INDX2CNTL = 0x5d6
                    0x05d8                  INDX2CNTH = 0x5d8
                    0x05d8                  _INDX2CNTH = 0x5d8
                    0x05da                  INDX2HLD = 0x5da
                    0x05da                  _INDX2HLD = 0x5da
                    0x05dc                  QEI2GECL = 0x5dc
                    0x05dc                  _QEI2GECL = 0x5dc
                    0x05dc                  QEI2ICL = 0x5dc
                    0x05dc                  _QEI2ICL = 0x5dc
                    0x05de                  QEI2GECH = 0x5de
                    0x05de                  _QEI2GECH = 0x5de
                    0x05de                  QEI2ICH = 0x5de
                    0x05de                  _QEI2ICH = 0x5de
                    0x05e0                  QEI2LECL = 0x5e0
                    0x05e0                  _QEI2LECL = 0x5e0
                    0x05e2                  QEI2LECH = 0x5e2
                    0x05e2                  _QEI2LECH = 0x5e2
                    0x0600                  PMCON = 0x600
                    0x0600                  _PMCON = 0x600
                    0x0600                  _PMCONbits = 0x600
                    0x0602                  PMMODE = 0x602
                    0x0602                  _PMMODE = 0x602
                    0x0602                  _PMMODEbits = 0x602
                    0x0604                  PMADDR = 0x604
                    0x0604                  _PMADDR = 0x604
                    0x0604                  _PMADDRbits = 0x604
                    0x0604                  PMDOUT1 = 0x604
                    0x0604                  _PMDOUT1 = 0x604
                    0x0604                  _PMDOUT1bits = 0x604
                    0x0606                  PMDOUT2 = 0x606
                    0x0606                  _PMDOUT2 = 0x606
                    0x0608                  PMDIN1 = 0x608
                    0x0608                  _PMDIN1 = 0x608
                    0x060a                  PMDIN2 = 0x60a
                    0x060a                  _PMDIN2 = 0x60a
                    0x060c                  PMAEN = 0x60c
                    0x060c                  _PMAEN = 0x60c
                    0x060c                  _PMAENbits = 0x60c
                    0x060e                  PMSTAT = 0x60e
                    0x060e                  _PMSTAT = 0x60e
                    0x060e                  _PMSTATbits = 0x60e
                    0x0620                  ALRMVAL = 0x620
                    0x0620                  _ALRMVAL = 0x620
                    0x0622                  ALCFGRPT = 0x622
                    0x0622                  _ALCFGRPT = 0x622
                    0x0622                  _ALCFGRPTbits = 0x622
                    0x0624                  RTCVAL = 0x624
                    0x0624                  _RTCVAL = 0x624
                    0x0626                  RCFGCAL = 0x626
                    0x0626                  _RCFGCAL = 0x626
                    0x0626                  _RCFGCALbits = 0x626
                    0x0640                  CRCCON1 = 0x640
                    0x0640                  _CRCCON1 = 0x640
                    0x0640                  _CRCCON1bits = 0x640
                    0x0642                  CRCCON2 = 0x642
                    0x0642                  _CRCCON2 = 0x642
                    0x0642                  _CRCCON2bits = 0x642
                    0x0644                  CRCXORL = 0x644
                    0x0644                  _CRCXORL = 0x644
                    0x0644                  _CRCXORLbits = 0x644
                    0x0646                  CRCXORH = 0x646
                    0x0646                  _CRCXORH = 0x646
                    0x0646                  _CRCXORHbits = 0x646
                    0x0648                  CRCDAT = 0x648
                    0x0648                  _CRCDAT = 0x648
                    0x0648                  CRCDATL = 0x648
                    0x0648                  _CRCDATL = 0x648
                    0x064a                  CRCDATH = 0x64a
                    0x064a                  _CRCDATH = 0x64a
                    0x064c                  CRCWDAT = 0x64c
                    0x064c                  _CRCWDAT = 0x64c
                    0x064c                  CRCWDATL = 0x64c
                    0x064c                  _CRCWDATL = 0x64c
                    0x064e                  CRCWDATH = 0x64e
                    0x064e                  _CRCWDATH = 0x64e
                    0x0680                  RPOR0 = 0x680
                    0x0680                  _RPOR0 = 0x680
                    0x0680                  _RPOR0bits = 0x680
                    0x0682                  RPOR1 = 0x682
                    0x0682                  _RPOR1 = 0x682
                    0x0682                  _RPOR1bits = 0x682
                    0x0684                  RPOR2 = 0x684
                    0x0684                  _RPOR2 = 0x684
                    0x0684                  _RPOR2bits = 0x684
                    0x0686                  RPOR3 = 0x686
                    0x0686                  _RPOR3 = 0x686
                    0x0686                  _RPOR3bits = 0x686
                    0x0688                  RPOR4 = 0x688
                    0x0688                  _RPOR4 = 0x688
                    0x0688                  _RPOR4bits = 0x688
                    0x068a                  RPOR5 = 0x68a
                    0x068a                  _RPOR5 = 0x68a
                    0x068a                  _RPOR5bits = 0x68a
                    0x068c                  RPOR6 = 0x68c
                    0x068c                  _RPOR6 = 0x68c
                    0x068c                  _RPOR6bits = 0x68c
                    0x068e                  RPOR7 = 0x68e
                    0x068e                  _RPOR7 = 0x68e
                    0x068e                  _RPOR7bits = 0x68e
                    0x0690                  RPOR8 = 0x690
                    0x0690                  _RPOR8 = 0x690
                    0x0690                  _RPOR8bits = 0x690
                    0x0692                  RPOR9 = 0x692
                    0x0692                  _RPOR9 = 0x692
                    0x0692                  _RPOR9bits = 0x692
                    0x0696                  RPOR11 = 0x696
                    0x0696                  _RPOR11 = 0x696
                    0x0696                  _RPOR11bits = 0x696
                    0x0698                  RPOR12 = 0x698
                    0x0698                  _RPOR12 = 0x698
                    0x0698                  _RPOR12bits = 0x698
                    0x069a                  RPOR13 = 0x69a
                    0x069a                  _RPOR13 = 0x69a
                    0x069a                  _RPOR13bits = 0x69a
                    0x069c                  RPOR14 = 0x69c
                    0x069c                  _RPOR14 = 0x69c
                    0x069c                  _RPOR14bits = 0x69c
                    0x069e                  RPOR15 = 0x69e
                    0x069e                  _RPOR15 = 0x69e
                    0x069e                  _RPOR15bits = 0x69e
                    0x06a0                  RPINR0 = 0x6a0
                    0x06a0                  _RPINR0 = 0x6a0
                    0x06a0                  _RPINR0bits = 0x6a0
                    0x06a2                  RPINR1 = 0x6a2
                    0x06a2                  _RPINR1 = 0x6a2
                    0x06a2                  _RPINR1bits = 0x6a2
                    0x06a4                  RPINR2 = 0x6a4
                    0x06a4                  _RPINR2 = 0x6a4
                    0x06a4                  _RPINR2bits = 0x6a4
                    0x06a6                  RPINR3 = 0x6a6
                    0x06a6                  _RPINR3 = 0x6a6
                    0x06a6                  _RPINR3bits = 0x6a6
                    0x06a8                  RPINR4 = 0x6a8
                    0x06a8                  _RPINR4 = 0x6a8
                    0x06a8                  _RPINR4bits = 0x6a8
                    0x06aa                  RPINR5 = 0x6aa
                    0x06aa                  _RPINR5 = 0x6aa
                    0x06aa                  _RPINR5bits = 0x6aa
                    0x06ac                  RPINR6 = 0x6ac
                    0x06ac                  _RPINR6 = 0x6ac
                    0x06ac                  _RPINR6bits = 0x6ac
                    0x06ae                  RPINR7 = 0x6ae
                    0x06ae                  _RPINR7 = 0x6ae
                    0x06ae                  _RPINR7bits = 0x6ae
                    0x06b0                  RPINR8 = 0x6b0
                    0x06b0                  _RPINR8 = 0x6b0
                    0x06b0                  _RPINR8bits = 0x6b0
                    0x06b2                  RPINR9 = 0x6b2
                    0x06b2                  _RPINR9 = 0x6b2
                    0x06b2                  _RPINR9bits = 0x6b2
                    0x06b4                  RPINR10 = 0x6b4
                    0x06b4                  _RPINR10 = 0x6b4
                    0x06b4                  _RPINR10bits = 0x6b4
                    0x06b6                  RPINR11 = 0x6b6
                    0x06b6                  _RPINR11 = 0x6b6
                    0x06b6                  _RPINR11bits = 0x6b6
                    0x06b8                  RPINR12 = 0x6b8
                    0x06b8                  _RPINR12 = 0x6b8
                    0x06b8                  _RPINR12bits = 0x6b8
                    0x06ba                  RPINR13 = 0x6ba
                    0x06ba                  _RPINR13 = 0x6ba
                    0x06ba                  _RPINR13bits = 0x6ba
                    0x06bc                  RPINR14 = 0x6bc
                    0x06bc                  _RPINR14 = 0x6bc
                    0x06bc                  _RPINR14bits = 0x6bc
                    0x06be                  RPINR15 = 0x6be
                    0x06be                  _RPINR15 = 0x6be
                    0x06be                  _RPINR15bits = 0x6be
                    0x06c0                  RPINR16 = 0x6c0
                    0x06c0                  _RPINR16 = 0x6c0
                    0x06c0                  _RPINR16bits = 0x6c0
                    0x06c2                  RPINR17 = 0x6c2
                    0x06c2                  _RPINR17 = 0x6c2
                    0x06c2                  _RPINR17bits = 0x6c2
                    0x06c4                  RPINR18 = 0x6c4
                    0x06c4                  _RPINR18 = 0x6c4
                    0x06c4                  _RPINR18bits = 0x6c4
                    0x06c6                  RPINR19 = 0x6c6
                    0x06c6                  _RPINR19 = 0x6c6
                    0x06c6                  _RPINR19bits = 0x6c6
                    0x06c8                  RPINR20 = 0x6c8
                    0x06c8                  _RPINR20 = 0x6c8
                    0x06c8                  _RPINR20bits = 0x6c8
                    0x06ca                  RPINR21 = 0x6ca
                    0x06ca                  _RPINR21 = 0x6ca
                    0x06ca                  _RPINR21bits = 0x6ca
                    0x06ce                  RPINR23 = 0x6ce
                    0x06ce                  _RPINR23 = 0x6ce
                    0x06ce                  _RPINR23bits = 0x6ce
                    0x06d0                  RPINR24 = 0x6d0
                    0x06d0                  _RPINR24 = 0x6d0
                    0x06d0                  _RPINR24bits = 0x6d0
                    0x06d2                  RPINR25 = 0x6d2
                    0x06d2                  _RPINR25 = 0x6d2
                    0x06d2                  _RPINR25bits = 0x6d2
                    0x06d4                  RPINR26 = 0x6d4
                    0x06d4                  _RPINR26 = 0x6d4
                    0x06d4                  _RPINR26bits = 0x6d4
                    0x06d6                  RPINR27 = 0x6d6
                    0x06d6                  _RPINR27 = 0x6d6
                    0x06d6                  _RPINR27bits = 0x6d6
                    0x06d8                  RPINR28 = 0x6d8
                    0x06d8                  _RPINR28 = 0x6d8
                    0x06d8                  _RPINR28bits = 0x6d8
                    0x06da                  RPINR29 = 0x6da
                    0x06da                  _RPINR29 = 0x6da
                    0x06da                  _RPINR29bits = 0x6da
                    0x06dc                  RPINR30 = 0x6dc
                    0x06dc                  _RPINR30 = 0x6dc
                    0x06dc                  _RPINR30bits = 0x6dc
                    0x06de                  RPINR31 = 0x6de
                    0x06de                  _RPINR31 = 0x6de
                    0x06de                  _RPINR31bits = 0x6de
                    0x06e0                  RPINR32 = 0x6e0
                    0x06e0                  _RPINR32 = 0x6e0
                    0x06e0                  _RPINR32bits = 0x6e0
                    0x06e2                  RPINR33 = 0x6e2
                    0x06e2                  _RPINR33 = 0x6e2
                    0x06e2                  _RPINR33bits = 0x6e2
                    0x06e4                  RPINR34 = 0x6e4
                    0x06e4                  _RPINR34 = 0x6e4
                    0x06e4                  _RPINR34bits = 0x6e4
                    0x06e6                  RPINR35 = 0x6e6
                    0x06e6                  _RPINR35 = 0x6e6
                    0x06e6                  _RPINR35bits = 0x6e6
                    0x06e8                  RPINR36 = 0x6e8
                    0x06e8                  _RPINR36 = 0x6e8
                    0x06e8                  _RPINR36bits = 0x6e8
                    0x06ea                  RPINR37 = 0x6ea
                    0x06ea                  _RPINR37 = 0x6ea
                    0x06ea                  _RPINR37bits = 0x6ea
                    0x06ec                  RPINR38 = 0x6ec
                    0x06ec                  _RPINR38 = 0x6ec
                    0x06ec                  _RPINR38bits = 0x6ec
                    0x06ee                  RPINR39 = 0x6ee
                    0x06ee                  _RPINR39 = 0x6ee
                    0x06ee                  _RPINR39bits = 0x6ee
                    0x06f0                  RPINR40 = 0x6f0
                    0x06f0                  _RPINR40 = 0x6f0
                    0x06f0                  _RPINR40bits = 0x6f0
                    0x06f2                  RPINR41 = 0x6f2
                    0x06f2                  _RPINR41 = 0x6f2
                    0x06f2                  _RPINR41bits = 0x6f2
                    0x06f4                  RPINR42 = 0x6f4
                    0x06f4                  _RPINR42 = 0x6f4
                    0x06f4                  _RPINR42bits = 0x6f4
                    0x06f6                  RPINR43 = 0x6f6
                    0x06f6                  _RPINR43 = 0x6f6
                    0x06f6                  _RPINR43bits = 0x6f6
                    0x0728                  NVMCON = 0x728
                    0x0728                  _NVMCON = 0x728
                    0x0728                  _NVMCONbits = 0x728
                    0x072a                  NVMADR = 0x72a
                    0x072a                  _NVMADR = 0x72a
                    0x072c                  NVMADRU = 0x72c
                    0x072c                  _NVMADRU = 0x72c
                    0x072c                  _NVMADRUbits = 0x72c
                    0x072e                  NVMKEY = 0x72e
                    0x072e                  _NVMKEY = 0x72e
                    0x0740                  RCON = 0x740
                    0x0740                  _RCON = 0x740
                    0x0740                  _RCONbits = 0x740
                    0x0742                  OSCCON = 0x742
                    0x0742                  _OSCCON = 0x742
                    0x0742                  _OSCCONbits = 0x742
                    0x0742                  OSCCONL = 0x742
                    0x0742                  _OSCCONL = 0x742
                    0x0743                  OSCCONH = 0x743
                    0x0743                  _OSCCONH = 0x743
                    0x0744                  CLKDIV = 0x744
                    0x0744                  _CLKDIV = 0x744
                    0x0744                  _CLKDIVbits = 0x744
                    0x0746                  PLLFBD = 0x746
                    0x0746                  _PLLFBD = 0x746
                    0x0746                  _PLLFBDbits = 0x746
                    0x0748                  OSCTUN = 0x748
                    0x0748                  _OSCTUN = 0x748
                    0x0748                  _OSCTUNbits = 0x748
                    0x074e                  REFOCON = 0x74e
                    0x074e                  _REFOCON = 0x74e
                    0x074e                  _REFOCONbits = 0x74e
                    0x0758                  ACLKCON3 = 0x758
                    0x0758                  _ACLKCON3 = 0x758
                    0x0758                  _ACLKCON3bits = 0x758
                    0x075a                  ACLKDIV3 = 0x75a
                    0x075a                  _ACLKDIV3 = 0x75a
                    0x075a                  _ACLKDIV3bits = 0x75a
                    0x0760                  PMD1 = 0x760
                    0x0760                  _PMD1 = 0x760
                    0x0760                  _PMD1bits = 0x760
                    0x0762                  PMD2 = 0x762
                    0x0762                  _PMD2 = 0x762
                    0x0762                  _PMD2bits = 0x762
                    0x0764                  PMD3 = 0x764
                    0x0764                  _PMD3 = 0x764
                    0x0764                  _PMD3bits = 0x764
                    0x0766                  PMD4 = 0x766
                    0x0766                  _PMD4 = 0x766
                    0x0766                  _PMD4bits = 0x766
                    0x0768                  PMD5 = 0x768
                    0x0768                  _PMD5 = 0x768
                    0x0768                  _PMD5bits = 0x768
                    0x076a                  PMD6 = 0x76a
                    0x076a                  _PMD6 = 0x76a
                    0x076a                  _PMD6bits = 0x76a
                    0x076c                  PMD7 = 0x76c
                    0x076c                  _PMD7 = 0x76c
                    0x076c                  _PMD7bits = 0x76c
                    0x0800                  IFS0 = 0x800
                    0x0800                  _IFS0 = 0x800
                    0x0800                  _IFS0bits = 0x800
                    0x0802                  IFS1 = 0x802
                    0x0802                  _IFS1 = 0x802
                    0x0802                  _IFS1bits = 0x802
                    0x0804                  IFS2 = 0x804
                    0x0804                  _IFS2 = 0x804
                    0x0804                  _IFS2bits = 0x804
                    0x0806                  IFS3 = 0x806
                    0x0806                  _IFS3 = 0x806
                    0x0806                  _IFS3bits = 0x806
                    0x0808                  IFS4 = 0x808
                    0x0808                  _IFS4 = 0x808
                    0x0808                  _IFS4bits = 0x808
                    0x080a                  IFS5 = 0x80a
                    0x080a                  _IFS5 = 0x80a
                    0x080a                  _IFS5bits = 0x80a
                    0x080c                  IFS6 = 0x80c
                    0x080c                  _IFS6 = 0x80c
                    0x080c                  _IFS6bits = 0x80c
                    0x080e                  IFS7 = 0x80e
                    0x080e                  _IFS7 = 0x80e
                    0x080e                  _IFS7bits = 0x80e
                    0x0810                  IFS8 = 0x810
                    0x0810                  _IFS8 = 0x810
                    0x0810                  _IFS8bits = 0x810
                    0x0820                  IEC0 = 0x820
                    0x0820                  _IEC0 = 0x820
                    0x0820                  _IEC0bits = 0x820
                    0x0822                  IEC1 = 0x822
                    0x0822                  _IEC1 = 0x822
                    0x0822                  _IEC1bits = 0x822
                    0x0824                  IEC2 = 0x824
                    0x0824                  _IEC2 = 0x824
                    0x0824                  _IEC2bits = 0x824
                    0x0826                  IEC3 = 0x826
                    0x0826                  _IEC3 = 0x826
                    0x0826                  _IEC3bits = 0x826
                    0x0828                  IEC4 = 0x828
                    0x0828                  _IEC4 = 0x828
                    0x0828                  _IEC4bits = 0x828
                    0x082a                  IEC5 = 0x82a
                    0x082a                  _IEC5 = 0x82a
                    0x082a                  _IEC5bits = 0x82a
                    0x082c                  IEC6 = 0x82c
                    0x082c                  _IEC6 = 0x82c
                    0x082c                  _IEC6bits = 0x82c
                    0x082e                  IEC7 = 0x82e
                    0x082e                  _IEC7 = 0x82e
                    0x082e                  _IEC7bits = 0x82e
                    0x0830                  IEC8 = 0x830
                    0x0830                  _IEC8 = 0x830
                    0x0830                  _IEC8bits = 0x830
                    0x0840                  IPC0 = 0x840
                    0x0840                  _IPC0 = 0x840
                    0x0840                  _IPC0bits = 0x840
                    0x0842                  IPC1 = 0x842
                    0x0842                  _IPC1 = 0x842
                    0x0842                  _IPC1bits = 0x842
                    0x0844                  IPC2 = 0x844
                    0x0844                  _IPC2 = 0x844
                    0x0844                  _IPC2bits = 0x844
                    0x0846                  IPC3 = 0x846
                    0x0846                  _IPC3 = 0x846
                    0x0846                  _IPC3bits = 0x846
                    0x0848                  IPC4 = 0x848
                    0x0848                  _IPC4 = 0x848
                    0x0848                  _IPC4bits = 0x848
                    0x084a                  IPC5 = 0x84a
                    0x084a                  _IPC5 = 0x84a
                    0x084a                  _IPC5bits = 0x84a
                    0x084c                  IPC6 = 0x84c
                    0x084c                  _IPC6 = 0x84c
                    0x084c                  _IPC6bits = 0x84c
                    0x084e                  IPC7 = 0x84e
                    0x084e                  _IPC7 = 0x84e
                    0x084e                  _IPC7bits = 0x84e
                    0x0850                  IPC8 = 0x850
                    0x0850                  _IPC8 = 0x850
                    0x0850                  _IPC8bits = 0x850
                    0x0852                  IPC9 = 0x852
                    0x0852                  _IPC9 = 0x852
                    0x0852                  _IPC9bits = 0x852
                    0x0854                  IPC10 = 0x854
                    0x0854                  _IPC10 = 0x854
                    0x0854                  _IPC10bits = 0x854
                    0x0856                  IPC11 = 0x856
                    0x0856                  _IPC11 = 0x856
                    0x0856                  _IPC11bits = 0x856
                    0x0858                  IPC12 = 0x858
                    0x0858                  _IPC12 = 0x858
                    0x0858                  _IPC12bits = 0x858
                    0x085a                  IPC13 = 0x85a
                    0x085a                  _IPC13 = 0x85a
                    0x085a                  _IPC13bits = 0x85a
                    0x085c                  IPC14 = 0x85c
                    0x085c                  _IPC14 = 0x85c
                    0x085c                  _IPC14bits = 0x85c
                    0x085e                  IPC15 = 0x85e
                    0x085e                  _IPC15 = 0x85e
                    0x085e                  _IPC15bits = 0x85e
                    0x0860                  IPC16 = 0x860
                    0x0860                  _IPC16 = 0x860
                    0x0860                  _IPC16bits = 0x860
                    0x0862                  IPC17 = 0x862
                    0x0862                  _IPC17 = 0x862
                    0x0862                  _IPC17bits = 0x862
                    0x0864                  IPC18 = 0x864
                    0x0864                  _IPC18 = 0x864
                    0x0864                  _IPC18bits = 0x864
                    0x0868                  IPC20 = 0x868
                    0x0868                  _IPC20 = 0x868
                    0x0868                  _IPC20bits = 0x868
                    0x086a                  IPC21 = 0x86a
                    0x086a                  _IPC21 = 0x86a
                    0x086a                  _IPC21bits = 0x86a
                    0x086c                  IPC22 = 0x86c
                    0x086c                  _IPC22 = 0x86c
                    0x086c                  _IPC22bits = 0x86c
                    0x086e                  IPC23 = 0x86e
                    0x086e                  _IPC23 = 0x86e
                    0x086e                  _IPC23bits = 0x86e
                    0x0870                  IPC24 = 0x870
                    0x0870                  _IPC24 = 0x870
                    0x0870                  _IPC24bits = 0x870
                    0x087a                  IPC29 = 0x87a
                    0x087a                  _IPC29 = 0x87a
                    0x087a                  _IPC29bits = 0x87a
                    0x087c                  IPC30 = 0x87c
                    0x087c                  _IPC30 = 0x87c
                    0x087c                  _IPC30bits = 0x87c
                    0x087e                  IPC31 = 0x87e
                    0x087e                  _IPC31 = 0x87e
                    0x087e                  _IPC31bits = 0x87e
                    0x0880                  IPC32 = 0x880
                    0x0880                  _IPC32 = 0x880
                    0x0880                  _IPC32bits = 0x880
                    0x0882                  IPC33 = 0x882
                    0x0882                  _IPC33 = 0x882
                    0x0882                  _IPC33bits = 0x882
                    0x0884                  IPC34 = 0x884
                    0x0884                  _IPC34 = 0x884
                    0x0884                  _IPC34bits = 0x884
                    0x0886                  IPC35 = 0x886
                    0x0886                  _IPC35 = 0x886
                    0x0886                  _IPC35bits = 0x886
                    0x08c0                  INTCON1 = 0x8c0
                    0x08c0                  _INTCON1 = 0x8c0
                    0x08c0                  _INTCON1bits = 0x8c0
                    0x08c2                  INTCON2 = 0x8c2
                    0x08c2                  _INTCON2 = 0x8c2
                    0x08c2                  _INTCON2bits = 0x8c2
                    0x08c4                  INTCON3 = 0x8c4
                    0x08c4                  _INTCON3 = 0x8c4
                    0x08c4                  _INTCON3bits = 0x8c4
                    0x08c6                  INTCON4 = 0x8c6
                    0x08c6                  _INTCON4 = 0x8c6
                    0x08c6                  _INTCON4bits = 0x8c6
                    0x08c8                  INTTREG = 0x8c8
                    0x08c8                  _INTTREG = 0x8c8
                    0x08c8                  _INTTREGbits = 0x8c8
                    0x0900                  OC1CON1 = 0x900
                    0x0900                  _OC1CON1 = 0x900
                    0x0900                  _OC1CON1bits = 0x900
                    0x0902                  OC1CON2 = 0x902
                    0x0902                  _OC1CON2 = 0x902
                    0x0902                  _OC1CON2bits = 0x902
                    0x0904                  OC1RS = 0x904
                    0x0904                  _OC1RS = 0x904
                    0x0906                  OC1R = 0x906
                    0x0906                  _OC1R = 0x906
                    0x0908                  OC1TMR = 0x908
                    0x0908                  _OC1TMR = 0x908
                    0x090a                  OC2CON1 = 0x90a
                    0x090a                  _OC2CON1 = 0x90a
                    0x090a                  _OC2CON1bits = 0x90a
                    0x090c                  OC2CON2 = 0x90c
                    0x090c                  _OC2CON2 = 0x90c
                    0x090c                  _OC2CON2bits = 0x90c
                    0x090e                  OC2RS = 0x90e
                    0x090e                  _OC2RS = 0x90e
                    0x0910                  OC2R = 0x910
                    0x0910                  _OC2R = 0x910
                    0x0912                  OC2TMR = 0x912
                    0x0912                  _OC2TMR = 0x912
                    0x0914                  OC3CON1 = 0x914
                    0x0914                  _OC3CON1 = 0x914
                    0x0914                  _OC3CON1bits = 0x914
                    0x0916                  OC3CON2 = 0x916
                    0x0916                  _OC3CON2 = 0x916
                    0x0916                  _OC3CON2bits = 0x916
                    0x0918                  OC3RS = 0x918
                    0x0918                  _OC3RS = 0x918
                    0x091a                  OC3R = 0x91a
                    0x091a                  _OC3R = 0x91a
                    0x091c                  OC3TMR = 0x91c
                    0x091c                  _OC3TMR = 0x91c
                    0x091e                  OC4CON1 = 0x91e
                    0x091e                  _OC4CON1 = 0x91e
                    0x091e                  _OC4CON1bits = 0x91e
                    0x0920                  OC4CON2 = 0x920
                    0x0920                  _OC4CON2 = 0x920
                    0x0920                  _OC4CON2bits = 0x920
                    0x0922                  OC4RS = 0x922
                    0x0922                  _OC4RS = 0x922
                    0x0924                  OC4R = 0x924
                    0x0924                  _OC4R = 0x924
                    0x0926                  OC4TMR = 0x926
                    0x0926                  _OC4TMR = 0x926
                    0x0928                  OC5CON1 = 0x928
                    0x0928                  _OC5CON1 = 0x928
                    0x0928                  _OC5CON1bits = 0x928
                    0x092a                  OC5CON2 = 0x92a
                    0x092a                  _OC5CON2 = 0x92a
                    0x092a                  _OC5CON2bits = 0x92a
                    0x092c                  OC5RS = 0x92c
                    0x092c                  _OC5RS = 0x92c
                    0x092e                  OC5R = 0x92e
                    0x092e                  _OC5R = 0x92e
                    0x0930                  OC5TMR = 0x930
                    0x0930                  _OC5TMR = 0x930
                    0x0932                  OC6CON1 = 0x932
                    0x0932                  _OC6CON1 = 0x932
                    0x0932                  _OC6CON1bits = 0x932
                    0x0934                  OC6CON2 = 0x934
                    0x0934                  _OC6CON2 = 0x934
                    0x0934                  _OC6CON2bits = 0x934
                    0x0936                  OC6RS = 0x936
                    0x0936                  _OC6RS = 0x936
                    0x0938                  OC6R = 0x938
                    0x0938                  _OC6R = 0x938
                    0x093a                  OC6TMR = 0x93a
                    0x093a                  _OC6TMR = 0x93a
                    0x093c                  OC7CON1 = 0x93c
                    0x093c                  _OC7CON1 = 0x93c
                    0x093c                  _OC7CON1bits = 0x93c
                    0x093e                  OC7CON2 = 0x93e
                    0x093e                  _OC7CON2 = 0x93e
                    0x093e                  _OC7CON2bits = 0x93e
                    0x0940                  OC7RS = 0x940
                    0x0940                  _OC7RS = 0x940
                    0x0942                  OC7R = 0x942
                    0x0942                  _OC7R = 0x942
                    0x0944                  OC7TMR = 0x944
                    0x0944                  _OC7TMR = 0x944
                    0x0946                  OC8CON1 = 0x946
                    0x0946                  _OC8CON1 = 0x946
                    0x0946                  _OC8CON1bits = 0x946
                    0x0948                  OC8CON2 = 0x948
                    0x0948                  _OC8CON2 = 0x948
                    0x0948                  _OC8CON2bits = 0x948
                    0x094a                  OC8RS = 0x94a
                    0x094a                  _OC8RS = 0x94a
                    0x094c                  OC8R = 0x94c
                    0x094c                  _OC8R = 0x94c
                    0x094e                  OC8TMR = 0x94e
                    0x094e                  _OC8TMR = 0x94e
                    0x0950                  OC9CON1 = 0x950
                    0x0950                  _OC9CON1 = 0x950
                    0x0950                  _OC9CON1bits = 0x950
                    0x0952                  OC9CON2 = 0x952
                    0x0952                  _OC9CON2 = 0x952
                    0x0952                  _OC9CON2bits = 0x952
                    0x0954                  OC9RS = 0x954
                    0x0954                  _OC9RS = 0x954
                    0x0956                  OC9R = 0x956
                    0x0956                  _OC9R = 0x956
                    0x0958                  OC9TMR = 0x958
                    0x0958                  _OC9TMR = 0x958
                    0x095a                  OC10CON1 = 0x95a
                    0x095a                  _OC10CON1 = 0x95a
                    0x095a                  _OC10CON1bits = 0x95a
                    0x095c                  OC10CON2 = 0x95c
                    0x095c                  _OC10CON2 = 0x95c
                    0x095c                  _OC10CON2bits = 0x95c
                    0x095e                  OC10RS = 0x95e
                    0x095e                  _OC10RS = 0x95e
                    0x0960                  OC10R = 0x960
                    0x0960                  _OC10R = 0x960
                    0x0962                  OC10TMR = 0x962
                    0x0962                  _OC10TMR = 0x962
                    0x0964                  OC11CON1 = 0x964
                    0x0964                  _OC11CON1 = 0x964
                    0x0964                  _OC11CON1bits = 0x964
                    0x0966                  OC11CON2 = 0x966
                    0x0966                  _OC11CON2 = 0x966
                    0x0966                  _OC11CON2bits = 0x966
                    0x0968                  OC11RS = 0x968
                    0x0968                  _OC11RS = 0x968
                    0x096a                  OC11R = 0x96a
                    0x096a                  _OC11R = 0x96a
                    0x096c                  OC11TMR = 0x96c
                    0x096c                  _OC11TMR = 0x96c
                    0x096e                  OC12CON1 = 0x96e
                    0x096e                  _OC12CON1 = 0x96e
                    0x096e                  _OC12CON1bits = 0x96e
                    0x0970                  OC12CON2 = 0x970
                    0x0970                  _OC12CON2 = 0x970
                    0x0970                  _OC12CON2bits = 0x970
                    0x0972                  OC12RS = 0x972
                    0x0972                  _OC12RS = 0x972
                    0x0974                  OC12R = 0x974
                    0x0974                  _OC12R = 0x974
                    0x0976                  OC12TMR = 0x976
                    0x0976                  _OC12TMR = 0x976
                    0x0978                  OC13CON1 = 0x978
                    0x0978                  _OC13CON1 = 0x978
                    0x0978                  _OC13CON1bits = 0x978
                    0x097a                  OC13CON2 = 0x97a
                    0x097a                  _OC13CON2 = 0x97a
                    0x097a                  _OC13CON2bits = 0x97a
                    0x097c                  OC13RS = 0x97c
                    0x097c                  _OC13RS = 0x97c
                    0x097e                  OC13R = 0x97e
                    0x097e                  _OC13R = 0x97e
                    0x0980                  OC13TMR = 0x980
                    0x0980                  _OC13TMR = 0x980
                    0x0982                  OC14CON1 = 0x982
                    0x0982                  _OC14CON1 = 0x982
                    0x0982                  _OC14CON1bits = 0x982
                    0x0984                  OC14CON2 = 0x984
                    0x0984                  _OC14CON2 = 0x984
                    0x0984                  _OC14CON2bits = 0x984
                    0x0986                  OC14RS = 0x986
                    0x0986                  _OC14RS = 0x986
                    0x0988                  OC14R = 0x988
                    0x0988                  _OC14R = 0x988
                    0x098a                  OC14TMR = 0x98a
                    0x098a                  _OC14TMR = 0x98a
                    0x098c                  OC15CON1 = 0x98c
                    0x098c                  _OC15CON1 = 0x98c
                    0x098c                  _OC15CON1bits = 0x98c
                    0x098e                  OC15CON2 = 0x98e
                    0x098e                  _OC15CON2 = 0x98e
                    0x098e                  _OC15CON2bits = 0x98e
                    0x0990                  OC15RS = 0x990
                    0x0990                  _OC15RS = 0x990
                    0x0992                  OC15R = 0x992
                    0x0992                  _OC15R = 0x992
                    0x0994                  OC15TMR = 0x994
                    0x0994                  _OC15TMR = 0x994
                    0x0996                  OC16CON1 = 0x996
                    0x0996                  _OC16CON1 = 0x996
                    0x0996                  _OC16CON1bits = 0x996
                    0x0998                  OC16CON2 = 0x998
                    0x0998                  _OC16CON2 = 0x998
                    0x0998                  _OC16CON2bits = 0x998
                    0x099a                  OC16RS = 0x99a
                    0x099a                  _OC16RS = 0x99a
                    0x099c                  OC16R = 0x99c
                    0x099c                  _OC16R = 0x99c
                    0x099e                  OC16TMR = 0x99e
                    0x099e                  _OC16TMR = 0x99e
                    0x0a80                  CMSTAT = 0xa80
                    0x0a80                  _CMSTAT = 0xa80
                    0x0a80                  _CMSTATbits = 0xa80
                    0x0a82                  CVRCON = 0xa82
                    0x0a82                  _CVRCON = 0xa82
                    0x0a82                  _CVRCONbits = 0xa82
                    0x0a84                  CM1CON = 0xa84
                    0x0a84                  _CM1CON = 0xa84
                    0x0a84                  _CM1CONbits = 0xa84
                    0x0a86                  CM1MSKSRC = 0xa86
                    0x0a86                  _CM1MSKSRC = 0xa86
                    0x0a86                  _CM1MSKSRCbits = 0xa86
                    0x0a88                  CM1MSKCON = 0xa88
                    0x0a88                  _CM1MSKCON = 0xa88
                    0x0a88                  _CM1MSKCONbits = 0xa88
                    0x0a8a                  CM1FLTR = 0xa8a
                    0x0a8a                  _CM1FLTR = 0xa8a
                    0x0a8a                  _CM1FLTRbits = 0xa8a
                    0x0a8c                  CM2CON = 0xa8c
                    0x0a8c                  _CM2CON = 0xa8c
                    0x0a8c                  _CM2CONbits = 0xa8c
                    0x0a8e                  CM2MSKSRC = 0xa8e
                    0x0a8e                  _CM2MSKSRC = 0xa8e
                    0x0a8e                  _CM2MSKSRCbits = 0xa8e
                    0x0a90                  CM2MSKCON = 0xa90
                    0x0a90                  _CM2MSKCON = 0xa90
                    0x0a90                  _CM2MSKCONbits = 0xa90
                    0x0a92                  CM2FLTR = 0xa92
                    0x0a92                  _CM2FLTR = 0xa92
                    0x0a92                  _CM2FLTRbits = 0xa92
                    0x0a94                  CM3CON = 0xa94
                    0x0a94                  _CM3CON = 0xa94
                    0x0a94                  _CM3CONbits = 0xa94
                    0x0a96                  CM3MSKSRC = 0xa96
                    0x0a96                  _CM3MSKSRC = 0xa96
                    0x0a96                  _CM3MSKSRCbits = 0xa96
                    0x0a98                  CM3MSKCON = 0xa98
                    0x0a98                  _CM3MSKCON = 0xa98
                    0x0a98                  _CM3MSKCONbits = 0xa98
                    0x0a9a                  CM3FLTR = 0xa9a
                    0x0a9a                  _CM3FLTR = 0xa9a
                    0x0a9a                  _CM3FLTRbits = 0xa9a
                    0x0b00                  DMA0CON = 0xb00
                    0x0b00                  _DMA0CON = 0xb00
                    0x0b00                  _DMA0CONbits = 0xb00
                    0x0b02                  DMA0REQ = 0xb02
                    0x0b02                  _DMA0REQ = 0xb02
                    0x0b02                  _DMA0REQbits = 0xb02
                    0x0b04                  DMA0STAL = 0xb04
                    0x0b04                  _DMA0STAL = 0xb04
                    0x0b06                  DMA0STAH = 0xb06
                    0x0b06                  _DMA0STAH = 0xb06
                    0x0b06                  _DMA0STAHbits = 0xb06
                    0x0b08                  DMA0STBL = 0xb08
                    0x0b08                  _DMA0STBL = 0xb08
                    0x0b0a                  DMA0STBH = 0xb0a
                    0x0b0a                  _DMA0STBH = 0xb0a
                    0x0b0a                  _DMA0STBHbits = 0xb0a
                    0x0b0c                  DMA0PAD = 0xb0c
                    0x0b0c                  _DMA0PAD = 0xb0c
                    0x0b0e                  DMA0CNT = 0xb0e
                    0x0b0e                  _DMA0CNT = 0xb0e
                    0x0b0e                  _DMA0CNTbits = 0xb0e
                    0x0b10                  DMA1CON = 0xb10
                    0x0b10                  _DMA1CON = 0xb10
                    0x0b10                  _DMA1CONbits = 0xb10
                    0x0b12                  DMA1REQ = 0xb12
                    0x0b12                  _DMA1REQ = 0xb12
                    0x0b12                  _DMA1REQbits = 0xb12
                    0x0b14                  DMA1STAL = 0xb14
                    0x0b14                  _DMA1STAL = 0xb14
                    0x0b16                  DMA1STAH = 0xb16
                    0x0b16                  _DMA1STAH = 0xb16
                    0x0b16                  _DMA1STAHbits = 0xb16
                    0x0b18                  DMA1STBL = 0xb18
                    0x0b18                  _DMA1STBL = 0xb18
                    0x0b1a                  DMA1STBH = 0xb1a
                    0x0b1a                  _DMA1STBH = 0xb1a
                    0x0b1a                  _DMA1STBHbits = 0xb1a
                    0x0b1c                  DMA1PAD = 0xb1c
                    0x0b1c                  _DMA1PAD = 0xb1c
                    0x0b1e                  DMA1CNT = 0xb1e
                    0x0b1e                  _DMA1CNT = 0xb1e
                    0x0b1e                  _DMA1CNTbits = 0xb1e
                    0x0b20                  DMA2CON = 0xb20
                    0x0b20                  _DMA2CON = 0xb20
                    0x0b20                  _DMA2CONbits = 0xb20
                    0x0b22                  DMA2REQ = 0xb22
                    0x0b22                  _DMA2REQ = 0xb22
                    0x0b22                  _DMA2REQbits = 0xb22
                    0x0b24                  DMA2STAL = 0xb24
                    0x0b24                  _DMA2STAL = 0xb24
                    0x0b26                  DMA2STAH = 0xb26
                    0x0b26                  _DMA2STAH = 0xb26
                    0x0b26                  _DMA2STAHbits = 0xb26
                    0x0b28                  DMA2STBL = 0xb28
                    0x0b28                  _DMA2STBL = 0xb28
                    0x0b2a                  DMA2STBH = 0xb2a
                    0x0b2a                  _DMA2STBH = 0xb2a
                    0x0b2a                  _DMA2STBHbits = 0xb2a
                    0x0b2c                  DMA2PAD = 0xb2c
                    0x0b2c                  _DMA2PAD = 0xb2c
                    0x0b2e                  DMA2CNT = 0xb2e
                    0x0b2e                  _DMA2CNT = 0xb2e
                    0x0b2e                  _DMA2CNTbits = 0xb2e
                    0x0b30                  DMA3CON = 0xb30
                    0x0b30                  _DMA3CON = 0xb30
                    0x0b30                  _DMA3CONbits = 0xb30
                    0x0b32                  DMA3REQ = 0xb32
                    0x0b32                  _DMA3REQ = 0xb32
                    0x0b32                  _DMA3REQbits = 0xb32
                    0x0b34                  DMA3STAL = 0xb34
                    0x0b34                  _DMA3STAL = 0xb34
                    0x0b36                  DMA3STAH = 0xb36
                    0x0b36                  _DMA3STAH = 0xb36
                    0x0b36                  _DMA3STAHbits = 0xb36
                    0x0b38                  DMA3STBL = 0xb38
                    0x0b38                  _DMA3STBL = 0xb38
                    0x0b3a                  DMA3STBH = 0xb3a
                    0x0b3a                  _DMA3STBH = 0xb3a
                    0x0b3a                  _DMA3STBHbits = 0xb3a
                    0x0b3c                  DMA3PAD = 0xb3c
                    0x0b3c                  _DMA3PAD = 0xb3c
                    0x0b3e                  DMA3CNT = 0xb3e
                    0x0b3e                  _DMA3CNT = 0xb3e
                    0x0b3e                  _DMA3CNTbits = 0xb3e
                    0x0b40                  DMA4CON = 0xb40
                    0x0b40                  _DMA4CON = 0xb40
                    0x0b40                  _DMA4CONbits = 0xb40
                    0x0b42                  DMA4REQ = 0xb42
                    0x0b42                  _DMA4REQ = 0xb42
                    0x0b42                  _DMA4REQbits = 0xb42
                    0x0b44                  DMA4STAL = 0xb44
                    0x0b44                  _DMA4STAL = 0xb44
                    0x0b46                  DMA4STAH = 0xb46
                    0x0b46                  _DMA4STAH = 0xb46
                    0x0b46                  _DMA4STAHbits = 0xb46
                    0x0b48                  DMA4STBL = 0xb48
                    0x0b48                  _DMA4STBL = 0xb48
                    0x0b4a                  DMA4STBH = 0xb4a
                    0x0b4a                  _DMA4STBH = 0xb4a
                    0x0b4a                  _DMA4STBHbits = 0xb4a
                    0x0b4c                  DMA4PAD = 0xb4c
                    0x0b4c                  _DMA4PAD = 0xb4c
                    0x0b4e                  DMA4CNT = 0xb4e
                    0x0b4e                  _DMA4CNT = 0xb4e
                    0x0b4e                  _DMA4CNTbits = 0xb4e
                    0x0b50                  DMA5CON = 0xb50
                    0x0b50                  _DMA5CON = 0xb50
                    0x0b50                  _DMA5CONbits = 0xb50
                    0x0b52                  DMA5REQ = 0xb52
                    0x0b52                  _DMA5REQ = 0xb52
                    0x0b52                  _DMA5REQbits = 0xb52
                    0x0b54                  DMA5STAL = 0xb54
                    0x0b54                  _DMA5STAL = 0xb54
                    0x0b56                  DMA5STAH = 0xb56
                    0x0b56                  _DMA5STAH = 0xb56
                    0x0b56                  _DMA5STAHbits = 0xb56
                    0x0b58                  DMA5STBL = 0xb58
                    0x0b58                  _DMA5STBL = 0xb58
                    0x0b5a                  DMA5STBH = 0xb5a
                    0x0b5a                  _DMA5STBH = 0xb5a
                    0x0b5a                  _DMA5STBHbits = 0xb5a
                    0x0b5c                  DMA5PAD = 0xb5c
                    0x0b5c                  _DMA5PAD = 0xb5c
                    0x0b5e                  DMA5CNT = 0xb5e
                    0x0b5e                  _DMA5CNT = 0xb5e
                    0x0b5e                  _DMA5CNTbits = 0xb5e
                    0x0b60                  DMA6CON = 0xb60
                    0x0b60                  _DMA6CON = 0xb60
                    0x0b60                  _DMA6CONbits = 0xb60
                    0x0b62                  DMA6REQ = 0xb62
                    0x0b62                  _DMA6REQ = 0xb62
                    0x0b62                  _DMA6REQbits = 0xb62
                    0x0b64                  DMA6STAL = 0xb64
                    0x0b64                  _DMA6STAL = 0xb64
                    0x0b66                  DMA6STAH = 0xb66
                    0x0b66                  _DMA6STAH = 0xb66
                    0x0b66                  _DMA6STAHbits = 0xb66
                    0x0b68                  DMA6STBL = 0xb68
                    0x0b68                  _DMA6STBL = 0xb68
                    0x0b6a                  DMA6STBH = 0xb6a
                    0x0b6a                  _DMA6STBH = 0xb6a
                    0x0b6a                  _DMA6STBHbits = 0xb6a
                    0x0b6c                  DMA6PAD = 0xb6c
                    0x0b6c                  _DMA6PAD = 0xb6c
                    0x0b6e                  DMA6CNT = 0xb6e
                    0x0b6e                  _DMA6CNT = 0xb6e
                    0x0b6e                  _DMA6CNTbits = 0xb6e
                    0x0b70                  DMA7CON = 0xb70
                    0x0b70                  _DMA7CON = 0xb70
                    0x0b70                  _DMA7CONbits = 0xb70
                    0x0b72                  DMA7REQ = 0xb72
                    0x0b72                  _DMA7REQ = 0xb72
                    0x0b72                  _DMA7REQbits = 0xb72
                    0x0b74                  DMA7STAL = 0xb74
                    0x0b74                  _DMA7STAL = 0xb74
                    0x0b76                  DMA7STAH = 0xb76
                    0x0b76                  _DMA7STAH = 0xb76
                    0x0b76                  _DMA7STAHbits = 0xb76
                    0x0b78                  DMA7STBL = 0xb78
                    0x0b78                  _DMA7STBL = 0xb78
                    0x0b7a                  DMA7STBH = 0xb7a
                    0x0b7a                  _DMA7STBH = 0xb7a
                    0x0b7a                  _DMA7STBHbits = 0xb7a
                    0x0b7c                  DMA7PAD = 0xb7c
                    0x0b7c                  _DMA7PAD = 0xb7c
                    0x0b7e                  DMA7CNT = 0xb7e
                    0x0b7e                  _DMA7CNT = 0xb7e
                    0x0b7e                  _DMA7CNTbits = 0xb7e
                    0x0b80                  DMA8CON = 0xb80
                    0x0b80                  _DMA8CON = 0xb80
                    0x0b80                  _DMA8CONbits = 0xb80
                    0x0b82                  DMA8REQ = 0xb82
                    0x0b82                  _DMA8REQ = 0xb82
                    0x0b82                  _DMA8REQbits = 0xb82
                    0x0b84                  DMA8STAL = 0xb84
                    0x0b84                  _DMA8STAL = 0xb84
                    0x0b86                  DMA8STAH = 0xb86
                    0x0b86                  _DMA8STAH = 0xb86
                    0x0b86                  _DMA8STAHbits = 0xb86
                    0x0b88                  DMA8STBL = 0xb88
                    0x0b88                  _DMA8STBL = 0xb88
                    0x0b8a                  DMA8STBH = 0xb8a
                    0x0b8a                  _DMA8STBH = 0xb8a
                    0x0b8a                  _DMA8STBHbits = 0xb8a
                    0x0b8c                  DMA8PAD = 0xb8c
                    0x0b8c                  _DMA8PAD = 0xb8c
                    0x0b8e                  DMA8CNT = 0xb8e
                    0x0b8e                  _DMA8CNT = 0xb8e
                    0x0b8e                  _DMA8CNTbits = 0xb8e
                    0x0b90                  DMA9CON = 0xb90
                    0x0b90                  _DMA9CON = 0xb90
                    0x0b90                  _DMA9CONbits = 0xb90
                    0x0b92                  DMA9REQ = 0xb92
                    0x0b92                  _DMA9REQ = 0xb92
                    0x0b92                  _DMA9REQbits = 0xb92
                    0x0b94                  DMA9STAL = 0xb94
                    0x0b94                  _DMA9STAL = 0xb94
                    0x0b96                  DMA9STAH = 0xb96
                    0x0b96                  _DMA9STAH = 0xb96
                    0x0b96                  _DMA9STAHbits = 0xb96
                    0x0b98                  DMA9STBL = 0xb98
                    0x0b98                  _DMA9STBL = 0xb98
                    0x0b9a                  DMA9STBH = 0xb9a
                    0x0b9a                  _DMA9STBH = 0xb9a
                    0x0b9a                  _DMA9STBHbits = 0xb9a
                    0x0b9c                  DMA9PAD = 0xb9c
                    0x0b9c                  _DMA9PAD = 0xb9c
                    0x0b9e                  DMA9CNT = 0xb9e
                    0x0b9e                  _DMA9CNT = 0xb9e
                    0x0b9e                  _DMA9CNTbits = 0xb9e
                    0x0ba0                  DMA10CON = 0xba0
                    0x0ba0                  _DMA10CON = 0xba0
                    0x0ba0                  _DMA10CONbits = 0xba0
                    0x0ba2                  DMA10REQ = 0xba2
                    0x0ba2                  _DMA10REQ = 0xba2
                    0x0ba2                  _DMA10REQbits = 0xba2
                    0x0ba4                  DMA10STAL = 0xba4
                    0x0ba4                  _DMA10STAL = 0xba4
                    0x0ba6                  DMA10STAH = 0xba6
                    0x0ba6                  _DMA10STAH = 0xba6
                    0x0ba6                  _DMA10STAHbits = 0xba6
                    0x0ba8                  DMA10STBL = 0xba8
                    0x0ba8                  _DMA10STBL = 0xba8
                    0x0baa                  DMA10STBH = 0xbaa
                    0x0baa                  _DMA10STBH = 0xbaa
                    0x0baa                  _DMA10STBHbits = 0xbaa
                    0x0bac                  DMA10PAD = 0xbac
                    0x0bac                  _DMA10PAD = 0xbac
                    0x0bae                  DMA10CNT = 0xbae
                    0x0bae                  _DMA10CNT = 0xbae
                    0x0bae                  _DMA10CNTbits = 0xbae
                    0x0bb0                  DMA11CON = 0xbb0
                    0x0bb0                  _DMA11CON = 0xbb0
                    0x0bb0                  _DMA11CONbits = 0xbb0
                    0x0bb2                  DMA11REQ = 0xbb2
                    0x0bb2                  _DMA11REQ = 0xbb2
                    0x0bb2                  _DMA11REQbits = 0xbb2
                    0x0bb4                  DMA11STAL = 0xbb4
                    0x0bb4                  _DMA11STAL = 0xbb4
                    0x0bb6                  DMA11STAH = 0xbb6
                    0x0bb6                  _DMA11STAH = 0xbb6
                    0x0bb6                  _DMA11STAHbits = 0xbb6
                    0x0bb8                  DMA11STBL = 0xbb8
                    0x0bb8                  _DMA11STBL = 0xbb8
                    0x0bba                  DMA11STBH = 0xbba
                    0x0bba                  _DMA11STBH = 0xbba
                    0x0bba                  _DMA11STBHbits = 0xbba
                    0x0bbc                  DMA11PAD = 0xbbc
                    0x0bbc                  _DMA11PAD = 0xbbc
                    0x0bbe                  DMA11CNT = 0xbbe
                    0x0bbe                  _DMA11CNT = 0xbbe
                    0x0bbe                  _DMA11CNTbits = 0xbbe
                    0x0bc0                  DMA12CON = 0xbc0
                    0x0bc0                  _DMA12CON = 0xbc0
                    0x0bc0                  _DMA12CONbits = 0xbc0
                    0x0bc2                  DMA12REQ = 0xbc2
                    0x0bc2                  _DMA12REQ = 0xbc2
                    0x0bc2                  _DMA12REQbits = 0xbc2
                    0x0bc4                  DMA12STAL = 0xbc4
                    0x0bc4                  _DMA12STAL = 0xbc4
                    0x0bc6                  DMA12STAH = 0xbc6
                    0x0bc6                  _DMA12STAH = 0xbc6
                    0x0bc6                  _DMA12STAHbits = 0xbc6
                    0x0bc8                  DMA12STBL = 0xbc8
                    0x0bc8                  _DMA12STBL = 0xbc8
                    0x0bca                  DMA12STBH = 0xbca
                    0x0bca                  _DMA12STBH = 0xbca
                    0x0bca                  _DMA12STBHbits = 0xbca
                    0x0bcc                  DMA12PAD = 0xbcc
                    0x0bcc                  _DMA12PAD = 0xbcc
                    0x0bce                  DMA12CNT = 0xbce
                    0x0bce                  _DMA12CNT = 0xbce
                    0x0bce                  _DMA12CNTbits = 0xbce
                    0x0bd0                  DMA13CON = 0xbd0
                    0x0bd0                  _DMA13CON = 0xbd0
                    0x0bd0                  _DMA13CONbits = 0xbd0
                    0x0bd2                  DMA13REQ = 0xbd2
                    0x0bd2                  _DMA13REQ = 0xbd2
                    0x0bd2                  _DMA13REQbits = 0xbd2
                    0x0bd4                  DMA13STAL = 0xbd4
                    0x0bd4                  _DMA13STAL = 0xbd4
                    0x0bd6                  DMA13STAH = 0xbd6
                    0x0bd6                  _DMA13STAH = 0xbd6
                    0x0bd6                  _DMA13STAHbits = 0xbd6
                    0x0bd8                  DMA13STBL = 0xbd8
                    0x0bd8                  _DMA13STBL = 0xbd8
                    0x0bda                  DMA13STBH = 0xbda
                    0x0bda                  _DMA13STBH = 0xbda
                    0x0bda                  _DMA13STBHbits = 0xbda
                    0x0bdc                  DMA13PAD = 0xbdc
                    0x0bdc                  _DMA13PAD = 0xbdc
                    0x0bde                  DMA13CNT = 0xbde
                    0x0bde                  _DMA13CNT = 0xbde
                    0x0bde                  _DMA13CNTbits = 0xbde
                    0x0be0                  DMA14CON = 0xbe0
                    0x0be0                  _DMA14CON = 0xbe0
                    0x0be0                  _DMA14CONbits = 0xbe0
                    0x0be2                  DMA14REQ = 0xbe2
                    0x0be2                  _DMA14REQ = 0xbe2
                    0x0be2                  _DMA14REQbits = 0xbe2
                    0x0be4                  DMA14STAL = 0xbe4
                    0x0be4                  _DMA14STAL = 0xbe4
                    0x0be6                  DMA14STAH = 0xbe6
                    0x0be6                  _DMA14STAH = 0xbe6
                    0x0be6                  _DMA14STAHbits = 0xbe6
                    0x0be8                  DMA14STBL = 0xbe8
                    0x0be8                  _DMA14STBL = 0xbe8
                    0x0bea                  DMA14STBH = 0xbea
                    0x0bea                  _DMA14STBH = 0xbea
                    0x0bea                  _DMA14STBHbits = 0xbea
                    0x0bec                  DMA14PAD = 0xbec
                    0x0bec                  _DMA14PAD = 0xbec
                    0x0bee                  DMA14CNT = 0xbee
                    0x0bee                  _DMA14CNT = 0xbee
                    0x0bee                  _DMA14CNTbits = 0xbee
                    0x0bf0                  DMAPWC = 0xbf0
                    0x0bf0                  _DMAPWC = 0xbf0
                    0x0bf0                  _DMAPWCbits = 0xbf0
                    0x0bf2                  DMARQC = 0xbf2
                    0x0bf2                  _DMARQC = 0xbf2
                    0x0bf2                  _DMARQCbits = 0xbf2
                    0x0bf4                  DMAPPS = 0xbf4
                    0x0bf4                  _DMAPPS = 0xbf4
                    0x0bf4                  _DMAPPSbits = 0xbf4
                    0x0bf6                  DMALCA = 0xbf6
                    0x0bf6                  _DMALCA = 0xbf6
                    0x0bf6                  _DMALCAbits = 0xbf6
                    0x0bf8                  DSADRL = 0xbf8
                    0x0bf8                  _DSADRL = 0xbf8
                    0x0bfa                  DSADRH = 0xbfa
                    0x0bfa                  _DSADRH = 0xbfa
                    0x0bfa                  _DSADRHbits = 0xbfa
                    0x0c00                  PTCON = 0xc00
                    0x0c00                  _PTCON = 0xc00
                    0x0c00                  _PTCONbits = 0xc00
                    0x0c02                  PTCON2 = 0xc02
                    0x0c02                  _PTCON2 = 0xc02
                    0x0c02                  _PTCON2bits = 0xc02
                    0x0c04                  PTPER = 0xc04
                    0x0c04                  _PTPER = 0xc04
                    0x0c06                  SEVTCMP = 0xc06
                    0x0c06                  _SEVTCMP = 0xc06
                    0x0c06                  _SEVTCMPbits = 0xc06
                    0x0c0a                  MDC = 0xc0a
                    0x0c0a                  _MDC = 0xc0a
                    0x0c0e                  STCON = 0xc0e
                    0x0c0e                  _STCON = 0xc0e
                    0x0c0e                  _STCONbits = 0xc0e
                    0x0c10                  STCON2 = 0xc10
                    0x0c10                  _STCON2 = 0xc10
                    0x0c10                  _STCON2bits = 0xc10
                    0x0c12                  STPER = 0xc12
                    0x0c12                  _STPER = 0xc12
                    0x0c14                  SSEVTCMP = 0xc14
                    0x0c14                  _SSEVTCMP = 0xc14
                    0x0c14                  _SSEVTCMPbits = 0xc14
                    0x0c1a                  CHOP = 0xc1a
                    0x0c1a                  _CHOP = 0xc1a
                    0x0c1a                  _CHOPbits = 0xc1a
                    0x0c20                  PWMCON1 = 0xc20
                    0x0c20                  _PWMCON1 = 0xc20
                    0x0c20                  _PWMCON1bits = 0xc20
                    0x0c22                  IOCON1 = 0xc22
                    0x0c22                  _IOCON1 = 0xc22
                    0x0c22                  _IOCON1bits = 0xc22
                    0x0c24                  FCLCON1 = 0xc24
                    0x0c24                  _FCLCON1 = 0xc24
                    0x0c24                  _FCLCON1bits = 0xc24
                    0x0c26                  PDC1 = 0xc26
                    0x0c26                  _PDC1 = 0xc26
                    0x0c28                  PHASE1 = 0xc28
                    0x0c28                  _PHASE1 = 0xc28
                    0x0c2a                  DTR1 = 0xc2a
                    0x0c2a                  _DTR1 = 0xc2a
                    0x0c2c                  ALTDTR1 = 0xc2c
                    0x0c2c                  _ALTDTR1 = 0xc2c
                    0x0c2e                  SDC1 = 0xc2e
                    0x0c2e                  _SDC1 = 0xc2e
                    0x0c30                  SPHASE1 = 0xc30
                    0x0c30                  _SPHASE1 = 0xc30
                    0x0c32                  TRIG1 = 0xc32
                    0x0c32                  _TRIG1 = 0xc32
                    0x0c32                  _TRIG1bits = 0xc32
                    0x0c34                  TRGCON1 = 0xc34
                    0x0c34                  _TRGCON1 = 0xc34
                    0x0c34                  _TRGCON1bits = 0xc34
                    0x0c38                  PWMCAP1 = 0xc38
                    0x0c38                  _PWMCAP1 = 0xc38
                    0x0c38                  _PWMCAP1bits = 0xc38
                    0x0c3a                  LEBCON1 = 0xc3a
                    0x0c3a                  _LEBCON1 = 0xc3a
                    0x0c3a                  _LEBCON1bits = 0xc3a
                    0x0c3c                  LEBDLY1 = 0xc3c
                    0x0c3c                  _LEBDLY1 = 0xc3c
                    0x0c3c                  _LEBDLY1bits = 0xc3c
                    0x0c3e                  AUXCON1 = 0xc3e
                    0x0c3e                  _AUXCON1 = 0xc3e
                    0x0c3e                  _AUXCON1bits = 0xc3e
                    0x0c40                  PWMCON2 = 0xc40
                    0x0c40                  _PWMCON2 = 0xc40
                    0x0c40                  _PWMCON2bits = 0xc40
                    0x0c42                  IOCON2 = 0xc42
                    0x0c42                  _IOCON2 = 0xc42
                    0x0c42                  _IOCON2bits = 0xc42
                    0x0c44                  FCLCON2 = 0xc44
                    0x0c44                  _FCLCON2 = 0xc44
                    0x0c44                  _FCLCON2bits = 0xc44
                    0x0c46                  PDC2 = 0xc46
                    0x0c46                  _PDC2 = 0xc46
                    0x0c48                  PHASE2 = 0xc48
                    0x0c48                  _PHASE2 = 0xc48
                    0x0c4a                  DTR2 = 0xc4a
                    0x0c4a                  _DTR2 = 0xc4a
                    0x0c4c                  ALTDTR2 = 0xc4c
                    0x0c4c                  _ALTDTR2 = 0xc4c
                    0x0c4e                  SDC2 = 0xc4e
                    0x0c4e                  _SDC2 = 0xc4e
                    0x0c50                  SPHASE2 = 0xc50
                    0x0c50                  _SPHASE2 = 0xc50
                    0x0c52                  TRIG2 = 0xc52
                    0x0c52                  _TRIG2 = 0xc52
                    0x0c52                  _TRIG2bits = 0xc52
                    0x0c54                  TRGCON2 = 0xc54
                    0x0c54                  _TRGCON2 = 0xc54
                    0x0c54                  _TRGCON2bits = 0xc54
                    0x0c58                  PWMCAP2 = 0xc58
                    0x0c58                  _PWMCAP2 = 0xc58
                    0x0c58                  _PWMCAP2bits = 0xc58
                    0x0c5a                  LEBCON2 = 0xc5a
                    0x0c5a                  _LEBCON2 = 0xc5a
                    0x0c5a                  _LEBCON2bits = 0xc5a
                    0x0c5c                  LEBDLY2 = 0xc5c
                    0x0c5c                  _LEBDLY2 = 0xc5c
                    0x0c5c                  _LEBDLY2bits = 0xc5c
                    0x0c5e                  AUXCON2 = 0xc5e
                    0x0c5e                  _AUXCON2 = 0xc5e
                    0x0c5e                  _AUXCON2bits = 0xc5e
                    0x0c60                  PWMCON3 = 0xc60
                    0x0c60                  _PWMCON3 = 0xc60
                    0x0c60                  _PWMCON3bits = 0xc60
                    0x0c62                  IOCON3 = 0xc62
                    0x0c62                  _IOCON3 = 0xc62
                    0x0c62                  _IOCON3bits = 0xc62
                    0x0c64                  FCLCON3 = 0xc64
                    0x0c64                  _FCLCON3 = 0xc64
                    0x0c64                  _FCLCON3bits = 0xc64
                    0x0c66                  PDC3 = 0xc66
                    0x0c66                  _PDC3 = 0xc66
                    0x0c68                  PHASE3 = 0xc68
                    0x0c68                  _PHASE3 = 0xc68
                    0x0c6a                  DTR3 = 0xc6a
                    0x0c6a                  _DTR3 = 0xc6a
                    0x0c6c                  ALTDTR3 = 0xc6c
                    0x0c6c                  _ALTDTR3 = 0xc6c
                    0x0c6e                  SDC3 = 0xc6e
                    0x0c6e                  _SDC3 = 0xc6e
                    0x0c70                  SPHASE3 = 0xc70
                    0x0c70                  _SPHASE3 = 0xc70
                    0x0c72                  TRIG3 = 0xc72
                    0x0c72                  _TRIG3 = 0xc72
                    0x0c72                  _TRIG3bits = 0xc72
                    0x0c74                  TRGCON3 = 0xc74
                    0x0c74                  _TRGCON3 = 0xc74
                    0x0c74                  _TRGCON3bits = 0xc74
                    0x0c78                  PWMCAP3 = 0xc78
                    0x0c78                  _PWMCAP3 = 0xc78
                    0x0c78                  _PWMCAP3bits = 0xc78
                    0x0c7a                  LEBCON3 = 0xc7a
                    0x0c7a                  _LEBCON3 = 0xc7a
                    0x0c7a                  _LEBCON3bits = 0xc7a
                    0x0c7c                  LEBDLY3 = 0xc7c
                    0x0c7c                  _LEBDLY3 = 0xc7c
                    0x0c7c                  _LEBDLY3bits = 0xc7c
                    0x0c7e                  AUXCON3 = 0xc7e
                    0x0c7e                  _AUXCON3 = 0xc7e
                    0x0c7e                  _AUXCON3bits = 0xc7e
                    0x0c80                  PWMCON4 = 0xc80
                    0x0c80                  _PWMCON4 = 0xc80
                    0x0c80                  _PWMCON4bits = 0xc80
                    0x0c82                  IOCON4 = 0xc82
                    0x0c82                  _IOCON4 = 0xc82
                    0x0c82                  _IOCON4bits = 0xc82
                    0x0c84                  FCLCON4 = 0xc84
                    0x0c84                  _FCLCON4 = 0xc84
                    0x0c84                  _FCLCON4bits = 0xc84
                    0x0c86                  PDC4 = 0xc86
                    0x0c86                  _PDC4 = 0xc86
                    0x0c88                  PHASE4 = 0xc88
                    0x0c88                  _PHASE4 = 0xc88
                    0x0c8a                  DTR4 = 0xc8a
                    0x0c8a                  _DTR4 = 0xc8a
                    0x0c8c                  ALTDTR4 = 0xc8c
                    0x0c8c                  _ALTDTR4 = 0xc8c
                    0x0c8e                  SDC4 = 0xc8e
                    0x0c8e                  _SDC4 = 0xc8e
                    0x0c90                  SPHASE4 = 0xc90
                    0x0c90                  _SPHASE4 = 0xc90
                    0x0c92                  TRIG4 = 0xc92
                    0x0c92                  _TRIG4 = 0xc92
                    0x0c92                  _TRIG4bits = 0xc92
                    0x0c94                  TRGCON4 = 0xc94
                    0x0c94                  _TRGCON4 = 0xc94
                    0x0c94                  _TRGCON4bits = 0xc94
                    0x0c98                  PWMCAP4 = 0xc98
                    0x0c98                  _PWMCAP4 = 0xc98
                    0x0c98                  _PWMCAP4bits = 0xc98
                    0x0c9a                  LEBCON4 = 0xc9a
                    0x0c9a                  _LEBCON4 = 0xc9a
                    0x0c9a                  _LEBCON4bits = 0xc9a
                    0x0c9c                  LEBDLY4 = 0xc9c
                    0x0c9c                  _LEBDLY4 = 0xc9c
                    0x0c9c                  _LEBDLY4bits = 0xc9c
                    0x0c9e                  AUXCON4 = 0xc9e
                    0x0c9e                  _AUXCON4 = 0xc9e
                    0x0c9e                  _AUXCON4bits = 0xc9e
                    0x0ca0                  PWMCON5 = 0xca0
                    0x0ca0                  _PWMCON5 = 0xca0
                    0x0ca0                  _PWMCON5bits = 0xca0
                    0x0ca2                  IOCON5 = 0xca2
                    0x0ca2                  _IOCON5 = 0xca2
                    0x0ca2                  _IOCON5bits = 0xca2
                    0x0ca4                  FCLCON5 = 0xca4
                    0x0ca4                  _FCLCON5 = 0xca4
                    0x0ca4                  _FCLCON5bits = 0xca4
                    0x0ca6                  PDC5 = 0xca6
                    0x0ca6                  _PDC5 = 0xca6
                    0x0ca8                  PHASE5 = 0xca8
                    0x0ca8                  _PHASE5 = 0xca8
                    0x0caa                  DTR5 = 0xcaa
                    0x0caa                  _DTR5 = 0xcaa
                    0x0cac                  ALTDTR5 = 0xcac
                    0x0cac                  _ALTDTR5 = 0xcac
                    0x0cae                  SDC5 = 0xcae
                    0x0cae                  _SDC5 = 0xcae
                    0x0cb0                  SPHASE5 = 0xcb0
                    0x0cb0                  _SPHASE5 = 0xcb0
                    0x0cb2                  TRIG5 = 0xcb2
                    0x0cb2                  _TRIG5 = 0xcb2
                    0x0cb2                  _TRIG5bits = 0xcb2
                    0x0cb4                  TRGCON5 = 0xcb4
                    0x0cb4                  _TRGCON5 = 0xcb4
                    0x0cb4                  _TRGCON5bits = 0xcb4
                    0x0cb8                  PWMCAP5 = 0xcb8
                    0x0cb8                  _PWMCAP5 = 0xcb8
                    0x0cb8                  _PWMCAP5bits = 0xcb8
                    0x0cba                  LEBCON5 = 0xcba
                    0x0cba                  _LEBCON5 = 0xcba
                    0x0cba                  _LEBCON5bits = 0xcba
                    0x0cbc                  LEBDLY5 = 0xcbc
                    0x0cbc                  _LEBDLY5 = 0xcbc
                    0x0cbc                  _LEBDLY5bits = 0xcbc
                    0x0cbe                  AUXCON5 = 0xcbe
                    0x0cbe                  _AUXCON5 = 0xcbe
                    0x0cbe                  _AUXCON5bits = 0xcbe
                    0x0cc0                  PWMCON6 = 0xcc0
                    0x0cc0                  _PWMCON6 = 0xcc0
                    0x0cc0                  _PWMCON6bits = 0xcc0
                    0x0cc2                  IOCON6 = 0xcc2
                    0x0cc2                  _IOCON6 = 0xcc2
                    0x0cc2                  _IOCON6bits = 0xcc2
                    0x0cc4                  FCLCON6 = 0xcc4
                    0x0cc4                  _FCLCON6 = 0xcc4
                    0x0cc4                  _FCLCON6bits = 0xcc4
                    0x0cc6                  PDC6 = 0xcc6
                    0x0cc6                  _PDC6 = 0xcc6
                    0x0cc8                  PHASE6 = 0xcc8
                    0x0cc8                  _PHASE6 = 0xcc8
                    0x0cca                  DTR6 = 0xcca
                    0x0cca                  _DTR6 = 0xcca
                    0x0ccc                  ALTDTR6 = 0xccc
                    0x0ccc                  _ALTDTR6 = 0xccc
                    0x0cce                  SDC6 = 0xcce
                    0x0cce                  _SDC6 = 0xcce
                    0x0cd0                  SPHASE6 = 0xcd0
                    0x0cd0                  _SPHASE6 = 0xcd0
                    0x0cd2                  TRIG6 = 0xcd2
                    0x0cd2                  _TRIG6 = 0xcd2
                    0x0cd2                  _TRIG6bits = 0xcd2
                    0x0cd4                  TRGCON6 = 0xcd4
                    0x0cd4                  _TRGCON6 = 0xcd4
                    0x0cd4                  _TRGCON6bits = 0xcd4
                    0x0cd8                  PWMCAP6 = 0xcd8
                    0x0cd8                  _PWMCAP6 = 0xcd8
                    0x0cd8                  _PWMCAP6bits = 0xcd8
                    0x0cda                  LEBCON6 = 0xcda
                    0x0cda                  _LEBCON6 = 0xcda
                    0x0cda                  _LEBCON6bits = 0xcda
                    0x0cdc                  LEBDLY6 = 0xcdc
                    0x0cdc                  _LEBDLY6 = 0xcdc
                    0x0cdc                  _LEBDLY6bits = 0xcdc
                    0x0cde                  AUXCON6 = 0xcde
                    0x0cde                  _AUXCON6 = 0xcde
                    0x0cde                  _AUXCON6bits = 0xcde
                    0x0e00                  TRISA = 0xe00
                    0x0e00                  _TRISA = 0xe00
                    0x0e00                  _TRISAbits = 0xe00
                    0x0e02                  PORTA = 0xe02
                    0x0e02                  _PORTA = 0xe02
                    0x0e02                  _PORTAbits = 0xe02
                    0x0e04                  LATA = 0xe04
                    0x0e04                  _LATA = 0xe04
                    0x0e04                  _LATAbits = 0xe04
                    0x0e06                  ODCA = 0xe06
                    0x0e06                  _ODCA = 0xe06
                    0x0e06                  _ODCAbits = 0xe06
                    0x0e08                  CNENA = 0xe08
                    0x0e08                  _CNENA = 0xe08
                    0x0e08                  _CNENAbits = 0xe08
                    0x0e0a                  CNPUA = 0xe0a
                    0x0e0a                  _CNPUA = 0xe0a
                    0x0e0a                  _CNPUAbits = 0xe0a
                    0x0e0c                  CNPDA = 0xe0c
                    0x0e0c                  _CNPDA = 0xe0c
                    0x0e0c                  _CNPDAbits = 0xe0c
                    0x0e0e                  ANSELA = 0xe0e
                    0x0e0e                  _ANSELA = 0xe0e
                    0x0e0e                  _ANSELAbits = 0xe0e
                    0x0e10                  TRISB = 0xe10
                    0x0e10                  _TRISB = 0xe10
                    0x0e10                  _TRISBbits = 0xe10
                    0x0e12                  PORTB = 0xe12
                    0x0e12                  _PORTB = 0xe12
                    0x0e12                  _PORTBbits = 0xe12
                    0x0e14                  LATB = 0xe14
                    0x0e14                  _LATB = 0xe14
                    0x0e14                  _LATBbits = 0xe14
                    0x0e18                  CNENB = 0xe18
                    0x0e18                  _CNENB = 0xe18
                    0x0e18                  _CNENBbits = 0xe18
                    0x0e1a                  CNPUB = 0xe1a
                    0x0e1a                  _CNPUB = 0xe1a
                    0x0e1a                  _CNPUBbits = 0xe1a
                    0x0e1c                  CNPDB = 0xe1c
                    0x0e1c                  _CNPDB = 0xe1c
                    0x0e1c                  _CNPDBbits = 0xe1c
                    0x0e1e                  ANSELB = 0xe1e
                    0x0e1e                  _ANSELB = 0xe1e
                    0x0e1e                  _ANSELBbits = 0xe1e
                    0x0e20                  TRISC = 0xe20
                    0x0e20                  _TRISC = 0xe20
                    0x0e20                  _TRISCbits = 0xe20
                    0x0e22                  PORTC = 0xe22
                    0x0e22                  _PORTC = 0xe22
                    0x0e22                  _PORTCbits = 0xe22
                    0x0e24                  LATC = 0xe24
                    0x0e24                  _LATC = 0xe24
                    0x0e24                  _LATCbits = 0xe24
                    0x0e28                  CNENC = 0xe28
                    0x0e28                  _CNENC = 0xe28
                    0x0e28                  _CNENCbits = 0xe28
                    0x0e2a                  CNPUC = 0xe2a
                    0x0e2a                  _CNPUC = 0xe2a
                    0x0e2a                  _CNPUCbits = 0xe2a
                    0x0e2c                  CNPDC = 0xe2c
                    0x0e2c                  _CNPDC = 0xe2c
                    0x0e2c                  _CNPDCbits = 0xe2c
                    0x0e2e                  ANSELC = 0xe2e
                    0x0e2e                  _ANSELC = 0xe2e
                    0x0e2e                  _ANSELCbits = 0xe2e
                    0x0e30                  TRISD = 0xe30
                    0x0e30                  _TRISD = 0xe30
                    0x0e30                  _TRISDbits = 0xe30
                    0x0e32                  PORTD = 0xe32
                    0x0e32                  _PORTD = 0xe32
                    0x0e32                  _PORTDbits = 0xe32
                    0x0e34                  LATD = 0xe34
                    0x0e34                  _LATD = 0xe34
                    0x0e34                  _LATDbits = 0xe34
                    0x0e36                  ODCD = 0xe36
                    0x0e36                  _ODCD = 0xe36
                    0x0e36                  _ODCDbits = 0xe36
                    0x0e38                  CNEND = 0xe38
                    0x0e38                  _CNEND = 0xe38
                    0x0e38                  _CNENDbits = 0xe38
                    0x0e3a                  CNPUD = 0xe3a
                    0x0e3a                  _CNPUD = 0xe3a
                    0x0e3a                  _CNPUDbits = 0xe3a
                    0x0e3c                  CNPDD = 0xe3c
                    0x0e3c                  _CNPDD = 0xe3c
                    0x0e3c                  _CNPDDbits = 0xe3c
                    0x0e3e                  ANSELD = 0xe3e
                    0x0e3e                  _ANSELD = 0xe3e
                    0x0e3e                  _ANSELDbits = 0xe3e
                    0x0e40                  TRISE = 0xe40
                    0x0e40                  _TRISE = 0xe40
                    0x0e40                  _TRISEbits = 0xe40
                    0x0e42                  PORTE = 0xe42
                    0x0e42                  _PORTE = 0xe42
                    0x0e42                  _PORTEbits = 0xe42
                    0x0e44                  LATE = 0xe44
                    0x0e44                  _LATE = 0xe44
                    0x0e44                  _LATEbits = 0xe44
                    0x0e48                  CNENE = 0xe48
                    0x0e48                  _CNENE = 0xe48
                    0x0e48                  _CNENEbits = 0xe48
                    0x0e4a                  CNPUE = 0xe4a
                    0x0e4a                  _CNPUE = 0xe4a
                    0x0e4a                  _CNPUEbits = 0xe4a
                    0x0e4c                  CNPDE = 0xe4c
                    0x0e4c                  _CNPDE = 0xe4c
                    0x0e4c                  _CNPDEbits = 0xe4c
                    0x0e4e                  ANSELE = 0xe4e
                    0x0e4e                  _ANSELE = 0xe4e
                    0x0e4e                  _ANSELEbits = 0xe4e
                    0x0e50                  TRISF = 0xe50
                    0x0e50                  _TRISF = 0xe50
                    0x0e50                  _TRISFbits = 0xe50
                    0x0e52                  PORTF = 0xe52
                    0x0e52                  _PORTF = 0xe52
                    0x0e52                  _PORTFbits = 0xe52
                    0x0e54                  LATF = 0xe54
                    0x0e54                  _LATF = 0xe54
                    0x0e54                  _LATFbits = 0xe54
                    0x0e56                  ODCF = 0xe56
                    0x0e56                  _ODCF = 0xe56
                    0x0e56                  _ODCFbits = 0xe56
                    0x0e58                  CNENF = 0xe58
                    0x0e58                  _CNENF = 0xe58
                    0x0e58                  _CNENFbits = 0xe58
                    0x0e5a                  CNPUF = 0xe5a
                    0x0e5a                  _CNPUF = 0xe5a
                    0x0e5a                  _CNPUFbits = 0xe5a
                    0x0e5c                  CNPDF = 0xe5c
                    0x0e5c                  _CNPDF = 0xe5c
                    0x0e5c                  _CNPDFbits = 0xe5c
                    0x0e60                  TRISG = 0xe60
                    0x0e60                  _TRISG = 0xe60
                    0x0e60                  _TRISGbits = 0xe60
                    0x0e62                  PORTG = 0xe62
                    0x0e62                  _PORTG = 0xe62
                    0x0e62                  _PORTGbits = 0xe62
                    0x0e64                  LATG = 0xe64
                    0x0e64                  _LATG = 0xe64
                    0x0e64                  _LATGbits = 0xe64
                    0x0e66                  ODCG = 0xe66
                    0x0e66                  _ODCG = 0xe66
                    0x0e66                  _ODCGbits = 0xe66
                    0x0e68                  CNENG = 0xe68
                    0x0e68                  _CNENG = 0xe68
                    0x0e68                  _CNENGbits = 0xe68
                    0x0e6a                  CNPUG = 0xe6a
                    0x0e6a                  _CNPUG = 0xe6a
                    0x0e6a                  _CNPUGbits = 0xe6a
                    0x0e6c                  CNPDG = 0xe6c
                    0x0e6c                  _CNPDG = 0xe6c
                    0x0e6c                  _CNPDGbits = 0xe6c
                    0x0e6e                  ANSELG = 0xe6e
                    0x0e6e                  _ANSELG = 0xe6e
                    0x0e6e                  _ANSELGbits = 0xe6e
                    0x0efe                  PADCFG1 = 0xefe
                    0x0efe                  _PADCFG1 = 0xefe
                    0x0efe                  _PADCFG1bits = 0xefe
                    0x0022                  ACCA = 0x22
                    0x0022                  _ACCA = 0x22
                    0x0028                  ACCB = 0x28
                    0x0028                  _ACCB = 0x28
                    0x0440                  CAN1 = 0x440
                    0x0440                  _CAN1 = 0x440
                    0x0540                  CAN2 = 0x540
                    0x0540                  _CAN2 = 0x540
                    0x0144                  IC1 = 0x144
                    0x0144                  _IC1 = 0x144
                    0x014c                  IC2 = 0x14c
                    0x014c                  _IC2 = 0x14c
                    0x0154                  IC3 = 0x154
                    0x0154                  _IC3 = 0x154
                    0x015c                  IC4 = 0x15c
                    0x015c                  _IC4 = 0x15c
                    0x0164                  IC5 = 0x164
                    0x0164                  _IC5 = 0x164
                    0x016c                  IC6 = 0x16c
                    0x016c                  _IC6 = 0x16c
                    0x0174                  IC7 = 0x174
                    0x0174                  _IC7 = 0x174
                    0x017c                  IC8 = 0x17c
                    0x017c                  _IC8 = 0x17c
                    0x0904                  OC1 = 0x904
                    0x0904                  _OC1 = 0x904
                    0x090e                  OC2 = 0x90e
                    0x090e                  _OC2 = 0x90e
                    0x0918                  OC3 = 0x918
                    0x0918                  _OC3 = 0x918
                    0x0922                  OC4 = 0x922
                    0x0922                  _OC4 = 0x922
                    0x092c                  OC5 = 0x92c
                    0x092c                  _OC5 = 0x92c
                    0x0936                  OC6 = 0x936
                    0x0936                  _OC6 = 0x936
                    0x0940                  OC7 = 0x940
                    0x0940                  _OC7 = 0x940
                    0x094a                  OC8 = 0x94a
                    0x094a                  _OC8 = 0x94a
                    0x0240                  SPI1 = 0x240
                    0x0240                  _SPI1 = 0x240
                    0x0260                  SPI2 = 0x260
                    0x0260                  _SPI2 = 0x260
                    0x0220                  UART1 = 0x220
                    0x0220                  _UART1 = 0x220
                    0x0230                  UART2 = 0x230
                    0x0230                  _UART2 = 0x230
START GROUP
LOAD c:/program files (x86)/microchip/xc16/v1.24/bin/bin/../../lib\libpic30-elf.a
LOAD c:/program files (x86)/microchip/xc16/v1.24/bin/bin/../../lib\libm-elf.a
LOAD c:/program files (x86)/microchip/xc16/v1.24/bin/bin/../../lib\libc-elf.a
END GROUP
OUTPUT(dist/XC16_dsPIC33EP512MU810/debug/PLCD_P01V45.debug.elf elf32-pic30)
LOAD jump_table
LOAD data_init

.debug_pubtypes
                  0x000590       0x4504
 .debug_pubtypes
                  0x000590         0x12 build/XC16_dsPIC33EP512MU810/debug/B40/par/abcc_handler_par.o
 .debug_pubtypes
                  0x0005a2         0x12 build/XC16_dsPIC33EP512MU810/debug/B40/par/abcc_par_drv.o
 .debug_pubtypes
                  0x0005b4         0x32 build/XC16_dsPIC33EP512MU810/debug/B40/spi/abcc_crc32.o
 .debug_pubtypes
                  0x0005e6         0xcf build/XC16_dsPIC33EP512MU810/debug/B40/spi/abcc_handler_spi.o
 .debug_pubtypes
                  0x0006b5        0x206 build/XC16_dsPIC33EP512MU810/debug/B40/spi/abcc_spi_drv.o
 .debug_pubtypes
                  0x0008bb        0x2ba build/XC16_dsPIC33EP512MU810/debug/B40/abcc_cbf.o
 .debug_pubtypes
                  0x000b75         0x8e build/XC16_dsPIC33EP512MU810/debug/B40/abcc_debug_err.o
 .debug_pubtypes
                  0x000c03        0x1f7 build/XC16_dsPIC33EP512MU810/debug/B40/abcc_handler.o
 .debug_pubtypes
                  0x000dfa        0x1a7 build/XC16_dsPIC33EP512MU810/debug/B40/abcc_link.o
 .debug_pubtypes
                  0x000fa1         0x3f build/XC16_dsPIC33EP512MU810/debug/B40/abcc_mem.o
 .debug_pubtypes
                  0x000fe0         0x8a build/XC16_dsPIC33EP512MU810/debug/B40/abcc_remap.o
 .debug_pubtypes
                  0x00106a        0x359 build/XC16_dsPIC33EP512MU810/debug/B40/abcc_setup.o
 .debug_pubtypes
                  0x0013c3        0x142 build/XC16_dsPIC33EP512MU810/debug/B40/abcc_sys_adapt.o
 .debug_pubtypes
                  0x001505        0x12b build/XC16_dsPIC33EP512MU810/debug/B40/abcc_timer.o
 .debug_pubtypes
                  0x001630        0x315 build/XC16_dsPIC33EP512MU810/debug/B40/ad_obj.o
 .debug_pubtypes
                  0x001945        0x11c build/XC16_dsPIC33EP512MU810/debug/B40/app_obj.o
 .debug_pubtypes
                  0x001a61        0x100 build/XC16_dsPIC33EP512MU810/debug/B40/dpv1.o
 .debug_pubtypes
                  0x001b61        0x1e8 build/XC16_dsPIC33EP512MU810/debug/B40/user_adi.o
 .debug_pubtypes
                  0x001d49         0x8e build/XC16_dsPIC33EP512MU810/debug/B40/user_setup.o
 .debug_pubtypes
                  0x001dd7        0x224 build/XC16_dsPIC33EP512MU810/debug/ECAN/ECAN1Drv.o
 .debug_pubtypes
                  0x001ffb         0x9c build/XC16_dsPIC33EP512MU810/debug/BerkeleyTCPClient.o
 .debug_pubtypes
                  0x002097         0x62 build/XC16_dsPIC33EP512MU810/debug/BerkeleyTCPServer.o
 .debug_pubtypes
                  0x0020f9         0x9f build/XC16_dsPIC33EP512MU810/debug/BerkeleyUDPClient.o
 .debug_pubtypes
                  0x002198         0x53 build/XC16_dsPIC33EP512MU810/debug/MODBUSTCPServer.o
 .debug_pubtypes
                  0x0021eb         0x33 build/XC16_dsPIC33EP512MU810/debug/Regul.o
 .debug_pubtypes
                  0x00221e         0x33 build/XC16_dsPIC33EP512MU810/debug/Pesage.o
 .debug_pubtypes
                  0x002251        0x1d0 build/XC16_dsPIC33EP512MU810/debug/Process.o
 .debug_pubtypes
                  0x002421         0xc5 build/XC16_dsPIC33EP512MU810/debug/TCPIPStack/Announce.o
 .debug_pubtypes
                  0x0024e6         0x12 build/XC16_dsPIC33EP512MU810/debug/TCPIPStack/ARCFOUR.o
 .debug_pubtypes
                  0x0024f8         0xa9 build/XC16_dsPIC33EP512MU810/debug/TCPIPStack/ARP.o
 .debug_pubtypes
                  0x0025a1         0x12 build/XC16_dsPIC33EP512MU810/debug/TCPIPStack/AutoIP.o
 .debug_pubtypes
                  0x0025b3        0x146 build/XC16_dsPIC33EP512MU810/debug/TCPIPStack/BerkeleyAPI.o
 .debug_pubtypes
                  0x0026f9         0x12 build/XC16_dsPIC33EP512MU810/debug/TCPIPStack/BigInt.o
 .debug_pubtypes
                  0x00270b         0x25 build/XC16_dsPIC33EP512MU810/debug/TCPIPStack/Delay.o
 .debug_pubtypes
                  0x002730         0x12 build/XC16_dsPIC33EP512MU810/debug/TCPIPStack/DHCP.o
 .debug_pubtypes
                  0x002742         0x12 build/XC16_dsPIC33EP512MU810/debug/TCPIPStack/DHCPs.o
 .debug_pubtypes
                  0x002754         0xd8 build/XC16_dsPIC33EP512MU810/debug/TCPIPStack/DNS.o
 .debug_pubtypes
                  0x00282c         0x12 build/XC16_dsPIC33EP512MU810/debug/TCPIPStack/DNSs.o
 .debug_pubtypes
                  0x00283e         0x12 build/XC16_dsPIC33EP512MU810/debug/TCPIPStack/DynDNS.o
 .debug_pubtypes
                  0x002850        0x166 build/XC16_dsPIC33EP512MU810/debug/TCPIPStack/ENC28J60.o
 .debug_pubtypes
                  0x0029b6         0x12 build/XC16_dsPIC33EP512MU810/debug/TCPIPStack/FileSystem.o
 .debug_pubtypes
                  0x0029c8         0x12 build/XC16_dsPIC33EP512MU810/debug/TCPIPStack/FTP.o
 .debug_pubtypes
                  0x0029da         0x12 build/XC16_dsPIC33EP512MU810/debug/TCPIPStack/Hashes.o
 .debug_pubtypes
                  0x0029ec         0x90 build/XC16_dsPIC33EP512MU810/debug/TCPIPStack/Helpers.o
 .debug_pubtypes
                  0x002a7c         0xef build/XC16_dsPIC33EP512MU810/debug/TCPIPStack/HTTP2.o
 .debug_pubtypes
                  0x002b6b         0x9a build/XC16_dsPIC33EP512MU810/debug/TCPIPStack/ICMP.o
 .debug_pubtypes
                  0x002c05         0xb7 build/XC16_dsPIC33EP512MU810/debug/TCPIPStack/IP.o
 .debug_pubtypes
                  0x002cbc         0x12 build/XC16_dsPIC33EP512MU810/debug/TCPIPStack/LCDBlocking.o
 .debug_pubtypes
                  0x002cce         0xae build/XC16_dsPIC33EP512MU810/debug/TCPIPStack/MPFS2.o
 .debug_pubtypes
                  0x002d7c         0xe6 build/XC16_dsPIC33EP512MU810/debug/TCPIPStack/NBNS.o
 .debug_pubtypes
                  0x002e62         0x12 build/XC16_dsPIC33EP512MU810/debug/TCPIPStack/Random.o
 .debug_pubtypes
                  0x002e74         0xb3 build/XC16_dsPIC33EP512MU810/debug/TCPIPStack/Reboot.o
 .debug_pubtypes
                  0x002f27         0x12 build/XC16_dsPIC33EP512MU810/debug/TCPIPStack/RSA.o
 .debug_pubtypes
                  0x002f39         0x12 build/XC16_dsPIC33EP512MU810/debug/TCPIPStack/SMTP.o
 .debug_pubtypes
                  0x002f4b         0x12 build/XC16_dsPIC33EP512MU810/debug/TCPIPStack/SNMP.o
 .debug_pubtypes
                  0x002f5d         0x12 build/XC16_dsPIC33EP512MU810/debug/TCPIPStack/SNMPv3.o
 .debug_pubtypes
                  0x002f6f         0x12 build/XC16_dsPIC33EP512MU810/debug/TCPIPStack/SNMPv3USM.o
 .debug_pubtypes
                  0x002f81         0x12 build/XC16_dsPIC33EP512MU810/debug/TCPIPStack/SNTP.o
 .debug_pubtypes
                  0x002f93         0xf8 build/XC16_dsPIC33EP512MU810/debug/TCPIPStack/SPIEEPROM.o
 .debug_pubtypes
                  0x00308b         0x12 build/XC16_dsPIC33EP512MU810/debug/TCPIPStack/SPIFlash.o
 .debug_pubtypes
                  0x00309d         0x12 build/XC16_dsPIC33EP512MU810/debug/TCPIPStack/SPIRAM.o
 .debug_pubtypes
                  0x0030af         0x12 build/XC16_dsPIC33EP512MU810/debug/TCPIPStack/SSL.o
 .debug_pubtypes
                  0x0030c1         0xa7 build/XC16_dsPIC33EP512MU810/debug/TCPIPStack/StackTsk.o
 .debug_pubtypes
                  0x003168        0x14f build/XC16_dsPIC33EP512MU810/debug/TCPIPStack/TCP.o
 .debug_pubtypes
                  0x0032b7         0x12 build/XC16_dsPIC33EP512MU810/debug/TCPIPStack/TCPPerformanceTest.o
 .debug_pubtypes
                  0x0032c9         0x12 build/XC16_dsPIC33EP512MU810/debug/TCPIPStack/Telnet.o
 .debug_pubtypes
                  0x0032db         0x12 build/XC16_dsPIC33EP512MU810/debug/TCPIPStack/TFTPc.o
 .debug_pubtypes
                  0x0032ed         0xb1 build/XC16_dsPIC33EP512MU810/debug/TCPIPStack/Tick.o
 .debug_pubtypes
                  0x00339e         0x12 build/XC16_dsPIC33EP512MU810/debug/TCPIPStack/UART.o
 .debug_pubtypes
                  0x0033b0         0x12 build/XC16_dsPIC33EP512MU810/debug/TCPIPStack/UART2TCPBridge.o
 .debug_pubtypes
                  0x0033c2        0x116 build/XC16_dsPIC33EP512MU810/debug/TCPIPStack/UDP.o
 .debug_pubtypes
                  0x0034d8         0x12 build/XC16_dsPIC33EP512MU810/debug/TCPIPStack/UDPPerformanceTest.o
 .debug_pubtypes
                  0x0034ea         0x12 build/XC16_dsPIC33EP512MU810/debug/TCPIPStack/ZeroconfHelper.o
 .debug_pubtypes
                  0x0034fc         0x12 build/XC16_dsPIC33EP512MU810/debug/TCPIPStack/ZeroconfLinkLocal.o
 .debug_pubtypes
                  0x00350e         0x12 build/XC16_dsPIC33EP512MU810/debug/TCPIPStack/ZeroconfMulticastDNS.o
 .debug_pubtypes
                  0x003520        0x295 build/XC16_dsPIC33EP512MU810/debug/usb/src/usb_device.o
 .debug_pubtypes
                  0x0037b5        0x15f build/XC16_dsPIC33EP512MU810/debug/usb/src/usb_device_cdc.o
 .debug_pubtypes
                  0x003914         0x6f build/XC16_dsPIC33EP512MU810/debug/usb/src/usb_hal_dspic33e.o
 .debug_pubtypes
                  0x003983         0x12 build/XC16_dsPIC33EP512MU810/debug/configuration_bits.o
 .debug_pubtypes
                  0x003995        0x17b build/XC16_dsPIC33EP512MU810/debug/interrupts.o
 .debug_pubtypes
                  0x003b10        0x685 build/XC16_dsPIC33EP512MU810/debug/main.o
 .debug_pubtypes
                  0x004195         0x96 build/XC16_dsPIC33EP512MU810/debug/system.o
 .debug_pubtypes
                  0x00422b         0x35 build/XC16_dsPIC33EP512MU810/debug/traps.o
 .debug_pubtypes
                  0x004260        0x1ed build/XC16_dsPIC33EP512MU810/debug/user.o
 .debug_pubtypes
                  0x00444d        0x146 build/XC16_dsPIC33EP512MU810/debug/CustomHTTPApp.o
 .debug_pubtypes
                  0x004593         0x90 build/XC16_dsPIC33EP512MU810/debug/AD7190.o
 .debug_pubtypes
                  0x004623         0x56 build/XC16_dsPIC33EP512MU810/debug/ADComm.o
 .debug_pubtypes
                  0x004679         0x85 build/XC16_dsPIC33EP512MU810/debug/UARTsComm.o
 .debug_pubtypes
                  0x0046fe         0x65 build/XC16_dsPIC33EP512MU810/debug/MemFlash.o
 .debug_pubtypes
                  0x004763        0x146 build/XC16_dsPIC33EP512MU810/debug/ADC10bitsDrv.o
 .debug_pubtypes
                  0x0048a9         0xca build/XC16_dsPIC33EP512MU810/debug/SPIFRAM.o
 .debug_pubtypes
                  0x004973         0x60 build/XC16_dsPIC33EP512MU810/debug/usb_descriptors.o
 .debug_pubtypes
                  0x0049d3         0xc1 build/XC16_dsPIC33EP512MU810/debug/ModbusUartServer.o

__c30_signature
                  0x004a94        0x4bc
 __c30_signature
                  0x004a94          0x6 build/XC16_dsPIC33EP512MU810/debug/B40/par/abcc_handler_par.o
 __c30_signature
                  0x004a9a          0x6 build/XC16_dsPIC33EP512MU810/debug/B40/par/abcc_par_drv.o
 __c30_signature
                  0x004aa0          0x6 build/XC16_dsPIC33EP512MU810/debug/B40/spi/abcc_crc32.o
 __c30_signature
                  0x004aa6          0x6 build/XC16_dsPIC33EP512MU810/debug/B40/spi/abcc_handler_spi.o
 __c30_signature
                  0x004aac          0x6 build/XC16_dsPIC33EP512MU810/debug/B40/spi/abcc_spi_drv.o
 __c30_signature
                  0x004ab2          0x6 build/XC16_dsPIC33EP512MU810/debug/B40/abcc_cbf.o
 __c30_signature
                  0x004ab8          0x6 build/XC16_dsPIC33EP512MU810/debug/B40/abcc_debug_err.o
 __c30_signature
                  0x004abe          0x6 build/XC16_dsPIC33EP512MU810/debug/B40/abcc_handler.o
 __c30_signature
                  0x004ac4          0x6 build/XC16_dsPIC33EP512MU810/debug/B40/abcc_link.o
 __c30_signature
                  0x004aca          0x6 build/XC16_dsPIC33EP512MU810/debug/B40/abcc_mem.o
 __c30_signature
                  0x004ad0          0x6 build/XC16_dsPIC33EP512MU810/debug/B40/abcc_remap.o
 __c30_signature
                  0x004ad6          0x6 build/XC16_dsPIC33EP512MU810/debug/B40/abcc_setup.o
 __c30_signature
                  0x004adc          0x6 build/XC16_dsPIC33EP512MU810/debug/B40/abcc_sys_adapt.o
 __c30_signature
                  0x004ae2          0x6 build/XC16_dsPIC33EP512MU810/debug/B40/abcc_timer.o
 __c30_signature
                  0x004ae8          0x6 build/XC16_dsPIC33EP512MU810/debug/B40/ad_obj.o
 __c30_signature
                  0x004aee          0x6 build/XC16_dsPIC33EP512MU810/debug/B40/app_obj.o
 __c30_signature
                  0x004af4          0x6 build/XC16_dsPIC33EP512MU810/debug/B40/dpv1.o
 __c30_signature
                  0x004afa          0x6 build/XC16_dsPIC33EP512MU810/debug/B40/user_adi.o
 __c30_signature
                  0x004b00          0x6 build/XC16_dsPIC33EP512MU810/debug/B40/user_setup.o
 __c30_signature
                  0x004b06          0x6 build/XC16_dsPIC33EP512MU810/debug/ECAN/ECAN1Drv.o
 __c30_signature
                  0x004b0c          0x6 build/XC16_dsPIC33EP512MU810/debug/BerkeleyTCPClient.o
 __c30_signature
                  0x004b12          0x6 build/XC16_dsPIC33EP512MU810/debug/BerkeleyTCPServer.o
 __c30_signature
                  0x004b18          0x6 build/XC16_dsPIC33EP512MU810/debug/BerkeleyUDPClient.o
 __c30_signature
                  0x004b1e          0x6 build/XC16_dsPIC33EP512MU810/debug/MODBUSTCPServer.o
 __c30_signature
                  0x004b24          0x6 build/XC16_dsPIC33EP512MU810/debug/Regul.o
 __c30_signature
                  0x004b2a          0x6 build/XC16_dsPIC33EP512MU810/debug/Pesage.o
 __c30_signature
                  0x004b30          0x6 build/XC16_dsPIC33EP512MU810/debug/Process.o
 __c30_signature
                  0x004b36          0x6 build/XC16_dsPIC33EP512MU810/debug/TCPIPStack/Announce.o
 __c30_signature
                  0x004b3c          0x6 build/XC16_dsPIC33EP512MU810/debug/TCPIPStack/ARCFOUR.o
 __c30_signature
                  0x004b42          0x6 build/XC16_dsPIC33EP512MU810/debug/TCPIPStack/ARP.o
 __c30_signature
                  0x004b48          0x6 build/XC16_dsPIC33EP512MU810/debug/TCPIPStack/AutoIP.o
 __c30_signature
                  0x004b4e          0x6 build/XC16_dsPIC33EP512MU810/debug/TCPIPStack/BerkeleyAPI.o
 __c30_signature
                  0x004b54          0x6 build/XC16_dsPIC33EP512MU810/debug/TCPIPStack/BigInt.o
 __c30_signature
                  0x004b5a          0x6 build/XC16_dsPIC33EP512MU810/debug/TCPIPStack/Delay.o
 __c30_signature
                  0x004b60          0x6 build/XC16_dsPIC33EP512MU810/debug/TCPIPStack/DHCP.o
 __c30_signature
                  0x004b66          0x6 build/XC16_dsPIC33EP512MU810/debug/TCPIPStack/DHCPs.o
 __c30_signature
                  0x004b6c          0x6 build/XC16_dsPIC33EP512MU810/debug/TCPIPStack/DNS.o
 __c30_signature
                  0x004b72          0x6 build/XC16_dsPIC33EP512MU810/debug/TCPIPStack/DNSs.o
 __c30_signature
                  0x004b78          0x6 build/XC16_dsPIC33EP512MU810/debug/TCPIPStack/DynDNS.o
 __c30_signature
                  0x004b7e          0x6 build/XC16_dsPIC33EP512MU810/debug/TCPIPStack/ENC28J60.o
 __c30_signature
                  0x004b84          0x6 build/XC16_dsPIC33EP512MU810/debug/TCPIPStack/FileSystem.o
 __c30_signature
                  0x004b8a          0x6 build/XC16_dsPIC33EP512MU810/debug/TCPIPStack/FTP.o
 __c30_signature
                  0x004b90          0x6 build/XC16_dsPIC33EP512MU810/debug/TCPIPStack/Hashes.o
 __c30_signature
                  0x004b96          0x6 build/XC16_dsPIC33EP512MU810/debug/TCPIPStack/Helpers.o
 __c30_signature
                  0x004b9c          0x6 build/XC16_dsPIC33EP512MU810/debug/TCPIPStack/HTTP2.o
 __c30_signature
                  0x004ba2          0x6 build/XC16_dsPIC33EP512MU810/debug/TCPIPStack/ICMP.o
 __c30_signature
                  0x004ba8          0x6 build/XC16_dsPIC33EP512MU810/debug/TCPIPStack/IP.o
 __c30_signature
                  0x004bae          0x6 build/XC16_dsPIC33EP512MU810/debug/TCPIPStack/LCDBlocking.o
 __c30_signature
                  0x004bb4          0x6 build/XC16_dsPIC33EP512MU810/debug/TCPIPStack/MPFS2.o
 __c30_signature
                  0x004bba          0x6 build/XC16_dsPIC33EP512MU810/debug/TCPIPStack/NBNS.o
 __c30_signature
                  0x004bc0          0x6 build/XC16_dsPIC33EP512MU810/debug/TCPIPStack/Random.o
 __c30_signature
                  0x004bc6          0x6 build/XC16_dsPIC33EP512MU810/debug/TCPIPStack/Reboot.o
 __c30_signature
                  0x004bcc          0x6 build/XC16_dsPIC33EP512MU810/debug/TCPIPStack/RSA.o
 __c30_signature
                  0x004bd2          0x6 build/XC16_dsPIC33EP512MU810/debug/TCPIPStack/SMTP.o
 __c30_signature
                  0x004bd8          0x6 build/XC16_dsPIC33EP512MU810/debug/TCPIPStack/SNMP.o
 __c30_signature
                  0x004bde          0x6 build/XC16_dsPIC33EP512MU810/debug/TCPIPStack/SNMPv3.o
 __c30_signature
                  0x004be4          0x6 build/XC16_dsPIC33EP512MU810/debug/TCPIPStack/SNMPv3USM.o
 __c30_signature
                  0x004bea          0x6 build/XC16_dsPIC33EP512MU810/debug/TCPIPStack/SNTP.o
 __c30_signature
                  0x004bf0          0x6 build/XC16_dsPIC33EP512MU810/debug/TCPIPStack/SPIEEPROM.o
 __c30_signature
                  0x004bf6          0x6 build/XC16_dsPIC33EP512MU810/debug/TCPIPStack/SPIFlash.o
 __c30_signature
                  0x004bfc          0x6 build/XC16_dsPIC33EP512MU810/debug/TCPIPStack/SPIRAM.o
 __c30_signature
                  0x004c02          0x6 build/XC16_dsPIC33EP512MU810/debug/TCPIPStack/SSL.o
 __c30_signature
                  0x004c08          0x6 build/XC16_dsPIC33EP512MU810/debug/TCPIPStack/StackTsk.o
 __c30_signature
                  0x004c0e          0x6 build/XC16_dsPIC33EP512MU810/debug/TCPIPStack/TCP.o
 __c30_signature
                  0x004c14          0x6 build/XC16_dsPIC33EP512MU810/debug/TCPIPStack/TCPPerformanceTest.o
 __c30_signature
                  0x004c1a          0x6 build/XC16_dsPIC33EP512MU810/debug/TCPIPStack/Telnet.o
 __c30_signature
                  0x004c20          0x6 build/XC16_dsPIC33EP512MU810/debug/TCPIPStack/TFTPc.o
 __c30_signature
                  0x004c26          0x6 build/XC16_dsPIC33EP512MU810/debug/TCPIPStack/Tick.o
 __c30_signature
                  0x004c2c          0x6 build/XC16_dsPIC33EP512MU810/debug/TCPIPStack/UART.o
 __c30_signature
                  0x004c32          0x6 build/XC16_dsPIC33EP512MU810/debug/TCPIPStack/UART2TCPBridge.o
 __c30_signature
                  0x004c38          0x6 build/XC16_dsPIC33EP512MU810/debug/TCPIPStack/UDP.o
 __c30_signature
                  0x004c3e          0x6 build/XC16_dsPIC33EP512MU810/debug/TCPIPStack/UDPPerformanceTest.o
 __c30_signature
                  0x004c44          0x6 build/XC16_dsPIC33EP512MU810/debug/TCPIPStack/ZeroconfHelper.o
 __c30_signature
                  0x004c4a          0x6 build/XC16_dsPIC33EP512MU810/debug/TCPIPStack/ZeroconfLinkLocal.o
 __c30_signature
                  0x004c50          0x6 build/XC16_dsPIC33EP512MU810/debug/TCPIPStack/ZeroconfMulticastDNS.o
 __c30_signature
                  0x004c56          0x6 build/XC16_dsPIC33EP512MU810/debug/usb/src/usb_device.o
 __c30_signature
                  0x004c5c          0x6 build/XC16_dsPIC33EP512MU810/debug/usb/src/usb_device_cdc.o
 __c30_signature
                  0x004c62          0x6 build/XC16_dsPIC33EP512MU810/debug/usb/src/usb_hal_dspic33e.o
 __c30_signature
                  0x004c68          0x6 build/XC16_dsPIC33EP512MU810/debug/configuration_bits.o
 __c30_signature
                  0x004c6e          0x6 build/XC16_dsPIC33EP512MU810/debug/interrupts.o
 __c30_signature
                  0x004c74          0x6 build/XC16_dsPIC33EP512MU810/debug/main.o
 __c30_signature
                  0x004c7a          0x6 build/XC16_dsPIC33EP512MU810/debug/system.o
 __c30_signature
                  0x004c80          0x6 build/XC16_dsPIC33EP512MU810/debug/traps.o
 __c30_signature
                  0x004c86          0x6 build/XC16_dsPIC33EP512MU810/debug/user.o
 __c30_signature
                  0x004c8c          0x6 build/XC16_dsPIC33EP512MU810/debug/CustomHTTPApp.o
 __c30_signature
                  0x004c92          0x6 build/XC16_dsPIC33EP512MU810/debug/AD7190.o
 __c30_signature
                  0x004c98          0x6 build/XC16_dsPIC33EP512MU810/debug/ADComm.o
 __c30_signature
                  0x004c9e          0x6 build/XC16_dsPIC33EP512MU810/debug/UARTsComm.o
 __c30_signature
                  0x004ca4          0x6 build/XC16_dsPIC33EP512MU810/debug/MemFlash.o
 __c30_signature
                  0x004caa          0x6 build/XC16_dsPIC33EP512MU810/debug/ADC10bitsDrv.o
 __c30_signature
                  0x004cb0          0x6 build/XC16_dsPIC33EP512MU810/debug/SPIFRAM.o
 __c30_signature
                  0x004cb6          0x6 build/XC16_dsPIC33EP512MU810/debug/usb_descriptors.o
 __c30_signature
                  0x004cbc          0x6 build/XC16_dsPIC33EP512MU810/debug/ModbusUartServer.o
 __c30_signature
                  0x004cc2          0x6 c:/program files (x86)/microchip/xc16/v1.24/bin/bin/../../lib/dsPIC33E\libp33EP512MU810-elf.a(CloseSPI1.o)
 __c30_signature
                  0x004cc8          0x6 c:/program files (x86)/microchip/xc16/v1.24/bin/bin/../../lib/dsPIC33E\libp33EP512MU810-elf.a(CloseSPI3.o)
 __c30_signature
                  0x004cce          0x6 c:/program files (x86)/microchip/xc16/v1.24/bin/bin/../../lib/dsPIC33E\libp33EP512MU810-elf.a(DataRdySPI1.o)
 __c30_signature
                  0x004cd4          0x6 c:/program files (x86)/microchip/xc16/v1.24/bin/bin/../../lib/dsPIC33E\libp33EP512MU810-elf.a(DataRdySPI3.o)
 __c30_signature
                  0x004cda          0x6 c:/program files (x86)/microchip/xc16/v1.24/bin/bin/../../lib/dsPIC33E\libp33EP512MU810-elf.a(OpenSPI1.o)
 __c30_signature
                  0x004ce0          0x6 c:/program files (x86)/microchip/xc16/v1.24/bin/bin/../../lib/dsPIC33E\libp33EP512MU810-elf.a(OpenSPI3.o)
 __c30_signature
                  0x004ce6          0x6 c:/program files (x86)/microchip/xc16/v1.24/bin/bin/../../lib/dsPIC33E\libp33EP512MU810-elf.a(ReadSPI1.o)
 __c30_signature
                  0x004cec          0x6 c:/program files (x86)/microchip/xc16/v1.24/bin/bin/../../lib/dsPIC33E\libp33EP512MU810-elf.a(ReadSPI3.o)
 __c30_signature
                  0x004cf2          0x6 c:/program files (x86)/microchip/xc16/v1.24/bin/bin/../../lib/dsPIC33E\libp33EP512MU810-elf.a(WriteSPI1.o)
 __c30_signature
                  0x004cf8          0x6 c:/program files (x86)/microchip/xc16/v1.24/bin/bin/../../lib/dsPIC33E\libp33EP512MU810-elf.a(WriteSPI3.o)
 __c30_signature
                  0x004cfe          0x6 c:/program files (x86)/microchip/xc16/v1.24/bin/bin/../../lib/dsPIC33E\libp33EP512MU810-elf.a(BusyUART2.o)
 __c30_signature
                  0x004d04          0x6 c:/program files (x86)/microchip/xc16/v1.24/bin/bin/../../lib/dsPIC33E\libp33EP512MU810-elf.a(BusyUART3.o)
 __c30_signature
                  0x004d0a          0x6 c:/program files (x86)/microchip/xc16/v1.24/bin/bin/../../lib/dsPIC33E\libp33EP512MU810-elf.a(BusyUART4.o)
 __c30_signature
                  0x004d10          0x6 c:/program files (x86)/microchip/xc16/v1.24/bin/bin/../../lib/dsPIC33E\libp33EP512MU810-elf.a(CloseUART1.o)
 __c30_signature
                  0x004d16          0x6 c:/program files (x86)/microchip/xc16/v1.24/bin/bin/../../lib/dsPIC33E\libp33EP512MU810-elf.a(CloseUART2.o)
 __c30_signature
                  0x004d1c          0x6 c:/program files (x86)/microchip/xc16/v1.24/bin/bin/../../lib/dsPIC33E\libp33EP512MU810-elf.a(CloseUART3.o)
 __c30_signature
                  0x004d22          0x6 c:/program files (x86)/microchip/xc16/v1.24/bin/bin/../../lib/dsPIC33E\libp33EP512MU810-elf.a(CloseUART4.o)
 __c30_signature
                  0x004d28          0x6 c:/program files (x86)/microchip/xc16/v1.24/bin/bin/../../lib/dsPIC33E\libp33EP512MU810-elf.a(ConfigIntUART1.o)
 __c30_signature
                  0x004d2e          0x6 c:/program files (x86)/microchip/xc16/v1.24/bin/bin/../../lib/dsPIC33E\libp33EP512MU810-elf.a(ConfigIntUART2.o)
 __c30_signature
                  0x004d34          0x6 c:/program files (x86)/microchip/xc16/v1.24/bin/bin/../../lib/dsPIC33E\libp33EP512MU810-elf.a(ConfigIntUART3.o)
 __c30_signature
                  0x004d3a          0x6 c:/program files (x86)/microchip/xc16/v1.24/bin/bin/../../lib/dsPIC33E\libp33EP512MU810-elf.a(ConfigIntUART4.o)
 __c30_signature
                  0x004d40          0x6 c:/program files (x86)/microchip/xc16/v1.24/bin/bin/../../lib/dsPIC33E\libp33EP512MU810-elf.a(DataRdyUART1.o)
 __c30_signature
                  0x004d46          0x6 c:/program files (x86)/microchip/xc16/v1.24/bin/bin/../../lib/dsPIC33E\libp33EP512MU810-elf.a(DataRdyUART2.o)
 __c30_signature
                  0x004d4c          0x6 c:/program files (x86)/microchip/xc16/v1.24/bin/bin/../../lib/dsPIC33E\libp33EP512MU810-elf.a(DataRdyUART3.o)
 __c30_signature
                  0x004d52          0x6 c:/program files (x86)/microchip/xc16/v1.24/bin/bin/../../lib/dsPIC33E\libp33EP512MU810-elf.a(DataRdyUART4.o)
 __c30_signature
                  0x004d58          0x6 c:/program files (x86)/microchip/xc16/v1.24/bin/bin/../../lib/dsPIC33E\libp33EP512MU810-elf.a(OpenUART1.o)
 __c30_signature
                  0x004d5e          0x6 c:/program files (x86)/microchip/xc16/v1.24/bin/bin/../../lib/dsPIC33E\libp33EP512MU810-elf.a(OpenUART2.o)
 __c30_signature
                  0x004d64          0x6 c:/program files (x86)/microchip/xc16/v1.24/bin/bin/../../lib/dsPIC33E\libp33EP512MU810-elf.a(OpenUART3.o)
 __c30_signature
                  0x004d6a          0x6 c:/program files (x86)/microchip/xc16/v1.24/bin/bin/../../lib/dsPIC33E\libp33EP512MU810-elf.a(OpenUART4.o)
 __c30_signature
                  0x004d70          0x6 c:/program files (x86)/microchip/xc16/v1.24/bin/bin/../../lib/dsPIC33E\libp33EP512MU810-elf.a(putsUART1.o)
 __c30_signature
                  0x004d76          0x6 c:/program files (x86)/microchip/xc16/v1.24/bin/bin/../../lib/dsPIC33E\libp33EP512MU810-elf.a(putsUART2.o)
 __c30_signature
                  0x004d7c          0x6 c:/program files (x86)/microchip/xc16/v1.24/bin/bin/../../lib/dsPIC33E\libp33EP512MU810-elf.a(putsUART3.o)
 __c30_signature
                  0x004d82          0x6 c:/program files (x86)/microchip/xc16/v1.24/bin/bin/../../lib/dsPIC33E\libp33EP512MU810-elf.a(putsUART4.o)
 __c30_signature
                  0x004d88          0x6 c:/program files (x86)/microchip/xc16/v1.24/bin/bin/../../lib/dsPIC33E\libp33EP512MU810-elf.a(ReadUART1.o)
 __c30_signature
                  0x004d8e          0x6 c:/program files (x86)/microchip/xc16/v1.24/bin/bin/../../lib/dsPIC33E\libp33EP512MU810-elf.a(ReadUART2.o)
 __c30_signature
                  0x004d94          0x6 c:/program files (x86)/microchip/xc16/v1.24/bin/bin/../../lib/dsPIC33E\libp33EP512MU810-elf.a(ReadUART3.o)
 __c30_signature
                  0x004d9a          0x6 c:/program files (x86)/microchip/xc16/v1.24/bin/bin/../../lib/dsPIC33E\libp33EP512MU810-elf.a(ReadUART4.o)
 __c30_signature
                  0x004da0          0x6 c:/program files (x86)/microchip/xc16/v1.24/bin/bin/../../lib\libpic30-elf.a(crt0_extendedep.o)
 __c30_signature
                  0x004da6          0x6 c:/program files (x86)/microchip/xc16/v1.24/bin/bin/../../lib\libpic30-elf.a(data_init_extendedep.o)
 __c30_signature
                  0x004dac          0x6 c:/program files (x86)/microchip/xc16/v1.24/bin/bin/../../lib\libm-elf.a(addsf3.epeo)
 __c30_signature
                  0x004db2          0x6 c:/program files (x86)/microchip/xc16/v1.24/bin/bin/../../lib\libm-elf.a(divsf3.epeo)
 __c30_signature
                  0x004db8          0x6 c:/program files (x86)/microchip/xc16/v1.24/bin/bin/../../lib\libm-elf.a(divsi3.epeo)
 __c30_signature
                  0x004dbe          0x6 c:/program files (x86)/microchip/xc16/v1.24/bin/bin/../../lib\libm-elf.a(feqltle.epeo)
 __c30_signature
                  0x004dc4          0x6 c:/program files (x86)/microchip/xc16/v1.24/bin/bin/../../lib\libm-elf.a(fgtge.epeo)
 __c30_signature
                  0x004dca          0x6 c:/program files (x86)/microchip/xc16/v1.24/bin/bin/../../lib\libm-elf.a(fixsfsi.epeo)
 __c30_signature
                  0x004dd0          0x6 c:/program files (x86)/microchip/xc16/v1.24/bin/bin/../../lib\libm-elf.a(fixunssfsi.epeo)
 __c30_signature
                  0x004dd6          0x6 c:/program files (x86)/microchip/xc16/v1.24/bin/bin/../../lib\libm-elf.a(floatsisf.epeo)
 __c30_signature
                  0x004ddc          0x6 c:/program files (x86)/microchip/xc16/v1.24/bin/bin/../../lib\libm-elf.a(floatunsisf.epeo)
 __c30_signature
                  0x004de2          0x6 c:/program files (x86)/microchip/xc16/v1.24/bin/bin/../../lib\libm-elf.a(fpack.epeo)
 __c30_signature
                  0x004de8          0x6 c:/program files (x86)/microchip/xc16/v1.24/bin/bin/../../lib\libm-elf.a(funpack.epeo)
 __c30_signature
                  0x004dee          0x6 c:/program files (x86)/microchip/xc16/v1.24/bin/bin/../../lib\libm-elf.a(funpack2.epeo)
 __c30_signature
                  0x004df4          0x6 c:/program files (x86)/microchip/xc16/v1.24/bin/bin/../../lib\libm-elf.a(futil.epeo)
 __c30_signature
                  0x004dfa          0x6 c:/program files (x86)/microchip/xc16/v1.24/bin/bin/../../lib\libm-elf.a(mulsf3.epeo)
 __c30_signature
                  0x004e00          0x6 c:/program files (x86)/microchip/xc16/v1.24/bin/bin/../../lib\libm-elf.a(udivsi3.epeo)
 __c30_signature
                  0x004e06          0x6 c:/program files (x86)/microchip/xc16/v1.24/bin/bin/../../lib\libm-elf.a(umodsi3.epeo)
 __c30_signature
                  0x004e0c          0x6 c:/program files (x86)/microchip/xc16/v1.24/bin/bin/../../lib\libm-elf.a(fcompare.epeo)
 __c30_signature
                  0x004e12          0x6 c:/program files (x86)/microchip/xc16/v1.24/bin/bin/../../lib\libm-elf.a(floatdisf.epeo)
 __c30_signature
                  0x004e18          0x6 c:/program files (x86)/microchip/xc16/v1.24/bin/bin/../../lib\libm-elf.a(floatundisf.epeo)
 __c30_signature
                  0x004e1e          0x6 c:/program files (x86)/microchip/xc16/v1.24/bin/bin/../../lib\libc-elf.a(atof.epeo)
 __c30_signature
                  0x004e24          0x6 c:/program files (x86)/microchip/xc16/v1.24/bin/bin/../../lib\libc-elf.a(atoi.epeo)
 __c30_signature
                  0x004e2a          0x6 c:/program files (x86)/microchip/xc16/v1.24/bin/bin/../../lib\libc-elf.a(atol.epeo)
 __c30_signature
                  0x004e30          0x6 c:/program files (x86)/microchip/xc16/v1.24/bin/bin/../../lib\libc-elf.a(errno.epeo)
 __c30_signature
                  0x004e36          0x6 c:/program files (x86)/microchip/xc16/v1.24/bin/bin/../../lib\libc-elf.a(ltoa.epeo)
 __c30_signature
                  0x004e3c          0x6 c:/program files (x86)/microchip/xc16/v1.24/bin/bin/../../lib\libc-elf.a(memcmp.epeo)
 __c30_signature
                  0x004e42          0x6 c:/program files (x86)/microchip/xc16/v1.24/bin/bin/../../lib\libc-elf.a(memcpy.epeo)
 __c30_signature
                  0x004e48          0x6 c:/program files (x86)/microchip/xc16/v1.24/bin/bin/../../lib\libc-elf.a(memset.epeo)
 __c30_signature
                  0x004e4e          0x6 c:/program files (x86)/microchip/xc16/v1.24/bin/bin/../../lib\libc-elf.a(rand.epeo)
 __c30_signature
                  0x004e54          0x6 c:/program files (x86)/microchip/xc16/v1.24/bin/bin/../../lib\libc-elf.a(sprintf.epeo)
 __c30_signature
                  0x004e5a          0x6 c:/program files (x86)/microchip/xc16/v1.24/bin/bin/../../lib\libc-elf.a(strcmp.epeo)
 __c30_signature
                  0x004e60          0x6 c:/program files (x86)/microchip/xc16/v1.24/bin/bin/../../lib\libc-elf.a(strcpy.epeo)
 __c30_signature
                  0x004e66          0x6 c:/program files (x86)/microchip/xc16/v1.24/bin/bin/../../lib\libc-elf.a(strlen.epeo)
 __c30_signature
                  0x004e6c          0x6 c:/program files (x86)/microchip/xc16/v1.24/bin/bin/../../lib\libc-elf.a(strncpy.epeo)
 __c30_signature
                  0x004e72          0x6 c:/program files (x86)/microchip/xc16/v1.24/bin/bin/../../lib\libc-elf.a(strtok.epeo)
 __c30_signature
                  0x004e78          0x6 c:/program files (x86)/microchip/xc16/v1.24/bin/bin/../../lib\libc-elf.a(putchar.epeo)
 __c30_signature
                  0x004e7e          0x6 c:/program files (x86)/microchip/xc16/v1.24/bin/bin/../../lib\libc-elf.a(_iob.epeo)
 __c30_signature
                  0x004e84          0x6 c:/program files (x86)/microchip/xc16/v1.24/bin/bin/../../lib\libc-elf.a(sprintf_cdfFnopsuxX.EPeo)
 __c30_signature
                  0x004e8a          0x6 c:/program files (x86)/microchip/xc16/v1.24/bin/bin/../../lib\libc-elf.a(doprnt_cdfFnopsuxX.EPeo)
 __c30_signature
                  0x004e90          0x6 c:/program files (x86)/microchip/xc16/v1.24/bin/bin/../../lib\libc-elf.a(printf_cdnopsuxX.EPeo)
 __c30_signature
                  0x004e96          0x6 c:/program files (x86)/microchip/xc16/v1.24/bin/bin/../../lib\libc-elf.a(doprnt.epeo)
 __c30_signature
                  0x004e9c          0x6 c:/program files (x86)/microchip/xc16/v1.24/bin/bin/../../lib\libc-elf.a(fputc.epeo)
 __c30_signature
                  0x004ea2          0x6 c:/program files (x86)/microchip/xc16/v1.24/bin/bin/../../lib\libc-elf.a(powers.epeo)
 __c30_signature
                  0x004ea8          0x6 c:/program files (x86)/microchip/xc16/v1.24/bin/bin/../../lib\libc-elf.a(strcspn.epeo)
 __c30_signature
                  0x004eae          0x6 c:/program files (x86)/microchip/xc16/v1.24/bin/bin/../../lib\libc-elf.a(strspn.epeo)
 __c30_signature
                  0x004eb4          0x6 c:/program files (x86)/microchip/xc16/v1.24/bin/bin/../../lib\libc-elf.a(strchr.epelo)
 __c30_signature
                  0x004eba          0x6 c:/program files (x86)/microchip/xc16/v1.24/bin/bin/../../lib\libc-elf.a(flsbuf.epeo)
 __c30_signature
                  0x004ec0          0x6 c:/program files (x86)/microchip/xc16/v1.24/bin/bin/../../lib\libpic30-elf.a(writeep.eo)
 __c30_signature
                  0x004ec6          0x6 c:/program files (x86)/microchip/xc16/v1.24/bin/bin/../../lib\libm-elf.a(adddf3.epeo)
 __c30_signature
                  0x004ecc          0x6 c:/program files (x86)/microchip/xc16/v1.24/bin/bin/../../lib\libm-elf.a(deqltle.epeo)
 __c30_signature
                  0x004ed2          0x6 c:/program files (x86)/microchip/xc16/v1.24/bin/bin/../../lib\libm-elf.a(dgtge.epeo)
 __c30_signature
                  0x004ed8          0x6 c:/program files (x86)/microchip/xc16/v1.24/bin/bin/../../lib\libm-elf.a(divdf3.epeo)
 __c30_signature
                  0x004ede          0x6 c:/program files (x86)/microchip/xc16/v1.24/bin/bin/../../lib\libm-elf.a(dne.epeo)
 __c30_signature
                  0x004ee4          0x6 c:/program files (x86)/microchip/xc16/v1.24/bin/bin/../../lib\libm-elf.a(dpack.epeo)
 __c30_signature
                  0x004eea          0x6 c:/program files (x86)/microchip/xc16/v1.24/bin/bin/../../lib\libm-elf.a(dunpack2.epeo)
 __c30_signature
                  0x004ef0          0x6 c:/program files (x86)/microchip/xc16/v1.24/bin/bin/../../lib\libm-elf.a(extendsfdf.epeo)
 __c30_signature
                  0x004ef6          0x6 c:/program files (x86)/microchip/xc16/v1.24/bin/bin/../../lib\libm-elf.a(fixunsdfdi.epeo)
 __c30_signature
                  0x004efc          0x6 c:/program files (x86)/microchip/xc16/v1.24/bin/bin/../../lib\libm-elf.a(fixunsdfsi.epeo)
 __c30_signature
                  0x004f02          0x6 c:/program files (x86)/microchip/xc16/v1.24/bin/bin/../../lib\libm-elf.a(floatundidf.epeo)
 __c30_signature
                  0x004f08          0x6 c:/program files (x86)/microchip/xc16/v1.24/bin/bin/../../lib\libm-elf.a(floatunsidf.epeo)
 __c30_signature
                  0x004f0e          0x6 c:/program files (x86)/microchip/xc16/v1.24/bin/bin/../../lib\libm-elf.a(frexp.epeo)
 __c30_signature
                  0x004f14          0x6 c:/program files (x86)/microchip/xc16/v1.24/bin/bin/../../lib\libm-elf.a(muldf3.epeo)
 __c30_signature
                  0x004f1a          0x6 c:/program files (x86)/microchip/xc16/v1.24/bin/bin/../../lib\libm-elf.a(subdf3.epeo)
 __c30_signature
                  0x004f20          0x6 c:/program files (x86)/microchip/xc16/v1.24/bin/bin/../../lib\libm-elf.a(mulsi3.epeo)
 __c30_signature
                  0x004f26          0x6 c:/program files (x86)/microchip/xc16/v1.24/bin/bin/../../lib\libm-elf.a(divmoddi3.epeo)
 __c30_signature
                  0x004f2c          0x6 c:/program files (x86)/microchip/xc16/v1.24/bin/bin/../../lib\libm-elf.a(muldi3.epeo)
 __c30_signature
                  0x004f32          0x6 c:/program files (x86)/microchip/xc16/v1.24/bin/bin/../../lib\libm-elf.a(dcompare.epeo)
 __c30_signature
                  0x004f38          0x6 c:/program files (x86)/microchip/xc16/v1.24/bin/bin/../../lib\libm-elf.a(dpropagateNaN.epeo)
 __c30_signature
                  0x004f3e          0x6 c:/program files (x86)/microchip/xc16/v1.24/bin/bin/../../lib\libm-elf.a(dtype.epeo)
 __c30_signature
                  0x004f44          0x6 c:/program files (x86)/microchip/xc16/v1.24/bin/bin/../../lib\libm-elf.a(dunpack.epeo)
 __c30_signature
                  0x004f4a          0x6 c:/program files (x86)/microchip/xc16/v1.24/bin/bin/../../lib\libm-elf.a(umuldi3.epeo)

_04697840560ab195
                    0xdc00        0x210
 _04697840560ab195
                    0xdc00        0x210 build/XC16_dsPIC33EP512MU810/debug/ADC10bitsDrv.o
                    0xdc00                  _BufferA

_04697A20560ab195
                    0xd800        0x210
 _04697A20560ab195
                    0xd800        0x210 build/XC16_dsPIC33EP512MU810/debug/ADC10bitsDrv.o
                    0xd800                  _BufferB

_047939C0560ab17d
                    0xdf00         0x80
 _047939C0560ab17d
                    0xdf00         0x80 build/XC16_dsPIC33EP512MU810/debug/ECAN/ECAN1Drv.o
                    0xdf00                  _ecanRxMsgBuffer

_04793780560ab17d
                    0xdb00          0xe
 _04793780560ab17d
                    0xdb00          0xe build/XC16_dsPIC33EP512MU810/debug/ECAN/ECAN1Drv.o
                    0xdb00                  _ecanTxMsgBuffer

.bss                0x1050       0x1ee4
 .bss               0x1050        0x820 build/XC16_dsPIC33EP512MU810/debug/UARTsComm.o
                    0x1050                  _U1Baudvalue
                    0x1052                  _U2Baudvalue
                    0x1054                  _U3Baudvalue
                    0x1056                  _U4Baudvalue
                    0x1058                  _U1MODEvalue
                    0x105a                  _U1STAvalue
                    0x105c                  _U2MODEvalue
                    0x105e                  _U2STAvalue
                    0x1060                  _U3MODEvalue
                    0x1062                  _U3STAvalue
                    0x1064                  _U4MODEvalue
                    0x1066                  _U4STAvalue
                    0x1068                  _TrameU1
                    0x126a                  _TrameU2
                    0x146c                  _TrameU3
                    0x166e                  _TrameU4
 .bss               0x1870        0x75c build/XC16_dsPIC33EP512MU810/debug/Process.o
                    0x1870                  _PAR
                    0x1b38                  _EXP
                    0x1f4e                  _sorTOR
                    0x1f58                  _entTOR
                    0x1f62                  _Cav_USR1
                    0x1f64                  _Cav_CLR
                    0x1f66                  _T100
                    0x1fa2                  _T10
                    0x1fb6                  _AD7190_PoidsPret
                    0x1fb8                  _Compteur
                    0x1fba                  _NbTopTotal
                    0x1fbe                  _CompteurTot
                    0x1fc2                  _entreeTorVitesseMem
 .bss               0x1fcc        0x48e build/XC16_dsPIC33EP512MU810/debug/B40/spi/abcc_spi_drv.o
 .bss               0x245a        0x46e build/XC16_dsPIC33EP512MU810/debug/B40/abcc_link.o
                    0x245c                  _link_bPool
 .bss               0x28c8        0x418 build/XC16_dsPIC33EP512MU810/debug/MODBUSTCPServer.o
                    0x28c8                  _MODBUS_COMMAND
                    0x28d4                  _WriteByteReverse
                    0x28d6                  _MODBUS_RX
                    0x2ad6                  _MODBUS_TX
                    0x2cd6                  _COIL
                    0x2cd8                  _COIL_REG
 .bss               0x2ce0        0x142 build/XC16_dsPIC33EP512MU810/debug/TCPIPStack/TCP.o
 .bss               0x2e22        0x112 build/XC16_dsPIC33EP512MU810/debug/user.o
                    0x2e22                  _USB_In_Buffer
                    0x2e62                  _USB_Mess_head
                    0x2e64                  _USB_Mess
                    0x2f30                  _USB_list_count

.data._powers_      0x2f34         0xb0
 .data._powers_
                    0x2f34         0xb0 c:/program files (x86)/microchip/xc16/v1.24/bin/bin/../../lib\libc-elf.a(powers.epeo)
                    0x2f34                  __powers_

.data._npowers_
                    0x2fe4         0xb0
 .data._npowers_
                    0x2fe4         0xb0 c:/program files (x86)/microchip/xc16/v1.24/bin/bin/../../lib\libc-elf.a(powers.epeo)
                    0x2fe4                  __npowers_

.bss                0x3094         0xac
 .bss               0x3094         0xac build/XC16_dsPIC33EP512MU810/debug/usb/src/usb_device_cdc.o
                    0x3094                  _cdc_data_tx
                    0x30d4                  _cdc_data_rx
                    0x3114                  _line_coding
                    0x311c                  _cdc_notice
                    0x3126                  _cdc_rx_len
                    0x3127                  _cdc_trf_state
                    0x3128                  _pCDCSrc
                    0x312a                  _pCDCDst
                    0x312c                  _cdc_tx_len
                    0x312d                  _cdc_mem_type
                    0x312e                  _CDCDataOutHandle
                    0x3130                  _CDCDataInHandle
                    0x3132                  _control_signal_bitmap
                    0x3134                  _BaudRateGen
                    0x3138                  _dummy_encapsulated_cmd_response

.data.dpowers       0x3140        0x140
 .data.dpowers      0x3140         0xa0 c:/program files (x86)/microchip/xc16/v1.24/bin/bin/../../lib\libc-elf.a(doprnt_cdfFnopsuxX.EPeo)
 .data.dpowers      0x31e0         0xa0 c:/program files (x86)/microchip/xc16/v1.24/bin/bin/../../lib\libc-elf.a(doprnt.epeo)

_04C8D600560ab18f
                    0x3400         0x60
 _04C8D600560ab18f
                    0x3400         0x60 build/XC16_dsPIC33EP512MU810/debug/usb/src/usb_device.o
                    0x3400                  _BDT

.bss                0x3280         0xfc
 .bss               0x3280         0xfc build/XC16_dsPIC33EP512MU810/debug/TCPIPStack/UDP.o
                    0x3280                  _UDPSocketInfo
                    0x3370                  _activeUDPSocket
                    0x3372                  _UDPTxCount
                    0x3374                  _UDPRxCount

.bss                0x3460        0x206
 .bss               0x3460         0xe6 build/XC16_dsPIC33EP512MU810/debug/B40/ad_obj.o
                    0x3460                  _AD_asDefaultMap
                    0x3462                  _AD_asADIEntryList
 .bss               0x3546         0x94 build/XC16_dsPIC33EP512MU810/debug/TCPIPStack/BerkeleyAPI.o
 .bss               0x35da         0x8c build/XC16_dsPIC33EP512MU810/debug/TCPIPStack/HTTP2.o
                    0x35da                  _curHTTP
                    0x365c                  _httpStubs
                    0x3664                  _curHTTPID

.data               0x337c         0x70
 .data              0x337c         0x70 build/XC16_dsPIC33EP512MU810/debug/BerkeleyTCPClient.o

.bss                0x3666         0x6c
 .bss               0x3666         0x6c build/XC16_dsPIC33EP512MU810/debug/TCPIPStack/MPFS2.o

.data               0x36d2         0x66
 .data              0x36d2         0x66 build/XC16_dsPIC33EP512MU810/debug/MODBUSTCPServer.o
                    0x36d2                  _ReadByteReverse
                    0x36d3                  _InputByteReverse
                    0x36d4                  _HOLDING_REG
                    0x3706                  _INPUT_REG

.bss                0x3738         0x9a
 .bss               0x3738         0x50 build/XC16_dsPIC33EP512MU810/debug/main.o
                    0x3738                  _fResetABCC
                    0x373a                  _ABCCPowerState
                    0x373c                  _address
                    0x3740                  _AppConfig
 .bss               0x3788         0x4a build/XC16_dsPIC33EP512MU810/debug/usb/src/usb_device.o
                    0x3788                  _USBDeviceState
                    0x378a                  _USBActiveConfiguration
                    0x378b                  _USBAlternateInterface
                    0x378e                  _pBDTEntryEP0OutCurrent
                    0x3790                  _pBDTEntryEP0OutNext
                    0x3792                  _pBDTEntryOut
                    0x3798                  _pBDTEntryIn
                    0x379e                  _shortPacketStatus
                    0x379f                  _controlTransferState
                    0x37a0                  _inPipes
                    0x37a6                  _outPipes
                    0x37ae                  _pDst
                    0x37b0                  _RemoteWakeup
                    0x37b1                  _USBBusIsSuspended
                    0x37b2                  _USTATcopy
                    0x37b3                  _endpoint_number
                    0x37b4                  _BothEP0OutUOWNsSet
                    0x37b5                  _ep_data_in
                    0x37b8                  _ep_data_out
                    0x37bb                  _USBStatusStageTimeoutCounter
                    0x37bc                  _USBDeferStatusStagePacket
                    0x37bd                  _USBStatusStageEnabledFlag1
                    0x37be                  _USBStatusStageEnabledFlag2
                    0x37bf                  _USBDeferINDataStagePackets
                    0x37c0                  _USBDeferOUTDataStagePackets
                    0x37c1                  _SetupPkt
                    0x37c9                  _CtrlTrfData

.data               0x37d2         0x54
 .data              0x37d2         0x2a c:/program files (x86)/microchip/xc16/v1.24/bin/bin/../../lib\libc-elf.a(doprnt_cdfFnopsuxX.EPeo)
 .data              0x37fc         0x2a c:/program files (x86)/microchip/xc16/v1.24/bin/bin/../../lib\libc-elf.a(doprnt.epeo)

.bss                0x3826         0x24
 .bss               0x3826         0x24 build/XC16_dsPIC33EP512MU810/debug/BerkeleyUDPClient.o

.data._iob          0x384a         0x24
 .data._iob         0x384a         0x24 c:/program files (x86)/microchip/xc16/v1.24/bin/bin/../../lib\libc-elf.a(_iob.epeo)
                    0x384a                  __iob

.bss                0x386e         0x5a
 .bss               0x386e         0x18 build/XC16_dsPIC33EP512MU810/debug/TCPIPStack/DNS.o
 .bss               0x3886         0x16 build/XC16_dsPIC33EP512MU810/debug/TCPIPStack/ARP.o
 .bss               0x389c         0x16 build/XC16_dsPIC33EP512MU810/debug/TCPIPStack/SPIEEPROM.o
 .bss               0x38b2         0x16 build/XC16_dsPIC33EP512MU810/debug/SPIFRAM.o

.bss                0x33ec         0x14
 .bss               0x33ec         0x14 build/XC16_dsPIC33EP512MU810/debug/TCPIPStack/ICMP.o

.bss                0x38c8         0x12
 .bss               0x38c8         0x12 build/XC16_dsPIC33EP512MU810/debug/BerkeleyTCPClient.o

.data               0x38da         0x74
 .data              0x38da         0x74 build/XC16_dsPIC33EP512MU810/debug/B40/user_adi.o

.bss                0x394e         0x90
 .bss               0x394e         0x3e build/XC16_dsPIC33EP512MU810/debug/B40/abcc_handler.o
                    0x394e                  _ABCC_RunDriver
                    0x3950                  _ABCC_ISR
                    0x3952                  _pnABCC_DrvInit
                    0x3954                  _pnABCC_DrvISR
                    0x3956                  _pnABCC_DrvRunDriverTx
                    0x3958                  _pnABCC_DrvRunDriverRx
                    0x395a                  _pnABCC_DrvWriteMessage
                    0x395c                  _pnABCC_DrvWriteProcessData
                    0x395e                  _pnABCC_DrvISReadyForWrPd
                    0x3960                  _pnABCC_DrvISReadyForWriteMessage
                    0x3962                  _pnABCC_DrvISReadyForCmd
                    0x3964                  _pnABCC_DrvSetNbrOfCmds
                    0x3966                  _pnABCC_DrvSetAppStatus
                    0x3968                  _pnABCC_DrvSetPdSize
                    0x396a                  _pnABCC_DrvSetMsgReceiverBuffer
                    0x396c                  _pnABCC_DrvSetIntMask
                    0x396e                  _pnABCC_DrvGetWrPdBuffer
                    0x3970                  _pnABCC_DrvGetModCap
                    0x3972                  _pnABCC_DrvGetLedStatus
                    0x3974                  _pnABCC_DrvGetIntStatus
                    0x3976                  _pnABCC_DrvGetAnybusState
                    0x3978                  _pnABCC_DrvReadProcessData
                    0x397a                  _pnABCC_DrvReadMessage
                    0x397c                  _pnABCC_DrvIsSupervised
                    0x397e                  _pnABCC_DrvGetAnbStatus
 .bss               0x398c         0x26 build/XC16_dsPIC33EP512MU810/debug/B40/user_adi.o
                    0x398c                  _ADI_DebitInstan
                    0x3990                  _ADI_PoidsInstan
                    0x3994                  _ADI_PoidsMetre
                    0x3998                  _ADI_Vitesse
                    0x399c                  _ADI_TotalPartiel
                    0x39a0                  _ADI_TotalGlobal
                    0x39a4                  _ADI_Tare
                    0x39a8                  _ADI_EtatBascule
                    0x39ac                  _ADI_CmdsBascule
                    0x39b0                  _ADI_DigitalInput
                    0x39b1                  _ADI_DigitalOutput
 .bss               0x39b2         0x18 build/XC16_dsPIC33EP512MU810/debug/B40/abcc_timer.o
 .bss               0x39ca         0x14 build/XC16_dsPIC33EP512MU810/debug/B40/abcc_setup.o

.data               0x39de         0x10
 .data              0x39de         0x10 build/XC16_dsPIC33EP512MU810/debug/B40/abcc_cbf.o

.bss                0x39ee         0x28
 .bss               0x39ee          0xe build/XC16_dsPIC33EP512MU810/debug/TCPIPStack/StackTsk.o
                    0x39f0                  _remoteNode
 .bss               0x39fc          0xa build/XC16_dsPIC33EP512MU810/debug/ECAN/ECAN1Drv.o
                    0x39fc                  _receivedECANmsg
                    0x39fe                  _transmitNextECANmsg
                    0x3a00                  _sentPacketECANMSG
                    0x3a02                  _rxECANIndex
                    0x3a04                  _txECANBufferIndex
 .bss               0x3a06          0x8 build/XC16_dsPIC33EP512MU810/debug/B40/abcc_sys_adapt.o
                    0x3a06                  _SPI3CON1Value
                    0x3a08                  _SPI3CON2Value
                    0x3a0a                  _SPI3STATValue
 .bss               0x3a0e          0x8 build/XC16_dsPIC33EP512MU810/debug/TCPIPStack/ENC28J60.o

.data               0x3a16          0x6
 .data              0x3a16          0x6 build/XC16_dsPIC33EP512MU810/debug/B40/app_obj.o
                    0x3a16                  _app_aacLanguages
                    0x3a18                  _app_sInstance

.bss                0x3a1c          0xc
 .bss               0x3a1c          0x6 build/XC16_dsPIC33EP512MU810/debug/B40/user_setup.o
                    0x3a1c                  _us_bSwitch1
                    0x3a1d                  _us_bSwitch2
                    0x3a1e                  _us_fSwitch1Set
                    0x3a1f                  _us_fSwitch2Set
 .bss               0x3a22          0x6 build/XC16_dsPIC33EP512MU810/debug/BerkeleyTCPServer.o

_04DDDD20560ab18d
                    0x3a28          0x6
 _04DDDD20560ab18d
                    0x3a28          0x6 build/XC16_dsPIC33EP512MU810/debug/TCPIPStack/Tick.o

.bss                0x3a2e          0xe
 .bss               0x3a2e          0x6 build/XC16_dsPIC33EP512MU810/debug/ADComm.o
                    0x3a2e                  _SPICON1Value
                    0x3a30                  _SPICON2Value
                    0x3a32                  _SPISTATValue
 .bss               0x3a34          0x4 build/XC16_dsPIC33EP512MU810/debug/B40/abcc_remap.o
 .bss               0x3a38          0x4 build/XC16_dsPIC33EP512MU810/debug/TCPIPStack/Announce.o

.data               0x3a3c          0x8
 .data              0x3a3c          0x4 build/XC16_dsPIC33EP512MU810/debug/TCPIPStack/DNS.o
 .data              0x3a40          0x4 build/XC16_dsPIC33EP512MU810/debug/TCPIPStack/Helpers.o

.bss                0x3a44          0xc
 .bss               0x3a44          0x4 build/XC16_dsPIC33EP512MU810/debug/TCPIPStack/IP.o
 .bss               0x3a48          0x4 build/XC16_dsPIC33EP512MU810/debug/TCPIPStack/NBNS.o
 .bss               0x3a4c          0x4 build/XC16_dsPIC33EP512MU810/debug/TCPIPStack/Tick.o

.data               0x3a50          0x4
 .data              0x3a50          0x4 build/XC16_dsPIC33EP512MU810/debug/main.o
                    0x3a50                  _ABCC_StateMachineEnabled
                    0x3a52                  ___C30_UART

.bss                0x3a54          0x8
 .bss               0x3a54          0x4 build/XC16_dsPIC33EP512MU810/debug/CustomHTTPApp.o
 .bss               0x3a58          0x4 build/XC16_dsPIC33EP512MU810/debug/MemFlash.o
                    0x3a58                  _Nb_Octets_Log
                    0x3a5a                  _Address_Log_L
                    0x3a5b                  _Address_Log_B

.bss.randx          0x3a5c          0x4
 .bss.randx         0x3a5c          0x4 c:/program files (x86)/microchip/xc16/v1.24/bin/bin/../../lib\libc-elf.a(rand.epeo)

.bss                0x3a60          0x2
 .bss               0x3a60          0x2 build/XC16_dsPIC33EP512MU810/debug/B40/abcc_debug_err.o
                    0x3a60                  _ErrorReporter

.data               0x3a62          0x8
 .data              0x3a62          0x2 build/XC16_dsPIC33EP512MU810/debug/B40/dpv1.o
                    0x3a62                  _dpv_sInstance
 .data              0x3a64          0x2 build/XC16_dsPIC33EP512MU810/debug/ECAN/ECAN1Drv.o
                    0x3a64                  _rxECANBufferIndex
 .data              0x3a66          0x2 build/XC16_dsPIC33EP512MU810/debug/Process.o
                    0x3a66                  _Demarrage1er
 .data              0x3a68          0x2 build/XC16_dsPIC33EP512MU810/debug/TCPIPStack/BerkeleyAPI.o

.pbss               0x3a6a          0x2
 .pbss              0x3a6a          0x2 build/XC16_dsPIC33EP512MU810/debug/TCPIPStack/DNS.o

.data               0x3a6c          0x4
 .data              0x3a6c          0x2 build/XC16_dsPIC33EP512MU810/debug/TCPIPStack/Reboot.o
 .data              0x3a6e          0x2 build/XC16_dsPIC33EP512MU810/debug/TCPIPStack/TCP.o

.pbss               0x3a70          0x2
 .pbss              0x3a70          0x2 build/XC16_dsPIC33EP512MU810/debug/TCPIPStack/TCP.o

.data               0x3a72          0x2
 .data              0x3a72          0x2 build/XC16_dsPIC33EP512MU810/debug/TCPIPStack/UDP.o

.pbss               0x3a74          0x2
 .pbss              0x3a74          0x2 build/XC16_dsPIC33EP512MU810/debug/TCPIPStack/UDP.o

.bss                0x3a76          0x4
 .bss               0x3a76          0x2 build/XC16_dsPIC33EP512MU810/debug/ADC10bitsDrv.o
                    0x3a76                  _DmaBufferSwitch
 .bss               0x3a78          0x2 build/XC16_dsPIC33EP512MU810/debug/ModbusUartServer.o

.bss.errno          0x3a7a          0x2
 .bss.errno         0x3a7a          0x2 c:/program files (x86)/microchip/xc16/v1.24/bin/bin/../../lib\libc-elf.a(errno.epeo)
                    0x3a7a                  _errno

.bss.randf          0x3a7c          0x2
 .bss.randf         0x3a7c          0x2 c:/program files (x86)/microchip/xc16/v1.24/bin/bin/../../lib\libc-elf.a(rand.epeo)

.bss.sp.1310        0x3a7e          0x2
 .bss.sp.1310       0x3a7e          0x2 c:/program files (x86)/microchip/xc16/v1.24/bin/bin/../../lib\libc-elf.a(strtok.epeo)

.data._Files        0x3a80          0x2
 .data._Files       0x3a80          0x2 c:/program files (x86)/microchip/xc16/v1.24/bin/bin/../../lib\libc-elf.a(_iob.epeo)
                    0x3a80                  __Files

.bss._outdone       0x3a82          0x2
 .bss._outdone      0x3a82          0x2 c:/program files (x86)/microchip/xc16/v1.24/bin/bin/../../lib\libc-elf.a(_iob.epeo)
                    0x3a82                  __outdone

.bss._sibuf         0x3a84          0x2
 .bss._sibuf        0x3a84          0x2 c:/program files (x86)/microchip/xc16/v1.24/bin/bin/../../lib\libc-elf.a(_iob.epeo)
                    0x3a84                  __sibuf

.bss._sobuf         0x3a86          0x2
 .bss._sobuf        0x3a86          0x2 c:/program files (x86)/microchip/xc16/v1.24/bin/bin/../../lib\libc-elf.a(_iob.epeo)
                    0x3a86                  __sobuf

.config_APLK      0xf80010          0x2
 .config_APLK     0xf80010          0x2 build/XC16_dsPIC33EP512MU810/debug/configuration_bits.o

.config_JTAGEN    0xf8000e          0x2
 .config_JTAGEN
                  0xf8000e          0x2 build/XC16_dsPIC33EP512MU810/debug/configuration_bits.o

.config_ALTI2C2
                  0xf8000c          0x2
 .config_ALTI2C2
                  0xf8000c          0x2 build/XC16_dsPIC33EP512MU810/debug/configuration_bits.o

.config_FWDTEN    0xf8000a          0x2
 .config_FWDTEN
                  0xf8000a          0x2 build/XC16_dsPIC33EP512MU810/debug/configuration_bits.o

.config_FCKSM     0xf80008          0x2
 .config_FCKSM    0xf80008          0x2 build/XC16_dsPIC33EP512MU810/debug/configuration_bits.o

.config_IESO      0xf80006          0x2
 .config_IESO     0xf80006          0x2 build/XC16_dsPIC33EP512MU810/debug/configuration_bits.o

.config_GSSK      0xf80004          0x2
 .config_GSSK     0xf80004          0x2 build/XC16_dsPIC33EP512MU810/debug/configuration_bits.o

.const              0xc0e0       0x16fe load address 0x0040e0  
 .const             0xc0e0        0x4c0 build/XC16_dsPIC33EP512MU810/debug/TCPIPStack/HTTP2.o
 .const             0xc5a0        0x2c8 build/XC16_dsPIC33EP512MU810/debug/Process.o
 .const             0xc868        0x2aa build/XC16_dsPIC33EP512MU810/debug/B40/abcc_setup.o
 .const             0xcb12        0x268 build/XC16_dsPIC33EP512MU810/debug/user.o
                    0xcb12                  _DELIMITER
                    0xcb16                  _DELIMITER_NULL
 .const             0xcd7a        0x18c build/XC16_dsPIC33EP512MU810/debug/B40/spi/abcc_spi_drv.o
 .const             0xcf06        0x164 build/XC16_dsPIC33EP512MU810/debug/B40/abcc_handler.o
 .const             0xd06a        0x158 build/XC16_dsPIC33EP512MU810/debug/B40/user_adi.o
 .const             0xd1c2        0x14a build/XC16_dsPIC33EP512MU810/debug/CustomHTTPApp.o
                    0xd285                  _HTML_UP_ARROW
                    0xd288                  _HTML_DOWN_ARROW
 .const             0xd30c        0x114 build/XC16_dsPIC33EP512MU810/debug/B40/abcc_cbf.o
 .const             0xd420         0xe6 build/XC16_dsPIC33EP512MU810/debug/B40/abcc_link.o
 .const             0xd506         0xa0 build/XC16_dsPIC33EP512MU810/debug/B40/user_setup.o
 .const             0xd5a6         0x92 build/XC16_dsPIC33EP512MU810/debug/usb_descriptors.o
                    0xd5a6                  _device_dsc
                    0xd5b8                  _configDescriptor1
                    0xd5fc                  _sd000
                    0xd600                  _sd001
                    0xd618                  _sd002
                    0xd630                  _USB_CD_Ptr
                    0xd632                  _USB_SD_Ptr
 .const             0xd638         0x50 build/XC16_dsPIC33EP512MU810/debug/B40/spi/abcc_crc32.o
                    0xd638                  _abBitReverseTable16
                    0xd648                  _crc_table32
 .const             0xd688         0x34 build/XC16_dsPIC33EP512MU810/debug/main.o
 .const             0xd6bc         0x2e build/XC16_dsPIC33EP512MU810/debug/B40/spi/abcc_handler_spi.o
 .const             0xd6ea         0x24 build/XC16_dsPIC33EP512MU810/debug/B40/abcc_timer.o
 .const             0xd70e         0x24 build/XC16_dsPIC33EP512MU810/debug/TCPIPStack/TCP.o
                    0xd70e                  _TCPSocketInitializer
 .const             0xd732         0x1c build/XC16_dsPIC33EP512MU810/debug/B40/app_obj.o
                    0xd746                  _app_sObject
 .const             0xd74e         0x1c build/XC16_dsPIC33EP512MU810/debug/TCPIPStack/Announce.o
 .const             0xd76a         0x1a build/XC16_dsPIC33EP512MU810/debug/AD7190.o
 .const             0xd784         0x18 build/XC16_dsPIC33EP512MU810/debug/B40/dpv1.o
                    0xd794                  _dpv1_sObject
 .const             0xd79c         0x12 build/XC16_dsPIC33EP512MU810/debug/B40/ad_obj.o
 .const             0xd7ae         0x10 build/XC16_dsPIC33EP512MU810/debug/BerkeleyTCPClient.o
 .const             0xd7be          0xe build/XC16_dsPIC33EP512MU810/debug/BerkeleyUDPClient.o
 .const             0xd7cc          0x8 build/XC16_dsPIC33EP512MU810/debug/TCPIPStack/MPFS2.o
 .const             0xd7d4          0x6 build/XC16_dsPIC33EP512MU810/debug/ModbusUartServer.o
 .const             0xd7da          0x4 build/XC16_dsPIC33EP512MU810/debug/MPFSImg2.o
                    0xd7da                  _MPFS_Start

.text             0x0057de       0x56ea
 .text            0x0057de       0x56ea build/XC16_dsPIC33EP512MU810/debug/ModbusUartServer.o
                  0x0057de                  _ModbusUartServer
                  0x005886                  _ProcessMessageRecu
                  0x00592e                  _LectureMots
                  0x007f5a                  _LectureModbus
                  0x008018                  _envoieLongPF
                  0x008078                  _envoieLongPf
                  0x0080a4                  _envoieReelPF
                  0x008150                  _envoieReelPf
                  0x008202                  _EcritureMots
                  0x009dc6                  _AffectationIO
                  0x009e04                  _ModifParamMetro
                  0x00aa3e                  _LectureLong
                  0x00ab20                  _LectureReel
                  0x00ac4a                  _ValidationCodeMetrologie
                  0x00ad66                  _ModbusErreur
                  0x00ad94                  _Random
                  0x00adc4                  _ModifieVitesseComm

MPFSData          0x00aec8       0x51ea
 MPFSData         0x00aec8       0x51ea build/XC16_dsPIC33EP512MU810/debug/MPFSImg2.o
                  0x00aecc                  BEGIN_MPFS

.text             0x0100b2      0x13658
 .text            0x0100b2       0x2840 build/XC16_dsPIC33EP512MU810/debug/Process.o
                  0x0100b2                  _EcrFRAM_Param
                  0x0100fa                  _EcrFRAM
                  0x010142                  _LecFRAM_Param
                  0x0101a6                  _LecFRAM
                  0x0101ee                  _InitParams
                  0x010618                  _gestion_profibus
                  0x010844                  _process_plcd
                  0x010cc2                  _gestion_defauts
                  0x010f5a                  _gestion_cycle
                  0x0111a8                  _ValEntTOR
                  0x0111e0                  _gestion_vitesse
                  0x011472                  _EnvoieSerie
                  0x011554                  _gestion_totalisateurs
                  0x01186c                  _verif_totaux
                  0x011ac2                  _etatSortieTOR
                  0x011af6                  _sortiesTOR
                  0x011d42                  _gestion_poids_debit
                  0x011ff6                  _gestion_comm_serie
                  0x012054                  _envoyer_reel
                  0x012132                  _moyenne_glissante_debit
                  0x012156                  _moyenne_glissante_poids
                  0x0123b8                  _conversion_poids
                  0x012438                  _lecture_entrees_TOR
                  0x0124e4                  _EcritSortieAna
 .text            0x0128f2       0x249c build/XC16_dsPIC33EP512MU810/debug/TCPIPStack/TCP.o
                  0x0129ba                  _TCPInit
                  0x012a8a                  _TCPOpen
                  0x012be4                  _TCPWasReset
                  0x012c12                  _TCPIsConnected
                  0x012c36                  _TCPDisconnect
                  0x012cd6                  _TCPClose
                  0x012cf6                  _TCPGetRemoteInfo
                  0x012d20                  _TCPFlush
                  0x012d46                  _TCPIsPutReady
                  0x012d94                  _TCPPut
                  0x012e3a                  _TCPPutArray
                  0x012f20                  _TCPPutString
                  0x012f44                  _TCPGetTxFIFOFull
                  0x012f70                  _TCPDiscard
                  0x012f90                  _TCPIsGetReady
                  0x012fc8                  _TCPGet
                  0x013042                  _TCPGetArray
                  0x01310e                  _TCPGetRxFIFOFree
                  0x013138                  _TCPPeekArray
                  0x0131e2                  _TCPPeek
                  0x0131fa                  _TCPFindArrayEx
                  0x01346a                  _TCPFindEx
                  0x01348e                  _TCPTick
                  0x01397e                  _TCPProcess
                  0x014b8c                  _TCPAdjustFIFOSize
 .text            0x014d8e       0x1dd8 build/XC16_dsPIC33EP512MU810/debug/B40/ad_obj.o
                  0x014d8e                  _AD_Init
                  0x014f24                  _AD_GetAdiIndex
                  0x014f5a                  _AD_GetAdiInstEntry
                  0x014f80                  _AD_ProcObjectRequest
                  0x015f20                  _AD_GetAdiValue
                  0x0160c0                  _AD_SetAdiValue
                  0x01663a                  _AD_UpdatePdReadData
                  0x01668c                  _AD_UpdatePdWriteData
                  0x0166ee                  _AD_NewWrPd
                  0x0166f8                  _AD_AdiMappingReq
                  0x016b3e                  _AD_RemapDone
 .text            0x016b66       0x1a80 build/XC16_dsPIC33EP512MU810/debug/TCPIPStack/HTTP2.o
                  0x016b66                  _HTTPPrint
                  0x016db4                  _HTTPPrint_
                  0x016dd2                  _HTTPInit
                  0x016e60                  _HTTPServer
                  0x01818e                  _HTTPURLDecode
                  0x018262                  _HTTPGetArg
                  0x0182b8                  _HTTPReadPostName
                  0x0182e4                  _HTTPReadPostValue
                  0x018500                  _HTTPIncFile
 .text            0x0185e6       0x18ce build/XC16_dsPIC33EP512MU810/debug/usb/src/usb_device.o
                  0x0185e6                  _USBDeviceInit
                  0x0186fa                  _USBDeviceTasks
                  0x018896                  _USBEnableEndpoint
                  0x0188d0                  _USBTransferOnePacket
                  0x018a0a                  _USBStallEndpoint
                  0x018b98                  _USBCancelIO
                  0x018d2a                  _USBDeviceDetach
                  0x018d3c                  _USBDeviceAttach
                  0x018d7e                  _USBCtrlEPAllowStatusStage
                  0x018eb6                  _USBCtrlEPAllowDataStage
 .text            0x019eb4       0x122a build/XC16_dsPIC33EP512MU810/debug/Pesage.o
                  0x019eb4                  _GestionCyclePesage
 .text            0x01b0de        0xd92 build/XC16_dsPIC33EP512MU810/debug/TCPIPStack/ENC28J60.o
                  0x01b0de                  _MACInit
                  0x01b20e                  _MACIsLinked
                  0x01b224                  _MACIsTxReady
                  0x01b23c                  _MACDiscardRx
                  0x01b278                  _MACGetFreeRxSize
                  0x01b302                  _MACGetHeader
                  0x01b3d4                  _MACPutHeader
                  0x01b42a                  _MACFlush
                  0x01b56c                  _MACSetReadPtrInRx
                  0x01b59e                  _MACSetWritePtr
                  0x01b5d4                  _MACSetReadPtr
                  0x01b60a                  _MACCalcRxChecksum
                  0x01b670                  _CalcIPBufferChecksum
                  0x01b726                  _MACMemCopyAsync
                  0x01b92c                  _MACIsMemCopyDone
                  0x01b944                  _MACGet
                  0x01b976                  _MACGetArray
                  0x01ba54                  _MACPut
                  0x01ba8c                  _MACPutArray
                  0x01bc46                  _ReadPHYReg
                  0x01bd8e                  _WritePHYReg
                  0x01bde6                  _MACPowerDown
                  0x01be1a                  _MACPowerUp
                  0x01be3c                  _SetCLKOUT
                  0x01be52                  _GetCLKOUT
 .text            0x01be70        0xbb4 build/XC16_dsPIC33EP512MU810/debug/user.o
                  0x01be70                  _InitApp
                  0x01be8c                  _putsUSB
                  0x01bef0                  _USB_enqMsg
                  0x01bf3c                  _DeviceCDCInitialize
                  0x01bf60                  _DeviceCDCTasks
                  0x01bffe                  _ProccessCmd
                  0x01c76e                  _CRC_Init
                  0x01c77e                  _CRC_ChecksumWord
                  0x01c7e4                  _ResetCounterMillis
                  0x01c7ee                  _GetCounterMillis
                  0x01c804                  _UpdateB40ADI
 .text            0x01ca24        0xb5e build/XC16_dsPIC33EP512MU810/debug/TCPIPStack/BerkeleyAPI.o
                  0x01ca24                  _BerkeleySocketInit
                  0x01ca50                  _socket
                  0x01caea                  _bind
                  0x01cb8a                  _listen
                  0x01cca6                  _accept
                  0x01cdec                  _connect
                  0x01cf6c                  _send
                  0x01cf8c                  _sendto
                  0x01d150                  _recv
                  0x01d1e8                  _recvfrom
                  0x01d348                  _gethostname
                  0x01d3aa                  _closesocket
 .text            0x01d582        0xb08 build/XC16_dsPIC33EP512MU810/debug/CustomHTTPApp.o
                  0x01d582                  _HTTPNeedsAuth
                  0x01d5b6                  _HTTPCheckAuth
                  0x01d5e8                  _HTTPExecuteGet
                  0x01d66c                  _HTTPExecutePost
                  0x01d9de                  _HTTPPrint_builddate
                  0x01da2c                  _HTTPPrint_version
                  0x01da4c                  _HTTPPrint_btn
                  0x01daa2                  _HTTPPrint_led
                  0x01daf6                  _HTTPPrint_ledSelected
                  0x01db5a                  _HTTPPrint_pot
                  0x01db88                  _HTTPPrint_lcdtext
                  0x01dbc2                  _HTTPPrint_hellomsg
                  0x01dc0e                  _HTTPPrint_cookiename
                  0x01dc5c                  _HTTPPrint_uploadeImage
                  0x01dc62                  _HTTPPrint_uploadedmd5
                  0x01dcb4                  _HTTPPrintIP
                  0x01dd1a                  _HTTPPrint_config_hostname
                  0x01dd38                  _HTTPPrint_config_dhcpchecked
                  0x01dd62                  _HTTPPrint_config_ip
                  0x01dd90                  _HTTPPrint_config_gw
                  0x01ddbe                  _HTTPPrint_config_subnet
                  0x01ddec                  _HTTPPrint_config_dns1
                  0x01de1a                  _HTTPPrint_config_dns2
                  0x01de48                  _HTTPPrint_config_mac
                  0x01df00                  _HTTPPrint_read_comm
                  0x01df08                  _HTTPPrint_write_comm
                  0x01df10                  _HTTPPrint_reboot
                  0x01df18                  _HTTPPrint_rebootaddr
                  0x01df36                  _HTTPPrint_ddns_user
                  0x01df3c                  _HTTPPrint_ddns_pass
                  0x01df42                  _HTTPPrint_ddns_host
                  0x01df48                  _HTTPPrint_ddns_service
                  0x01df50                  _HTTPPrint_ddns_status
                  0x01df70                  _HTTPPrint_ddns_status_msg
                  0x01dfbe                  _HTTPPrint_smtps_en
                  0x01dfde                  _HTTPPrint_snmp_en
                  0x01dffe                  _HTTPPrint_status_ok
                  0x01e044                  _HTTPPrint_status_fail
 .text            0x01e08a        0xaf2 build/XC16_dsPIC33EP512MU810/debug/TCPIPStack/MPFS2.o
                  0x01e08a                  _MPFSInit
                  0x01e0b6                  _MPFSOpen
                  0x01e20c                  _MPFSOpenID
                  0x01e296                  _MPFSClose
                  0x01e2bc                  _MPFSGet
                  0x01e44c                  _MPFSGetArray
                  0x01e676                  _MPFSGetLong
                  0x01e698                  _MPFSSeek
                  0x01e8aa                  _MPFSGetTimestamp
                  0x01e8f0                  _MPFSGetMicrotime
                  0x01e936                  _MPFSGetFlags
                  0x01e97a                  _MPFSGetSize
                  0x01e9c0                  _MPFSGetBytesRem
                  0x01e9fe                  _MPFSGetStartAddr
                  0x01ea46                  _MPFSGetEndAddr
                  0x01ea98                  _MPFSGetFilename
                  0x01eafc                  _MPFSGetPosition
                  0x01eb22                  _MPFSGetID
 .text            0x01eb7c        0x9b8 build/XC16_dsPIC33EP512MU810/debug/main.o
                  0x01eb7c                  _main
                  0x01ecac                  _ABCCMainStateMachine
                  0x01ed52                  _DisplayIPValue
                  0x01ed88                  _GestionReponseModbus
                  0x01eef4                  _ProcessIO
                  0x01f12a                  _InitTCPIPAppConfig
                  0x01f206                  _InitializeBoard
                  0x01f3d8                  _SaveAppConfig
                  0x01f410                  _ADInit
                  0x01f462                  _LEDUpdateUSBStatus
                  0x01f4d0                  _USER_USB_CALLBACK_EVENT_HANDLER
 .text            0x01f534        0x8b4 build/XC16_dsPIC33EP512MU810/debug/TCPIPStack/Helpers.o
                  0x01f534                  _LFSRSeedRand
                  0x01f576                  _LFSRRand
                  0x01f5e6                  _GenerateRandomDWORD
                  0x01f6f0                  _StringToIPAddress
                  0x01f86a                  _Base64Decode
                  0x01f9d2                  _uitoa
                  0x01fa52                  _hexatob
                  0x01fabc                  _btohexa_high
                  0x01fade                  _btohexa_low
                  0x01fafc                  _stricmppgm2ram
                  0x01fb94                  _swaps
                  0x01fbb0                  _swapl
                  0x01fc10                  _CalcIPChecksum
                  0x01fc92                  _strupr
                  0x01fcd2                  _FormatNetBIOSName
                  0x01fd1c                  _strnchr
                  0x01fd6a                  _strncpy_m
 .text            0x01fde8        0x896 build/XC16_dsPIC33EP512MU810/debug/TCPIPStack/DNS.o
                  0x01fde8                  _DNSBeginUsage
                  0x01fe08                  _DNSEndUsage
                  0x01fe40                  _DNSResolve
                  0x01fe80                  _DNSIsResolved
 .text            0x02067e        0x87a build/XC16_dsPIC33EP512MU810/debug/TCPIPStack/UDP.o
                  0x02067e                  _UDPInit
                  0x02069e                  _UDPOpenEx
                  0x0207b8                  _UDPTask
                  0x0209fa                  _UDPIsOpened
                  0x020a1c                  _UDPClose
                  0x020a5e                  _UDPSetTxBuffer
                  0x020a74                  _UDPSetRxBuffer
                  0x020a8a                  _UDPIsPutReady
                  0x020ac0                  _UDPPut
                  0x020af0                  _UDPPutArray
                  0x020b2c                  _UDPPutString
                  0x020b4a                  _UDPFlush
                  0x020c44                  _UDPIsGetReady
                  0x020c7a                  _UDPGet
                  0x020cae                  _UDPGetArray
                  0x020cfa                  _UDPDiscard
                  0x020d20                  _UDPProcess
 .text            0x020ef8        0x866 build/XC16_dsPIC33EP512MU810/debug/UARTsComm.o
                  0x020ef8                  _UARTs_Init
                  0x020fee                  _BaudrateIsValid
                  0x02105e                  _UART1_SetBaudrate
                  0x0210b4                  _UART2_SetBaudrate
                  0x02110a                  _UART3_SetBaudrate
                  0x021160                  _UART4_SetBaudrate
                  0x0211b6                  _UART1_SetStopBit
                  0x0211f4                  _UART2_SetStopBit
                  0x021232                  _UART1_SetParityNBits
                  0x02128a                  _UART2_SetParityNBits
                  0x0212e2                  _ReceiveUART1
                  0x021358                  _ReceiveUART2
                  0x021496                  _ReceiveUART3
                  0x0215c8                  _ReceiveUART4
                  0x0216fa                  _SendStrUART3
                  0x021726                  _SendStrUART4
 .text            0x02175e        0x748 build/XC16_dsPIC33EP512MU810/debug/B40/abcc_setup.o
                  0x02175e                  _ABCC_SetupInit
                  0x02178c                  _ABCC_SetupCommands
                  0x021abc                  _ABCC_SetupResponses
                  0x021e46                  _ABCC_UserInitComplete
                  0x021e7e                  _ABCC_NetworkType
                  0x021e88                  _ABCC_ModuleType
                  0x021e92                  _ABCC_NetFormatType
                  0x021e9c                  _ABCC_ParameterSupport
 .text            0x021ea6        0x6a2 build/XC16_dsPIC33EP512MU810/debug/B40/spi/abcc_spi_drv.o
                  0x021ed4                  _ABCC_DrvSpiRunDriverTx
                  0x022010                  _ABCC_DrvSpiRunDriverRx
                  0x0221a2                  build/XC16_dsPIC33EP512MU810/debug/B40/spi/abcc_spi_drv.o:_spi_drv_DataReceived
                  0x0221e8                  build/XC16_dsPIC33EP512MU810/debug/B40/spi/abcc_spi_drv.o:_drv_WdTimeoutHandler
                  0x0221f6                  _ABCC_DrvSpiInit
                  0x02229e                  _ABCC_DrvSpiWriteMessage
                  0x02231a                  _ABCC_DrvSpiWriteProcessData
                  0x022350                  _ABCC_DrvSpiIsReadyForWriteMessage
                  0x022376                  _ABCC_DrvSpiIsReadyForCmd
                  0x022396                  _ABCC_DrvSpiSetNbrOfCmds
                  0x0223a2                  _ABCC_DrvSpiSetAppStatus
                  0x0223b2                  _ABCC_DrvSpiSetPdSize
                  0x02240e                  _ABCC_DrvSpiSetMsgReceiverBuffer
                  0x022456                  _ABCC_DrvSpiGetIntStatus
                  0x02247a                  _ABCC_DrvSpiGetAnybusState
                  0x022488                  _ABCC_DrvSpiReadProcessData
                  0x0224a0                  _ABCC_DrvSpiReadMessage
                  0x0224c2                  _ABCC_DrvSpiSetIntMask
                  0x0224d2                  _ABCC_DrvSpiGetWrPdBuffer
                  0x0224e2                  _ABCC_DrvSpiGetModCap
                  0x022506                  _ABCC_DrvSpiGetLedStatus
                  0x022510                  _ABCC_DrvSpiIsReadyForWrPd
                  0x022524                  _ABCC_DrvSpiIsSupervised
                  0x02253a                  _ABCC_DrvSpiGetAnbStatus
 .text            0x022548        0x62a build/XC16_dsPIC33EP512MU810/debug/AD7190.o
                  0x022548                  _AD7190_SetRegisterValue
                  0x02259a                  _AD7190_GetRegisterValue
                  0x02260c                  _AD7190_Init
                  0x022640                  _AD7190_Reset
                  0x02266c                  _AD7190_SetPower
                  0x0226fc                  _AD7190_WaitRdyGoLow
                  0x022730                  _AD7190_ChannelSelect
                  0x022790                  _AD7190_Calibrate
                  0x02281e                  _AD7190_RangeSetup
                  0x0228a4                  _AD7190_SingleConversion
                  0x0228e4                  _AD7190_ContinuousReadAvg
                  0x02294c                  _AD7190_TemperatureRead
                  0x0229ae                  _AD7190_StartContinuousRead
                  0x022a16                  _AD7190_StopContinuousRead
                  0x022a38                  _AD7190_PrintRegisters
 .text            0x022b72        0x628 build/XC16_dsPIC33EP512MU810/debug/B40/abcc_handler.o
                  0x022b72                  _ABCC_SetReadyForCommunication
                  0x022b7c                  _ABCC_SetMainStateError
                  0x022b86                  _ABCC_GetMainState
                  0x022b90                  _ABCC_CheckAnbStatus
                  0x022bb0                  _ABCC_CheckSendMessage
                  0x022bba                  _ABCC_StartDriver
                  0x022d52                  _ABCC_isReadyForCommunication
                  0x022dda                  _ABCC_NewWrPdEvent
                  0x022e08                  _ABCC_RdPdEvent
                  0x022e2c                  _ABCC_RdMsgEvent
                  0x022eb4                  _ABCC_SendCmdMsg
                  0x022f04                  _ABCC_GetCmdQueueSize
                  0x022f12                  _ABCC_SendRespMsg
                  0x022f24                  _ABCC_MsgAlloc
                  0x022f32                  _ABCC_MsgFree
                  0x022f44                  _ABCC_SetPdSize
                  0x022f6c                  _ABCC_HWReset
                  0x022f88                  _ABCC_ShutdownDriver
                  0x022faa                  _ABCC_ModuleDetect
                  0x022fb8                  _ABCC_ModCap
                  0x022fc6                  _ABCC_LedStatus
                  0x022fd4                  _ABCC_AnbState
                  0x022fe2                  _ABCC_IsSupervised
                  0x022ff0                  _ABCC_HWReleaseReset
                  0x022ffa                  _ABCC_SetAppStatus
                  0x023008                  _ABCC_ReadModuleId
                  0x023016                  _ABCC_RunTimerSystem
                  0x023024                  _ABCC_GetNewSourceId
                  0x023054                  _ABCC_GetOpmode
                  0x023062                  _ABCC_GetAttribute
                  0x0230ba                  _ABCC_SetByteAttribute
                  0x02311c                  _ABCC_VerifyMessage
                  0x023130                  _SetErrorReporter
                  0x02313c                  _ABCC_GetDataTypeSize
 .text            0x02319a        0x570 build/XC16_dsPIC33EP512MU810/debug/B40/abcc_link.o
                  0x023278                  _ABCC_LinkInit
                  0x023302                  _ABCC_LinkReadMessage
                  0x023382                  _ABCC_LinkCheckSendMessage
                  0x02340c                  _ABCC_LinkRunDriverRx
                  0x02342a                  _ABCC_LinkGetNumCmdQueueEntries
                  0x02343e                  _ABCC_LinkWriteMessage
                  0x02355c                  _ABCC_LinkWrMsgWithNotification
                  0x0235a0                  _ABCC_LinkAlloc
                  0x0235b6                  _ABCC_LinkFree
                  0x023614                  _ABCC_LinkMapMsgHandler
                  0x023668                  _ABCC_LinkGetMsgHandler
                  0x0236c6                  _ABCC_LinkIsSrcIdUsed

.dinit            0x02370a        0x4fa
 .dinit           0x02370a        0x4fa data_init

.text             0x023c04       0x4336
 .text            0x023c04        0x4aa build/XC16_dsPIC33EP512MU810/debug/MemFlash.o
                  0x023c04                  _Flash_N_Clock
                  0x023c22                  _Active_Flash
                  0x023c2a                  _Desactive_Flash
                  0x023c38                  _Flash_Ready
                  0x023c5a                  _Wait_Flash_Ready
                  0x023c6a                  _Write_Flash
                  0x023c9c                  _Charge_Pointeurs
                  0x023cb4                  _Lecture_Byte_In_Flash
                  0x023cd0                  _Direct_Byte_Write_In_Page
                  0x023ce8                  _Transfert_Page_To_Buffer
                  0x023d00                  _Read_Flash
                  0x023d3c                  _Incremente_Adresse_FlashDB32
                  0x023e0a                  _Incremente_Adresse_FlashDB64
                  0x023ed8                  _MakeAddrDB32
                  0x023f34                  _MakeAddrDB64
                  0x023f96                  _Ecriture_Memoire_Flash_Ligne_Str
                  0x024026                  _Lecture_Memoire_Flash_Ligne_Str
 .text            0x0240ae        0x44e build/XC16_dsPIC33EP512MU810/debug/usb/src/usb_device_cdc.o
                  0x0240ae                  _USBCheckCDCRequest
                  0x0241f8                  _CDCInitEP
                  0x024248                  _USBCDCEventHandler
                  0x02428e                  _getsUSBUSART
                  0x024322                  _putUSBUSART
                  0x02434e                  _putsUSBUSART
                  0x0243a4                  _putrsUSBUSART
                  0x0243fa                  _CDCTxService
 .text            0x0244fc        0x440 build/XC16_dsPIC33EP512MU810/debug/B40/app_obj.o
                  0x0244fc                  _APP_IsResetRequestAllowed
                  0x024512                  _APP_ProcResetRequest
                  0x02453e                  _APP_ProcessCmdMsg
                  0x024568                  _app_InstanceCommand
                  0x024772                  _app_ObjectCommand
 .text            0x02493c        0x3ae build/XC16_dsPIC33EP512MU810/debug/TCPIPStack/NBNS.o
                  0x02493c                  _NBNSTask
 .text            0x024cea        0x3a8 build/XC16_dsPIC33EP512MU810/debug/TCPIPStack/ARP.o
                  0x024cea                  _ARPSendPkt
                  0x024dbe                  _ARPInit
                  0x024df0                  _ARPProcess
                  0x024ec8                  _ARPResolve
                  0x024f92                  _ARPIsResolved
                  0x02505a                  _SwapARPPacket
 .text            0x025092        0x358 build/XC16_dsPIC33EP512MU810/debug/SPIFRAM.o
                  0x025092                  _FRAMInit
                  0x0250aa                  _FRAMBeginRead
                  0x0250c2                  _FRAMRead
                  0x025106                  _FRAMReadArray
                  0x0251e2                  _FRAMBeginWrite
                  0x0251fa                  _FRAMWrite
                  0x02523c                  _FRAMWriteArray
                  0x02526a                  _FRAMEndWrite
                  0x025378                  _FRAMIsBusy
 .text            0x0253ea        0x336 build/XC16_dsPIC33EP512MU810/debug/TCPIPStack/SPIEEPROM.o
                  0x0253ea                  _XEEInit
                  0x025408                  _XEEBeginRead
                  0x025420                  _XEERead
                  0x025464                  _XEEEndRead
                  0x02546e                  _XEEReadArray
                  0x02552c                  _XEEBeginWrite
                  0x025544                  _XEEWrite
                  0x025586                  _XEEWriteArray
                  0x0255b4                  _XEEEndWrite
                  0x0256ae                  _XEEIsBusy
 .text            0x025720        0x2ec build/XC16_dsPIC33EP512MU810/debug/ECAN/ECAN1Drv.o
                  0x025720                  _ECANFilterSID
                  0x025750                  _ECANFilterEID
                  0x025762                  _ECAN1DMAConfig
                  0x0257aa                  _ECAN1ClockConfig
                  0x0257ba                  _ECAN1InterruptConfig
                  0x0257e4                  _ECAN1TxRxBuffersConfig
                  0x0257ee                  _ECAN1RxFiltersConfig
                  0x02585a                  _ECAN1SendPacket
                  0x025890                  _ECAN1SetOPMode
                  0x0258ac                  _ECANCreateSIDPacket
                  0x025900                  _ECANCreateEIDPacket
 .text            0x025a0c        0x2e4 build/XC16_dsPIC33EP512MU810/debug/B40/dpv1.o
                  0x025a0c                  _DPV1_ProcessCmdMsg
                  0x025a36                  _dpv1_InstanceCommand
                  0x025b92                  _dpv1_ObjectCommand
 .text            0x025cf0        0x2c2 build/XC16_dsPIC33EP512MU810/debug/TCPIPStack/ICMP.o
                  0x025cf0                  _ICMPProcess
                  0x025ddc                  _ICMPSendPing
                  0x025e00                  _ICMPSendPingToHost
                  0x025e2a                  _ICMPGetReply
                  0x025f84                  _ICMPBeginUsage
                  0x025fa4                  _ICMPEndUsage
 .text            0x025fb2        0x27a build/XC16_dsPIC33EP512MU810/debug/BerkeleyUDPClient.o
                  0x025fb2                  _BerkeleyUDPClient
                  0x0261da                  _BerkeleySNTPGetUTCSeconds
 .text            0x02622c        0x270 build/XC16_dsPIC33EP512MU810/debug/Regul.o
                  0x02622c                  _RegulationDoseur
                  0x02632c                  _RegulationPID
 .text            0x02649c        0x252 build/XC16_dsPIC33EP512MU810/debug/B40/spi/abcc_crc32.o
                  0x02649c                  _CRC_Crc32
 .text            0x0266ee        0x23c build/XC16_dsPIC33EP512MU810/debug/B40/user_setup.o
                  0x0266ee                  _US_Init
                  0x0266f8                  _US_RunUserInitStateMachine
                  0x0267ee                  build/XC16_dsPIC33EP512MU810/debug/B40/user_setup.o:_US_ProcessRespMsg
                  0x026906                  _US_SetSwitch1
                  0x026918                  _US_SetSwitch2
 .text            0x02692a        0x23c build/XC16_dsPIC33EP512MU810/debug/BerkeleyTCPServer.o
                  0x02692a                  _TestModbus
                  0x02698e                  _BerkeleyTCPServer
 .text            0x026b66        0x1f4 build/XC16_dsPIC33EP512MU810/debug/B40/abcc_timer.o
                  0x026b66                  _ABCC_TimerInit
                  0x026b88                  _ABCC_TimerCreate
                  0x026bfa                  _ABCC_TimerStart
                  0x026c78                  _ABCC_TimerStop
                  0x026cba                  _ABCC_TimerTick
 .text            0x026d5a        0x1ca build/XC16_dsPIC33EP512MU810/debug/TCPIPStack/IP.o
                  0x026d5a                  _IPGetHeader
                  0x026e24                  _IPPutHeader
                  0x026ed6                  _IPSetRxBuffer
 .text            0x026f24        0x1c2 build/XC16_dsPIC33EP512MU810/debug/TCPIPStack/Announce.o
                  0x026f24                  _AnnounceIP
                  0x026fce                  _DiscoveryTask
 .text            0x0270e6        0x1c2 build/XC16_dsPIC33EP512MU810/debug/TCPIPStack/StackTsk.o
                  0x0270e6                  _StackInit
                  0x02711e                  _StackTask
                  0x027292                  _StackApplications
 .text            0x0272a8        0x16a build/XC16_dsPIC33EP512MU810/debug/B40/abcc_cbf.o
                  0x0272a8                  _ABCC_CbfUserInitReq
                  0x0272b6                  _ABCC_CbfAdiMappingReq
                  0x0272c8                  _ABCC_CbfRemapDone
                  0x0272d2                  _ABCC_CbfUpdateWriteProcessData
                  0x0272e4                  _ABCC_CbfNewReadPd
                  0x0272f2                  _ABCC_CbfDriverError
                  0x027314                  _ABCC_CbfReceiveMsg
                  0x027384                  _ABCC_CbfWdTimeout
                  0x02739a                  _ABCC_CbfWdTimeoutRecovered
                  0x0273b0                  _ABCC_CbfEvent
                  0x0273ea                  _ABCC_CbfAnbStatusChanged
 .text            0x027412        0x160 build/XC16_dsPIC33EP512MU810/debug/MODBUSTCPServer.o
                  0x027412                  _MODBUSTCPServer
                  0x0274b0                  _ProcessReceivedMessage
                  0x027544                  _ModbusError
 .text            0x027572        0x15a build/XC16_dsPIC33EP512MU810/debug/TCPIPStack/Tick.o
                  0x027572                  _TickInit
                  0x027604                  _TickGet
                  0x027636                  _TickGetDiv256
                  0x027668                  _TickGetDiv64K
                  0x02769a                  _TickConvertToMilliseconds
                  0x0276b4                  __T1Interrupt
 .text            0x0276cc        0x12e build/XC16_dsPIC33EP512MU810/debug/BerkeleyTCPClient.o
                  0x0276cc                  _BerkeleyTCPClient
 .text            0x0277fa        0x118 build/XC16_dsPIC33EP512MU810/debug/B40/abcc_sys_adapt.o
                  0x0277fa                  _ABCC_SYS_Init
                  0x027824                  _ABCC_SYS_Close
                  0x02782e                  _ABCC_SYS_SetOpmode
                  0x027836                  _ABCC_SYS_GetOpmode
                  0x027840                  _ABCC_SYS_HWReset
                  0x027848                  _ABCC_SYS_HWReleaseReset
                  0x027850                  _ABCC_SYS_ReadModuleId
                  0x02785a                  _ABCC_SYS_ModuleDetect
                  0x027872                  _ABCC_SYS_AbccInterruptEnable
                  0x02787e                  _ABCC_SYS_AbccInterruptDisable
                  0x027886                  _ABCC_SYS_EnterCriticalImpl
                  0x02788c                  _ABCC_SYS_ExitCriticalImpl
                  0x027892                  _ABCC_SYS_UseCriticalImpl
                  0x027898                  _ABCC_SYS_SpiRegDataReceived
                  0x0278a4                  _ABCC_SYS_SpiSendReceive
 .text            0x027912        0x118 build/XC16_dsPIC33EP512MU810/debug/TCPIPStack/Reboot.o
                  0x027912                  _RebootTask
 .text            0x027a2a        0x116 build/XC16_dsPIC33EP512MU810/debug/ADC10bitsDrv.o
                  0x027a2a                  _InitAdc1
                  0x027a8a                  _InitTmr3
                  0x027a9e                  _InitDma0
                  0x027ad6                  _ProcessADCSamples
 .text            0x027b40        0x100 build/XC16_dsPIC33EP512MU810/debug/ADComm.o
                  0x027b40                  _ADSPI_Init
                  0x027b66                  _SPI_Read
                  0x027bd8                  _SPI_Write
 .text            0x027c40         0xc8 build/XC16_dsPIC33EP512MU810/debug/B40/abcc_mem.o
                  0x027c40                  _ABCC_MemCreatePool
                  0x027c8c                  _ABCC_MemAlloc
                  0x027cc8                  _ABCC_MemFree
 .text            0x027d08         0x86 build/XC16_dsPIC33EP512MU810/debug/B40/spi/abcc_handler_spi.o
                  0x027d08                  _ABCC_SpiRunDriver
                  0x027d64                  _ABCC_SpiISR
 .text            0x027d8e         0x7e build/XC16_dsPIC33EP512MU810/debug/system.o
                  0x027d8e                  _ConfigureOscillator
 .text            0x027e0c         0x78 build/XC16_dsPIC33EP512MU810/debug/TCPIPStack/Delay.o
                  0x027e0c                  _DelayMs
                  0x027e48                  _Delay10us
 .text            0x027e84         0x56 build/XC16_dsPIC33EP512MU810/debug/usb/src/usb_hal_dspic33e.o
                  0x027e84                  _USBSleepOnSuspend
 .text            0x027eda         0x42 build/XC16_dsPIC33EP512MU810/debug/B40/abcc_remap.o
                  0x027eda                  build/XC16_dsPIC33EP512MU810/debug/B40/abcc_remap.o:_abcc_RemapRespMsgSent
                  0x027ef0                  _ABCC_SendRemapRespMsg
 .text            0x027f1c         0x1e build/XC16_dsPIC33EP512MU810/debug/B40/user_adi.o
                  0x027f1c                  _AD_GetNumAdi
                  0x027f26                  _ADI_GetDefaultMap
                  0x027f30                  _ADI_GetADIEntryList

MPFSHelpers       0x027f3a          0xe
 MPFSHelpers      0x027f3a          0xe build/XC16_dsPIC33EP512MU810/debug/MPFSImg2.o
                  0x027f3a                  _ReadProgramMemory
